 surface_hid_mini

 Timestamp is 66d24ca1 (Fri Aug 30 22:50:09 2024)

 Preferred load address is 0000000180000000

 Start         Length     Name                   Class
 0001:00000000 00005e20H .text                   CODE
 0001:00005e20 0001e3b0H .text$mn                CODE
 0001:000241d0 000000b0H .text$mn$00             CODE
 0001:00024280 000004c0H .text$mn$21             CODE
 0001:00024740 00001310H .text$s                 CODE
 0001:00025a50 000000cfH .text$unlikely          CODE
 0002:00000000 00000280H .idata$5                DATA
 0002:00000280 00000030H .00cfg                  DATA
 0002:000002b0 00000014H .gehcont                DATA
 0002:000002c4 0000080cH .gfids                  DATA
 0002:00000acc 00000000H .gfids$y                DATA
 0002:00000acc 00000000H .giats$y                DATA
 0002:00000acc 00000000H .gljmp$y                DATA
 0002:00000ad0 00002630H .rdata                  DATA
 0002:00003100 00000000H .rdata$CastGuardVftablesA DATA
 0002:00003100 00000000H .rdata$CastGuardVftablesC DATA
 0002:00003100 00000000H .rdata$zETW0            DATA
 0002:00003100 00000000H .rdata$zETW9            DATA
 0002:00003100 000002d0H .rdata$zzzdbg           DATA
 0002:000033d0 000019f0H .xdata                  DATA
 0003:00000000 00000d60H .data                   DATA
 0003:00000d60 00000010H .kmdfclassbind$a        DATA
 0003:00000d70 00000008H .kmdfclassbind$c        DATA
 0003:00000d78 00000008H .kmdfclassbind$d        DATA
 0003:00000d80 00000010H .kmdftypeinit$a         DATA
 0003:00000d90 00000010H .kmdftypeinit$c         DATA
 0003:00000da0 00000410H .bss                    DATA
 0004:00000000 00002274H .pdata                  DATA
 0005:00000000 0001aec0H PAGE                    CODE
 0005:0001aec0 00000768H PAGE$s                  CODE
 0006:00000000 000001a0H PAGED                   CODE
 0006:000001a0 00000007H PAGED$s                 CODE
 0007:00000000 00000083H .edata                  DATA
 0008:00000000 00000648H INIT                    CODE
 0008:00000648 00000050H .idata$2                CODE
 0008:00000698 00000018H .idata$3                CODE
 0008:000006b0 00000280H .idata$4                CODE
 0008:00000930 00000714H .idata$6                CODE

  Address         Publics by Value              Rva+Base               Lib:Object

 0000:00000000       __AbsoluteZero             0000000000000000     <absolute>
 0000:00000000       ___safe_se_handler_count   0000000000000000     <absolute>
 0000:00000000       ___safe_se_handler_table   0000000000000000     <absolute>
 0000:00000000       __arm64x_extra_rfe_table   0000000000000000     <absolute>
 0000:00000000       __arm64x_extra_rfe_table_size 0000000000000000     <absolute>
 0000:00000000       __arm64x_native_entrypoint 0000000000000000     <absolute>
 0000:00000000       __arm64x_redirection_metadata 0000000000000000     <absolute>
 0000:00000000       __arm64x_redirection_metadata_count 0000000000000000     <absolute>
 0000:00000000       __dynamic_value_reloc_table 0000000000000000     <absolute>
 0000:00000000       __enclave_config           0000000000000000     <absolute>
 0000:00000000       __guard_check_icall_a64n_fptr 0000000000000000     <absolute>
 0000:00000000       __guard_iat_count          0000000000000000     <absolute>
 0000:00000000       __guard_iat_table          0000000000000000     <absolute>
 0000:00000000       __guard_longjmp_count      0000000000000000     <absolute>
 0000:00000000       __guard_longjmp_table      0000000000000000     <absolute>
 0000:00000000       __hybrid_auxiliary_delayload_iat 0000000000000000     <absolute>
 0000:00000000       __hybrid_auxiliary_delayload_iat_copy 0000000000000000     <absolute>
 0000:00000000       __hybrid_auxiliary_iat     0000000000000000     <absolute>
 0000:00000000       __hybrid_auxiliary_iat_copy 0000000000000000     <absolute>
 0000:00000000       __hybrid_code_map          0000000000000000     <absolute>
 0000:00000000       __hybrid_code_map_count    0000000000000000     <absolute>
 0000:00000000       __hybrid_image_info_bitfield 0000000000000000     <absolute>
 0000:00000000       __volatile_metadata        0000000000000000     <absolute>
 0000:00000000       __x64_code_ranges_to_entry_points 0000000000000000     <absolute>
 0000:00000000       __x64_code_ranges_to_entry_points_count 0000000000000000     <absolute>
 0000:00000004       __guard_eh_cont_count      0000000000000004     <absolute>
 0000:0000019b       __guard_fids_count         000000000000019b     <absolute>
 0000:10414500       __guard_flags              0000000010414500     <absolute>
 0000:00000000       __ImageBase                0000000180000000     <linker-defined>
 0001:00005e10       __CxxFrameHandler3         0000000180006e10 f   surface_hid_mini.surface_hid_mini.3efcb60154bd7459-cgu.0.rcgu.o
 0001:00005e20       __report_gsfailure         0000000180006e20 f   BufferOverflowFastFailK:gs_report.obj
 0001:00005e30       _guard_check_icall_nop     0000000180006e30 f i BufferOverflowFastFailK:guard_check.obj
 0001:00005e40       EtwWriteTransfer           0000000180006e40 f   ntoskrnl:ntoskrnl.exe
 0001:00005e50       ExAllocatePool2            0000000180006e50 f   ntoskrnl:ntoskrnl.exe
 0001:00005e56       EtwUnregister              0000000180006e56 f   ntoskrnl:ntoskrnl.exe
 0001:00005e5c       ExFreePool                 0000000180006e5c f   ntoskrnl:ntoskrnl.exe
 0001:00005e62       RtlInitUnicodeString       0000000180006e62 f   ntoskrnl:ntoskrnl.exe
 0001:00005e68       RtlEqualUnicodeString      0000000180006e68 f   ntoskrnl:ntoskrnl.exe
 0001:00005e6e       PoRegisterPowerSettingCallback 0000000180006e6e f   ntoskrnl:ntoskrnl.exe
 0001:00005e74       PoUnregisterPowerSettingCallback 0000000180006e74 f   ntoskrnl:ntoskrnl.exe
 0001:00005e7a       EtwRegister                0000000180006e7a f   ntoskrnl:ntoskrnl.exe
 0001:00005e80       EtwSetInformation          0000000180006e80 f   ntoskrnl:ntoskrnl.exe
 0001:00005e90       __cpu_features_init        0000000180006e90 f   ntoskrnl:cpuinfo.obj
 0001:00005f50       ?FxStubDriverEntryFailure@@YAXXZ 0000000180006f50 f   WdfDriverEntry:stub.obj
 0001:00005fa8       ?FxStubDriverUnloadCommon@@YAXXZ 0000000180006fa8 f   WdfDriverEntry:stub.obj
 0001:00005fe0       FxDriverEntry              0000000180006fe0 f   WdfDriverEntry:stub.obj
 0001:0000600c       FxDriverEntryWorker        000000018000700c f   WdfDriverEntry:stub.obj
 0001:00006160       FxStubDriverMiniportUnload 0000000180007160 f   WdfDriverEntry:stub.obj
 0001:00006170       FxStubDriverUnload         0000000180007170 f   WdfDriverEntry:stub.obj
 0001:0000619c       ?FxStubInitTypes@@YAJXZ    000000018000719c f   WdfDriverEntry:inittypes.obj
 0001:00006260       ?FxStubBindClasses@@YAJPEAU_WDF_BIND_INFO@@@Z 0000000180007260 f   WdfDriverEntry:classbind.obj
 0001:000063dc       ?FxStubIsClassBound@@YAEXZ 00000001800073dc f   WdfDriverEntry:classbind.obj
 0001:000063f0       ?FxStubUnbindClasses@@YAXPEAU_WDF_BIND_INFO@@@Z 00000001800073f0 f   WdfDriverEntry:classbind.obj
 0001:000064d0       WPP_RECORDER_SF_           00000001800074d0 f i libms_surface_wpp-b83efe80b23bd200:2e40c9e35e9506f4-wpp.o
 0001:000065a0       WppClassicProviderCallback 00000001800075a0 f   libms_surface_wpp-b83efe80b23bd200:2e40c9e35e9506f4-wpp.o
 0001:000065f0       WppCleanup                 00000001800075f0 f   libms_surface_wpp-b83efe80b23bd200:2e40c9e35e9506f4-wpp.o
 0001:00006660       WppInitialize              0000000180007660 f   libms_surface_wpp-b83efe80b23bd200:2e40c9e35e9506f4-wpp.o
 0001:00006710       ?BufferPool_BufferGet@@YAPEAXPEAUDMFMODULE__@@@Z 0000000180007710 f   DmfK:Dmf_BufferPool.obj
 0001:00006884       ?BufferPool_BufferPoolCreate@@YAJPEAUDMFMODULE__@@@Z 0000000180007884 f   DmfK:Dmf_BufferPool.obj
 0001:00006bdc       ?BufferPool_BufferPoolEntryCreateAndAddToList@@YAJPEAUDMFMODULE__@@@Z 0000000180007bdc f   DmfK:Dmf_BufferPool.obj
 0001:0000707c       ?BufferPool_BufferPoolEntryGet@@YAPEAUWDFMEMORY__@@PEAUDMFMODULE__@@PEAPEAUBUFFERPOOL_ENTRY@@@Z 000000018000807c f   DmfK:Dmf_BufferPool.obj
 0001:000072c0       ?BufferPool_BufferPoolEntryGetFromClientBuffer@@YAPEAUBUFFERPOOL_ENTRY@@PEAX@Z 00000001800082c0 f   DmfK:Dmf_BufferPool.obj
 0001:000073bc       ?BufferPool_BufferPoolEntryPut@@YAXPEAUDMFMODULE__@@PEAUBUFFERPOOL_ENTRY@@P6AXPEAU_DMF_CONTEXT_BufferPool@@1@Z@Z 00000001800083bc f   DmfK:Dmf_BufferPool.obj
 0001:000075c0       ?BufferPool_BufferPoolEntryTimerHandler@@YAXPEAUWDFTIMER__@@@Z 00000001800085c0 f   DmfK:Dmf_BufferPool.obj
 0001:00007814       ?BufferPool_InsertList@@YAXPEAUDMFMODULE__@@PEAU_DMF_CONTEXT_BufferPool@@PEAUBUFFERPOOL_ENTRY@@P6AX12@Z@Z 0000000180008814 f   DmfK:Dmf_BufferPool.obj
 0001:00007870       ?BufferPool_InsertTailList@@YAXPEAU_DMF_CONTEXT_BufferPool@@PEAUBUFFERPOOL_ENTRY@@@Z 0000000180008870 f   DmfK:Dmf_BufferPool.obj
 0001:00007894       ?BufferPool_ListFlushAndDestroy@@YAXPEAUDMFMODULE__@@@Z 0000000180008894 f   DmfK:Dmf_BufferPool.obj
 0001:00007b54       ?BufferPool_Put@@YAXPEAUDMFMODULE__@@PEAXP6AXPEAU_DMF_CONTEXT_BufferPool@@PEAUBUFFERPOOL_ENTRY@@@Z@Z 0000000180008b54 f   DmfK:Dmf_BufferPool.obj
 0001:00007d28       ?BufferPool_RemoveEntryList@@YAXPEAUDMFMODULE__@@PEAU_DMF_CONTEXT_BufferPool@@PEAUBUFFERPOOL_ENTRY@@@Z 0000000180008d28 f   DmfK:Dmf_BufferPool.obj
 0001:00007d7c       ?BufferPool_RemoveHeadList@@YAPEAUBUFFERPOOL_ENTRY@@PEAUDMFMODULE__@@PEAU_DMF_CONTEXT_BufferPool@@@Z 0000000180008d7c f   DmfK:Dmf_BufferPool.obj
 0001:00007e60       ?DMF_BufferPool_LiveKernelDumpInitialize@@YAXPEAUDMFMODULE__@@@Z 0000000180008e60 f   DmfK:Dmf_BufferPool.obj
 0001:00007ec0       DMF_BufferPool_ContextGet  0000000180008ec0 f   DmfK:Dmf_BufferPool.obj
 0001:00007fa8       DMF_BufferPool_Count       0000000180008fa8 f   DmfK:Dmf_BufferPool.obj
 0001:00008158       DMF_BufferPool_Get         0000000180009158 f   DmfK:Dmf_BufferPool.obj
 0001:00008274       DMF_BufferPool_GetWithMemory 0000000180009274 f   DmfK:Dmf_BufferPool.obj
 0001:00008394       DMF_BufferPool_Put         0000000180009394 f   DmfK:Dmf_BufferPool.obj
 0001:00008480       WPP_RECORDER_SF_D          0000000180009480 f i DmfK:DmfPortable.obj
 0001:00008480       WPP_RECORDER_SF_d          0000000180009480 f i DmfK:Dmf_BufferPool.obj
 0001:00008570       WPP_RECORDER_SF_Dd         0000000180009570 f i DmfK:Dmf_IoctlHandler.obj
 0001:00008570       WPP_RECORDER_SF_dd         0000000180009570 f i DmfK:Dmf_BufferPool.obj
 0001:0000868c       WPP_RECORDER_SF_q          000000018000968c f i DmfK:Dmf_BufferPool.obj
 0001:0000877c       WPP_RECORDER_SF_ID         000000018000977c f i DmfK:SurfaceTelemetry.obj
 0001:0000877c       WPP_RECORDER_SF_qd         000000018000977c f i DmfK:Dmf_BufferPool.obj
 0001:0000889c       WPP_RECORDER_SF_qdq        000000018000989c f i DmfK:Dmf_BufferPool.obj
 0001:000089e0       WdfObjectAddCustomType_DMF_BufferPool 00000001800099e0 f i DmfK:Dmf_BufferPool.obj
 0001:00008a70       ?DMF_SamCommunicationViaSsh_BranchTrackInitialize@@YAXPEAUDMFMODULE__@@@Z 0000000180009a70 f   DmfK:Dmf_SamCommunicationViaSsh.obj
 0001:00008b20       ?DMF_SamCommunicationViaSsh_LiveKernelDumpInitialize@@YAXPEAUDMFMODULE__@@@Z 0000000180009b20 f   DmfK:Dmf_SamCommunicationViaSsh.obj
 0001:00008b80       ?SamCommunicationViaSsh_OnDeviceArrivalNotification@@YAXPEAUDMFMODULE__@@@Z 0000000180009b80 f   DmfK:Dmf_SamCommunicationViaSsh.obj
 0001:00008cb0       ?SamCommunicationViaSsh_OnDeviceRemovalNotification@@YAXPEAUDMFMODULE__@@@Z 0000000180009cb0 f   DmfK:Dmf_SamCommunicationViaSsh.obj
 0001:00008dc4       DMF_SamCommunicationViaSsh_Send 0000000180009dc4 f   DmfK:Dmf_SamCommunicationViaSsh.obj
 0001:00008f34       DMF_SamCommunicationViaSsh_SendSynchronously 0000000180009f34 f   DmfK:Dmf_SamCommunicationViaSsh.obj
 0001:00009098       WPP_RECORDER_SF_c          000000018000a098 f i DmfK:Dmf_SamCommunicationViaSsh.obj
 0001:00009190       WdfObjectAddCustomType_DMF_SamCommunicationViaSsh 000000018000a190 f i DmfK:Dmf_SamCommunicationViaSsh.obj
 0001:0000921c       ?DMF_FeatureHandleGetFromModuleCollection@@YAPEAU_DMF_OBJECT_@@PEAUDMFCOLLECTION__@@W4DmfFeatureType@@@Z 000000018000a21c f   DmfK:DmfHelpers.obj
 0001:00009254       ?DMF_GenericMemoryAllocate@@YAPEAX_K0K@Z 000000018000a254 f   DmfK:DmfHelpers.obj
 0001:00009338       ?DMF_GenericMemoryFree@@YAXPEAXK@Z 000000018000a338 f   DmfK:DmfHelpers.obj
 0001:00009340       ?DMF_GenericSpinLockAcquire@@YAXPEA_KPEAE@Z 000000018000a340 f   DmfK:DmfHelpers.obj
 0001:00009358       ?DMF_GenericSpinLockCreate@@YAJPEAU_WDF_OBJECT_ATTRIBUTES@@PEA_K@Z 000000018000a358 f   DmfK:DmfHelpers.obj
 0001:00009370       ?DMF_GenericSpinLockDestroy@@YAXPEA_K@Z 000000018000a370 f   DmfK:DmfHelpers.obj
 0001:00009370       ?DMF_HandleValidate_Close@@YAXPEAU_DMF_OBJECT_@@@Z 000000018000a370 f   DmfK:DmfValidate.obj
 0001:00009370       ?DMF_HandleValidate_Destroy@@YAXPEAU_DMF_OBJECT_@@@Z 000000018000a370 f   DmfK:DmfValidate.obj
 0001:00009370       ?DMF_HandleValidate_IsAvailable@@YAXPEAU_DMF_OBJECT_@@@Z 000000018000a370 f   DmfK:DmfValidate.obj
 0001:00009370       ?DMF_HandleValidate_IsClosing@@YAXPEAU_DMF_OBJECT_@@@Z 000000018000a370 f   DmfK:DmfValidate.obj
 0001:00009370       ?DMF_HandleValidate_IsCreated@@YAXPEAU_DMF_OBJECT_@@@Z 000000018000a370 f   DmfK:DmfValidate.obj
 0001:00009370       ?DMF_HandleValidate_IsCreatedOrClosed@@YAXPEAU_DMF_OBJECT_@@@Z 000000018000a370 f   DmfK:DmfValidate.obj
 0001:00009370       ?DMF_HandleValidate_IsCreatedOrOpened@@YAXPEAU_DMF_OBJECT_@@@Z 000000018000a370 f   DmfK:DmfValidate.obj
 0001:00009370       ?DMF_HandleValidate_IsOpen@@YAXPEAU_DMF_OBJECT_@@@Z 000000018000a370 f   DmfK:DmfValidate.obj
 0001:00009370       ?DMF_HandleValidate_IsOpening@@YAXPEAU_DMF_OBJECT_@@@Z 000000018000a370 f   DmfK:DmfValidate.obj
 0001:00009370       ?DMF_HandleValidate_Open@@YAXPEAU_DMF_OBJECT_@@@Z 000000018000a370 f   DmfK:DmfValidate.obj
 0001:00009370       ?DMF_String_LiveKernelDumpInitialize@@YAXPEAUDMFMODULE__@@@Z 000000018000a370 f   DmfK:Dmf_String.obj
 0001:00009370       DMF_HandleValidate_ClosingOk 000000018000a370 f   DmfK:DmfValidate.obj
 0001:00009370       DMF_HandleValidate_ModuleMethod 000000018000a370 f   DmfK:DmfValidate.obj
 0001:00009370       DMF_HandleValidate_OpeningOk 000000018000a370 f   DmfK:DmfValidate.obj
 0001:00009370       DMF_ObjectValidate         000000018000a370 f   DmfK:DmfValidate.obj
 0001:00009374       ?DMF_GenericSpinLockRelease@@YAXPEA_KE@Z 000000018000a374 f   DmfK:DmfHelpers.obj
 0001:0000937c       ?DMF_RequestPassthru@@YAXPEAUWDFDEVICE__@@PEAUWDFREQUEST__@@@Z 000000018000a37c f   DmfK:DmfHelpers.obj
 0001:000094d0       ?DMF_RequestPassthruWithCompletion@@YAXPEAUWDFDEVICE__@@PEAUWDFREQUEST__@@P6AX1PEAUWDFIOTARGET__@@PEAU_WDF_REQUEST_COMPLETION_PARAMS@@PEAX@Z4@Z 000000018000a4d0 f   DmfK:DmfHelpers.obj
 0001:00009630       DMF_FeatureModuleGetFromModule 000000018000a630 f   DmfK:DmfHelpers.obj
 0001:00009694       DMF_IsModuleDynamic        000000018000a694 f   DmfK:DmfHelpers.obj
 0001:000096d4       DMF_IsModulePassiveLevel   000000018000a6d4 f   DmfK:DmfHelpers.obj
 0001:00009714       DMF_ModuleConfigGet        000000018000a714 f   DmfK:DmfHelpers.obj
 0001:00009750       DMF_ModuleIsInFilterDriver 000000018000a750 f   DmfK:DmfHelpers.obj
 0001:00009794       DMF_ModuleLockPrivate      000000018000a794 f   DmfK:DmfHelpers.obj
 0001:000097f4       DMF_ModuleUnlockPrivate    000000018000a7f4 f   DmfK:DmfHelpers.obj
 0001:00009840       DMF_ParentDeviceGet        000000018000a840 f   DmfK:DmfHelpers.obj
 0001:0000987c       DMF_ParentModuleGet        000000018000a87c f   DmfK:DmfHelpers.obj
 0001:000098c8       WPP_RECORDER_SF_qs         000000018000a8c8 f i DmfK:DmfHelpers.obj
 0001:00009a40       WPP_RECORDER_SF_qsd        000000018000aa40 f i DmfK:DmfHelpers.obj
 0001:00009bf0       ?DMF_SamNotificationViaSsh_BranchTrackInitialize@@YAXPEAUDMFMODULE__@@@Z 000000018000abf0 f   DmfK:Dmf_SamNotificationViaSsh.obj
 0001:0000a530       ?DMF_SamNotificationViaSsh_LiveKernelDumpInitialize@@YAXPEAUDMFMODULE__@@@Z 000000018000b530 f   DmfK:Dmf_SamNotificationViaSsh.obj
 0001:0000b290       ?SamNotificationViaSsh_RegisterCompletion@@YAXPEAUDMFMODULE__@@PEAX1_K12J@Z 000000018000c290 f   DmfK:Dmf_SamNotificationViaSsh.obj
 0001:0000ca50       ?SamNotificationViaSsh_UnregisterCompletion@@YAXPEAUDMFMODULE__@@PEAX1_K12J@Z 000000018000da50 f   DmfK:Dmf_SamNotificationViaSsh.obj
 0001:0000cc4c       DMF_SamNotificationViaSsh_ClientBufferPutOutput 000000018000dc4c f   DmfK:Dmf_SamNotificationViaSsh.obj
 0001:0000cd60       WPP_RECORDER_SF_dP         000000018000dd60 f i DmfK:Dmf_SamNotificationViaSsh.obj
 0001:0000cd60       WPP_RECORDER_SF_dq         000000018000dd60 f i DmfK:DmfInterfaceInternal.obj
 0001:0000ce80       WPP_RECORDER_SF_ddP        000000018000de80 f i DmfK:Dmf_SamNotificationViaSsh.obj
 0001:0000cfc4       WPP_RECORDER_SF_s          000000018000dfc4 f i DmfK:Dmf_SamNotificationViaSsh.obj
 0001:0000d110       WdfObjectAddCustomType_DMF_SamNotificationViaSsh 000000018000e110 f i DmfK:Dmf_SamNotificationViaSsh.obj
 0001:0000d19c       ?SurfaceTelemetry_ReadConsentFile@@YAJXZ 000000018000e19c f   DmfK:SurfaceTelemetry.obj
 0001:0000d430       SurfaceTelemetry_Initialize 000000018000e430 f   DmfK:SurfaceTelemetry.obj
 0001:0000d540       SurfaceTelemetry_IsTelemetryEventTypeAllowed 000000018000e540 f   DmfK:SurfaceTelemetry.obj
 0001:0000d674       SurfaceTelemetry_Update    000000018000e674 f   DmfK:SurfaceTelemetry.obj
 0001:0000d780       ?DMF_QueuedWorkItem_LiveKernelDumpInitialize@@YAXPEAUDMFMODULE__@@@Z 000000018000e780 f   DmfK:Dmf_QueuedWorkItem.obj
 0001:0000d7e0       ?QueuedWorkItem_CallbackScheduledTask@@YA?AW4ScheduledTask_Result_Type@@PEAUDMFMODULE__@@PEAXW4_WDF_POWER_DEVICE_STATE@@@Z 000000018000e7e0 f   DmfK:Dmf_QueuedWorkItem.obj
 0001:0000d964       DMF_QueuedWorkItem_Enqueue 000000018000e964 f   DmfK:Dmf_QueuedWorkItem.obj
 0001:0000db50       WdfObjectAddCustomType_DMF_QueuedWorkItem 000000018000eb50 f i DmfK:Dmf_QueuedWorkItem.obj
 0001:0000dd5c       ?DMF_ModuleCollectionD0Entry@@YAJPEAUDMFCOLLECTION__@@W4_WDF_POWER_DEVICE_STATE@@@Z 000000018000ed5c f   DmfK:DmfModuleCollection.obj
 0001:0000df1c       ?DMF_ModuleCollectionD0EntryCleanup@@YAXPEAUDMFCOLLECTION__@@@Z 000000018000ef1c f   DmfK:DmfModuleCollection.obj
 0001:0000e000       ?DMF_ModuleCollectionD0EntryPostInterruptsEnabled@@YAJPEAUDMFCOLLECTION__@@W4_WDF_POWER_DEVICE_STATE@@@Z 000000018000f000 f   DmfK:DmfModuleCollection.obj
 0001:0000e1c0       ?DMF_ModuleCollectionD0Exit@@YAJPEAUDMFCOLLECTION__@@W4_WDF_POWER_DEVICE_STATE@@@Z 000000018000f1c0 f   DmfK:DmfModuleCollection.obj
 0001:0000e378       ?DMF_ModuleCollectionD0ExitPreInterruptsDisabled@@YAJPEAUDMFCOLLECTION__@@W4_WDF_POWER_DEVICE_STATE@@@Z 000000018000f378 f   DmfK:DmfModuleCollection.obj
 0001:0000e530       ?DMF_ModuleCollectionDestroy@@YAXPEAX@Z 000000018000f530 f   DmfK:DmfModuleCollection.obj
 0001:0000e69c       ?DMF_ModuleCollectionDeviceIoControl@@YAEPEAUDMFCOLLECTION__@@PEAUWDFQUEUE__@@PEAUWDFREQUEST__@@_K3K@Z 000000018000f69c f   DmfK:DmfModuleCollection.obj
 0001:0000e844       ?DMF_ModuleCollectionDispatchNtStatus@@YAJPEAU_DMF_MODULE_COLLECTION_@@P6AJPEAUDMFMODULE__@@@Z@Z 000000018000f844 f   DmfK:DmfModuleCollection.obj
 0001:0000e944       ?DMF_ModuleCollectionDispatchVoid@@YAXPEAU_DMF_MODULE_COLLECTION_@@P6AXPEAUDMFMODULE__@@@Z@Z 000000018000f944 f   DmfK:DmfModuleCollection.obj
 0001:0000ea2c       ?DMF_ModuleCollectionInternalDeviceIoControl@@YAEPEAUDMFCOLLECTION__@@PEAUWDFQUEUE__@@PEAUWDFREQUEST__@@_K3K@Z 000000018000fa2c f   DmfK:DmfModuleCollection.obj
 0001:0000ebd4       ?DMF_ModuleCollectionQueueIoRead@@YAEPEAUDMFCOLLECTION__@@PEAUWDFQUEUE__@@PEAUWDFREQUEST__@@_K@Z 000000018000fbd4 f   DmfK:DmfModuleCollection.obj
 0001:0000ed5c       ?DMF_ModuleCollectionQueueIoWrite@@YAEPEAUDMFCOLLECTION__@@PEAUWDFQUEUE__@@PEAUWDFREQUEST__@@_K@Z 000000018000fd5c f   DmfK:DmfModuleCollection.obj
 0001:0000eee4       ?DMF_ModuleCollectionSelfManagedIoRestart@@YAJPEAUDMFCOLLECTION__@@@Z 000000018000fee4 f   DmfK:DmfModuleCollection.obj
 0001:0000f004       ?DMF_ModuleCollectionSelfManagedIoSuspend@@YAJPEAUDMFCOLLECTION__@@@Z 0000000180010004 f   DmfK:DmfModuleCollection.obj
 0001:0000f124       ?DMF_ModuleCollectionSurpriseRemoval@@YAXPEAUDMFCOLLECTION__@@@Z 0000000180010124 f   DmfK:DmfModuleCollection.obj
 0001:0000f22c       WPP_RECORDER_SF_qq         000000018001022c f i DmfK:DmfModuleCollection.obj
 0001:0000f350       ?DMF_SurfaceTelemetryConsentSettingsNotification_LiveKernelDumpInitialize@@YAXPEAUDMFMODULE__@@@Z 0000000180010350 f   DmfK:Dmf_SurfaceTelemetryConsentSettingsNotification.obj
 0001:0000f3b0       WdfObjectAddCustomType_DMF_SurfaceTelemetryConsentSettingsNotification 00000001800103b0 f i DmfK:Dmf_SurfaceTelemetryConsentSettingsNotification.obj
 0001:0000f43c       DMF_DmfDeviceInitFree      000000018001043c f   DmfK:DmfDeviceInit.obj
 0001:0000f4b0       ?DMF_LiveKernelDump_LiveKernelDumpInitialize@@YAXPEAUDMFMODULE__@@@Z 00000001800104b0 f   DmfK:Dmf_LiveKernelDump.obj
 0001:0000f510       ?LiveDump_CrashDumpStoreTriageDumpDataCallback@@YAXPEAUDMFMODULE__@@K_K111@Z 0000000180010510 f   DmfK:Dmf_LiveKernelDump.obj
 0001:0000f518       ?LiveKernelDump_DataBufferSourceAdd@@YAJPEAUDMFMODULE__@@PEAXK@Z 0000000180010518 f   DmfK:Dmf_LiveKernelDump.obj
 0001:0000f6e0       ?LiveKernelDump_InsertDataBufferInCrashDump@@YAEPEAUDMFMODULE__@@PEAEKPEAX@Z 00000001800106e0 f   DmfK:Dmf_LiveKernelDump.obj
 0001:0000f7a0       ?LiveKernelDump_InsertDataBufferInLiveDump@@YAEPEAUDMFMODULE__@@PEAEKPEAX@Z 00000001800107a0 f   DmfK:Dmf_LiveKernelDump.obj
 0001:0000f964       ?LiveKernelDump_InsertDmfTriageDataToCrashDump@@YAJPEAUDMFMODULE__@@@Z 0000000180010964 f   DmfK:Dmf_LiveKernelDump.obj
 0001:0000f9c0       DMF_LiveKernelDump_DataBufferSourceAdd 00000001800109c0 f   DmfK:Dmf_LiveKernelDump.obj
 0001:0000fac8       WPP_RECORDER_SF_qddD       0000000180010ac8 f i DmfK:Dmf_LiveKernelDump.obj
 0001:0000fac8       WPP_RECORDER_SF_qddd       0000000180010ac8 f i DmfK:Dmf_CrashDump.obj
 0001:0000fc40       WdfObjectAddCustomType_DMF_LiveKernelDump 0000000180010c40 f i DmfK:Dmf_LiveKernelDump.obj
 0001:0000fccc       DMF_Portable_EventClose    0000000180010ccc f   DmfK:DmfPortable.obj
 0001:0000fd54       DMF_Portable_EventCreate   0000000180010d54 f   DmfK:DmfPortable.obj
 0001:0000fe10       DMF_Portable_EventReset    0000000180010e10 f   DmfK:DmfPortable.obj
 0001:0000feac       DMF_Portable_EventSet      0000000180010eac f   DmfK:DmfPortable.obj
 0001:0000ff4c       DMF_Portable_LookasideListCreate 0000000180010f4c f   DmfK:DmfPortable.obj
 0001:00010044       DMF_Portable_LookasideListCreateMemory 0000000180011044 f   DmfK:DmfPortable.obj
 0001:00010110       DMF_Portable_Rundown_Acquire 0000000180011110 f   DmfK:DmfPortable.obj
 0001:00010118       DMF_Portable_Rundown_Completed 0000000180011118 f   DmfK:DmfPortable.obj
 0001:00010120       DMF_Portable_Rundown_Initialize 0000000180011120 f   DmfK:DmfPortable.obj
 0001:00010128       DMF_Portable_Rundown_Reinitialize 0000000180011128 f   DmfK:DmfPortable.obj
 0001:00010130       DMF_Portable_Rundown_Release 0000000180011130 f   DmfK:DmfPortable.obj
 0001:00010138       DMF_Portable_Rundown_WaitForRundownProtectionRelease 0000000180011138 f   DmfK:DmfPortable.obj
 0001:00010140       ?DMF_ModuleDestroy@@YAXPEAUDMFMODULE__@@E@Z 0000000180011140 f   DmfK:DmfCore.obj
 0001:00010304       ?DMF_ModuleTransportSet@@YAXPEAUDMFMODULE__@@0@Z 0000000180011304 f   DmfK:DmfCore.obj
 0001:00010368       ?RtlStringCbPrintfA@@YAJPEAD_KPEBDZZ 0000000180011368 f i DmfK:DmfCore.obj
 0001:000103d0       DMF_ModuleRequestCompleteOrForward 00000001800113d0 f   DmfK:DmfCore.obj
 0001:00010430       ?DmfChildObjectLastGet@@YAPEAU_DMF_OBJECT_@@PEAU1@PEAUCHILD_OBJECT_INTERATION_CONTEXT@@@Z 0000000180011430 f   DmfK:DmfCall.obj
 0001:00010470       ?DmfChildObjectPreviousGet@@YAPEAU_DMF_OBJECT_@@PEAUCHILD_OBJECT_INTERATION_CONTEXT@@@Z 0000000180011470 f   DmfK:DmfCall.obj
 0001:000104b0       ?DmfChildObjectFirstGet@@YAPEAU_DMF_OBJECT_@@PEAU1@PEAUCHILD_OBJECT_INTERATION_CONTEXT@@@Z 00000001800114b0 f   DmfK:DmfCall.obj
 0001:000104f0       ?DmfChildObjectNextGet@@YAPEAU_DMF_OBJECT_@@PEAUCHILD_OBJECT_INTERATION_CONTEXT@@@Z 00000001800114f0 f   DmfK:DmfCall.obj
 0001:00010524       ?DMF_ChildDispatchSingleParameterNtStatus@@YAJPEAUDMFMODULE__@@P6AJ0@ZPEAU_DMF_ChildObjectGet@@@Z 0000000180011524 f   DmfK:DmfCall.obj
 0001:000105a8       ?DMF_ChildDispatchSingleParameterVoid@@YAXPEAUDMFMODULE__@@P6AX0@ZPEAU_DMF_ChildObjectGet@@@Z 00000001800115a8 f   DmfK:DmfCall.obj
 0001:00010618       ?DMF_ModuleReferenceAdd@@YAJPEAUDMFMODULE__@@@Z 0000000180011618 f   DmfK:DmfCall.obj
 0001:00010710       ?DMF_ModuleReferenceDelete@@YAJPEAUDMFMODULE__@@@Z 0000000180011710 f   DmfK:DmfCall.obj
 0001:00010810       ?DMF_ModuleTreeDestroy@@YAXPEAUDMFMODULE__@@@Z 0000000180011810 f   DmfK:DmfCall.obj
 0001:00010880       ?DMF_ModuleWaitForReferenceCountToClear@@YAXPEAUDMFMODULE__@@@Z 0000000180011880 f   DmfK:DmfCall.obj
 0001:00010a40       ?DMF_Module_ArmWakeFromS0@@YAJPEAUDMFMODULE__@@@Z 0000000180011a40 f   DmfK:DmfCall.obj
 0001:00010aa4       ?DMF_Module_ArmWakeFromSxWithReason@@YAJPEAUDMFMODULE__@@EE@Z 0000000180011aa4 f   DmfK:DmfCall.obj
 0001:00010b60       ?DMF_Module_CloseOrUnregisterNotificationOnDestroy@@YAXPEAUDMFMODULE__@@@Z 0000000180011b60 f   DmfK:DmfCall.obj
 0001:00010bfc       ?DMF_Module_D0Entry@@YAJPEAUDMFMODULE__@@W4_WDF_POWER_DEVICE_STATE@@@Z 0000000180011bfc f   DmfK:DmfCall.obj
 0001:00010c88       ?DMF_Module_D0EntryPostInterruptsEnabled@@YAJPEAUDMFMODULE__@@W4_WDF_POWER_DEVICE_STATE@@@Z 0000000180011c88 f   DmfK:DmfCall.obj
 0001:00010d14       ?DMF_Module_D0Exit@@YAJPEAUDMFMODULE__@@W4_WDF_POWER_DEVICE_STATE@@@Z 0000000180011d14 f   DmfK:DmfCall.obj
 0001:00010dac       ?DMF_Module_D0ExitPreInterruptsDisabled@@YAJPEAUDMFMODULE__@@W4_WDF_POWER_DEVICE_STATE@@@Z 0000000180011dac f   DmfK:DmfCall.obj
 0001:00010e44       ?DMF_Module_DeviceIoControl@@YAEPEAUDMFMODULE__@@PEAUWDFQUEUE__@@PEAUWDFREQUEST__@@_K3K@Z 0000000180011e44 f   DmfK:DmfCall.obj
 0001:00010f30       ?DMF_Module_DisarmWakeFromS0@@YAXPEAUDMFMODULE__@@@Z 0000000180011f30 f   DmfK:DmfCall.obj
 0001:00010fa0       ?DMF_Module_DisarmWakeFromSx@@YAXPEAUDMFMODULE__@@@Z 0000000180011fa0 f   DmfK:DmfCall.obj
 0001:0001100c       ?DMF_Module_FileCleanup@@YAEPEAUDMFMODULE__@@PEAUWDFFILEOBJECT__@@@Z 000000018001200c f   DmfK:DmfCall.obj
 0001:000110a8       ?DMF_Module_FileClose@@YAEPEAUDMFMODULE__@@PEAUWDFFILEOBJECT__@@@Z 00000001800120a8 f   DmfK:DmfCall.obj
 0001:00011144       ?DMF_Module_FileCreate@@YAEPEAUDMFMODULE__@@PEAUWDFDEVICE__@@PEAUWDFREQUEST__@@PEAUWDFFILEOBJECT__@@@Z 0000000180012144 f   DmfK:DmfCall.obj
 0001:00011208       ?DMF_Module_InternalDeviceIoControl@@YAEPEAUDMFMODULE__@@PEAUWDFQUEUE__@@PEAUWDFREQUEST__@@_K3K@Z 0000000180012208 f   DmfK:DmfCall.obj
 0001:00011300       ?DMF_Module_NotificationUnregister@@YAXPEAUDMFMODULE__@@@Z 0000000180012300 f   DmfK:DmfCall.obj
 0001:00011370       ?DMF_Module_OpenOrRegisterNotificationOnCreate@@YAJPEAUDMFMODULE__@@@Z 0000000180012370 f   DmfK:DmfCall.obj
 0001:00011474       ?DMF_Module_PrepareHardware@@YAJPEAUDMFMODULE__@@PEAUWDFCMRESLIST__@@1@Z 0000000180012474 f   DmfK:DmfCall.obj
 0001:00011510       ?DMF_Module_QueryRemove@@YAJPEAUDMFMODULE__@@@Z 0000000180012510 f   DmfK:DmfCall.obj
 0001:00011580       ?DMF_Module_QueryStop@@YAJPEAUDMFMODULE__@@@Z 0000000180012580 f   DmfK:DmfCall.obj
 0001:000115e4       ?DMF_Module_QueueIoRead@@YAEPEAUDMFMODULE__@@PEAUWDFQUEUE__@@PEAUWDFREQUEST__@@_K@Z 00000001800125e4 f   DmfK:DmfCall.obj
 0001:000116a4       ?DMF_Module_QueueIoWrite@@YAEPEAUDMFMODULE__@@PEAUWDFQUEUE__@@PEAUWDFREQUEST__@@_K@Z 00000001800126a4 f   DmfK:DmfCall.obj
 0001:00011764       ?DMF_Module_RelationsQuery@@YAXPEAUDMFMODULE__@@W4_DEVICE_RELATION_TYPE@@@Z 0000000180012764 f   DmfK:DmfCall.obj
 0001:000117ec       ?DMF_Module_ReleaseHardware@@YAJPEAUDMFMODULE__@@PEAUWDFCMRESLIST__@@@Z 00000001800127ec f   DmfK:DmfCall.obj
 0001:00011890       ?DMF_Module_SelfManagedIoCleanup@@YAXPEAUDMFMODULE__@@@Z 0000000180012890 f   DmfK:DmfCall.obj
 0001:000118f0       ?DMF_Module_SelfManagedIoFlush@@YAXPEAUDMFMODULE__@@@Z 00000001800128f0 f   DmfK:DmfCall.obj
 0001:00011950       ?DMF_Module_SelfManagedIoInit@@YAJPEAUDMFMODULE__@@@Z 0000000180012950 f   DmfK:DmfCall.obj
 0001:000119c0       ?DMF_Module_SelfManagedIoRestart@@YAJPEAUDMFMODULE__@@@Z 00000001800129c0 f   DmfK:DmfCall.obj
 0001:00011a30       ?DMF_Module_SelfManagedIoSuspend@@YAJPEAUDMFMODULE__@@@Z 0000000180012a30 f   DmfK:DmfCall.obj
 0001:00011aa0       ?DMF_Module_SurpriseRemoval@@YAXPEAUDMFMODULE__@@@Z 0000000180012aa0 f   DmfK:DmfCall.obj
 0001:00011afc       ?DMF_Module_UsageNotificationEx@@YAJPEAUDMFMODULE__@@W4_WDF_SPECIAL_FILE_TYPE@@E@Z 0000000180012afc f   DmfK:DmfCall.obj
 0001:00011ba0       ?DMF_Module_WakeFromS0Triggered@@YAXPEAUDMFMODULE__@@@Z 0000000180012ba0 f   DmfK:DmfCall.obj
 0001:00011c10       ?DMF_Module_WakeFromSxTriggered@@YAXPEAUDMFMODULE__@@@Z 0000000180012c10 f   DmfK:DmfCall.obj
 0001:00011c80       ?DmfEvtDynamicModuleCleanupCallback@@YAXPEAX@Z 0000000180012c80 f   DmfK:DmfCall.obj
 0001:00011d6c       DMF_IsPoolTypePassiveLevel 0000000180012d6c f   DmfK:DmfCall.obj
 0001:00011d74       DMF_ModuleClose            0000000180012d74 f   DmfK:DmfCall.obj
 0001:00011db4       DMF_ModuleDereference      0000000180012db4 f   DmfK:DmfCall.obj
 0001:00011e14       DMF_ModuleInContextSave    0000000180012e14 f   DmfK:DmfCall.obj
 0001:00011e4c       DMF_ModuleLockIsPassive    0000000180012e4c f   DmfK:DmfCall.obj
 0001:00011e80       DMF_ModuleOpen             0000000180012e80 f   DmfK:DmfCall.obj
 0001:00011ec0       DMF_ModuleReference        0000000180012ec0 f   DmfK:DmfCall.obj
 0001:00011f50       ?BranchTrack_CheckPointProcess@@YAXPEAUDMFMODULE__@@PEAD11KP6AE01_K2@Z2P6AX0PEAEK4PEAK@Z@Z 0000000180012f50 f   DmfK:Dmf_BranchTrack.obj
 0001:00012bf0       ?DMF_BranchTrack_LiveKernelDumpInitialize@@YAXPEAUDMFMODULE__@@@Z 0000000180013bf0 f   DmfK:Dmf_BranchTrack.obj
 0001:00012dd4       DMF_BranchTrack_CheckPointCreate 0000000180013dd4 f   DmfK:Dmf_BranchTrack.obj
 0001:00012f14       DMF_BranchTrack_CheckPointExecute 0000000180013f14 f   DmfK:Dmf_BranchTrack.obj
 0001:00013060       DMF_BranchTrack_Helper_BranchStatusQuery_AtLeast 0000000180014060 f   DmfK:Dmf_BranchTrack.obj
 0001:00013070       DMF_BranchTrack_Helper_BranchStatusQuery_Count 0000000180014070 f   DmfK:Dmf_BranchTrack.obj
 0001:00013080       DMF_BranchTrack_Helper_BranchStatusQuery_MoreThan 0000000180014080 f   DmfK:Dmf_BranchTrack.obj
 0001:00013090       WdfObjectAddCustomType_DMF_BranchTrack 0000000180014090 f i DmfK:Dmf_BranchTrack.obj
 0001:00013120       ?DMF_DeviceInterfaceTarget_LiveKernelDumpInitialize@@YAXPEAUDMFMODULE__@@@Z 0000000180014120 f   DmfK:Dmf_DeviceInterfaceTarget.obj
 0001:00013180       ?DeviceInterfaceTarget_EvtIoTargetQueryRemove@@YAJPEAUWDFIOTARGET__@@@Z 0000000180014180 f   DmfK:Dmf_DeviceInterfaceTarget.obj
 0001:00013310       ?DeviceInterfaceTarget_EvtIoTargetRemoveCancel@@YAXPEAUWDFIOTARGET__@@@Z 0000000180014310 f   DmfK:Dmf_DeviceInterfaceTarget.obj
 0001:000136e0       ?DeviceInterfaceTarget_EvtIoTargetRemoveComplete@@YAXPEAUWDFIOTARGET__@@@Z 00000001800146e0 f   DmfK:Dmf_DeviceInterfaceTarget.obj
 0001:00013884       ?DeviceInterfaceTarget_ModuleCloseReasonSet@@YA?AW4ModuleCloseReason_Type@@PEAUDMFMODULE__@@W41@@Z 0000000180014884 f   DmfK:Dmf_DeviceInterfaceTarget.obj
 0001:00013a40       ?DeviceInterfaceTarget_SendCompletion@@YAXPEAUDMFMODULE__@@PEAX1_K12J@Z 0000000180014a40 f   DmfK:Dmf_DeviceInterfaceTarget.obj
 0001:00013b00       ?DeviceInterfaceTarget_Stream_BufferInput@@YAXPEAUDMFMODULE__@@PEAXPEA_K1@Z 0000000180014b00 f   DmfK:Dmf_DeviceInterfaceTarget.obj
 0001:00013c10       ?DeviceInterfaceTarget_Stream_BufferOutput@@YA?AW4ContinuousRequestTarget_BufferDisposition@@PEAUDMFMODULE__@@PEAX_K1J@Z 0000000180014c10 f   DmfK:Dmf_DeviceInterfaceTarget.obj
 0001:00013d30       ?DeviceInterfaceTarget_Stream_Cancel@@YAEPEAUDMFMODULE__@@PEAURequestTarget_DmfRequest__@@@Z 0000000180014d30 f   DmfK:Dmf_DeviceInterfaceTarget.obj
 0001:00013d70       ?DeviceInterfaceTarget_Stream_IoTargetClear@@YAXPEAUDMFMODULE__@@@Z 0000000180014d70 f   DmfK:Dmf_DeviceInterfaceTarget.obj
 0001:00013db0       ?DeviceInterfaceTarget_Stream_IoTargetSet@@YAXPEAUDMFMODULE__@@PEAUWDFIOTARGET__@@@Z 0000000180014db0 f   DmfK:Dmf_DeviceInterfaceTarget.obj
 0001:00013df0       ?DeviceInterfaceTarget_Stream_Send@@YAJPEAUDMFMODULE__@@PEAX_K12W4ContinuousRequestTarget_RequestType@@KKP6AX011212J@Z1@Z 0000000180014df0 f   DmfK:Dmf_DeviceInterfaceTarget.obj
 0001:00013e50       ?DeviceInterfaceTarget_Stream_SendEx@@YAJPEAUDMFMODULE__@@PEAX_K12W4ContinuousRequestTarget_RequestType@@KKP6AX011212J@Z1PEAPEAURequestTarget_DmfRequest__@@@Z 0000000180014e50 f   DmfK:Dmf_DeviceInterfaceTarget.obj
 0001:00013f70       ?DeviceInterfaceTarget_Stream_SendSynchronously@@YAJPEAUDMFMODULE__@@PEAX_K12W4ContinuousRequestTarget_RequestType@@KKPEA_K@Z 0000000180014f70 f   DmfK:Dmf_DeviceInterfaceTarget.obj
 0001:00013fd0       ?DeviceInterfaceTarget_SymbolicLinkNameClear@@YAXPEAUDMFMODULE__@@@Z 0000000180014fd0 f   DmfK:Dmf_DeviceInterfaceTarget.obj
 0001:00014040       ?DeviceInterfaceTarget_SymbolicLinkNameStore@@YAJPEAUDMFMODULE__@@PEAU_UNICODE_STRING@@@Z 0000000180015040 f   DmfK:Dmf_DeviceInterfaceTarget.obj
 0001:00014250       ?DeviceInterfaceTarget_Target_Cancel@@YAEPEAUDMFMODULE__@@PEAURequestTarget_DmfRequest__@@@Z 0000000180015250 f   DmfK:Dmf_DeviceInterfaceTarget.obj
 0001:00014290       ?DeviceInterfaceTarget_Target_IoTargetClear@@YAXPEAUDMFMODULE__@@@Z 0000000180015290 f   DmfK:Dmf_DeviceInterfaceTarget.obj
 0001:000142d0       ?DeviceInterfaceTarget_Target_IoTargetSet@@YAXPEAUDMFMODULE__@@PEAUWDFIOTARGET__@@@Z 00000001800152d0 f   DmfK:Dmf_DeviceInterfaceTarget.obj
 0001:00014310       ?DeviceInterfaceTarget_Target_Send@@YAJPEAUDMFMODULE__@@PEAX_K12W4ContinuousRequestTarget_RequestType@@KKP6AX011212J@Z1@Z 0000000180015310 f   DmfK:Dmf_DeviceInterfaceTarget.obj
 0001:000143d0       ?DeviceInterfaceTarget_Target_SendEx@@YAJPEAUDMFMODULE__@@PEAX_K12W4ContinuousRequestTarget_RequestType@@KKP6AX011212J@Z1PEAPEAURequestTarget_DmfRequest__@@@Z 00000001800153d0 f   DmfK:Dmf_DeviceInterfaceTarget.obj
 0001:000144f0       ?DeviceInterfaceTarget_Target_SendSynchronously@@YAJPEAUDMFMODULE__@@PEAX_K12W4ContinuousRequestTarget_RequestType@@KKPEA_K@Z 00000001800154f0 f   DmfK:Dmf_DeviceInterfaceTarget.obj
 0001:00014550       ?RtlUnicodeStringCopy@@YAJPEAU_UNICODE_STRING@@PEBU1@@Z 0000000180015550 f i DmfK:Dmf_DeviceInterfaceTarget.obj
 0001:00014650       DMF_DeviceInterfaceTarget_BufferPut 0000000180015650 f   DmfK:Dmf_DeviceInterfaceTarget.obj
 0001:000147a8       DMF_DeviceInterfaceTarget_Send 00000001800157a8 f   DmfK:Dmf_DeviceInterfaceTarget.obj
 0001:0001497c       DMF_DeviceInterfaceTarget_SendEx 000000018001597c f   DmfK:Dmf_DeviceInterfaceTarget.obj
 0001:00014b5c       DMF_DeviceInterfaceTarget_SendSynchronously 0000000180015b5c f   DmfK:Dmf_DeviceInterfaceTarget.obj
 0001:00014d20       DMF_DeviceInterfaceTarget_StreamStart 0000000180015d20 f   DmfK:Dmf_DeviceInterfaceTarget.obj
 0001:00014e78       DMF_DeviceInterfaceTarget_StreamStop 0000000180015e78 f   DmfK:Dmf_DeviceInterfaceTarget.obj
 0001:00014fbc       WPP_RECORDER_SF_S          0000000180015fbc f i DmfK:Dmf_DeviceInterfaceTarget.obj
 0001:00015108       WPP_RECORDER_SF__guid_     0000000180016108 f i DmfK:Dmf_DeviceInterfaceTarget.obj
 0001:000151f8       WPP_RECORDER_SF_qdd        00000001800161f8 f i DmfK:Dmf_DeviceInterfaceTarget.obj
 0001:00015340       WdfObjectAddCustomType_DMF_DeviceInterfaceTarget 0000000180016340 f i DmfK:Dmf_DeviceInterfaceTarget.obj
 0001:000153d0       ?String_FindInListExactCharCallback@@YAJPEAUDMFMODULE__@@PEAD1@Z 00000001800163d0 f   DmfK:Dmf_String.obj
 0001:000153f0       ?String_FindInListLeftLookForMatchCharCallback@@YAJPEAUDMFMODULE__@@PEAD1@Z 00000001800163f0 f   DmfK:Dmf_String.obj
 0001:00015428       DMF_String_FindInListChar  0000000180016428 f   DmfK:Dmf_String.obj
 0001:00015590       DMF_String_FindInListExactChar 0000000180016590 f   DmfK:Dmf_String.obj
 0001:00015614       DMF_String_FindInListLookForLeftMatchChar 0000000180016614 f   DmfK:Dmf_String.obj
 0001:00015698       WPP_RECORDER_SF_Dss        0000000180016698 f i DmfK:Dmf_String.obj
 0001:00015880       WdfObjectAddCustomType_DMF_String 0000000180016880 f i DmfK:Dmf_String.obj
 0001:00015910       ?DMF_SmbiosWmi_LiveKernelDumpInitialize@@YAXPEAUDMFMODULE__@@@Z 0000000180016910 f   DmfK:Dmf_SmbiosWmi.obj
 0001:00015970       ?SmbioWmi_TablesSet@@YAJPEAUDMFMODULE__@@@Z 0000000180016970 f   DmfK:Dmf_SmbiosWmi.obj
 0001:00015e48       ?SmbiosViaWmi_StringAssign@@YAPEADDPEAPEAEPEAE@Z 0000000180016e48 f   DmfK:Dmf_SmbiosWmi.obj
 0001:00015e84       DMF_SmbiosWmi_TableType01Get 0000000180016e84 f   DmfK:Dmf_SmbiosWmi.obj
 0001:00015fdc       WPP_RECORDER_SF_DDDDDDDDDDDDDDDD 0000000180016fdc f i DmfK:Dmf_SmbiosWmi.obj
 0001:00016310       WdfObjectAddCustomType_DMF_SmbiosWmi 0000000180017310 f i DmfK:Dmf_SmbiosWmi.obj
 0001:0001639c       WPP_RECORDER_SF_Sd         000000018001739c f i DmfK:Dmf_File.obj
 0001:00016520       ?DMF_BufferQueue_LiveKernelDumpInitialize@@YAXPEAUDMFMODULE__@@@Z 0000000180017520 f   DmfK:Dmf_BufferQueue.obj
 0001:00016580       DMF_BufferQueue_Count      0000000180017580 f   DmfK:Dmf_BufferQueue.obj
 0001:00016684       DMF_BufferQueue_Dequeue    0000000180017684 f   DmfK:Dmf_BufferQueue.obj
 0001:0001679c       DMF_BufferQueue_Enqueue    000000018001779c f   DmfK:Dmf_BufferQueue.obj
 0001:000168a8       DMF_BufferQueue_Fetch      00000001800178a8 f   DmfK:Dmf_BufferQueue.obj
 0001:000169bc       DMF_BufferQueue_Flush      00000001800179bc f   DmfK:Dmf_BufferQueue.obj
 0001:00016ad4       DMF_BufferQueue_Reuse      0000000180017ad4 f   DmfK:Dmf_BufferQueue.obj
 0001:00016c20       WdfObjectAddCustomType_DMF_BufferQueue 0000000180017c20 f i DmfK:Dmf_BufferQueue.obj
 0001:00016cb0       ?DMF_ScheduledTask_LiveKernelDumpInitialize@@YAXPEAUDMFMODULE__@@@Z 0000000180017cb0 f   DmfK:Dmf_ScheduledTask.obj
 0001:0001706c       ?ScheduledTask_TimerRestart@@YAXPEAUDMFMODULE__@@W4ScheduledTask_Result_Type@@@Z 000000018001806c f   DmfK:Dmf_ScheduledTask.obj
 0001:0001719c       DMF_ScheduledTask_ExecuteNowDeferred 000000018001819c f   DmfK:Dmf_ScheduledTask.obj
 0001:000172c0       WdfObjectAddCustomType_DMF_ScheduledTask 00000001800182c0 f i DmfK:Dmf_ScheduledTask.obj
 0001:00017350       ?DmfContainerEvtWdfRequestCompletionRoutine_FileCreate@@YAXPEAUWDFREQUEST__@@PEAUWDFIOTARGET__@@PEAU_WDF_REQUEST_COMPLETION_PARAMS@@PEAX@Z 0000000180018350 f   DmfK:DmfContainer.obj
 0001:00017380       DmfContainerEvtDeviceD0Entry 0000000180018380 f   DmfK:DmfContainer.obj
 0001:000174b0       DmfContainerEvtDeviceD0EntryPostInterruptsEnabled 00000001800184b0 f   DmfK:DmfContainer.obj
 0001:000175d0       DmfContainerEvtDeviceD0Exit 00000001800185d0 f   DmfK:DmfContainer.obj
 0001:000176f0       DmfContainerEvtDeviceD0ExitPreInterruptsDisabled 00000001800186f0 f   DmfK:DmfContainer.obj
 0001:00017810       DmfContainerEvtDeviceIoControl 0000000180018810 f   DmfK:DmfContainer.obj
 0001:000179b0       DmfContainerEvtDeviceSelfManagedIoRestart 00000001800189b0 f   DmfK:DmfContainer.obj
 0001:00017a80       DmfContainerEvtDeviceSelfManagedIoSuspend 0000000180018a80 f   DmfK:DmfContainer.obj
 0001:00017b50       DmfContainerEvtDeviceSurpriseRemoval 0000000180018b50 f   DmfK:DmfContainer.obj
 0001:00017c10       DmfContainerEvtInternalDeviceIoControl 0000000180018c10 f   DmfK:DmfContainer.obj
 0001:00017db0       DmfContainerEvtQueueIoRead 0000000180018db0 f   DmfK:DmfContainer.obj
 0001:00017f30       DmfContainerEvtQueueIoWrite 0000000180018f30 f   DmfK:DmfContainer.obj
 0001:000180b0       ?Bridge_DefaultEvtDeviceContextCleanup@@YAXPEAX@Z 00000001800190b0 f   DmfK:Dmf_Bridge.obj
 0001:00018140       ?Bridge_DefaultEvtDeviceD0Entry@@YAJPEAUWDFDEVICE__@@W4_WDF_POWER_DEVICE_STATE@@@Z 0000000180019140 f   DmfK:Dmf_Bridge.obj
 0001:000181e0       ?Bridge_DefaultEvtDeviceD0EntryPostInterruptsEnabled@@YAJPEAUWDFDEVICE__@@W4_WDF_POWER_DEVICE_STATE@@@Z 00000001800191e0 f   DmfK:Dmf_Bridge.obj
 0001:00018280       ?Bridge_DefaultEvtDeviceD0Exit@@YAJPEAUWDFDEVICE__@@W4_WDF_POWER_DEVICE_STATE@@@Z 0000000180019280 f   DmfK:Dmf_Bridge.obj
 0001:00018320       ?Bridge_DefaultEvtDeviceD0ExitPreInterruptsDisabled@@YAJPEAUWDFDEVICE__@@W4_WDF_POWER_DEVICE_STATE@@@Z 0000000180019320 f   DmfK:Dmf_Bridge.obj
 0001:000183c0       ?Bridge_DefaultEvtDeviceSelfManagedIoRestart@@YAJPEAUWDFDEVICE__@@@Z 00000001800193c0 f   DmfK:Dmf_Bridge.obj
 0001:00018460       ?Bridge_DefaultEvtDeviceSelfManagedIoSuspend@@YAJPEAUWDFDEVICE__@@@Z 0000000180019460 f   DmfK:Dmf_Bridge.obj
 0001:00018500       ?Bridge_DefaultEvtDeviceSurpriseRemoval@@YAXPEAUWDFDEVICE__@@@Z 0000000180019500 f   DmfK:Dmf_Bridge.obj
 0001:00018590       ?DMF_Bridge_LiveKernelDumpInitialize@@YAXPEAUDMFMODULE__@@@Z 0000000180019590 f   DmfK:Dmf_Bridge.obj
 0001:00019250       WdfObjectAddCustomType_DMF_Bridge 000000018001a250 f i DmfK:Dmf_Bridge.obj
 0001:000192e0       ?DMF_Generic_AuxiliaryLock_Dispatch@@YAXPEAUDMFMODULE__@@K@Z 000000018001a2e0 f   DmfK:DmfGeneric.obj
 0001:00019360       ?DMF_Generic_AuxiliaryUnlock_Dispatch@@YAXPEAUDMFMODULE__@@K@Z 000000018001a360 f   DmfK:DmfGeneric.obj
 0001:000193e0       ?DMF_Generic_Destroy@@YAXPEAUDMFMODULE__@@@Z 000000018001a3e0 f   DmfK:DmfGeneric.obj
 0001:000194d0       ?DMF_Generic_Lock_Dispatch@@YAXPEAUDMFMODULE__@@@Z 000000018001a4d0 f   DmfK:DmfGeneric.obj
 0001:000194e0       ?DMF_Generic_ModuleD0Entry@@YAJPEAUDMFMODULE__@@W4_WDF_POWER_DEVICE_STATE@@@Z 000000018001a4e0 f   DmfK:DmfGeneric.obj
 0001:00019720       ?DMF_Generic_ModuleD0EntryPostInterruptsEnabled@@YAJPEAUDMFMODULE__@@W4_WDF_POWER_DEVICE_STATE@@@Z 000000018001a720 f   DmfK:DmfGeneric.obj
 0001:00019820       ?DMF_Generic_ModuleD0Exit@@YAJPEAUDMFMODULE__@@W4_WDF_POWER_DEVICE_STATE@@@Z 000000018001a820 f   DmfK:DmfGeneric.obj
 0001:000199d0       ?DMF_Generic_ModuleD0ExitPreInterruptsDisabled@@YAJPEAUDMFMODULE__@@W4_WDF_POWER_DEVICE_STATE@@@Z 000000018001a9d0 f   DmfK:DmfGeneric.obj
 0001:00019ad0       ?DMF_Generic_ModuleDeviceIoControl@@YAEPEAUDMFMODULE__@@PEAUWDFQUEUE__@@PEAUWDFREQUEST__@@_K3K@Z 000000018001aad0 f   DmfK:DmfGeneric.obj
 0001:00019bf0       ?DMF_Generic_ModuleInternalDeviceIoControl@@YAEPEAUDMFMODULE__@@PEAUWDFQUEUE__@@PEAUWDFREQUEST__@@_K3K@Z 000000018001abf0 f   DmfK:DmfGeneric.obj
 0001:00019ce0       ?DMF_Generic_ModuleQueueIoRead@@YAEPEAUDMFMODULE__@@PEAUWDFQUEUE__@@PEAUWDFREQUEST__@@_K@Z 000000018001ace0 f   DmfK:DmfGeneric.obj
 0001:00019dd0       ?DMF_Generic_ModuleQueueIoWrite@@YAEPEAUDMFMODULE__@@PEAUWDFQUEUE__@@PEAUWDFREQUEST__@@_K@Z 000000018001add0 f   DmfK:DmfGeneric.obj
 0001:00019ec0       ?DMF_Generic_ModuleSelfManagedIoRestart@@YAJPEAUDMFMODULE__@@@Z 000000018001aec0 f   DmfK:DmfGeneric.obj
 0001:00019fb0       ?DMF_Generic_ModuleSelfManagedIoSuspend@@YAJPEAUDMFMODULE__@@@Z 000000018001afb0 f   DmfK:DmfGeneric.obj
 0001:0001a0a0       ?DMF_Generic_ModuleSurpriseRemoval@@YAXPEAUDMFMODULE__@@@Z 000000018001b0a0 f   DmfK:DmfGeneric.obj
 0001:0001a190       ?DMF_Generic_Unlock_Dispatch@@YAXPEAUDMFMODULE__@@@Z 000000018001b190 f   DmfK:DmfGeneric.obj
 0001:0001a198       WPP_RECORDER_SF_qqs        000000018001b198 f i DmfK:DmfGeneric.obj
 0001:0001a33c       WPP_RECORDER_SF_qqsd       000000018001b33c f i DmfK:DmfGeneric.obj
 0001:0001a510       ?DMF_IoctlHandler_LiveKernelDumpInitialize@@YAXPEAUDMFMODULE__@@@Z 000000018001b510 f   DmfK:Dmf_IoctlHandler.obj
 0001:0001ab04       ?IoctlHandler_AssociatedFileObjectsLookUp@@YAEPEAUDMFMODULE__@@PEAUWDFFILEOBJECT__@@E@Z 000000018001bb04 f   DmfK:Dmf_IoctlHandler.obj
 0001:0001aca0       ?IoctlHandler_RequestForward@@YAJPEAUDMFMODULE__@@PEAUWDFREQUEST__@@@Z 000000018001bca0 f   DmfK:Dmf_IoctlHandler.obj
 0001:0001ade4       WPP_RECORDER_SF_ddd        000000018001bde4 f i DmfK:Dmf_IoctlHandler.obj
 0001:0001af30       WdfObjectAddCustomType_DMF_IoctlHandler 000000018001bf30 f i DmfK:Dmf_IoctlHandler.obj
 0001:0001afbc       LkmdTelInsertTriageDataBlock 000000018001bfbc f   DmfK:lkmdtel.obj
 0001:0001b128       RtlStringCbPrintfW         000000018001c128 f i DmfK:lkmdtel.obj
 0001:0001b1f0       DMF_Utility_DelayMilliseconds 000000018001c1f0 f   DmfK:DmfUtility.obj
 0001:0001b2a0       DMF_Utility_IsEqualGUID    000000018001c2a0 f   DmfK:DmfUtility.obj
 0001:0001b2c0       ?DMF_RingBuffer_LiveKernelDumpInitialize@@YAXPEAUDMFMODULE__@@@Z 000000018001c2c0 f   DmfK:Dmf_RingBuffer.obj
 0001:0001b320       ?RingBuffer_ItemProcessCallbackRead@@YAXPEAXPEAEK@Z 000000018001c320 f   DmfK:Dmf_RingBuffer.obj
 0001:0001b330       ?RingBuffer_ItemProcessCallbackWrite@@YAXPEAXPEAEK@Z 000000018001c330 f   DmfK:Dmf_RingBuffer.obj
 0001:0001b5f8       DMF_RingBuffer_Enumerate   000000018001c5f8 f   DmfK:Dmf_RingBuffer.obj
 0001:0001b78c       DMF_RingBuffer_Read        000000018001c78c f   DmfK:Dmf_RingBuffer.obj
 0001:0001b8dc       DMF_RingBuffer_ReadAll     000000018001c8dc f   DmfK:Dmf_RingBuffer.obj
 0001:0001ba48       DMF_RingBuffer_Reorder     000000018001ca48 f   DmfK:Dmf_RingBuffer.obj
 0001:0001bc2c       DMF_RingBuffer_TotalSizeGet 000000018001cc2c f   DmfK:Dmf_RingBuffer.obj
 0001:0001bca4       DMF_RingBuffer_Write       000000018001cca4 f   DmfK:Dmf_RingBuffer.obj
 0001:0001be00       WdfObjectAddCustomType_DMF_RingBuffer 000000018001ce00 f i DmfK:Dmf_RingBuffer.obj
 0001:0001be90       ?CrashDump_BugCheckSecondaryDumpDataCallbackAdditional@@YAXW4_KBUGCHECK_CALLBACK_REASON@@PEAU_KBUGCHECK_REASON_CALLBACK_RECORD@@PEAXK@Z 000000018001ce90 f   DmfK:Dmf_CrashDump.obj
 0001:0001bf40       ?CrashDump_BugCheckSecondaryDumpDataCallbackRingBuffer@@YAXW4_KBUGCHECK_CALLBACK_REASON@@PEAU_KBUGCHECK_REASON_CALLBACK_RECORD@@PEAXK@Z 000000018001cf40 f   DmfK:Dmf_CrashDump.obj
 0001:0001c040       ?CrashDump_BugCheckTriageDumpDataCallback@@YAXW4_KBUGCHECK_CALLBACK_REASON@@PEAU_KBUGCHECK_REASON_CALLBACK_RECORD@@PEAXK@Z 000000018001d040 f   DmfK:Dmf_CrashDump.obj
 0001:0001c0d4       ?CrashDump_DataSourceCaptureInternal@@YAJPEAUDMFMODULE__@@KPEAEKPEAK@Z 000000018001d0d4 f   DmfK:Dmf_CrashDump.obj
 0001:0001c13c       ?CrashDump_DataSourceReadInternal@@YAJPEAUDMFMODULE__@@KPEAEK@Z 000000018001d13c f   DmfK:Dmf_CrashDump.obj
 0001:0001c1a0       ?CrashDump_DataSourceWriteInternal@@YAJPEAUDMFMODULE__@@KPEAEK@Z 000000018001d1a0 f   DmfK:Dmf_CrashDump.obj
 0001:0001c210       ?CrashDump_RingBufferElementsFirstBufferGet@@YAEPEAUDMFMODULE__@@PEAEKPEAX@Z 000000018001d210 f   DmfK:Dmf_CrashDump.obj
 0001:0001c220       ?CrashDump_RingBufferElementsXor@@YAEPEAUDMFMODULE__@@PEAEKPEAX@Z 000000018001d220 f   DmfK:Dmf_CrashDump.obj
 0001:0001c260       ?DMF_CrashDump_LiveKernelDumpInitialize@@YAXPEAUDMFMODULE__@@@Z 000000018001d260 f   DmfK:Dmf_CrashDump.obj
 0001:0001c2c0       ?DMF_CrashDump_SurpriseRemoval@@YAXPEAUDMFMODULE__@@@Z 000000018001d2c0 f   DmfK:Dmf_CrashDump.obj
 0001:0001c380       DMF_CrashDump_TriageDumpDataAdd 000000018001d380 f   DmfK:Dmf_CrashDump.obj
 0001:0001c500       WdfObjectAddCustomType_DMF_CrashDump 000000018001d500 f i DmfK:Dmf_CrashDump.obj
 0001:0001c590       ?DMF_Internal_Close@@YAXPEAUDMFMODULE__@@@Z 000000018001d590 f   DmfK:DmfInternal.obj
 0001:0001c6e0       ?DMF_Internal_Destroy@@YAXPEAUDMFMODULE__@@@Z 000000018001d6e0 f   DmfK:DmfInternal.obj
 0001:0001c7e0       ?DMF_Internal_ModuleD0Entry@@YAJPEAUDMFMODULE__@@W4_WDF_POWER_DEVICE_STATE@@@Z 000000018001d7e0 f   DmfK:DmfInternal.obj
 0001:0001c8f0       ?DMF_Internal_ModuleD0EntryPostInterruptsEnabled@@YAJPEAUDMFMODULE__@@W4_WDF_POWER_DEVICE_STATE@@@Z 000000018001d8f0 f   DmfK:DmfInternal.obj
 0001:0001ca00       ?DMF_Internal_ModuleD0Exit@@YAJPEAUDMFMODULE__@@W4_WDF_POWER_DEVICE_STATE@@@Z 000000018001da00 f   DmfK:DmfInternal.obj
 0001:0001cb10       ?DMF_Internal_ModuleD0ExitPreInterruptsDisabled@@YAJPEAUDMFMODULE__@@W4_WDF_POWER_DEVICE_STATE@@@Z 000000018001db10 f   DmfK:DmfInternal.obj
 0001:0001cc20       ?DMF_Internal_ModuleDeviceIoControl@@YAEPEAUDMFMODULE__@@PEAUWDFQUEUE__@@PEAUWDFREQUEST__@@_K3K@Z 000000018001dc20 f   DmfK:DmfInternal.obj
 0001:0001cd70       ?DMF_Internal_ModuleInternalDeviceIoControl@@YAEPEAUDMFMODULE__@@PEAUWDFQUEUE__@@PEAUWDFREQUEST__@@_K3K@Z 000000018001dd70 f   DmfK:DmfInternal.obj
 0001:0001cec0       ?DMF_Internal_ModuleQueueIoRead@@YAEPEAUDMFMODULE__@@PEAUWDFQUEUE__@@PEAUWDFREQUEST__@@_K@Z 000000018001dec0 f   DmfK:DmfInternal.obj
 0001:0001cff0       ?DMF_Internal_ModuleQueueIoWrite@@YAEPEAUDMFMODULE__@@PEAUWDFQUEUE__@@PEAUWDFREQUEST__@@_K@Z 000000018001dff0 f   DmfK:DmfInternal.obj
 0001:0001d120       ?DMF_Internal_ModuleSelfManagedIoRestart@@YAJPEAUDMFMODULE__@@@Z 000000018001e120 f   DmfK:DmfInternal.obj
 0001:0001d230       ?DMF_Internal_ModuleSelfManagedIoSuspend@@YAJPEAUDMFMODULE__@@@Z 000000018001e230 f   DmfK:DmfInternal.obj
 0001:0001d340       ?DMF_Internal_ModuleSurpriseRemoval@@YAXPEAUDMFMODULE__@@@Z 000000018001e340 f   DmfK:DmfInternal.obj
 0001:0001d440       ?DMF_Internal_Open@@YAJPEAUDMFMODULE__@@@Z 000000018001e440 f   DmfK:DmfInternal.obj
 0001:0001d5b8       ?DMF_ModuleIsClosed@@YAEPEAUDMFMODULE__@@@Z 000000018001e5b8 f   DmfK:DmfInternal.obj
 0001:0001d628       WPP_RECORDER_SF_qsq        000000018001e628 f i DmfK:DmfInternal.obj
 0001:0001d7cc       ?DMF_ModuleInterfaceDestroy@@YAXPEAU_DMF_INTERFACE_OBJECT@@@Z 000000018001e7cc f   DmfK:DmfInterfaceInternal.obj
 0001:0001d86c       ?DMF_ModuleInterfaceFindAndRemove@@YAEPEAUDMFMODULE__@@0PEAPEAU_DMF_INTERFACE_OBJECT@@@Z 000000018001e86c f   DmfK:DmfInterfaceInternal.obj
 0001:0001da24       ?DMF_ModuleInterfaceWaitToClose@@YAXPEAU_DMF_INTERFACE_OBJECT@@@Z 000000018001ea24 f   DmfK:DmfInterfaceInternal.obj
 0001:0001db14       ?DMF_ModuleInterfacesUnbind@@YAXPEAUDMFMODULE__@@@Z 000000018001eb14 f   DmfK:DmfInterfaceInternal.obj
 0001:0001dc00       DMF_ModuleInterfaceUnbind  000000018001ec00 f   DmfK:DmfInterfaceInternal.obj
 0001:0001dd10       ?DMF_HashTable_LiveKernelDumpInitialize@@YAXPEAUDMFMODULE__@@@Z 000000018001ed10 f   DmfK:Dmf_HashTable.obj
 0001:0001df94       DMF_HashTable_Enumerate    000000018001ef94 f   DmfK:Dmf_HashTable.obj
 0001:0001e19c       DMF_HashTable_Find         000000018001f19c f   DmfK:Dmf_HashTable.obj
 0001:0001e324       WPP_RECORDER_SF_DDDD       000000018001f324 f i DmfK:Dmf_HashTable.obj
 0001:0001e490       WdfObjectAddCustomType_DMF_HashTable 000000018001f490 f i DmfK:Dmf_HashTable.obj
 0001:0001e520       ?DMF_RequestTarget_LiveKernelDumpInitialize@@YAXPEAUDMFMODULE__@@@Z 000000018001f520 f   DmfK:Dmf_RequestTarget.obj
 0001:0001e580       ?RequestTarget_CompletionRoutine@@YAXPEAUWDFREQUEST__@@PEAUWDFIOTARGET__@@PEAU_WDF_REQUEST_COMPLETION_PARAMS@@PEAX@Z 000000018001f580 f   DmfK:Dmf_RequestTarget.obj
 0001:0001e640       ?RequestTarget_CompletionRoutinePassive@@YAXPEAUWDFREQUEST__@@PEAUWDFIOTARGET__@@PEAU_WDF_REQUEST_COMPLETION_PARAMS@@PEAX@Z 000000018001f640 f   DmfK:Dmf_RequestTarget.obj
 0001:0001ed10       ?RequestTarget_ProcessAsynchronousRequestSingle@@YAXPEAUDMFMODULE__@@PEAUWDFREQUEST__@@PEAU_WDF_REQUEST_COMPLETION_PARAMS@@PEAURequestTarget_SingleAsynchronousRequestContext@@@Z 000000018001fd10 f   DmfK:Dmf_RequestTarget.obj
 0001:0001f170       ?RequestTarget_QueuedWorkitemCallbackSingle@@YA?AW4ScheduledTask_Result_Type@@PEAUDMFMODULE__@@PEAX1@Z 0000000180020170 f   DmfK:Dmf_RequestTarget.obj
 0001:0001f898       DMF_RequestTarget_Cancel   0000000180020898 f   DmfK:Dmf_RequestTarget.obj
 0001:0001fb10       DMF_RequestTarget_IoTargetClear 0000000180020b10 f   DmfK:Dmf_RequestTarget.obj
 0001:0001fc08       DMF_RequestTarget_IoTargetSet 0000000180020c08 f   DmfK:Dmf_RequestTarget.obj
 0001:0001fd0c       DMF_RequestTarget_SendEx   0000000180020d0c f   DmfK:Dmf_RequestTarget.obj
 0001:0001fe84       DMF_RequestTarget_SendSynchronously 0000000180020e84 f   DmfK:Dmf_RequestTarget.obj
 0001:0001ffe0       WdfObjectAddCustomType_DMF_RequestTarget 0000000180020fe0 f i DmfK:Dmf_RequestTarget.obj
 0001:000201f0       ?ContinuousRequestTarget_CompletionRoutine@@YAXPEAUWDFREQUEST__@@PEAUWDFIOTARGET__@@PEAU_WDF_REQUEST_COMPLETION_PARAMS@@PEAX@Z 00000001800211f0 f   DmfK:Dmf_ContinuousRequestTarget.obj
 0001:000202f0       ?ContinuousRequestTarget_CompletionRoutinePassive@@YAXPEAUWDFREQUEST__@@PEAUWDFIOTARGET__@@PEAU_WDF_REQUEST_COMPLETION_PARAMS@@PEAX@Z 00000001800212f0 f   DmfK:Dmf_ContinuousRequestTarget.obj
 0001:00020f10       ?ContinuousRequestTarget_ProcessAsynchronousRequestSingle@@YAXPEAUDMFMODULE__@@PEAUWDFREQUEST__@@PEAU_WDF_REQUEST_COMPLETION_PARAMS@@PEAUContinuousRequestTarget_SingleAsynchronousRequestContext@@@Z 0000000180021f10 f   DmfK:Dmf_ContinuousRequestTarget.obj
 0001:000216c0       ?ContinuousRequestTarget_QueuedWorkitemCallbackSingle@@YA?AW4ScheduledTask_Result_Type@@PEAUDMFMODULE__@@PEAX1@Z 00000001800226c0 f   DmfK:Dmf_ContinuousRequestTarget.obj
 0001:000216f0       ?ContinuousRequestTarget_QueuedWorkitemCallbackStream@@YA?AW4ScheduledTask_Result_Type@@PEAUDMFMODULE__@@PEAX1@Z 00000001800226f0 f   DmfK:Dmf_ContinuousRequestTarget.obj
 0001:00021e78       ?ContinuousRequestTarget_RequestsCancel@@YAXPEAUDMFMODULE__@@@Z 0000000180022e78 f   DmfK:Dmf_ContinuousRequestTarget.obj
 0001:000220c8       ?ContinuousRequestTarget_StopAndWait@@YAXPEAUDMFMODULE__@@@Z 00000001800230c8 f   DmfK:Dmf_ContinuousRequestTarget.obj
 0001:00022250       ?ContinuousRequestTarget_StreamCompletionRoutine@@YAXPEAUWDFREQUEST__@@PEAUWDFIOTARGET__@@PEAU_WDF_REQUEST_COMPLETION_PARAMS@@PEAX@Z 0000000180023250 f   DmfK:Dmf_ContinuousRequestTarget.obj
 0001:00022320       ?ContinuousRequestTarget_StreamCompletionRoutinePassive@@YAXPEAUWDFREQUEST__@@PEAUWDFIOTARGET__@@PEAU_WDF_REQUEST_COMPLETION_PARAMS@@PEAX@Z 0000000180023320 f   DmfK:Dmf_ContinuousRequestTarget.obj
 0001:00022740       ?DMF_ContinuousRequestTarget_LiveKernelDumpInitialize@@YAXPEAUDMFMODULE__@@@Z 0000000180023740 f   DmfK:Dmf_ContinuousRequestTarget.obj
 0001:00022a10       DMF_ContinuousRequestTarget_BufferPut 0000000180023a10 f   DmfK:Dmf_ContinuousRequestTarget.obj
 0001:00022b34       DMF_ContinuousRequestTarget_Cancel 0000000180023b34 f   DmfK:Dmf_ContinuousRequestTarget.obj
 0001:00022c58       DMF_ContinuousRequestTarget_IoTargetClear 0000000180023c58 f   DmfK:Dmf_ContinuousRequestTarget.obj
 0001:00022d68       DMF_ContinuousRequestTarget_IoTargetSet 0000000180023d68 f   DmfK:Dmf_ContinuousRequestTarget.obj
 0001:00022e88       DMF_ContinuousRequestTarget_SendEx 0000000180023e88 f   DmfK:Dmf_ContinuousRequestTarget.obj
 0001:00023024       DMF_ContinuousRequestTarget_SendSynchronously 0000000180024024 f   DmfK:Dmf_ContinuousRequestTarget.obj
 0001:000231a0       DMF_ContinuousRequestTarget_Start 00000001800241a0 f   DmfK:Dmf_ContinuousRequestTarget.obj
 0001:000233bc       DMF_ContinuousRequestTarget_StopAndWait 00000001800243bc f   DmfK:Dmf_ContinuousRequestTarget.obj
 0001:000234e0       WdfObjectAddCustomType_DMF_ContinuousRequestTarget 00000001800244e0 f i DmfK:Dmf_ContinuousRequestTarget.obj
 0001:00023570       ?DMF_Rundown_LiveKernelDumpInitialize@@YAXPEAUDMFMODULE__@@@Z 0000000180024570 f   DmfK:Dmf_Rundown.obj
 0001:000235d0       ?Rundown_Close@@YAXPEAUDMFMODULE__@@@Z 00000001800245d0 f   DmfK:Dmf_Rundown.obj
 0001:00023770       ?Rundown_ReferenceAdd@@YAJPEAUDMFMODULE__@@@Z 0000000180024770 f   DmfK:Dmf_Rundown.obj
 0001:0002385c       ?Rundown_ReferenceDelete@@YAJPEAUDMFMODULE__@@@Z 000000018002485c f   DmfK:Dmf_Rundown.obj
 0001:00023944       DMF_Rundown_Dereference    0000000180024944 f   DmfK:Dmf_Rundown.obj
 0001:00023a5c       DMF_Rundown_EndAndWait     0000000180024a5c f   DmfK:Dmf_Rundown.obj
 0001:00023d10       DMF_Rundown_Reference      0000000180024d10 f   DmfK:Dmf_Rundown.obj
 0001:00023e4c       DMF_Rundown_Start          0000000180024e4c f   DmfK:Dmf_Rundown.obj
 0001:00023fc0       WdfObjectAddCustomType_DMF_Rundown 0000000180024fc0 f i DmfK:Dmf_Rundown.obj
 0001:0002404c       WerLiveKernelCloseHandle   000000018002504c f   DmfK:ext-ms-win-ntos-werkernel-l1-1-1.dll
 0001:00024058       WerLiveKernelOpenDumpFile  0000000180025058 f   DmfK:ext-ms-win-ntos-werkernel-l1-1-1.dll
 0001:00024064       WerLiveKernelCancelReport  0000000180025064 f   DmfK:ext-ms-win-ntos-werkernel-l1-1-1.dll
 0001:00024070       WerLiveKernelCreateReport  0000000180025070 f   DmfK:ext-ms-win-ntos-werkernel-l1-1-1.dll
 0001:0002407c       WerLiveKernelSubmitReport  000000018002507c f   DmfK:ext-ms-win-ntos-werkernel-l1-1-1.dll
 0001:00024090       ext_ms_win_ntos_werkernel_l1_1_1_WerLiveKernelCancelReport 0000000180025090 f   DmfK:stubgen_data.obj
 0001:00024090       ext_ms_win_ntos_werkernel_l1_1_1_WerLiveKernelCloseHandle 0000000180025090 f   DmfK:stubgen_data.obj
 0001:00024090       ext_ms_win_ntos_werkernel_l1_1_1_WerLiveKernelCreateReport 0000000180025090 f   DmfK:stubgen_data.obj
 0001:00024090       ext_ms_win_ntos_werkernel_l1_1_1_WerLiveKernelOpenDumpFile 0000000180025090 f   DmfK:stubgen_data.obj
 0001:00024090       ext_ms_win_ntos_werkernel_l1_1_1_WerLiveKernelSubmitReport 0000000180025090 f   DmfK:stubgen_data.obj
 0001:000240a0       WppAutoLogTrace            00000001800250a0 f   wpprecorder:WppRecorder.sys
 0001:000240b0       WppAutoLogStart            00000001800250b0 f   wpprecorder:WppRecorder.sys
 0001:000240c0       WppAutoLogStop             00000001800250c0 f   wpprecorder:WppRecorder.sys
 0001:000240d0       imp_WppRecorderReplay      00000001800250d0 f   wpprecorder:WppRecorder.sys
 0001:000240d6       imp_WppRecorderLogCreate   00000001800250d6 f   wpprecorder:WppRecorder.sys
 0001:000240dc       imp_WppRecorderLogDelete   00000001800250dc f   wpprecorder:WppRecorder.sys
 0001:000240e2       imp_WppRecorderLogGetDefault 00000001800250e2 f   wpprecorder:WppRecorder.sys
 0001:000240e8       imp_WppRecorderIsDefaultLogAvailable 00000001800250e8 f   wpprecorder:WppRecorder.sys
 0001:000240f0       __GSHandlerCheck           00000001800250f0 f   ntoskrnl:gshandler.obj
 0001:00024110       __GSHandlerCheckCommon     0000000180025110 f   ntoskrnl:gshandler.obj
 0001:00024170       strncpy_s                  0000000180025170 f   ntoskrnl:ntoskrnl.exe
 0001:00024176       strcmp                     0000000180025176 f   ntoskrnl:ntoskrnl.exe
 0001:0002417c       _vsnprintf                 000000018002517c f   ntoskrnl:ntoskrnl.exe
 0001:00024182       strncmp                    0000000180025182 f   ntoskrnl:ntoskrnl.exe
 0001:00024188       KeCapturePersistentThreadState 0000000180025188 f   ntoskrnl:ntoskrnl.exe
 0001:0002418e       _vsnwprintf                000000018002518e f   ntoskrnl:ntoskrnl.exe
 0001:00024194       sprintf_s                  0000000180025194 f   ntoskrnl:ntoskrnl.exe
 0001:0002419a       WdfVersionBind             000000018002519a f   WdfLdr:WDFLDR.SYS
 0001:000241a0       WdfLdrQueryInterface       00000001800251a0 f   WdfLdr:WDFLDR.SYS
 0001:000241a6       WdfVersionUnbind           00000001800251a6 f   WdfLdr:WDFLDR.SYS
 0001:000241b0       WdfVersionBindClass        00000001800251b0 f   WdfLdr:WDFLDR.SYS
 0001:000241c0       WdfVersionUnbindClass      00000001800251c0 f   WdfLdr:WDFLDR.SYS
 0001:000241e0       __security_check_cookie    00000001800251e0 f   BufferOverflowFastFailK:amdsecgs.obj
 0001:00024210       _guard_dispatch_icall_nop  0000000180025210 f   BufferOverflowFastFailK:guard_dispatch.obj
 0001:00024230       _guard_xfg_dispatch_icall_nop 0000000180025230 f   BufferOverflowFastFailK:guard_xfg_dispatch.obj
 0001:00024250       _guard_dispatch_icall      0000000180025250 f   BufferOverflowFastFailK:dispatchcfg.obj
 0001:00024250       _guard_dispatch_icall_$fo_default$ 0000000180025250     BufferOverflowFastFailK:dispatchcfg.obj
 0001:00024280       memset                     0000000180025280 f   ntoskrnl:memset.obj
 0001:00024280       memset_$fo_default$        0000000180025280     ntoskrnl:memset.obj
 0001:000243c0       __memset_repmovs           00000001800253c0 f   ntoskrnl:memset.obj
 0001:00024440       __memset_query             0000000180025440 f   ntoskrnl:memset.obj
 0001:00024480       memcpy                     0000000180025480 f   ntoskrnl:memcpy.obj
 0001:00024480       memmove                    0000000180025480 f   ntoskrnl:memcpy.obj
 0001:00024740       ??_C@_0EJ@IPCLCLNF@REPOSITORYDIR?2SurfaceLibrary?2Ke@FNODOBFM@ 0000000180025740     DmfK:Dmf_BufferPool.obj
 0001:00024790       ??_C@_0CE@IONBOFEE@Invalid?5Module?5Handle?5Passed?5?$CIL@FNODOBFM@ 0000000180025790     DmfK:Dmf_BufferPool.obj
 0001:000247c0       ??_C@_0CG@HBENCEPF@Invalid?5Module?5Handle?5Passed?5?$CIU@FNODOBFM@ 00000001800257c0     DmfK:Dmf_BufferPool.obj
 0001:000247f0       ??_C@_0CC@HAKALEAP@DMF_BufferPool?5signature?5mismat@FNODOBFM@ 00000001800257f0     DmfK:Dmf_BufferPool.obj
 0001:00024820       ??_C@_0CG@KGJELHIL@DMF_BufferPool?5data?5sentinel?5mi@FNODOBFM@ 0000000180025820     DmfK:Dmf_BufferPool.obj
 0001:00024850       ??_C@_0CJ@OMFNPCO@DMF_BufferPool?5context?5sentinel@FNODOBFM@ 0000000180025850     DmfK:Dmf_BufferPool.obj
 0001:00024880       ??_C@_00CNPNBAHC@@FNODOBFM@ 0000000180025880     DmfK:Dmf_SamCommunicationViaSsh.obj
 0001:00024890       ??_C@_0FF@HLOJMPAF@REPOSITORYDIR?2SurfaceLibrary?2Ke@FNODOBFM@ 0000000180025890     DmfK:Dmf_SamCommunicationViaSsh.obj
 0001:000248f0       ??_C@_08FNDBFMB@at?5least@FNODOBFM@ 00000001800258f0     DmfK:Dmf_SamCommunicationViaSsh.obj
 0001:00024900       ??_C@_0EI@FJBPHPGP@SamCommunicationViaSsh_OnDevice@FNODOBFM@ 0000000180025900     DmfK:Dmf_SamCommunicationViaSsh.obj
 0001:00024950       ??_C@_0FM@HDECLPKF@SamCommunicationViaSsh_OnDevice@FNODOBFM@ 0000000180025950     DmfK:Dmf_SamCommunicationViaSsh.obj
 0001:000249b0       ??_C@_04HIBGFPH@NULL@FNODOBFM@ 00000001800259b0     DmfK:DmfHelpers.obj
 0001:000249c0       ??_C@_1CA@LMCEOOKO@?$AAE?$AAx?$AAA?$AAl?$AAl?$AAo?$AAc?$AAa?$AAt?$AAe?$AAP?$AAo?$AAo?$AAl?$AA2@FNODOBFM@ 00000001800259c0     DmfK:DmfHelpers.obj
 0001:000249e0       ??_C@_1CM@DMLIEPAK@?$AAE?$AAx?$AAA?$AAl?$AAl?$AAo?$AAc?$AAa?$AAt?$AAe?$AAP?$AAo?$AAo?$AAl?$AAW@FNODOBFM@ 00000001800259e0     DmfK:DmfHelpers.obj
 0001:00024a10       ??_C@_0FE@CFNMELEB@REPOSITORYDIR?2SurfaceLibrary?2Ke@FNODOBFM@ 0000000180025a10     DmfK:Dmf_SamNotificationViaSsh.obj
 0001:00024a70       ??_C@_05DAFACFLE@never@FNODOBFM@ 0000000180025a70     DmfK:Dmf_SamNotificationViaSsh.obj
 0001:00024a80       ??_C@_0DG@HOMIOAHF@SamNotificationViaSsh_Unregiste@FNODOBFM@ 0000000180025a80     DmfK:Dmf_SamNotificationViaSsh.obj
 0001:00024ac0       ??_C@_0EA@PAKKEFEB@SamNotificationViaSsh_Unregiste@FNODOBFM@ 0000000180025ac0     DmfK:Dmf_SamNotificationViaSsh.obj
 0001:00024b00       ??_C@_0DE@OHLODENE@SamNotificationViaSsh_RegisterC@FNODOBFM@ 0000000180025b00     DmfK:Dmf_SamNotificationViaSsh.obj
 0001:00024b40       ??_C@_0DO@OPLEJPGD@SamNotificationViaSsh_RegisterC@FNODOBFM@ 0000000180025b40     DmfK:Dmf_SamNotificationViaSsh.obj
 0001:00024b80       ??_C@_0GE@GNHMAFBP@SamNotificationViaSsh_RegisterC@FNODOBFM@ 0000000180025b80     DmfK:Dmf_SamNotificationViaSsh.obj
 0001:00024bf0       ??_C@_0DH@DMKADBF@SamNotificationViaSsh_Streaming@FNODOBFM@ 0000000180025bf0     DmfK:Dmf_SamNotificationViaSsh.obj
 0001:00024c30       ??_C@_0EI@DCEJBBCE@SamNotificationViaSsh_Streaming@FNODOBFM@ 0000000180025c30     DmfK:Dmf_SamNotificationViaSsh.obj
 0001:00024c80       ??_C@_09MLEKNIHI@more?5than@FNODOBFM@ 0000000180025c80     DmfK:Dmf_SamNotificationViaSsh.obj
 0001:00024c90       ??_C@_0GA@HFAFKBD@SamNotificationViaSsh_Streaming@FNODOBFM@ 0000000180025c90     DmfK:Dmf_SamNotificationViaSsh.obj
 0001:00024cf0       ??_C@_0GI@GKOPJLLO@SamNotificationViaSsh_Streaming@FNODOBFM@ 0000000180025cf0     DmfK:Dmf_SamNotificationViaSsh.obj
 0001:00024d60       ??_C@_0DP@BFDBIJMK@SamNotificationViaSsh_RegisterF@FNODOBFM@ 0000000180025d60     DmfK:Dmf_SamNotificationViaSsh.obj
 0001:00024da0       ??_C@_0EM@DCBFGFII@SamNotificationViaSsh_RegisterF@FNODOBFM@ 0000000180025da0     DmfK:Dmf_SamNotificationViaSsh.obj
 0001:00024df0       ??_C@_0FG@CHGJHLKI@SamNotificationViaSsh_RegisterF@FNODOBFM@ 0000000180025df0     DmfK:Dmf_SamNotificationViaSsh.obj
 0001:00024e50       ??_C@_0HE@HNBHINLH@SamNotificationViaSsh_RegisterF@FNODOBFM@ 0000000180025e50     DmfK:Dmf_SamNotificationViaSsh.obj
 0001:00024ed0       ??_C@_0HM@ILLDINLJ@SamNotificationViaSsh_RegisterF@FNODOBFM@ 0000000180025ed0     DmfK:Dmf_SamNotificationViaSsh.obj
 0001:00024f50       ??_C@_0EJ@MFPBBJCC@SamNotificationViaSsh_Streaming@FNODOBFM@ 0000000180025f50     DmfK:Dmf_SamNotificationViaSsh.obj
 0001:00024fa0       ??_C@_0CI@DOKLJEDB@SamNotificationViaSsh_Streaming@FNODOBFM@ 0000000180025fa0     DmfK:Dmf_SamNotificationViaSsh.obj
 0001:00024fd0       ??_C@_0DA@JOPKCJGO@SamNotificationViaSsh_Streaming@FNODOBFM@ 0000000180025fd0     DmfK:Dmf_SamNotificationViaSsh.obj
 0001:00025000       ??_C@_0GJ@IJLGKMJG@SamNotificationViaSsh_Streaming@FNODOBFM@ 0000000180026000     DmfK:Dmf_SamNotificationViaSsh.obj
 0001:00025070       ??_C@_0FJ@DJGKCNPN@SamNotificationViaSsh_OnDeviceA@FNODOBFM@ 0000000180026070     DmfK:Dmf_SamNotificationViaSsh.obj
 0001:000250d0       ??_C@_0FI@GGKACCLE@SamNotificationViaSsh_OnDeviceR@FNODOBFM@ 00000001800260d0     DmfK:Dmf_SamNotificationViaSsh.obj
 0001:00025130       ??_C@_0GF@ELOIGPJN@SamNotificationViaSsh_StreamAsy@FNODOBFM@ 0000000180026130     DmfK:Dmf_SamNotificationViaSsh.obj
 0001:000251a0       ??_C@_0HJ@ICCDCJAH@SamNotificationViaSsh_StreamAsy@FNODOBFM@ 00000001800261a0     DmfK:Dmf_SamNotificationViaSsh.obj
 0001:00025220       ??_C@_0DJ@EGKDHFIN@SamNotificationViaSsh_ModuleD0E@FNODOBFM@ 0000000180026220     DmfK:Dmf_SamNotificationViaSsh.obj
 0001:00025260       ??_C@_0GD@GJCJKAII@SamNotificationViaSsh_ModuleD0E@FNODOBFM@ 0000000180026260     DmfK:Dmf_SamNotificationViaSsh.obj
 0001:000252d0       ??_C@_0EO@KDNCKFAP@SamNotificationViaSsh_ModuleD0E@FNODOBFM@ 00000001800262d0     DmfK:Dmf_SamNotificationViaSsh.obj
 0001:00025320       ??_C@_0FG@FBCHJGP@SamNotificationViaSsh_ModuleD0E@FNODOBFM@ 0000000180026320     DmfK:Dmf_SamNotificationViaSsh.obj
 0001:00025380       ??_C@_0DH@BNLKJOBD@SamNotificationViaSsh_ModuleD0E@FNODOBFM@ 0000000180026380     DmfK:Dmf_SamNotificationViaSsh.obj
 0001:000253c0       ??_C@_0GH@PACOOCBG@SamNotificationViaSsh_ModuleD0E@FNODOBFM@ 00000001800263c0     DmfK:Dmf_SamNotificationViaSsh.obj
 0001:00025430       ??_C@_0EF@EHHIGGFG@SamNotificationViaSsh_ModuleD0E@FNODOBFM@ 0000000180026430     DmfK:Dmf_SamNotificationViaSsh.obj
 0001:00025480       ??_C@_0DE@HFFMBFGL@DMF_SamNotificationViaSsh_Open?4@FNODOBFM@ 0000000180026480     DmfK:Dmf_SamNotificationViaSsh.obj
 0001:000254c0       ??_C@_0DE@GLNGJOEC@DMF_SamNotificationViaSsh_Close@FNODOBFM@ 00000001800264c0     DmfK:Dmf_SamNotificationViaSsh.obj
 0001:00025500       ??_C@_0FH@JNPFOGH@DMF_SamNotificationViaSsh_Close@FNODOBFM@ 0000000180026500     DmfK:Dmf_SamNotificationViaSsh.obj
 0001:00025560       ??_C@_0EJ@ILGEIGHJ@DMF_SamNotificationViaSsh_Close@FNODOBFM@ 0000000180026560     DmfK:Dmf_SamNotificationViaSsh.obj
 0001:000255b0       ??_C@_0FF@NNGNAPBD@DMF_SamNotificationViaSsh_Open?4@FNODOBFM@ 00000001800265b0     DmfK:Dmf_SamNotificationViaSsh.obj
 0001:00025610       ??_C@_1FA@LCJFFEMG@?$AA?2?$AAd?$AAr?$AAi?$AAv?$AAe?$AAr?$AAd?$AAa?$AAt?$AAa?$AA?2?$AAS?$AAu?$AAr@FNODOBFM@ 0000000180026610     DmfK:SurfaceTelemetry.obj
 0001:00025660       ??_C@_0FE@GGGCLLCL@REPOSITORYDIR?2SurfaceLibrary?2Ke@FNODOBFM@ 0000000180026660     DmfK:Dmf_LiveKernelDump.obj
 0001:000256c0       ??_C@_0DM@KPAAJLBB@REPOSITORYDIR?2SurfaceLibrary?2Ke@FNODOBFM@ 00000001800266c0     DmfK:DmfCall.obj
 0001:00025700       ??_C@_0FB@PJIFEEHB@REPOSITORYDIR?2SurfaceLibrary?2Ke@FNODOBFM@ 0000000180026700     DmfK:Dmf_BranchTrack.obj
 0001:00025760       ??_C@_19CIJIHAKK@?$AAN?$AAU?$AAL?$AAL@FNODOBFM@ 0000000180026760     DmfK:Dmf_DeviceInterfaceTarget.obj
 0001:00025770       ??_C@_0FE@JINLKCMF@REPOSITORYDIR?2SurfaceLibrary?2Ke@FNODOBFM@ 0000000180026770     DmfK:Dmf_DeviceInterfaceTarget.obj
 0001:000257d0       ??_C@_0EL@IPHAGBOF@REPOSITORYDIR?2SurfaceLibrary?2Ke@FNODOBFM@ 00000001800267d0     DmfK:Dmf_IoctlHandler.obj
 0001:00025820       ??_C@_0EJ@JNKALINH@REPOSITORYDIR?2SurfaceLibrary?2Ke@FNODOBFM@ 0000000180026820     DmfK:Dmf_RingBuffer.obj
 0001:00025870       ??_C@_0EI@GPLPDCOG@REPOSITORYDIR?2SurfaceLibrary?2Ke@FNODOBFM@ 0000000180026870     DmfK:Dmf_CrashDump.obj
 0001:000258c0       ??_C@_1DC@KLEDOEDH@?$AAK?$AAe?$AAA?$AAd?$AAd?$AAT?$AAr?$AAi?$AAa?$AAg?$AAe?$AAD?$AAu?$AAm?$AAp@FNODOBFM@ 00000001800268c0     DmfK:Dmf_CrashDump.obj
 0001:00025900       ??_C@_0EI@CPGEFFGM@REPOSITORYDIR?2SurfaceLibrary?2Ke@FNODOBFM@ 0000000180026900     DmfK:Dmf_HashTable.obj
 0001:00025950       ??_C@_0EM@MPAHBDJB@REPOSITORYDIR?2SurfaceLibrary?2Ke@FNODOBFM@ 0000000180026950     DmfK:Dmf_RequestTarget.obj
 0001:000259a0       ??_C@_0FG@CBDMDBNG@REPOSITORYDIR?2SurfaceLibrary?2Ke@FNODOBFM@ 00000001800269a0     DmfK:Dmf_ContinuousRequestTarget.obj
 0001:00025a00       ??_C@_0EG@CBNDIIGN@REPOSITORYDIR?2SurfaceLibrary?2Ke@FNODOBFM@ 0000000180026a00     DmfK:Dmf_Rundown.obj
 0002:00000000       __imp_WdfVersionUnbind     0000000180027000     WdfLdr:WDFLDR.SYS
 0002:00000008       __imp_WdfLdrQueryInterface 0000000180027008     WdfLdr:WDFLDR.SYS
 0002:00000010       __imp_WdfVersionBind       0000000180027010     WdfLdr:WDFLDR.SYS
 0002:00000018       __imp_WdfVersionUnbindClass 0000000180027018     WdfLdr:WDFLDR.SYS
 0002:00000020       __imp_WdfVersionBindClass  0000000180027020     WdfLdr:WDFLDR.SYS
 0002:00000028       \177WDFLDR_NULL_THUNK_DATA 0000000180027028     WdfLdr:WDFLDR.SYS
 0002:00000030       __imp_imp_WppRecorderReplay 0000000180027030     wpprecorder:WppRecorder.sys
 0002:00000038       __imp_imp_WppRecorderIsDefaultLogAvailable 0000000180027038     wpprecorder:WppRecorder.sys
 0002:00000040       __imp_imp_WppRecorderLogGetDefault 0000000180027040     wpprecorder:WppRecorder.sys
 0002:00000048       __imp_imp_WppRecorderLogDelete 0000000180027048     wpprecorder:WppRecorder.sys
 0002:00000050       __imp_imp_WppRecorderLogCreate 0000000180027050     wpprecorder:WppRecorder.sys
 0002:00000058       __imp_WppAutoLogStop       0000000180027058     wpprecorder:WppRecorder.sys
 0002:00000060       __imp_WppAutoLogStart      0000000180027060     wpprecorder:WppRecorder.sys
 0002:00000068       __imp_WppAutoLogTrace      0000000180027068     wpprecorder:WppRecorder.sys
 0002:00000070       \177WppRecorder_NULL_THUNK_DATA 0000000180027070     wpprecorder:WppRecorder.sys
 0002:00000078       __imp_WerLiveKernelCancelReport 0000000180027078     DmfK:ext-ms-win-ntos-werkernel-l1-1-1.dll
 0002:00000080       __imp_WerLiveKernelCreateReport 0000000180027080     DmfK:ext-ms-win-ntos-werkernel-l1-1-1.dll
 0002:00000088       __imp_WerLiveKernelOpenDumpFile 0000000180027088     DmfK:ext-ms-win-ntos-werkernel-l1-1-1.dll
 0002:00000090       __imp_WerLiveKernelCloseHandle 0000000180027090     DmfK:ext-ms-win-ntos-werkernel-l1-1-1.dll
 0002:00000098       __imp_WerLiveKernelSubmitReport 0000000180027098     DmfK:ext-ms-win-ntos-werkernel-l1-1-1.dll
 0002:000000a0       \177ext-ms-win-ntos-werkernel-l1-1-1_NULL_THUNK_DATA 00000001800270a0     DmfK:ext-ms-win-ntos-werkernel-l1-1-1.dll
 0002:000000a8       __imp_EtwSetInformation    00000001800270a8     ntoskrnl:ntoskrnl.exe
 0002:000000b0       __imp_EtwRegister          00000001800270b0     ntoskrnl:ntoskrnl.exe
 0002:000000b8       __imp_PoUnregisterPowerSettingCallback 00000001800270b8     ntoskrnl:ntoskrnl.exe
 0002:000000c0       __imp_PoRegisterPowerSettingCallback 00000001800270c0     ntoskrnl:ntoskrnl.exe
 0002:000000c8       __imp_RtlEqualUnicodeString 00000001800270c8     ntoskrnl:ntoskrnl.exe
 0002:000000d0       __imp_RtlCopyUnicodeString 00000001800270d0     ntoskrnl:ntoskrnl.exe
 0002:000000d8       __imp_DbgPrintEx           00000001800270d8     ntoskrnl:ntoskrnl.exe
 0002:000000e0       __imp_MmGetSystemRoutineAddress 00000001800270e0     ntoskrnl:ntoskrnl.exe
 0002:000000e8       __imp_IoWMIRegistrationControl 00000001800270e8     ntoskrnl:ntoskrnl.exe
 0002:000000f0       __imp_RtlAssert            00000001800270f0     ntoskrnl:ntoskrnl.exe
 0002:000000f8       __imp_KeInitializeSpinLock 00000001800270f8     ntoskrnl:ntoskrnl.exe
 0002:00000100       __imp_KeAcquireSpinLockRaiseToDpc 0000000180027100     ntoskrnl:ntoskrnl.exe
 0002:00000108       __imp_KeReleaseSpinLock    0000000180027108     ntoskrnl:ntoskrnl.exe
 0002:00000110       __imp_ExFreePoolWithTag    0000000180027110     ntoskrnl:ntoskrnl.exe
 0002:00000118       __imp_strncpy_s            0000000180027118     ntoskrnl:ntoskrnl.exe
 0002:00000120       __imp_strcmp               0000000180027120     ntoskrnl:ntoskrnl.exe
 0002:00000128       __imp_KeInitializeEvent    0000000180027128     ntoskrnl:ntoskrnl.exe
 0002:00000130       __imp_KeResetEvent         0000000180027130     ntoskrnl:ntoskrnl.exe
 0002:00000138       __imp_KeSetEvent           0000000180027138     ntoskrnl:ntoskrnl.exe
 0002:00000140       __imp_KeWaitForSingleObject 0000000180027140     ntoskrnl:ntoskrnl.exe
 0002:00000148       __imp_ExInitializeRundownProtection 0000000180027148     ntoskrnl:ntoskrnl.exe
 0002:00000150       __imp_ExReInitializeRundownProtection 0000000180027150     ntoskrnl:ntoskrnl.exe
 0002:00000158       __imp_ExAcquireRundownProtection 0000000180027158     ntoskrnl:ntoskrnl.exe
 0002:00000160       __imp_RtlInitUnicodeString 0000000180027160     ntoskrnl:ntoskrnl.exe
 0002:00000168       __imp_ExRundownCompleted   0000000180027168     ntoskrnl:ntoskrnl.exe
 0002:00000170       __imp_ExWaitForRundownProtectionRelease 0000000180027170     ntoskrnl:ntoskrnl.exe
 0002:00000178       __imp__vsnprintf           0000000180027178     ntoskrnl:ntoskrnl.exe
 0002:00000180       __imp_RtlCompareUnicodeString 0000000180027180     ntoskrnl:ntoskrnl.exe
 0002:00000188       __imp_IoRegisterPlugPlayNotification 0000000180027188     ntoskrnl:ntoskrnl.exe
 0002:00000190       __imp_IoUnregisterPlugPlayNotificationEx 0000000180027190     ntoskrnl:ntoskrnl.exe
 0002:00000198       __imp_strncmp              0000000180027198     ntoskrnl:ntoskrnl.exe
 0002:000001a0       __imp_IoWMIOpenBlock       00000001800271a0     ntoskrnl:ntoskrnl.exe
 0002:000001a8       __imp_IoWMIQueryAllData    00000001800271a8     ntoskrnl:ntoskrnl.exe
 0002:000001b0       __imp_ObfDereferenceObject 00000001800271b0     ntoskrnl:ntoskrnl.exe
 0002:000001b8       __imp_ZwOpenFile           00000001800271b8     ntoskrnl:ntoskrnl.exe
 0002:000001c0       __imp_ZwQueryInformationFile 00000001800271c0     ntoskrnl:ntoskrnl.exe
 0002:000001c8       __imp_ZwReadFile           00000001800271c8     ntoskrnl:ntoskrnl.exe
 0002:000001d0       __imp_ZwWriteFile          00000001800271d0     ntoskrnl:ntoskrnl.exe
 0002:000001d8       __imp_ZwClose              00000001800271d8     ntoskrnl:ntoskrnl.exe
 0002:000001e0       __imp_RtlCompareUnicodeStrings 00000001800271e0     ntoskrnl:ntoskrnl.exe
 0002:000001e8       __imp_SeTokenIsAdmin       00000001800271e8     ntoskrnl:ntoskrnl.exe
 0002:000001f0       __imp_ZwOpenKey            00000001800271f0     ntoskrnl:ntoskrnl.exe
 0002:000001f8       __imp_ZwQueryValueKey      00000001800271f8     ntoskrnl:ntoskrnl.exe
 0002:00000200       __imp_ExAllocatePoolWithTag 0000000180027200     ntoskrnl:ntoskrnl.exe
 0002:00000208       __imp_KeCapturePersistentThreadState 0000000180027208     ntoskrnl:ntoskrnl.exe
 0002:00000210       NtBuildNumber              0000000180027210     ntoskrnl:ntoskrnl.exe
 0002:00000210       __imp_NtBuildNumber        0000000180027210     ntoskrnl:ntoskrnl.exe
 0002:00000218       __imp_RtlCaptureContext    0000000180027218     ntoskrnl:ntoskrnl.exe
 0002:00000220       __imp__vsnwprintf          0000000180027220     ntoskrnl:ntoskrnl.exe
 0002:00000228       __imp_KeDelayExecutionThread 0000000180027228     ntoskrnl:ntoskrnl.exe
 0002:00000230       __imp_sprintf_s            0000000180027230     ntoskrnl:ntoskrnl.exe
 0002:00000238       __imp_RtlCompareMemory     0000000180027238     ntoskrnl:ntoskrnl.exe
 0002:00000240       __imp_KeDeregisterBugCheckReasonCallback 0000000180027240     ntoskrnl:ntoskrnl.exe
 0002:00000248       __imp_KeRegisterBugCheckReasonCallback 0000000180027248     ntoskrnl:ntoskrnl.exe
 0002:00000250       __imp_ExFreePool           0000000180027250     ntoskrnl:ntoskrnl.exe
 0002:00000258       __imp_EtwUnregister        0000000180027258     ntoskrnl:ntoskrnl.exe
 0002:00000260       __imp_ExAllocatePool2      0000000180027260     ntoskrnl:ntoskrnl.exe
 0002:00000268       __imp_ExReleaseRundownProtection 0000000180027268     ntoskrnl:ntoskrnl.exe
 0002:00000270       __imp_EtwWriteTransfer     0000000180027270     ntoskrnl:ntoskrnl.exe
 0002:00000278       \177ntoskrnl_NULL_THUNK_DATA 0000000180027278     ntoskrnl:ntoskrnl.exe
 0002:00000280       __guard_check_icall_fptr   0000000180027280     BufferOverflowFastFailK:guard_support.obj
 0002:00000288       __guard_dispatch_icall_fptr 0000000180027288     BufferOverflowFastFailK:guard_support.obj
 0002:00000290       __guard_xfg_check_icall_fptr 0000000180027290     BufferOverflowFastFailK:guard_support.obj
 0002:00000298       __guard_xfg_dispatch_icall_fptr 0000000180027298     BufferOverflowFastFailK:guard_support.obj
 0002:000002a0       __guard_xfg_table_dispatch_icall_fptr 00000001800272a0     BufferOverflowFastFailK:guard_support.obj
 0002:000002a8       __castguard_check_failure_os_handled_fptr 00000001800272a8     BufferOverflowFastFailK:guard_support.obj
 0002:000002b0       __guard_eh_cont_table      00000001800272b0     <linker-defined>
 0002:000002c4       __guard_fids_table         00000001800272c4     <linker-defined>
 0002:00000ad0       __xmm@00000001000000000000000800000001 0000000180027ad0     surface_hid_mini.surface_hid_mini.3efcb60154bd7459-cgu.0.rcgu.o
 0002:00000ae0       __xmm@00000000000000000000000028270e02 0000000180027ae0     surface_hid_mini.surface_hid_mini.3efcb60154bd7459-cgu.0.rcgu.o
 0002:00000af0       __xmm@00000000000000000000000002012101 0000000180027af0     surface_hid_mini.surface_hid_mini.3efcb60154bd7459-cgu.0.rcgu.o
 0002:00000b00       __xmm@00000000000000000000000002012102 0000000180027b00     surface_hid_mini.surface_hid_mini.3efcb60154bd7459-cgu.0.rcgu.o
 0002:00000b10       __xmm@0000000000000000000000000b0b0101 0000000180027b10     surface_hid_mini.surface_hid_mini.3efcb60154bd7459-cgu.0.rcgu.o
 0002:00000b20       __xmm@000000800000000a0000008000000008 0000000180027b20     surface_hid_mini.surface_hid_mini.3efcb60154bd7459-cgu.0.rcgu.o
 0002:00001c40       _fltused                   0000000180028c40     surface_hid_mini.surface_hid_mini.3efcb60154bd7459-cgu.0.rcgu.o
 0002:00001d50       ??_C@_1BI@BJCKEEDJ@?$AAK?$AAm?$AAd?$AAf?$AAL?$AAi?$AAb?$AAr?$AAa?$AAr?$AAy@ 0000000180028d50     WdfDriverEntry:stub.obj
 0002:00001d68       ??_C@_0CI@FGGECOFJ@DriverEntry?5failed?50x?$CFx?5for?5dri@ 0000000180028d68     WdfDriverEntry:stub.obj
 0002:00001d90       GUID_WDF_LOADER_INTERFACE_DRIVER_ENTRY_FAILURE 0000000180028d90     WdfDriverEntry:stub.obj
 0002:00001da0       ??_C@_0KH@DJLKAFDB@FxStubInitTypes?3?5invalid?5driver@ 0000000180028da0     WdfDriverEntry:inittypes.obj
 0002:00001e48       ??_C@_0CH@JKHNJGFB@FxGetNextObjectContextTypeInfo?5@ 0000000180028e48     WdfDriverEntry:inittypes.obj
 0002:00001e70       ??_C@_0KL@EAFAJNMK@FxStubBindClasses?3?5invalid?5driv@ 0000000180028e70     WdfDriverEntry:classbind.obj
 0002:00001f20       ??_C@_0BP@CNINNJGL@FxGetNextClassBindInfo?5failed?6@ 0000000180028f20     WdfDriverEntry:classbind.obj
 0002:00001f40       ??_C@_0GB@LEIJHLCM@FxStubBindClasses?3?5ClientBindCl@ 0000000180028f40     WdfDriverEntry:classbind.obj
 0002:00001fb0       ??_C@_0FO@DJFFLMAP@FxStubBindClasses?3?5VersionBindC@ 0000000180028fb0     WdfDriverEntry:classbind.obj
 0002:00002010       WPP_ThisDir_CTLGUID_surface_hid_mini 0000000180029010     libms_surface_wpp-b83efe80b23bd200:2e40c9e35e9506f4-wpp.o
 0002:00002020       WPP_bb87df9ebd4738b330287b206bac9014_Traceguids 0000000180029020     libms_surface_wpp-b83efe80b23bd200:2e40c9e35e9506f4-wpp.o
 0002:00002030       ??_C@_1BK@DHLDGJM@?$AAP?$AAs?$AAG?$AAe?$AAt?$AAV?$AAe?$AAr?$AAs?$AAi?$AAo?$AAn@ 0000000180029030     libms_surface_wpp-b83efe80b23bd200:2e40c9e35e9506f4-wpp.o
 0002:00002050       ??_C@_1CA@OFIBBPKJ@?$AAW?$AAm?$AAi?$AAT?$AAr?$AAa?$AAc?$AAe?$AAM?$AAe?$AAs?$AAs?$AAa?$AAg?$AAe@ 0000000180029050     libms_surface_wpp-b83efe80b23bd200:2e40c9e35e9506f4-wpp.o
 0002:00002070       ??_C@_1DC@DOCOAJH@?$AAW?$AAm?$AAi?$AAQ?$AAu?$AAe?$AAr?$AAy?$AAT?$AAr?$AAa?$AAc?$AAe?$AAI?$AAn@ 0000000180029070     libms_surface_wpp-b83efe80b23bd200:2e40c9e35e9506f4-wpp.o
 0002:000020a8       ??_C@_1DG@PFOPAIND@?$AAE?$AAt?$AAw?$AAR?$AAe?$AAg?$AAi?$AAs?$AAt?$AAe?$AAr?$AAC?$AAl?$AAa?$AAs@ 00000001800290a8     libms_surface_wpp-b83efe80b23bd200:2e40c9e35e9506f4-wpp.o
 0002:000020e0       ??_C@_1BM@CJMKDOJH@?$AAE?$AAt?$AAw?$AAU?$AAn?$AAr?$AAe?$AAg?$AAi?$AAs?$AAt?$AAe?$AAr@ 00000001800290e0     libms_surface_wpp-b83efe80b23bd200:2e40c9e35e9506f4-wpp.o
 0002:00002100       ??_C@_0BH@PIMJLMCH@WdfCustomType_DMF_File@ 0000000180029100     DmfK:Dmf_BufferPool.obj
 0002:00002118       ??_C@_0BK@HGGIFFEE@WdfCustomType_DMF_Rundown@ 0000000180029118     DmfK:Dmf_BufferPool.obj
 0002:00002138       ??_C@_0CA@PMAMDIMC@WdfCustomType_DMF_RequestTarget@ 0000000180029138     DmfK:Dmf_BufferPool.obj
 0002:00002158       ??_C@_0CK@CBFLEAOM@WdfCustomType_DMF_ContinuousReq@ 0000000180029158     DmfK:Dmf_BufferPool.obj
 0002:00002188       ??_C@_0CI@FDODINOB@WdfCustomType_DMF_DeviceInterfa@ 0000000180029188     DmfK:Dmf_BufferPool.obj
 0002:000021b0       ??_C@_0BM@MNCFDPLM@WdfCustomType_DMF_SmbiosWmi@ 00000001800291b0     DmfK:Dmf_BufferPool.obj
 0002:000021d0       ??_C@_0BO@IEINAGIE@WdfCustomType_DMF_BranchTrack@ 00000001800291d0     DmfK:Dmf_BufferPool.obj
 0002:000021f0       ??_C@_0CB@DJHHJFOM@WdfCustomType_DMF_LiveKernelDum@ 00000001800291f0     DmfK:Dmf_BufferPool.obj
 0002:00002218       ??_C@_0BN@ELKFMFCC@WdfCustomType_DMFMODULE_TYPE@ 0000000180029218     DmfK:Dmf_BufferPool.obj
 0002:00002238       ??_C@_0CB@OKEHELBH@WdfCustomType_DMFCOLLECTION_TYP@ 0000000180029238     DmfK:Dmf_BufferPool.obj
 0002:00002260       ??_C@_09DFPHHNJE@DMFMODULE@ 0000000180029260     DmfK:Dmf_BufferPool.obj
 0002:00002270       GUID_DEVINTERFACE_BranchTrack 0000000180029270     DmfK:Dmf_BufferPool.obj
 0002:00002280       ??_C@_0BN@KHBHIDEG@WdfCustomType_DMF_BufferPool@ 0000000180029280     DmfK:Dmf_BufferPool.obj
 0002:000022a0       ??_C@_0BM@PMCGJCJC@WdfCustomType_DMF_HashTable@ 00000001800292a0     DmfK:Dmf_BufferPool.obj
 0002:000022c0       ??_C@_0BN@NOKBALGC@WdfCustomType_DMF_RingBuffer@ 00000001800292c0     DmfK:Dmf_BufferPool.obj
 0002:000022e0       ??_C@_0BO@BKNEEINJ@WdfCustomType_DMF_BufferQueue@ 00000001800292e0     DmfK:Dmf_BufferPool.obj
 0002:00002300       ??_C@_0BP@NIFLHNKE@WdfCustomType_DMF_IoctlHandler@ 0000000180029300     DmfK:Dmf_BufferPool.obj
 0002:00002320       ??_C@_0BJ@GPEPJKDG@WdfCustomType_DMF_String@ 0000000180029320     DmfK:Dmf_BufferPool.obj
 0002:00002340       WPP_29de08c82c6d3c5dc2154f240775ac47_Traceguids 0000000180029340     DmfK:Dmf_BufferPool.obj
 0002:00002350       ??_C@_0BM@ELOMGNBE@WdfCustomType_DMF_CrashDump@ 0000000180029350     DmfK:Dmf_BufferPool.obj
 0002:00002370       ??_C@_0BJ@KAACMJBC@WdfCustomType_DMF_Bridge@ 0000000180029370     DmfK:Dmf_BufferPool.obj
 0002:00002390       GUID_DEVINTERFACE_CrashDump 0000000180029390     DmfK:Dmf_BufferPool.obj
 0002:000023a0       ??_C@_0BH@DKCMHNLF@DMF_CONTEXT_BufferPool@ 00000001800293a0     DmfK:Dmf_BufferPool.obj
 0002:000023b8       ??_C@_0CE@OCNEGNNO@WdfCustomType_DMF_BufferPool_Bu@ 00000001800293b8     DmfK:Dmf_BufferPool.obj
 0002:000023e0       GUID_DEVICE_INTERFACE_ARRIVAL 00000001800293e0     DmfK:Dmf_BufferPool.obj
 0002:000023f0       GUID_DEVICE_INTERFACE_REMOVAL 00000001800293f0     DmfK:Dmf_BufferPool.obj
 0002:00002400       ??_C@_0BJ@IABHEJKO@BUFFERPOOL_TIMER_CONTEXT@ 0000000180029400     DmfK:Dmf_BufferPool.obj
 0002:00002420       ??_C@_0CA@CNOFEGJE@WdfCustomType_DMF_ScheduledTask@ 0000000180029420     DmfK:Dmf_BufferPool.obj
 0002:00002440       ??_C@_0CB@PJECPGBD@WdfCustomType_DMF_QueuedWorkIte@ 0000000180029440     DmfK:Dmf_BufferPool.obj
 0002:00002468       GUID_DEVINTERFACE_SurfaceSerialHub 0000000180029468     DmfK:Dmf_SamCommunicationViaSsh.obj
 0002:00002478       ??_C@_0DO@PFDJMPEM@WdfCustomType_DMF_SurfaceTeleme@ 0000000180029478     DmfK:Dmf_SamCommunicationViaSsh.obj
 0002:000024b8       GUID_DEVINTERFACE_SurfaceTelemetryConsentSettingsNotification 00000001800294b8     DmfK:Dmf_SamCommunicationViaSsh.obj
 0002:000024c8       WPP_ede84a8d0a563aa725fe80e95971cc8c_Traceguids 00000001800294c8     DmfK:Dmf_SamCommunicationViaSsh.obj
 0002:000024d8       ??_C@_0CD@FKPKNDCE@DMF_CONTEXT_SamCommunicationVia@ 00000001800294d8     DmfK:Dmf_SamCommunicationViaSsh.obj
 0002:00002500       ??_C@_0CJ@BJJFHPAM@WdfCustomType_DMF_SamCommunicat@ 0000000180029500     DmfK:Dmf_SamCommunicationViaSsh.obj
 0002:00002530       ??_C@_0CI@OOKDEBLC@WdfCustomType_DMF_SamNotificati@ 0000000180029530     DmfK:Dmf_SamCommunicationViaSsh.obj
 0002:00002558       WPP_cf17d742a855303cbfc498ef2a8c7616_Traceguids 0000000180029558     DmfK:DmfHelpers.obj
 0002:00002568       ??_C@_0BD@JCLIEHEP@DMF_DEVICE_CONTEXT@ 0000000180029568     DmfK:DmfHelpers.obj
 0002:00002580       WPP_9cce8732a9a23fd5662e1d8a0c6faab4_Traceguids 0000000180029580     DmfK:Dmf_SamNotificationViaSsh.obj
 0002:00002590       ??_C@_0CC@OIOGADNK@DMF_CONTEXT_SamNotificationViaS@ 0000000180029590     DmfK:Dmf_SamNotificationViaSsh.obj
 0002:000025b8       WPP_76bed8964cf63f3cb49ef63508442285_Traceguids 00000001800295b8     DmfK:SurfaceTelemetry.obj
 0002:000025c8       WPP_c7b9ba003e2e36b2bb246be0f4fb8e9d_Traceguids 00000001800295c8     DmfK:Dmf_QueuedWorkItem.obj
 0002:000025d8       ??_C@_0BL@GAMHBBEB@DMF_CONTEXT_QueuedWorkItem@ 00000001800295d8     DmfK:Dmf_QueuedWorkItem.obj
 0002:000025f8       WPP_a304d9a05c763ae8997add1b3483044f_Traceguids 00000001800295f8     DmfK:DmfModuleCollection.obj
 0002:00002608       WPP_9ec23aa426a631bc7650fe4f969c9165_Traceguids 0000000180029608     DmfK:Dmf_SurfaceTelemetryConsentSettingsNotification.obj
 0002:00002618       ??_C@_0DI@JNCAGPNO@DMF_CONTEXT_SurfaceTelemetryCon@ 0000000180029618     DmfK:Dmf_SurfaceTelemetryConsentSettingsNotification.obj
 0002:00002650       WPP_6e34b21b3cd73c4f944fc51f8e334c7f_Traceguids 0000000180029650     DmfK:DmfDeviceInit.obj
 0002:00002660       WPP_c72a7a9e2ea5355f7444ce2c104975c3_Traceguids 0000000180029660     DmfK:Dmf_LiveKernelDump.obj
 0002:00002670       ??_C@_0BL@KAPCHCLO@DMF_CONTEXT_LiveKernelDump@ 0000000180029670     DmfK:Dmf_LiveKernelDump.obj
 0002:00002690       WPP_ce8bbdb318263124fab9de796f4fb53b_Traceguids 0000000180029690     DmfK:DmfPortable.obj
 0002:000026a0       WPP_9ee3043c4f2e38c1fe1cc3b0df10a756_Traceguids 00000001800296a0     DmfK:DmfCore.obj
 0002:000026b0       ??_C@_07MLMHLOOL@Generic@  00000001800296b0     DmfK:DmfCore.obj
 0002:000026b8       WPP_bea935c9f26a39b5f4cf2c3d9956e19c_Traceguids 00000001800296b8     DmfK:DmfCall.obj
 0002:000026c8       WPP_65120927b2083cf558636214b82181b4_Traceguids 00000001800296c8     DmfK:Dmf_BranchTrack.obj
 0002:000026d8       ??_C@_0BI@KAKEJONM@DMF_CONTEXT_BranchTrack@ 00000001800296d8     DmfK:Dmf_BranchTrack.obj
 0002:000026f0       WPP_50e18a4d9a09372e83e1a977eb7d463f_Traceguids 00000001800296f0     DmfK:Dmf_DeviceInterfaceTarget.obj
 0002:00002700       ??_C@_0CC@FFKGMPIJ@DMF_CONTEXT_DeviceInterfaceTarg@ 0000000180029700     DmfK:Dmf_DeviceInterfaceTarget.obj
 0002:00002728       WPP_599b9ccc13e63bd7de7bd52853cf32e4_Traceguids 0000000180029728     DmfK:Dmf_String.obj
 0002:00002738       WPP_1ce7a2e3a3b439ec3759b0f4cf5eea70_Traceguids 0000000180029738     DmfK:Dmf_SmbiosWmi.obj
 0002:00002748       ??_C@_0BG@CEKMGDDJ@DMF_CONTEXT_SmbiosWmi@ 0000000180029748     DmfK:Dmf_SmbiosWmi.obj
 0002:00002760       WPP_7d60093c7f093786bb3679cb8db10815_Traceguids 0000000180029760     DmfK:Dmf_File.obj
 0002:00002770       WPP_6d3d5bccc65433b634f8f15cb6360fcf_Traceguids 0000000180029770     DmfK:Dmf_BufferQueue.obj
 0002:00002780       ??_C@_0BI@DOPNNAIB@DMF_CONTEXT_BufferQueue@ 0000000180029780     DmfK:Dmf_BufferQueue.obj
 0002:00002798       WPP_bf28c7fd66b03dc245f3f6f58be93d4b_Traceguids 0000000180029798     DmfK:Dmf_ScheduledTask.obj
 0002:000027a8       ??_C@_0BK@KBFDKOJH@DMF_CONTEXT_ScheduledTask@ 00000001800297a8     DmfK:Dmf_ScheduledTask.obj
 0002:000027c8       WPP_9f0751f581513e827ab9bad83e0a256b_Traceguids 00000001800297c8     DmfK:DmfContainer.obj
 0002:000027d8       WPP_f5b28edfd0a3311703e0da264304d527_Traceguids 00000001800297d8     DmfK:Dmf_Bridge.obj
 0002:000027e8       ??_C@_0BD@IOKDMGKM@DMF_CONTEXT_Bridge@ 00000001800297e8     DmfK:Dmf_Bridge.obj
 0002:00002800       WPP_5c7dd15af4f2367cd5a8179e9d1efbcf_Traceguids 0000000180029800     DmfK:DmfBranchTrack.obj
 0002:00002810       WPP_29a93f16971e39db801151a1a58c434e_Traceguids 0000000180029810     DmfK:DmfLiveKernelDump.obj
 0002:00002820       WPP_281b8847791c3b1bef2436939410a9f3_Traceguids 0000000180029820     DmfK:DmfGeneric.obj
 0002:00002830       WPP_dcfa6ef3dfab331c8f04d7ba26e3554d_Traceguids 0000000180029830     DmfK:Dmf_IoctlHandler.obj
 0002:00002840       ??_C@_0BJ@LNMPINPK@DMF_CONTEXT_IoctlHandler@ 0000000180029840     DmfK:Dmf_IoctlHandler.obj
 0002:00002860       ??_C@_17EEOGHOKP@?$AA?$CF?$AAw?$AAs@ 0000000180029860     DmfK:lkmdtel.obj
 0002:00002868       ??_C@_0DM@MDCGBJNP@LKMDTEL?3?5WerLiveKernelCreateRep@ 0000000180029868     DmfK:lkmdtel.obj
 0002:000028b0       ??_C@_0EG@JBJCILOI@LKMDTEL?3?5WerPolicy?5is?5WerLiveKe@ 00000001800298b0     DmfK:lkmdtel.obj
 0002:000028f8       ??_C@_0DC@NDBFJGLB@LKMDTEL?3?5WerLiveCancelReport?5fa@ 00000001800298f8     DmfK:lkmdtel.obj
 0002:00002930       ??_C@_1CE@NGPJDKDL@?$AAM?$AAa?$AAx?$AAR?$AAe?$AAp?$AAo?$AAr?$AAt?$AAS?$AAi?$AAz?$AAe?$AAI?$AAn@ 0000000180029930     DmfK:lkmdtel.obj
 0002:00002960       ??_C@_1HG@OLOLOOHC@?$AA?2?$AAR?$AAe?$AAg?$AAi?$AAs?$AAt?$AAr?$AAy?$AA?2?$AAM?$AAa?$AAc?$AAh?$AAi@ 0000000180029960     DmfK:lkmdtel.obj
 0002:000029e0       ??_C@_0FF@EGBMKBNH@LKMDTEL?3?5Secondary?5size?5updated@ 00000001800299e0     DmfK:lkmdtel.obj
 0002:00002a40       ??_C@_0EP@JAKBNMKN@LKMDTEL?3?5LkmdTelpWriteDumpFile?3@ 0000000180029a40     DmfK:lkmdtel.obj
 0002:00002a90       ??_C@_0EJ@KNFLKGLB@LKMDTEL?3?5LkmdTelSubmitReport?3?5L@ 0000000180029a90     DmfK:lkmdtel.obj
 0002:00002ae0       ??_C@_0EN@BDGICLBJ@LKMDTEL?3?5LkmdTelSubmitReport?3?5W@ 0000000180029ae0     DmfK:lkmdtel.obj
 0002:00002b30       ??_C@_0EN@BGMPLCFC@LKMDTEL?3?5LkmdTelSubmitReport?3?5W@ 0000000180029b30     DmfK:lkmdtel.obj
 0002:00002b80       ??_C@_0EM@FOEELLKM@LKMDTEL?3?5LkmdTelSubmitReport?3?5W@ 0000000180029b80     DmfK:lkmdtel.obj
 0002:00002bd0       WPP_33c31c75c7fc36e9f63f061734fd4b35_Traceguids 0000000180029bd0     DmfK:DmfUtility.obj
 0002:00002de0       WPP_bdd69fd0b8ab31cd69b83ac1f0b9588e_Traceguids 0000000180029de0     DmfK:Dmf_RingBuffer.obj
 0002:00002df0       ??_C@_0BH@EDJKPFJB@DMF_CONTEXT_RingBuffer@ 0000000180029df0     DmfK:Dmf_RingBuffer.obj
 0002:00002e08       WPP_86e87043f1613111113d5bc8cc8434fd_Traceguids 0000000180029e08     DmfK:Dmf_CrashDump.obj
 0002:00002e18       ??_C@_0BG@KCGFDBJB@DMF_CONTEXT_CrashDump@ 0000000180029e18     DmfK:Dmf_CrashDump.obj
 0002:00002e30       WPP_0e5cf494fad4361ef8f2c02e9f07521c_Traceguids 0000000180029e30     DmfK:DmfInternal.obj
 0002:00002e40       WPP_c4bcc0e2d587391410fd2454268751a4_Traceguids 0000000180029e40     DmfK:DmfInterfaceInternal.obj
 0002:00002e50       WPP_8fee9584323a33da4995b45d8b967c7f_Traceguids 0000000180029e50     DmfK:Dmf_HashTable.obj
 0002:00002e60       ??_C@_0BG@BFKPMOBH@DMF_CONTEXT_HashTable@ 0000000180029e60     DmfK:Dmf_HashTable.obj
 0002:00002e78       WPP_2033769a05ed32eae9e9c09e9b61a8a4_Traceguids 0000000180029e78     DmfK:Dmf_RequestTarget.obj
 0002:00002e88       ??_C@_0BK@HALKNAMB@DMF_CONTEXT_RequestTarget@ 0000000180029e88     DmfK:Dmf_RequestTarget.obj
 0002:00002ea8       ??_C@_0P@HELBCPOP@UNIQUE_REQUEST@ 0000000180029ea8     DmfK:Dmf_RequestTarget.obj
 0002:00002eb8       WPP_51023f9795ab3a78548eea2addf100ba_Traceguids 0000000180029eb8     DmfK:Dmf_ContinuousRequestTarget.obj
 0002:00002ec8       ??_C@_0CE@BEKNIHLK@DMF_CONTEXT_ContinuousRequestTa@ 0000000180029ec8     DmfK:Dmf_ContinuousRequestTarget.obj
 0002:00002ef0       WPP_328a349032863cd674a185f0e2f4ff2d_Traceguids 0000000180029ef0     DmfK:Dmf_Rundown.obj
 0002:00002f00       ??_C@_0BE@FKJPGKMA@DMF_CONTEXT_Rundown@ 0000000180029f00     DmfK:Dmf_Rundown.obj
 0002:00002f30       _load_config_used          0000000180029f30     BufferOverflowFastFailK:loadcfg.obj
 0003:000000f0       __security_cookie          000000018002c0f0     BufferOverflowFastFailK:gs_support.obj
 0003:000000f8       __security_cookie_complement 000000018002c0f8     BufferOverflowFastFailK:gs_support.obj
 0003:00000100       __isa_info                 000000018002c100     ntoskrnl:cpuinfo.obj
 0003:00000140       WdfBindInfo                000000018002c140     WdfDriverEntry:stub.obj
 0003:00000170       WPP_GLOBAL_Control         000000018002c170     libms_surface_wpp-b83efe80b23bd200:2e40c9e35e9506f4-wpp.o
 0003:00000178       WPP_RECORDER_INITIALIZED   000000018002c178     libms_surface_wpp-b83efe80b23bd200:2e40c9e35e9506f4-wpp.o
 0003:00000180       _WDF_WdfCustomType_DMF_File_TYPE_INFO 000000018002c180     DmfK:Dmf_BufferPool.obj
 0003:000001a8       _WDF_WdfCustomType_DMF_Rundown_TYPE_INFO 000000018002c1a8     DmfK:Dmf_BufferPool.obj
 0003:000001d0       _WDF_WdfCustomType_DMF_RequestTarget_TYPE_INFO 000000018002c1d0     DmfK:Dmf_BufferPool.obj
 0003:000001f8       _WDF_WdfCustomType_DMF_ContinuousRequestTarget_TYPE_INFO 000000018002c1f8     DmfK:Dmf_BufferPool.obj
 0003:00000220       _WDF_WdfCustomType_DMF_DeviceInterfaceTarget_TYPE_INFO 000000018002c220     DmfK:Dmf_BufferPool.obj
 0003:00000248       _WDF_WdfCustomType_DMF_SmbiosWmi_TYPE_INFO 000000018002c248     DmfK:Dmf_BufferPool.obj
 0003:00000270       _WDF_WdfCustomType_DMF_BranchTrack_TYPE_INFO 000000018002c270     DmfK:Dmf_BufferPool.obj
 0003:00000298       _WDF_WdfCustomType_DMF_LiveKernelDump_TYPE_INFO 000000018002c298     DmfK:Dmf_BufferPool.obj
 0003:000002c0       _WDF_WdfCustomType_DMFMODULE_TYPE_TYPE_INFO 000000018002c2c0     DmfK:Dmf_BufferPool.obj
 0003:000002e8       _WDF_WdfCustomType_DMFCOLLECTION_TYPE_TYPE_INFO 000000018002c2e8     DmfK:Dmf_BufferPool.obj
 0003:00000310       _WDF_DMFMODULE_TYPE_INFO   000000018002c310     DmfK:Dmf_BufferPool.obj
 0003:00000338       _WDF_WdfCustomType_DMF_BufferPool_TYPE_INFO 000000018002c338     DmfK:Dmf_BufferPool.obj
 0003:00000360       _WDF_WdfCustomType_DMF_HashTable_TYPE_INFO 000000018002c360     DmfK:Dmf_BufferPool.obj
 0003:00000388       _WDF_WdfCustomType_DMF_RingBuffer_TYPE_INFO 000000018002c388     DmfK:Dmf_BufferPool.obj
 0003:000003b0       _WDF_WdfCustomType_DMF_BufferQueue_TYPE_INFO 000000018002c3b0     DmfK:Dmf_BufferPool.obj
 0003:000003d8       _WDF_WdfCustomType_DMF_IoctlHandler_TYPE_INFO 000000018002c3d8     DmfK:Dmf_BufferPool.obj
 0003:00000400       _WDF_WdfCustomType_DMF_String_TYPE_INFO 000000018002c400     DmfK:Dmf_BufferPool.obj
 0003:00000428       _WDF_WdfCustomType_DMF_CrashDump_TYPE_INFO 000000018002c428     DmfK:Dmf_BufferPool.obj
 0003:00000450       _WDF_WdfCustomType_DMF_Bridge_TYPE_INFO 000000018002c450     DmfK:Dmf_BufferPool.obj
 0003:00000478       _WDF_DMF_CONTEXT_BufferPool_TYPE_INFO 000000018002c478     DmfK:Dmf_BufferPool.obj
 0003:000004a0       _WDF_WdfCustomType_DMF_BufferPool_Buffer_TYPE_INFO 000000018002c4a0     DmfK:Dmf_BufferPool.obj
 0003:000004c8       _WDF_BUFFERPOOL_TIMER_CONTEXT_TYPE_INFO 000000018002c4c8     DmfK:Dmf_BufferPool.obj
 0003:000004f0       _WDF_WdfCustomType_DMF_ScheduledTask_TYPE_INFO 000000018002c4f0     DmfK:Dmf_BufferPool.obj
 0003:00000518       _WDF_WdfCustomType_DMF_QueuedWorkItem_TYPE_INFO 000000018002c518     DmfK:Dmf_BufferPool.obj
 0003:00000540       _WDF_WdfCustomType_DMF_SurfaceTelemetryConsentSettingsNotification_TYPE_INFO 000000018002c540     DmfK:Dmf_SamCommunicationViaSsh.obj
 0003:00000568       _WDF_DMF_CONTEXT_SamCommunicationViaSsh_TYPE_INFO 000000018002c568     DmfK:Dmf_SamCommunicationViaSsh.obj
 0003:00000590       _WDF_WdfCustomType_DMF_SamCommunicationViaSsh_TYPE_INFO 000000018002c590     DmfK:Dmf_SamCommunicationViaSsh.obj
 0003:000005b8       _WDF_WdfCustomType_DMF_SamNotificationViaSsh_TYPE_INFO 000000018002c5b8     DmfK:Dmf_SamCommunicationViaSsh.obj
 0003:000005e0       _WDF_DMF_DEVICE_CONTEXT_TYPE_INFO 000000018002c5e0     DmfK:DmfHelpers.obj
 0003:00000608       _WDF_DMF_CONTEXT_SamNotificationViaSsh_TYPE_INFO 000000018002c608     DmfK:Dmf_SamNotificationViaSsh.obj
 0003:00000630       _WDF_DMF_CONTEXT_QueuedWorkItem_TYPE_INFO 000000018002c630     DmfK:Dmf_QueuedWorkItem.obj
 0003:00000658       _WDF_DMF_CONTEXT_SurfaceTelemetryConsentSettingsNotification_TYPE_INFO 000000018002c658     DmfK:Dmf_SurfaceTelemetryConsentSettingsNotification.obj
 0003:00000680       ?SurfaceTelemetryConsentSettingsNotification_IoctlHandlerTable@@3PAUIoctlHandler_IoctlRecord@@A 000000018002c680     DmfK:Dmf_SurfaceTelemetryConsentSettingsNotification.obj
 0003:000006a0       ?LiveKernelDump_IoctlSpecification@@3PAUIoctlHandler_IoctlRecord@@A 000000018002c6a0     DmfK:Dmf_LiveKernelDump.obj
 0003:000006c0       _WDF_DMF_CONTEXT_LiveKernelDump_TYPE_INFO 000000018002c6c0     DmfK:Dmf_LiveKernelDump.obj
 0003:000006f0       ?DmfCallbacksDmf_Internal_Passive@@3UDMF_CALLBACKS_DMF@@A 000000018002c6f0     DmfK:DmfCore.obj
 0003:00000730       ?DmfCallbacksInternal_Internal_Passive@@3UDMF_CALLBACKS_INTERNAL@@A 000000018002c730     DmfK:DmfCore.obj
 0003:00000760       ?DmfCallbacksWdf_Internal_Passive@@3UDMF_CALLBACKS_WDF@@A 000000018002c760     DmfK:DmfCore.obj
 0003:00000850       ?DmfCallbacksDmf_Internal_Dispatch@@3UDMF_CALLBACKS_DMF@@A 000000018002c850     DmfK:DmfCore.obj
 0003:00000890       ?DmfCallbacksInternal_Internal_Dispatch@@3UDMF_CALLBACKS_INTERNAL@@A 000000018002c890     DmfK:DmfCore.obj
 0003:000008c0       ?DmfCallbacksWdf_Internal_Dispatch@@3UDMF_CALLBACKS_WDF@@A 000000018002c8c0     DmfK:DmfCore.obj
 0003:00000a38       ?DmfChildObjectIterateForward@@3U_DMF_ChildObjectGet@@A 000000018002ca38     DmfK:DmfCall.obj
 0003:00000a48       ?DmfChildObjectIterateBackward@@3U_DMF_ChildObjectGet@@A 000000018002ca48     DmfK:DmfCall.obj
 0003:00000a58       _WDF_DMF_CONTEXT_BranchTrack_TYPE_INFO 000000018002ca58     DmfK:Dmf_BranchTrack.obj
 0003:00000a80       _WDF_DMF_CONTEXT_DeviceInterfaceTarget_TYPE_INFO 000000018002ca80     DmfK:Dmf_DeviceInterfaceTarget.obj
 0003:00000aa8       _WDF_DMF_CONTEXT_SmbiosWmi_TYPE_INFO 000000018002caa8     DmfK:Dmf_SmbiosWmi.obj
 0003:00000ad0       _WDF_DMF_CONTEXT_BufferQueue_TYPE_INFO 000000018002cad0     DmfK:Dmf_BufferQueue.obj
 0003:00000af8       _WDF_DMF_CONTEXT_ScheduledTask_TYPE_INFO 000000018002caf8     DmfK:Dmf_ScheduledTask.obj
 0003:00000b20       _WDF_DMF_CONTEXT_Bridge_TYPE_INFO 000000018002cb20     DmfK:Dmf_Bridge.obj
 0003:00000b48       _WDF_DMF_CONTEXT_IoctlHandler_TYPE_INFO 000000018002cb48     DmfK:Dmf_IoctlHandler.obj
 0003:00000b70       gMaxReportSize             000000018002cb70     DmfK:lkmdtel.obj
 0003:00000b74       gMaxSecondarySize          000000018002cb74     DmfK:lkmdtel.obj
 0003:00000b78       _WDF_DMF_CONTEXT_RingBuffer_TYPE_INFO 000000018002cb78     DmfK:Dmf_RingBuffer.obj
 0003:00000ba0       _WDF_DMF_CONTEXT_CrashDump_TYPE_INFO 000000018002cba0     DmfK:Dmf_CrashDump.obj
 0003:00000bd0       ?CrashDump_IoctlSpecification@@3PAUIoctlHandler_IoctlRecord@@A 000000018002cbd0     DmfK:Dmf_CrashDump.obj
 0003:00000c90       _WDF_DMF_CONTEXT_HashTable_TYPE_INFO 000000018002cc90     DmfK:Dmf_HashTable.obj
 0003:00000cb8       _WDF_DMF_CONTEXT_RequestTarget_TYPE_INFO 000000018002ccb8     DmfK:Dmf_RequestTarget.obj
 0003:00000ce0       _WDF_UNIQUE_REQUEST_TYPE_INFO 000000018002cce0     DmfK:Dmf_RequestTarget.obj
 0003:00000d08       _WDF_DMF_CONTEXT_ContinuousRequestTarget_TYPE_INFO 000000018002cd08     DmfK:Dmf_ContinuousRequestTarget.obj
 0003:00000d30       ?g_ContinuousRequestTargetUniqueId@@3_JA 000000018002cd30     DmfK:Dmf_ContinuousRequestTarget.obj
 0003:00000d38       _WDF_DMF_CONTEXT_Rundown_TYPE_INFO 000000018002cd38     DmfK:Dmf_Rundown.obj
 0003:00000d60       ?__KMDF_CLASS_BIND_START@@3U_MARKER_TYPE@@A 000000018002cd60     WdfDriverEntry:classbind.obj
 0003:00000d60       _guard_check_icall_$fo_default$ 000000018002cd60 f   BufferOverflowFastFailK:checkcfg.obj
 0003:00000d70       ?__KMDF_CLASS_BIND_END@@3PEAXEA 000000018002cd70     WdfDriverEntry:classbind.obj
 0003:00000d80       ?__KMDF_TYPE_INIT_START@@3U_MARKER_TYPE@@A 000000018002cd80     WdfDriverEntry:inittypes.obj
 0003:00000d90       ?__KMDF_TYPE_INIT_END@@3PEAXEA 000000018002cd90     WdfDriverEntry:inittypes.obj
 0003:00000fc8       WdfDriverMiniportUnloadOverride 000000018002cfc8     WdfDriverEntry:stub.obj
 0003:00000fd0       typeWDF_IFR_HEADER         000000018002cfd0     WdfDriverEntry:stub.obj
 0003:00000fe8       WdfFunctions_01015         000000018002cfe8     WdfDriverEntry:stub.obj
 0003:00000ff0       WdfDriverGlobals           000000018002cff0     WdfDriverEntry:stub.obj
 0003:00001008       pfnWppQueryTraceInformation 000000018002d008     libms_surface_wpp-b83efe80b23bd200:2e40c9e35e9506f4-wpp.o
 0003:00001010       pfnWppTraceMessage         000000018002d010     libms_surface_wpp-b83efe80b23bd200:2e40c9e35e9506f4-wpp.o
 0003:00001018       pfnEtwUnregister           000000018002d018     libms_surface_wpp-b83efe80b23bd200:2e40c9e35e9506f4-wpp.o
 0003:00001020       pfnEtwRegisterClassicProvider 000000018002d020     libms_surface_wpp-b83efe80b23bd200:2e40c9e35e9506f4-wpp.o
 0003:00001028       pfnWppGetVersion           000000018002d028     libms_surface_wpp-b83efe80b23bd200:2e40c9e35e9506f4-wpp.o
 0003:00001030       WPPTraceSuite              000000018002d030     libms_surface_wpp-b83efe80b23bd200:2e40c9e35e9506f4-wpp.o
 0003:00001048       ?g_Initialized@@3EA        000000018002d048     DmfK:SurfaceTelemetry.obj
 0003:0000104c       ?g_MaximumEventTypeAllowed@@3JA 000000018002d04c     DmfK:SurfaceTelemetry.obj
 0003:00001050       ?g_DmfDefaultDeviceInit@@3UDMFDEVICE_INIT@@A 000000018002d050     DmfK:DmfDeviceInit.obj
 0003:00001140       ?g_DisableWppRecorder@@3EA 000000018002d140     DmfK:DmfDeviceInit.obj
 0003:0000114c       gMaxSizeInitialized        000000018002d14c     DmfK:lkmdtel.obj
 0003:00001150       ?g_DMF_IoGetActivityIdIrp@@3P6AJPEAU_IRP@@PEAU_GUID@@@ZEA 000000018002d150     DmfK:DmfUtility.obj
 0003:00001158       ?g_DmfModuleCrashDump@@3PEAUDMFMODULE__@@EA 000000018002d158     DmfK:Dmf_CrashDump.obj
 0003:00001160       WPP_MAIN_CB                000000018002d160     <common>
 0005:00001ca0       WppCleanupKm               0000000180032ca0 f   libms_surface_wpp-b83efe80b23bd200:2e40c9e35e9506f4-wpp.o
 0005:00001d50       WppInitKm                  0000000180032d50 f   libms_surface_wpp-b83efe80b23bd200:2e40c9e35e9506f4-wpp.o
 0005:00001e30       WppLoadTracingSupport      0000000180032e30 f   libms_surface_wpp-b83efe80b23bd200:2e40c9e35e9506f4-wpp.o
 0005:00001f30       WppTraceCallback           0000000180032f30 f   libms_surface_wpp-b83efe80b23bd200:2e40c9e35e9506f4-wpp.o
 0005:000021a0       ?BufferPool_BufferPoolDestroy@@YAXPEAUDMFMODULE__@@@Z 00000001800331a0 f   DmfK:Dmf_BufferPool.obj
 0005:000023f0       DMF_BufferPool_Create      00000001800333f0 f   DmfK:Dmf_BufferPool.obj
 0005:00002650       ?DMF_SamCommunicationViaSsh_ChildModulesAdd@@YAXPEAUDMFMODULE__@@PEAU_DMF_MODULE_ATTRIBUTES@@PEAX@Z 0000000180033650 f   DmfK:Dmf_SamCommunicationViaSsh.obj
 0005:000027f0       DMF_SamCommunicationViaSsh_Create 00000001800337f0 f   DmfK:Dmf_SamCommunicationViaSsh.obj
 0005:000029e0       ?DMF_SynchronizationCreate@@YAJPEAU_DMF_OBJECT_@@E@Z 00000001800339e0 f   DmfK:DmfHelpers.obj
 0005:00002cc0       ?DMF_SamNotificationViaSsh_ChildModulesAdd@@YAXPEAUDMFMODULE__@@PEAU_DMF_MODULE_ATTRIBUTES@@PEAX@Z 0000000180033cc0 f   DmfK:Dmf_SamNotificationViaSsh.obj
 0005:0000315c       ?SamNotificationViaSsh_LegacyModeQueryAndSet@@YAXPEAUDMFMODULE__@@@Z 000000018003415c f   DmfK:Dmf_SamNotificationViaSsh.obj
 0005:00003530       DMF_SamNotificationViaSsh_Create 0000000180034530 f   DmfK:Dmf_SamNotificationViaSsh.obj
 0005:000037c0       ?DMF_QueuedWorkItem_ChildModulesAdd@@YAXPEAUDMFMODULE__@@PEAU_DMF_MODULE_ATTRIBUTES@@PEAX@Z 00000001800347c0 f   DmfK:Dmf_QueuedWorkItem.obj
 0005:000039b0       DMF_QueuedWorkItem_Create  00000001800349b0 f   DmfK:Dmf_QueuedWorkItem.obj
 0005:00003b98       ?DMF_ModuleCollectionArmWakeFromS0@@YAJPEAUDMFCOLLECTION__@@@Z 0000000180034b98 f   DmfK:DmfModuleCollection.obj
 0005:00003cb8       ?DMF_ModuleCollectionArmWakeFromSxWithReason@@YAJPEAUDMFCOLLECTION__@@EE@Z 0000000180034cb8 f   DmfK:DmfModuleCollection.obj
 0005:00003e20       ?DMF_ModuleCollectionConfigAddAttributes@@YAXPEAUDMF_MODULE_COLLECTION_CONFIG@@PEAU_DMF_MODULE_ATTRIBUTES@@PEAU_WDF_OBJECT_ATTRIBUTES@@PEAPEAUDMFMODULE__@@@Z 0000000180034e20 f   DmfK:DmfModuleCollection.obj
 0005:00004044       ?DMF_ModuleCollectionConfigListInitialize@@YAJPEAUDMF_MODULE_COLLECTION_CONFIG@@@Z 0000000180035044 f   DmfK:DmfModuleCollection.obj
 0005:000041cc       ?DMF_ModuleCollectionCreate@@YAJPEAUDMFDEVICE_INIT@@PEAUDMF_MODULE_COLLECTION_CONFIG@@PEAPEAUDMFCOLLECTION__@@@Z 00000001800351cc f   DmfK:DmfModuleCollection.obj
 0005:00004810       ?DMF_ModuleCollectionDisarmWakeFromS0@@YAXPEAUDMFCOLLECTION__@@@Z 0000000180035810 f   DmfK:DmfModuleCollection.obj
 0005:00004918       ?DMF_ModuleCollectionDisarmWakeFromSx@@YAXPEAUDMFCOLLECTION__@@@Z 0000000180035918 f   DmfK:DmfModuleCollection.obj
 0005:00004a20       ?DMF_ModuleCollectionFeatureHandleGet@@YAPEAU_DMF_OBJECT_@@PEAU_DMF_MODULE_COLLECTION_@@W4DmfFeatureType@@@Z 0000000180035a20 f   DmfK:DmfModuleCollection.obj
 0005:00004aa4       ?DMF_ModuleCollectionFileCleanup@@YAEPEAUDMFCOLLECTION__@@PEAUWDFFILEOBJECT__@@@Z 0000000180035aa4 f   DmfK:DmfModuleCollection.obj
 0005:00004c08       ?DMF_ModuleCollectionFileClose@@YAEPEAUDMFCOLLECTION__@@PEAUWDFFILEOBJECT__@@@Z 0000000180035c08 f   DmfK:DmfModuleCollection.obj
 0005:00004d6c       ?DMF_ModuleCollectionFileCreate@@YAEPEAUDMFCOLLECTION__@@PEAUWDFDEVICE__@@PEAUWDFREQUEST__@@PEAUWDFFILEOBJECT__@@@Z 0000000180035d6c f   DmfK:DmfModuleCollection.obj
 0005:00004ef0       ?DMF_ModuleCollectionHandlePropagate@@YAXPEAU_DMF_MODULE_COLLECTION_@@J@Z 0000000180035ef0 f   DmfK:DmfModuleCollection.obj
 0005:00004f30       ?DMF_ModuleCollectionHandleSet@@YAXPEAU_DMF_OBJECT_@@@Z 0000000180035f30 f   DmfK:DmfModuleCollection.obj
 0005:00004f70       ?DMF_ModuleCollectionPostCreate@@YAJPEAUDMF_MODULE_COLLECTION_CONFIG@@PEAUDMFCOLLECTION__@@@Z 0000000180035f70 f   DmfK:DmfModuleCollection.obj
 0005:000050a4       ?DMF_ModuleCollectionPrepareHardware@@YAJPEAUDMFCOLLECTION__@@PEAUWDFCMRESLIST__@@1@Z 00000001800360a4 f   DmfK:DmfModuleCollection.obj
 0005:0000527c       ?DMF_ModuleCollectionQueryRemove@@YAJPEAUDMFCOLLECTION__@@@Z 000000018003627c f   DmfK:DmfModuleCollection.obj
 0005:0000539c       ?DMF_ModuleCollectionQueryStop@@YAJPEAUDMFCOLLECTION__@@@Z 000000018003639c f   DmfK:DmfModuleCollection.obj
 0005:000054bc       ?DMF_ModuleCollectionRelationsQuery@@YAXPEAUDMFCOLLECTION__@@W4_DEVICE_RELATION_TYPE@@@Z 00000001800364bc f   DmfK:DmfModuleCollection.obj
 0005:0000560c       ?DMF_ModuleCollectionReleaseHardware@@YAJPEAUDMFCOLLECTION__@@PEAUWDFCMRESLIST__@@@Z 000000018003660c f   DmfK:DmfModuleCollection.obj
 0005:000057b8       ?DMF_ModuleCollectionSelfManagedIoCleanup@@YAXPEAUDMFCOLLECTION__@@@Z 00000001800367b8 f   DmfK:DmfModuleCollection.obj
 0005:000058c0       ?DMF_ModuleCollectionSelfManagedIoFlush@@YAXPEAUDMFCOLLECTION__@@@Z 00000001800368c0 f   DmfK:DmfModuleCollection.obj
 0005:000059c8       ?DMF_ModuleCollectionSelfManagedIoInit@@YAJPEAUDMFCOLLECTION__@@@Z 00000001800369c8 f   DmfK:DmfModuleCollection.obj
 0005:00005ae8       ?DMF_ModuleCollectionUsageNotificationEx@@YAJPEAUDMFCOLLECTION__@@W4_WDF_SPECIAL_FILE_TYPE@@E@Z 0000000180036ae8 f   DmfK:DmfModuleCollection.obj
 0005:00005c50       ?DMF_ModuleCollectionWakeFromS0Triggered@@YAXPEAUDMFCOLLECTION__@@@Z 0000000180036c50 f   DmfK:DmfModuleCollection.obj
 0005:00005d58       ?DMF_ModuleCollectionWakeFromSxTriggered@@YAXPEAUDMFCOLLECTION__@@@Z 0000000180036d58 f   DmfK:DmfModuleCollection.obj
 0005:00005e60       ?DMF_ModuleCollection_ModuleValidate@@YAEPEAU_DMF_OBJECT_@@@Z 0000000180036e60 f   DmfK:DmfModuleCollection.obj
 0005:00006088       DMF_DmfModuleAdd           0000000180037088 f   DmfK:DmfModuleCollection.obj
 0005:00006090       DMF_ModulesCreate          0000000180037090 f   DmfK:DmfModuleCollection.obj
 0005:00006530       ?DMF_SurfaceTelemetryConsentSettingsNotification_ChildModulesAdd@@YAXPEAUDMFMODULE__@@PEAU_DMF_MODULE_ATTRIBUTES@@PEAX@Z 0000000180037530 f   DmfK:Dmf_SurfaceTelemetryConsentSettingsNotification.obj
 0005:000066b0       DMF_SurfaceTelemetryConsentSettingsNotification_Create 00000001800376b0 f   DmfK:Dmf_SurfaceTelemetryConsentSettingsNotification.obj
 0005:00006898       ?DMF_DmfControlDeviceInitClientDriverDeviceGet@@YAPEAUWDFDEVICE__@@PEAUDMFDEVICE_INIT@@@Z 0000000180037898 f   DmfK:DmfDeviceInit.obj
 0005:000068a0       ?DMF_DmfDeviceInitBranchTrackModuleConfigGet@@YAPEAUDMF_CONFIG_BranchTrack@@PEAUDMFDEVICE_INIT@@@Z 00000001800378a0 f   DmfK:DmfDeviceInit.obj
 0005:000068a8       ?DMF_DmfDeviceInitBridgeModuleConfigGet@@YAPEAUDMF_CONFIG_Bridge@@PEAUDMFDEVICE_INIT@@@Z 00000001800378a8 f   DmfK:DmfDeviceInit.obj
 0005:000068b0       ?DMF_DmfDeviceInitClientImplementsDeviceAdd@@YAEPEAUDMFDEVICE_INIT@@@Z 00000001800378b0 f   DmfK:DmfDeviceInit.obj
 0005:000068b4       ?DMF_DmfDeviceInitDefaultQueueConfigGet@@YAPEAU_WDF_IO_QUEUE_CONFIG@@PEAUDMFDEVICE_INIT@@@Z 00000001800378b4 f   DmfK:DmfDeviceInit.obj
 0005:000068bc       ?DMF_DmfDeviceInitDefaultQueueObjectAttributesGet@@YAPEAU_WDF_OBJECT_ATTRIBUTES@@PEAUDMFDEVICE_INIT@@@Z 00000001800378bc f   DmfK:DmfDeviceInit.obj
 0005:000068c4       ?DMF_DmfDeviceInitDmfEventCallbacksGet@@YAPEAU_DMF_EVENT_CALLBACKS@@PEAUDMFDEVICE_INIT@@@Z 00000001800378c4 f   DmfK:DmfDeviceInit.obj
 0005:000068cc       ?DMF_DmfDeviceInitIsBridgeEnabled@@YAEPEAUDMFDEVICE_INIT@@@Z 00000001800378cc f   DmfK:DmfDeviceInit.obj
 0005:000068d0       ?DMF_DmfDeviceInitIsControlDevice@@YAEPEAUDMFDEVICE_INIT@@@Z 00000001800378d0 f   DmfK:DmfDeviceInit.obj
 0005:000068d8       ?DMF_DmfDeviceInitIsDefaultQueueCreated@@YAEPEAUDMFDEVICE_INIT@@@Z 00000001800378d8 f   DmfK:DmfDeviceInit.obj
 0005:000068dc       ?DMF_DmfDeviceInitIsFilterDriver@@YAEPEAUDMFDEVICE_INIT@@@Z 00000001800378dc f   DmfK:DmfDeviceInit.obj
 0005:000068e4       ?DMF_DmfDeviceInitLiveKernelDumpModuleConfigGet@@YAPEAUDMF_CONFIG_LiveKernelDump@@PEAUDMFDEVICE_INIT@@@Z 00000001800378e4 f   DmfK:DmfDeviceInit.obj
 0005:000068ec       ?DMF_DmfDeviceInitValidate@@YAEPEAUDMFDEVICE_INIT@@@Z 00000001800378ec f   DmfK:DmfDeviceInit.obj
 0005:00006a4c       DMF_DmfDeviceInitAllocate  0000000180037a4c f   DmfK:DmfDeviceInit.obj
 0005:00006dbc       DMF_DmfDeviceInitDisableWppRecorder 0000000180037dbc f   DmfK:DmfDeviceInit.obj
 0005:00006dc4       DMF_DmfDeviceInitHookFileObjectConfig 0000000180037dc4 f   DmfK:DmfDeviceInit.obj
 0005:00006e40       DMF_DmfDeviceInitHookPnpPowerEventCallbacks 0000000180037e40 f   DmfK:DmfDeviceInit.obj
 0005:00006f10       DMF_DmfDeviceInitHookPowerPolicyEventCallbacks 0000000180037f10 f   DmfK:DmfDeviceInit.obj
 0005:00006f84       DMF_DmfDeviceInitHookQueueConfig 0000000180037f84 f   DmfK:DmfDeviceInit.obj
 0005:00006fd4       DMF_DmfDeviceInitIsWppRecorderDisabled 0000000180037fd4 f   DmfK:DmfDeviceInit.obj
 0005:00006fdc       DMF_DmfDeviceInitSetEventCallbacks 0000000180037fdc f   DmfK:DmfDeviceInit.obj
 0005:00006ff0       ?LiveKernelDump_IoctlHandler@@YAJPEAUDMFMODULE__@@PEAUWDFQUEUE__@@PEAUWDFREQUEST__@@KPEAX_K34PEA_K@Z 0000000180037ff0 f   DmfK:Dmf_LiveKernelDump.obj
 0005:00007170       ?DMF_LiveKernelDump_ChildModulesAdd@@YAXPEAUDMFMODULE__@@PEAU_DMF_MODULE_ATTRIBUTES@@PEAX@Z 0000000180038170 f   DmfK:Dmf_LiveKernelDump.obj
 0005:00007568       ?LiveKernelDump_InsertClientTriageDataToLiveDump@@YAJPEAXKPEAULIVEKERNELDUMP_CLIENT_STRUCTURE@@@Z 0000000180038568 f   DmfK:Dmf_LiveKernelDump.obj
 0005:00007684       ?LiveKernelDump_InsertDmfTriageDataToLiveDump@@YAJPEAUDMFMODULE__@@PEAX@Z 0000000180038684 f   DmfK:Dmf_LiveKernelDump.obj
 0005:000078cc       ?LiveKernelDump_LiveKernelMemoryDumpCreate@@YAJPEAUDMFMODULE__@@K_KEKPEAULIVEKERNELDUMP_CLIENT_STRUCTURE@@KPEAX@Z 00000001800388cc f   DmfK:Dmf_LiveKernelDump.obj
 0005:00007be0       DMF_LiveKernelDump_Create  0000000180038be0 f   DmfK:Dmf_LiveKernelDump.obj
 0005:00007d90       DMF_LiveKernelDump_StoreDmfCollectionAsBugcheckParameter 0000000180038d90 f   DmfK:Dmf_LiveKernelDump.obj
 0005:00007f0c       DMF_Portable_EventWaitForSingleObject 0000000180038f0c f   DmfK:DmfPortable.obj
 0005:00008d08       DMF_ModuleCreate           0000000180039d08 f   DmfK:DmfCore.obj
 0005:000096a0       ?DMF_BranchTrack_ChildModulesAdd@@YAXPEAUDMFMODULE__@@PEAU_DMF_MODULE_ATTRIBUTES@@PEAX@Z 000000018003a6a0 f   DmfK:Dmf_BranchTrack.obj
 0005:00009d50       DMF_BranchTrack_Create     000000018003ad50 f   DmfK:Dmf_BranchTrack.obj
 0005:00009fb0       ?DMF_DeviceInterfaceTarget_ChildModulesAdd@@YAXPEAUDMFMODULE__@@PEAU_DMF_MODULE_ATTRIBUTES@@PEAX@Z 000000018003afb0 f   DmfK:Dmf_DeviceInterfaceTarget.obj
 0005:0000af60       DMF_DeviceInterfaceTarget_Create 000000018003bf60 f   DmfK:Dmf_DeviceInterfaceTarget.obj
 0005:0000b1dc       ?SmbiosWmi_Read@@YAJPEAUDMFMODULE__@@@Z 000000018003c1dc f   DmfK:Dmf_SmbiosWmi.obj
 0005:0000b500       DMF_SmbiosWmi_Create       000000018003c500 f   DmfK:Dmf_SmbiosWmi.obj
 0005:0000b668       DMF_File_FileExists        000000018003c668 f   DmfK:Dmf_File.obj
 0005:0000b7a8       DMF_File_Read              000000018003c7a8 f   DmfK:Dmf_File.obj
 0005:0000bb04       DMF_File_ReadEx            000000018003cb04 f   DmfK:Dmf_File.obj
 0005:0000bd30       ?DMF_BufferQueue_ChildModulesAdd@@YAXPEAUDMFMODULE__@@PEAU_DMF_MODULE_ATTRIBUTES@@PEAX@Z 000000018003cd30 f   DmfK:Dmf_BufferQueue.obj
 0005:0000c000       DMF_BufferQueue_Create     000000018003d000 f   DmfK:Dmf_BufferQueue.obj
 0005:0000c200       ?DMF_ScheduledTask_ChildModulesAdd@@YAXPEAUDMFMODULE__@@PEAU_DMF_MODULE_ATTRIBUTES@@PEAX@Z 000000018003d200 f   DmfK:Dmf_ScheduledTask.obj
 0005:0000ca60       ?ScheduledTask_ClientWorkDo@@YA?AW4ScheduledTask_Result_Type@@PEAUDMFMODULE__@@PEAXW4_WDF_POWER_DEVICE_STATE@@@Z 000000018003da60 f   DmfK:Dmf_ScheduledTask.obj
 0005:0000cdc0       ?ScheduledTask_DeferredHandlerOnDemand@@YAXPEAUWDFWORKITEM__@@@Z 000000018003ddc0 f   DmfK:Dmf_ScheduledTask.obj
 0005:0000cf70       ?ScheduledTask_TimerHandler@@YAXPEAUWDFTIMER__@@@Z 000000018003df70 f   DmfK:Dmf_ScheduledTask.obj
 0005:0000d09c       DMF_ScheduledTask_Cancel   000000018003e09c f   DmfK:Dmf_ScheduledTask.obj
 0005:0000d1f0       DMF_ScheduledTask_Create   000000018003e1f0 f   DmfK:Dmf_ScheduledTask.obj
 0005:0000d498       DMF_ScheduledTask_TimesRunGet 000000018003e498 f   DmfK:Dmf_ScheduledTask.obj
 0005:0000d69c       DMF_ScheduledTask_TimesRunSet 000000018003e69c f   DmfK:Dmf_ScheduledTask.obj
 0005:0000d884       ?DMF_ContainerFileObjectConfigInit@@YAXPEAU_WDF_FILEOBJECT_CONFIG@@@Z 000000018003e884 f   DmfK:DmfContainer.obj
 0005:0000d8bc       ?DMF_ContainerPnpPowerCallbacksInit@@YAXPEAU_WDF_PNPPOWER_EVENT_CALLBACKS@@@Z 000000018003e8bc f   DmfK:DmfContainer.obj
 0005:0000d974       ?DMF_ContainerPowerPolicyCallbacksInit@@YAXPEAU_WDF_POWER_POLICY_EVENT_CALLBACKS@@@Z 000000018003e974 f   DmfK:DmfContainer.obj
 0005:0000d9b8       ?DMF_ContainerQueueConfigCallbacksInit@@YAXPEAU_WDF_IO_QUEUE_CONFIG@@@Z 000000018003e9b8 f   DmfK:DmfContainer.obj
 0005:0000d9e8       DMF_Invoke_DeviceCallbacksDestroy 000000018003e9e8 f   DmfK:DmfContainer.obj
 0005:0000dba0       DmfContainerEvtDeviceArmWakeFromS0 000000018003eba0 f   DmfK:DmfContainer.obj
 0005:0000dc70       DmfContainerEvtDeviceArmWakeFromSxWithReason 000000018003ec70 f   DmfK:DmfContainer.obj
 0005:0000dd60       DmfContainerEvtDeviceDisarmWakeFromS0 000000018003ed60 f   DmfK:DmfContainer.obj
 0005:0000de20       DmfContainerEvtDeviceDisarmWakeFromSx 000000018003ee20 f   DmfK:DmfContainer.obj
 0005:0000dee0       DmfContainerEvtDevicePrepareHardware 000000018003eee0 f   DmfK:DmfContainer.obj
 0005:0000e000       DmfContainerEvtDeviceQueryRemove 000000018003f000 f   DmfK:DmfContainer.obj
 0005:0000e0d0       DmfContainerEvtDeviceQueryStop 000000018003f0d0 f   DmfK:DmfContainer.obj
 0005:0000e1a0       DmfContainerEvtDeviceRelationsQuery 000000018003f1a0 f   DmfK:DmfContainer.obj
 0005:0000e270       DmfContainerEvtDeviceReleaseHardware 000000018003f270 f   DmfK:DmfContainer.obj
 0005:0000e390       DmfContainerEvtDeviceSelfManagedIoCleanup 000000018003f390 f   DmfK:DmfContainer.obj
 0005:0000e450       DmfContainerEvtDeviceSelfManagedIoFlush 000000018003f450 f   DmfK:DmfContainer.obj
 0005:0000e510       DmfContainerEvtDeviceSelfManagedIoInit 000000018003f510 f   DmfK:DmfContainer.obj
 0005:0000e5e0       DmfContainerEvtDeviceUsageNotificationEx 000000018003f5e0 f   DmfK:DmfContainer.obj
 0005:0000e6d0       DmfContainerEvtDeviceWakeFromS0Triggered 000000018003f6d0 f   DmfK:DmfContainer.obj
 0005:0000e790       DmfContainerEvtDeviceWakeFromSxTriggered 000000018003f790 f   DmfK:DmfContainer.obj
 0005:0000e850       DmfContainerEvtFileCleanup 000000018003f850 f   DmfK:DmfContainer.obj
 0005:0000e990       DmfContainerEvtFileClose   000000018003f990 f   DmfK:DmfContainer.obj
 0005:0000eac0       DmfContainerEvtFileCreate  000000018003fac0 f   DmfK:DmfContainer.obj
 0005:0000ebf0       ?Bridge_DefaultEvtDeviceArmWakeFromS0@@YAJPEAUWDFDEVICE__@@@Z 000000018003fbf0 f   DmfK:Dmf_Bridge.obj
 0005:0000ec90       ?Bridge_DefaultEvtDeviceArmWakeFromSxWithReason@@YAJPEAUWDFDEVICE__@@EE@Z 000000018003fc90 f   DmfK:Dmf_Bridge.obj
 0005:0000ed30       ?Bridge_DefaultEvtDeviceDisarmWakeFromS0@@YAXPEAUWDFDEVICE__@@@Z 000000018003fd30 f   DmfK:Dmf_Bridge.obj
 0005:0000edc0       ?Bridge_DefaultEvtDeviceDisarmWakeFromSx@@YAXPEAUWDFDEVICE__@@@Z 000000018003fdc0 f   DmfK:Dmf_Bridge.obj
 0005:0000ee50       ?Bridge_DefaultEvtDevicePrepareHardware@@YAJPEAUWDFDEVICE__@@PEAUWDFCMRESLIST__@@1@Z 000000018003fe50 f   DmfK:Dmf_Bridge.obj
 0005:0000eef0       ?Bridge_DefaultEvtDeviceQueryRemove@@YAJPEAUWDFDEVICE__@@@Z 000000018003fef0 f   DmfK:Dmf_Bridge.obj
 0005:0000ef90       ?Bridge_DefaultEvtDeviceQueryStop@@YAJPEAUWDFDEVICE__@@@Z 000000018003ff90 f   DmfK:Dmf_Bridge.obj
 0005:0000f030       ?Bridge_DefaultEvtDeviceRelationsQuery@@YAXPEAUWDFDEVICE__@@W4_DEVICE_RELATION_TYPE@@@Z 0000000180040030 f   DmfK:Dmf_Bridge.obj
 0005:0000f0c0       ?Bridge_DefaultEvtDeviceReleaseHardware@@YAJPEAUWDFDEVICE__@@PEAUWDFCMRESLIST__@@@Z 00000001800400c0 f   DmfK:Dmf_Bridge.obj
 0005:0000f160       ?Bridge_DefaultEvtDeviceSelfManagedIoCleanup@@YAXPEAUWDFDEVICE__@@@Z 0000000180040160 f   DmfK:Dmf_Bridge.obj
 0005:0000f1f0       ?Bridge_DefaultEvtDeviceSelfManagedIoFlush@@YAXPEAUWDFDEVICE__@@@Z 00000001800401f0 f   DmfK:Dmf_Bridge.obj
 0005:0000f280       ?Bridge_DefaultEvtDeviceSelfManagedIoInit@@YAJPEAUWDFDEVICE__@@@Z 0000000180040280 f   DmfK:Dmf_Bridge.obj
 0005:0000f320       ?Bridge_DefaultEvtDeviceUsageNotificationEx@@YAJPEAUWDFDEVICE__@@W4_WDF_SPECIAL_FILE_TYPE@@E@Z 0000000180040320 f   DmfK:Dmf_Bridge.obj
 0005:0000f3c0       ?Bridge_DefaultEvtDeviceWakeFromS0Triggered@@YAXPEAUWDFDEVICE__@@@Z 00000001800403c0 f   DmfK:Dmf_Bridge.obj
 0005:0000f450       ?Bridge_DefaultEvtDeviceWakeFromSxTriggered@@YAXPEAUWDFDEVICE__@@@Z 0000000180040450 f   DmfK:Dmf_Bridge.obj
 0005:00010c60       DMF_Bridge_Create          0000000180041c60 f   DmfK:Dmf_Bridge.obj
 0005:00010f58       ?DMF_ModuleBranchTrack_HasClientEnabledBranchTrack@@YAKPEAUWDFDEVICE__@@@Z 0000000180041f58 f   DmfK:DmfBranchTrack.obj
 0005:00011100       ?DMF_ModuleBranchTrack_ModuleCollectionInitialize@@YAXPEAU_DMF_MODULE_COLLECTION_@@@Z 0000000180042100 f   DmfK:DmfBranchTrack.obj
 0005:00011144       ?DMF_ModuleBranchTrack_ModuleInitialize@@YAXPEAU_DMF_OBJECT_@@@Z 0000000180042144 f   DmfK:DmfBranchTrack.obj
 0005:0001118c       ?DMF_LiveKernelDump_ModuleInitialize@@YAXPEAU_DMF_OBJECT_@@@Z 000000018004218c f   DmfK:DmfLiveKernelDump.obj
 0005:000112cc       ?DMF_ModuleLiveKernelDump_ModuleCollectionInitialize@@YAXPEAU_DMF_MODULE_COLLECTION_@@@Z 00000001800422cc f   DmfK:DmfLiveKernelDump.obj
 0005:00011410       ?DMF_Generic_AuxiliaryLock_Passive@@YAXPEAUDMFMODULE__@@K@Z 0000000180042410 f   DmfK:DmfGeneric.obj
 0005:00011490       ?DMF_Generic_AuxiliaryUnlock_Passive@@YAXPEAUDMFMODULE__@@K@Z 0000000180042490 f   DmfK:DmfGeneric.obj
 0005:00011510       ?DMF_Generic_ChildModulesAdd@@YAXPEAUDMFMODULE__@@PEAU_DMF_MODULE_ATTRIBUTES@@PEAX@Z 0000000180042510 f   DmfK:DmfGeneric.obj
 0005:00011610       ?DMF_Generic_Close@@YAXPEAUDMFMODULE__@@@Z 0000000180042610 f   DmfK:DmfGeneric.obj
 0005:00011710       ?DMF_Generic_Lock_Passive@@YAXPEAUDMFMODULE__@@@Z 0000000180042710 f   DmfK:DmfGeneric.obj
 0005:00011720       ?DMF_Generic_ModuleArmWakeFromS0@@YAJPEAUDMFMODULE__@@@Z 0000000180042720 f   DmfK:DmfGeneric.obj
 0005:00011810       ?DMF_Generic_ModuleArmWakeFromSxWithReason@@YAJPEAUDMFMODULE__@@EE@Z 0000000180042810 f   DmfK:DmfGeneric.obj
 0005:00011900       ?DMF_Generic_ModuleDisarmWakeFromS0@@YAXPEAUDMFMODULE__@@@Z 0000000180042900 f   DmfK:DmfGeneric.obj
 0005:000119f0       ?DMF_Generic_ModuleDisarmWakeFromSx@@YAXPEAUDMFMODULE__@@@Z 00000001800429f0 f   DmfK:DmfGeneric.obj
 0005:00011ae0       ?DMF_Generic_ModuleFileCleanup@@YAEPEAUDMFMODULE__@@PEAUWDFFILEOBJECT__@@@Z 0000000180042ae0 f   DmfK:DmfGeneric.obj
 0005:00011bd0       ?DMF_Generic_ModuleFileClose@@YAEPEAUDMFMODULE__@@PEAUWDFFILEOBJECT__@@@Z 0000000180042bd0 f   DmfK:DmfGeneric.obj
 0005:00011cc0       ?DMF_Generic_ModuleFileCreate@@YAEPEAUDMFMODULE__@@PEAUWDFDEVICE__@@PEAUWDFREQUEST__@@PEAUWDFFILEOBJECT__@@@Z 0000000180042cc0 f   DmfK:DmfGeneric.obj
 0005:00011db0       ?DMF_Generic_ModulePrepareHardware@@YAJPEAUDMFMODULE__@@PEAUWDFCMRESLIST__@@1@Z 0000000180042db0 f   DmfK:DmfGeneric.obj
 0005:00011fc0       ?DMF_Generic_ModuleQueryRemove@@YAJPEAUDMFMODULE__@@@Z 0000000180042fc0 f   DmfK:DmfGeneric.obj
 0005:000120b0       ?DMF_Generic_ModuleQueryStop@@YAJPEAUDMFMODULE__@@@Z 00000001800430b0 f   DmfK:DmfGeneric.obj
 0005:000121a0       ?DMF_Generic_ModuleRelationsQuery@@YAXPEAUDMFMODULE__@@W4_DEVICE_RELATION_TYPE@@@Z 00000001800431a0 f   DmfK:DmfGeneric.obj
 0005:00012290       ?DMF_Generic_ModuleReleaseHardware@@YAJPEAUDMFMODULE__@@PEAUWDFCMRESLIST__@@@Z 0000000180043290 f   DmfK:DmfGeneric.obj
 0005:000123f0       ?DMF_Generic_ModuleSelfManagedIoCleanup@@YAXPEAUDMFMODULE__@@@Z 00000001800433f0 f   DmfK:DmfGeneric.obj
 0005:000124e0       ?DMF_Generic_ModuleSelfManagedIoFlush@@YAXPEAUDMFMODULE__@@@Z 00000001800434e0 f   DmfK:DmfGeneric.obj
 0005:000125d0       ?DMF_Generic_ModuleSelfManagedIoInit@@YAJPEAUDMFMODULE__@@@Z 00000001800435d0 f   DmfK:DmfGeneric.obj
 0005:000126c0       ?DMF_Generic_ModuleUsageNotificationEx@@YAJPEAUDMFMODULE__@@W4_WDF_SPECIAL_FILE_TYPE@@E@Z 00000001800436c0 f   DmfK:DmfGeneric.obj
 0005:000127b0       ?DMF_Generic_ModuleWakeFromS0Triggered@@YAXPEAUDMFMODULE__@@@Z 00000001800437b0 f   DmfK:DmfGeneric.obj
 0005:000128a0       ?DMF_Generic_ModuleWakeFromSxTriggered@@YAXPEAUDMFMODULE__@@@Z 00000001800438a0 f   DmfK:DmfGeneric.obj
 0005:00012990       ?DMF_Generic_NotificationRegister@@YAJPEAUDMFMODULE__@@@Z 0000000180043990 f   DmfK:DmfGeneric.obj
 0005:00012a90       ?DMF_Generic_NotificationUnregister@@YAXPEAUDMFMODULE__@@@Z 0000000180043a90 f   DmfK:DmfGeneric.obj
 0005:00012b90       ?DMF_Generic_Open@@YAJPEAUDMFMODULE__@@@Z 0000000180043b90 f   DmfK:DmfGeneric.obj
 0005:00012c90       ?DMF_Generic_ResourcesAssign@@YAJPEAUDMFMODULE__@@PEAUWDFCMRESLIST__@@1@Z 0000000180043c90 f   DmfK:DmfGeneric.obj
 0005:00012d90       ?DMF_Generic_Unlock_Passive@@YAXPEAUDMFMODULE__@@@Z 0000000180043d90 f   DmfK:DmfGeneric.obj
 0005:00012da0       ?EVT_DMF_MODULE_Generic_OnDeviceNotificationPostOpen@@YAXPEAUDMFMODULE__@@@Z 0000000180043da0 f   DmfK:DmfGeneric.obj
 0005:00012e50       ?EVT_DMF_MODULE_Generic_OnDeviceNotificationPreClose@@YAXPEAUDMFMODULE__@@@Z 0000000180043e50 f   DmfK:DmfGeneric.obj
 0005:00013c60       ?IoctlHandler_DeviceInterfaceCreate@@YAJPEAUDMFMODULE__@@@Z 0000000180044c60 f   DmfK:Dmf_IoctlHandler.obj
 0005:00013df0       DMF_IoctlHandler_Create    0000000180044df0 f   DmfK:Dmf_IoctlHandler.obj
 0005:00014074       LkmdTelCloseHandle         0000000180045074 f   DmfK:lkmdtel.obj
 0005:000140bc       LkmdTelCreateReport        00000001800450bc f   DmfK:lkmdtel.obj
 0005:000142cc       LkmdTelSetSecondaryData    00000001800452cc f   DmfK:lkmdtel.obj
 0005:00014340       LkmdTelSubmitReport        0000000180045340 f   DmfK:lkmdtel.obj
 0005:00014418       LkmdTelpAllocateMem        0000000180045418 f   DmfK:lkmdtel.obj
 0005:0001443c       LkmdTelpGetRegistryKey     000000018004543c f   DmfK:lkmdtel.obj
 0005:000144ec       LkmdTelpGetRegistryUlongValue 00000001800454ec f   DmfK:lkmdtel.obj
 0005:000145b8       LkmdTelpSetMaxSize         00000001800455b8 f   DmfK:lkmdtel.obj
 0005:00014690       LkmdTelpWriteDumpFile      0000000180045690 f   DmfK:lkmdtel.obj
 0005:00014a40       DMF_RingBuffer_Create      0000000180045a40 f   DmfK:Dmf_RingBuffer.obj
 0005:00014bf0       ?CrashDump_IoctlHandler@@YAJPEAUDMFMODULE__@@PEAUWDFQUEUE__@@PEAUWDFREQUEST__@@KPEAX_K34PEA_K@Z 0000000180045bf0 f   DmfK:Dmf_CrashDump.obj
 0005:00014e04       ?CrashDump_DataSourceCaptureAuxiliary@@YAJPEAUDMFMODULE__@@PEAUWDFFILEOBJECT__@@PEAEKPEAK@Z 0000000180045e04 f   DmfK:Dmf_CrashDump.obj
 0005:00015098       ?CrashDump_DataSourceCreateAuxiliary@@YAJPEAUDMFMODULE__@@PEAUWDFFILEOBJECT__@@KKPEBU_GUID@@@Z 0000000180046098 f   DmfK:Dmf_CrashDump.obj
 0005:000156c8       ?CrashDump_DataSourceCreateSelf@@YAJPEAUDMFMODULE__@@KKPEBU_GUID@@@Z 00000001800466c8 f   DmfK:Dmf_CrashDump.obj
 0005:000157e8       ?CrashDump_DataSourceDestroyAuxiliary@@YAJPEAUDMFMODULE__@@PEAUWDFFILEOBJECT__@@@Z 00000001800467e8 f   DmfK:Dmf_CrashDump.obj
 0005:000158e4       ?CrashDump_DataSourceDestroyAuxiliaryInternal@@YAJPEAUDMFMODULE__@@PEAUWDFFILEOBJECT__@@@Z 00000001800468e4 f   DmfK:Dmf_CrashDump.obj
 0005:00015a28       ?CrashDump_DataSourceDestroySelf@@YAJPEAUDMFMODULE__@@@Z 0000000180046a28 f   DmfK:Dmf_CrashDump.obj
 0005:00015afc       ?CrashDump_DataSourceOpenAuxiliary@@YAJPEAUDMFMODULE__@@PEAUWDFFILEOBJECT__@@PEAKPEBU_GUID@@@Z 0000000180046afc f   DmfK:Dmf_CrashDump.obj
 0005:00015f04       ?CrashDump_DataSourceOrphanCreate@@YAXPEAUDMFMODULE__@@PEAUWDFFILEOBJECT__@@@Z 0000000180046f04 f   DmfK:Dmf_CrashDump.obj
 0005:00016034       ?CrashDump_DataSourceReadAuxiliary@@YAJPEAUDMFMODULE__@@PEAUWDFFILEOBJECT__@@PEAEK@Z 0000000180047034 f   DmfK:Dmf_CrashDump.obj
 0005:000162b4       ?CrashDump_DataSourceWriteAuxiliary@@YAJPEAUDMFMODULE__@@PEAUWDFFILEOBJECT__@@PEAEK@Z 00000001800472b4 f   DmfK:Dmf_CrashDump.obj
 0005:00016940       ?CrashDump_TriageDataCreateInternal@@YAJPEAUDMFMODULE__@@@Z 0000000180047940 f   DmfK:Dmf_CrashDump.obj
 0005:00016ce0       ?DMF_CrashDump_ChildModulesAdd@@YAXPEAUDMFMODULE__@@PEAU_DMF_MODULE_ATTRIBUTES@@PEAX@Z 0000000180047ce0 f   DmfK:Dmf_CrashDump.obj
 0005:00017180       ?DMF_CrashDump_FileClose@@YAEPEAUDMFMODULE__@@PEAUWDFFILEOBJECT__@@@Z 0000000180048180 f   DmfK:Dmf_CrashDump.obj
 0005:00017610       DMF_CrashDump_Create       0000000180048610 f   DmfK:Dmf_CrashDump.obj
 0005:00017900       ?DMF_Internal_ModuleArmWakeFromS0@@YAJPEAUDMFMODULE__@@@Z 0000000180048900 f   DmfK:DmfInternal.obj
 0005:00017a10       ?DMF_Internal_ModuleArmWakeFromSxWithReason@@YAJPEAUDMFMODULE__@@EE@Z 0000000180048a10 f   DmfK:DmfInternal.obj
 0005:00017b30       ?DMF_Internal_ModuleDisarmWakeFromS0@@YAXPEAUDMFMODULE__@@@Z 0000000180048b30 f   DmfK:DmfInternal.obj
 0005:00017c30       ?DMF_Internal_ModuleDisarmWakeFromSx@@YAXPEAUDMFMODULE__@@@Z 0000000180048c30 f   DmfK:DmfInternal.obj
 0005:00017d30       ?DMF_Internal_ModuleFileCleanup@@YAEPEAUDMFMODULE__@@PEAUWDFFILEOBJECT__@@@Z 0000000180048d30 f   DmfK:DmfInternal.obj
 0005:00017e50       ?DMF_Internal_ModuleFileClose@@YAEPEAUDMFMODULE__@@PEAUWDFFILEOBJECT__@@@Z 0000000180048e50 f   DmfK:DmfInternal.obj
 0005:00017f70       ?DMF_Internal_ModuleFileCreate@@YAEPEAUDMFMODULE__@@PEAUWDFDEVICE__@@PEAUWDFREQUEST__@@PEAUWDFFILEOBJECT__@@@Z 0000000180048f70 f   DmfK:DmfInternal.obj
 0005:000180a0       ?DMF_Internal_ModulePrepareHardware@@YAJPEAUDMFMODULE__@@PEAUWDFCMRESLIST__@@1@Z 00000001800490a0 f   DmfK:DmfInternal.obj
 0005:000181c0       ?DMF_Internal_ModuleQueryRemove@@YAJPEAUDMFMODULE__@@@Z 00000001800491c0 f   DmfK:DmfInternal.obj
 0005:000182d0       ?DMF_Internal_ModuleQueryStop@@YAJPEAUDMFMODULE__@@@Z 00000001800492d0 f   DmfK:DmfInternal.obj
 0005:000183e0       ?DMF_Internal_ModuleRelationsQuery@@YAXPEAUDMFMODULE__@@W4_DEVICE_RELATION_TYPE@@@Z 00000001800493e0 f   DmfK:DmfInternal.obj
 0005:000184f0       ?DMF_Internal_ModuleReleaseHardware@@YAJPEAUDMFMODULE__@@PEAUWDFCMRESLIST__@@@Z 00000001800494f0 f   DmfK:DmfInternal.obj
 0005:00018610       ?DMF_Internal_ModuleSelfManagedIoCleanup@@YAXPEAUDMFMODULE__@@@Z 0000000180049610 f   DmfK:DmfInternal.obj
 0005:00018710       ?DMF_Internal_ModuleSelfManagedIoFlush@@YAXPEAUDMFMODULE__@@@Z 0000000180049710 f   DmfK:DmfInternal.obj
 0005:00018810       ?DMF_Internal_ModuleSelfManagedIoInit@@YAJPEAUDMFMODULE__@@@Z 0000000180049810 f   DmfK:DmfInternal.obj
 0005:00018920       ?DMF_Internal_ModuleUsageNotificationEx@@YAJPEAUDMFMODULE__@@W4_WDF_SPECIAL_FILE_TYPE@@E@Z 0000000180049920 f   DmfK:DmfInternal.obj
 0005:00018a40       ?DMF_Internal_ModuleWakeFromS0Triggered@@YAXPEAUDMFMODULE__@@@Z 0000000180049a40 f   DmfK:DmfInternal.obj
 0005:00018b40       ?DMF_Internal_ModuleWakeFromSxTriggered@@YAXPEAUDMFMODULE__@@@Z 0000000180049b40 f   DmfK:DmfInternal.obj
 0005:00018c40       ?DMF_Internal_NotificationRegister@@YAJPEAUDMFMODULE__@@@Z 0000000180049c40 f   DmfK:DmfInternal.obj
 0005:00018d50       ?DMF_Internal_NotificationUnregister@@YAXPEAUDMFMODULE__@@@Z 0000000180049d50 f   DmfK:DmfInternal.obj
 0005:00018e50       ?DMF_Internal_ResourcesAssign@@YAJPEAUDMFMODULE__@@PEAUWDFCMRESLIST__@@1@Z 0000000180049e50 f   DmfK:DmfInternal.obj
 0005:00019510       DMF_HashTable_Create       000000018004a510 f   DmfK:Dmf_HashTable.obj
 0005:00019710       ?DMF_RequestTarget_ChildModulesAdd@@YAXPEAUDMFMODULE__@@PEAU_DMF_MODULE_ATTRIBUTES@@PEAX@Z 000000018004a710 f   DmfK:Dmf_RequestTarget.obj
 0005:00019c00       DMF_RequestTarget_Create   000000018004ac00 f   DmfK:Dmf_RequestTarget.obj
 0005:00019e00       ?DMF_ContinuousRequestTarget_ChildModulesAdd@@YAXPEAUDMFMODULE__@@PEAU_DMF_MODULE_ATTRIBUTES@@PEAX@Z 000000018004ae00 f   DmfK:Dmf_ContinuousRequestTarget.obj
 0005:0001a8d0       DMF_ContinuousRequestTarget_Create 000000018004b8d0 f   DmfK:Dmf_ContinuousRequestTarget.obj
 0005:0001acc0       DMF_Rundown_Create         000000018004bcc0 f   DmfK:Dmf_Rundown.obj
 0005:0001aec0       ??_C@_0L@HNDALOFD@BufferPool@NNGAKEGL@ 000000018004bec0     DmfK:Dmf_BufferPool.obj
 0005:0001aed0       ??_C@_0EJ@IPCLCLNF@REPOSITORYDIR?2SurfaceLibrary?2Ke@NNGAKEGL@ 000000018004bed0     DmfK:Dmf_BufferPool.obj
 0005:0001af20       ??_C@_0BO@MANCDNMF@Invalid?5Pool?1Lock?5combination@NNGAKEGL@ 000000018004bf20     DmfK:Dmf_BufferPool.obj
 0005:0001af40       ??_C@_0BH@ECHIDAPF@SamCommunicationViaSsh@NNGAKEGL@ 000000018004bf40     DmfK:Dmf_SamCommunicationViaSsh.obj
 0005:0001af60       ??_C@_0P@LBPDBOHH@Surface?5Laptop@NNGAKEGL@ 000000018004bf60     DmfK:Dmf_SamNotificationViaSsh.obj
 0005:0001af70       ??_C@_0M@NMIFGBBC@Surface?5Pro@NNGAKEGL@ 000000018004bf70     DmfK:Dmf_SamNotificationViaSsh.obj
 0005:0001af80       ??_C@_0P@IIIFKELK@Surface?5Book?52@NNGAKEGL@ 000000018004bf80     DmfK:Dmf_SamNotificationViaSsh.obj
 0005:0001af90       ??_C@_0P@EIHHGGJI@OEMLA?5Product?5@NNGAKEGL@ 000000018004bf90     DmfK:Dmf_SamNotificationViaSsh.obj
 0005:0001afa0       ??_C@_0P@DKODPJOJ@OEMCA?5Product?5@NNGAKEGL@ 000000018004bfa0     DmfK:Dmf_SamNotificationViaSsh.obj
 0005:0001afb0       ??_C@_0P@HDINJPOP@OEMSHP?5Product@NNGAKEGL@ 000000018004bfb0     DmfK:Dmf_SamNotificationViaSsh.obj
 0005:0001afc0       ??_C@_0P@GEKPAPCG@OEMSHZ?5Product@NNGAKEGL@ 000000018004bfc0     DmfK:Dmf_SamNotificationViaSsh.obj
 0005:0001afd0       ??_C@_0BH@JNPAHNF@BufferPoolRegistration@NNGAKEGL@ 000000018004bfd0     DmfK:Dmf_SamNotificationViaSsh.obj
 0005:0001aff0       ??_C@_0FE@CFNMELEB@REPOSITORYDIR?2SurfaceLibrary?2Ke@NNGAKEGL@ 000000018004bff0     DmfK:Dmf_SamNotificationViaSsh.obj
 0005:0001b050       ??_C@_09MLEKNIHI@more?5than@NNGAKEGL@ 000000018004c050     DmfK:Dmf_SamNotificationViaSsh.obj
 0005:0001b060       ??_C@_0EO@KDNCKFAP@SamNotificationViaSsh_ModuleD0E@NNGAKEGL@ 000000018004c060     DmfK:Dmf_SamNotificationViaSsh.obj
 0005:0001b0b0       ??_C@_08FNDBFMB@at?5least@NNGAKEGL@ 000000018004c0b0     DmfK:Dmf_SamNotificationViaSsh.obj
 0005:0001b0c0       ??_C@_0FG@FBCHJGP@SamNotificationViaSsh_ModuleD0E@NNGAKEGL@ 000000018004c0c0     DmfK:Dmf_SamNotificationViaSsh.obj
 0005:0001b120       ??_C@_0GA@HFAFKBD@SamNotificationViaSsh_Streaming@NNGAKEGL@ 000000018004c120     DmfK:Dmf_SamNotificationViaSsh.obj
 0005:0001b180       ??_C@_0GI@GKOPJLLO@SamNotificationViaSsh_Streaming@NNGAKEGL@ 000000018004c180     DmfK:Dmf_SamNotificationViaSsh.obj
 0005:0001b1f0       ??_C@_0GI@MLIDADOC@SamNotificationViaSsh_OnDeviceA@NNGAKEGL@ 000000018004c1f0     DmfK:Dmf_SamNotificationViaSsh.obj
 0005:0001b260       ??_C@_0FF@NNGNAPBD@DMF_SamNotificationViaSsh_Open?4@NNGAKEGL@ 000000018004c260     DmfK:Dmf_SamNotificationViaSsh.obj
 0005:0001b2c0       ??_C@_0BG@NNECKFAN@SamNotificationViaSsh@NNGAKEGL@ 000000018004c2c0     DmfK:Dmf_SamNotificationViaSsh.obj
 0005:0001b2e0       ??_C@_0P@OPFKONC@QueuedWorkItem@NNGAKEGL@ 000000018004c2e0     DmfK:Dmf_QueuedWorkItem.obj
 0005:0001b2f0       ??_C@_0M@OJIKMFFC@BranchTrack@NNGAKEGL@ 000000018004c2f0     DmfK:DmfModuleCollection.obj
 0005:0001b300       ??_C@_0P@MOMAMNCN@LiveKernelDump@NNGAKEGL@ 000000018004c300     DmfK:DmfModuleCollection.obj
 0005:0001b310       ??_C@_0CM@LDEHPPLA@SurfaceTelemetryConsentSettings@NNGAKEGL@ 000000018004c310     DmfK:Dmf_SurfaceTelemetryConsentSettingsNotification.obj
 0005:0001b340       ??_C@_0BB@KGCEIKCH@DataBufferSource@NNGAKEGL@ 000000018004c340     DmfK:Dmf_LiveKernelDump.obj
 0005:0001b360       ??_C@_0BK@OEFLKDBD@LiveKernelDumpBufferQueue@NNGAKEGL@ 000000018004c360     DmfK:Dmf_LiveKernelDump.obj
 0005:0001b380       ??_C@_03BEKMBJJJ@DMF@NNGAKEGL@ 000000018004c380     DmfK:Dmf_LiveKernelDump.obj
 0005:0001b390       ??_C@_0DM@DHNCJMAI@REPOSITORYDIR?2SurfaceLibrary?2Ke@NNGAKEGL@ 000000018004c390     DmfK:DmfCore.obj
 0005:0001b3d0       ??_C@_00CNPNBAHC@@NNGAKEGL@ 000000018004c3d0     DmfK:DmfCore.obj
 0005:0001b3e0       ??_C@_0BC@PDIABCOE@BufferPoolContext@NNGAKEGL@ 000000018004c3e0     DmfK:Dmf_DeviceInterfaceTarget.obj
 0005:0001b400       ??_C@_0BG@GAACGJFO@DeviceInterfaceTarget@NNGAKEGL@ 000000018004c400     DmfK:Dmf_DeviceInterfaceTarget.obj
 0005:0001b420       ??_C@_09IKKAPKNH@SmbiosWmi@NNGAKEGL@ 000000018004c420     DmfK:Dmf_SmbiosWmi.obj
 0005:0001b430       ??_C@_0BD@JHNDGADN@BufferPoolProducer@NNGAKEGL@ 000000018004c430     DmfK:Dmf_BufferQueue.obj
 0005:0001b450       ??_C@_0BD@LNFLHENH@BufferPoolConsumer@NNGAKEGL@ 000000018004c450     DmfK:Dmf_BufferQueue.obj
 0005:0001b470       ??_C@_0M@HHNDILAP@BufferQueue@NNGAKEGL@ 000000018004c470     DmfK:Dmf_BufferQueue.obj
 0005:0001b480       ??_C@_0O@PIOKNKAA@ScheduledTask@NNGAKEGL@ 000000018004c480     DmfK:Dmf_ScheduledTask.obj
 0005:0001b490       ??_C@_1BC@OCOFHKJN@?$AAT?$AAi?$AAm?$AAe?$AAs?$AAR?$AAu?$AAn@NNGAKEGL@ 000000018004c490     DmfK:Dmf_ScheduledTask.obj
 0005:0001b4b0       ??_C@_06ICJJNPDE@Bridge@NNGAKEGL@ 000000018004c4b0     DmfK:Dmf_Bridge.obj
 0005:0001b4c0       ??_C@_1CG@DKCFLCEN@?$AAB?$AAr?$AAa?$AAn?$AAc?$AAh?$AAT?$AAr?$AAa?$AAc?$AAk?$AAE?$AAn?$AAa?$AAb@NNGAKEGL@ 000000018004c4c0     DmfK:DmfBranchTrack.obj
 0005:0001b4f0       ??_C@_0N@LHIGANIG@IoctlHandler@NNGAKEGL@ 000000018004c4f0     DmfK:Dmf_IoctlHandler.obj
 0005:0001b500       ??_C@_0L@EIGDGHH@RingBuffer@NNGAKEGL@ 000000018004c500     DmfK:Dmf_RingBuffer.obj
 0005:0001b510       ??_C@_0BF@IIHFOBJD@DataSourceRingBuffer@NNGAKEGL@ 000000018004c510     DmfK:Dmf_CrashDump.obj
 0005:0001b530       ??_C@_0CN@FAHGKGKP@?$CF08X?$CF04X?$CF04X?$CF02X?$CF02X?$CF02X?$CF02X?$CF02@NNGAKEGL@ 000000018004c530     DmfK:Dmf_CrashDump.obj
 0005:0001b560       ??_C@_1EA@PMDNBEFP@?$AAK?$AAe?$AAI?$AAn?$AAi?$AAt?$AAi?$AAa?$AAl?$AAi?$AAz?$AAe?$AAT?$AAr?$AAi@NNGAKEGL@ 000000018004c560     DmfK:Dmf_CrashDump.obj
 0005:0001b5a0       ??_C@_09MGJKIHP@CrashDump@NNGAKEGL@ 000000018004c5a0     DmfK:Dmf_CrashDump.obj
 0005:0001b5b0       ??_C@_09LLKDFHPJ@HashTable@NNGAKEGL@ 000000018004c5b0     DmfK:Dmf_HashTable.obj
 0005:0001b5c0       ??_C@_0O@CJADKEFG@RequestTarget@NNGAKEGL@ 000000018004c5c0     DmfK:Dmf_RequestTarget.obj
 0005:0001b5d0       ??_C@_0BA@EAOHEKME@BufferPoolInput@NNGAKEGL@ 000000018004c5d0     DmfK:Dmf_ContinuousRequestTarget.obj
 0005:0001b5e0       ??_C@_0BB@BOEHKGLG@BufferPoolOutput@NNGAKEGL@ 000000018004c5e0     DmfK:Dmf_ContinuousRequestTarget.obj
 0005:0001b600       ??_C@_0BI@OFGBOHBL@ContinuousRequestTarget@NNGAKEGL@ 000000018004c600     DmfK:Dmf_ContinuousRequestTarget.obj
 0005:0001b620       ??_C@_07KEEHELKP@Rundown@NNGAKEGL@ 000000018004c620     DmfK:Dmf_Rundown.obj
 0006:00000000       DMF_String_Create          000000018004d000 f   DmfK:Dmf_String.obj
 0006:000001a0       ??_C@_06ENNEIMBA@String@KLAMFNPN@ 000000018004d1a0     DmfK:Dmf_String.obj
 0008:00000000       DriverEntry                000000018004f000 f   surface_hid_mini.surface_hid_mini.3efcb60154bd7459-cgu.0.rcgu.o
 0008:00000618       __security_init_cookie     000000018004f618 f   BufferOverflowFastFailK:gs_support.obj
 0008:00000648       __IMPORT_DESCRIPTOR_ntoskrnl 000000018004f648     ntoskrnl:ntoskrnl.exe
 0008:0000065c       __IMPORT_DESCRIPTOR_ext-ms-win-ntos-werkernel-l1-1-1 000000018004f65c     DmfK:ext-ms-win-ntos-werkernel-l1-1-1.dll
 0008:00000670       __IMPORT_DESCRIPTOR_WppRecorder 000000018004f670     wpprecorder:WppRecorder.sys
 0008:00000684       __IMPORT_DESCRIPTOR_WDFLDR 000000018004f684     WdfLdr:WDFLDR.SYS
 0008:00000698       __NULL_IMPORT_DESCRIPTOR   000000018004f698     ntoskrnl:ntoskrnl.exe

 entry point at        0001:00005fe0

 Static symbols

 0000:fffae000       .debug$S                   0000000180000000     surface_hid_mini.dll.exp
 0002:fffd9000       __guard_fids__             0000000180000000     BufferOverflowFastFailK:guard_support.obj
 0002:fffd9000       __guard_fids__             0000000180000000     BufferOverflowFastFailK:guard_support.obj
 0002:fffd9000       __guard_fids__guard_icall_checks_enforced 0000000180000000     BufferOverflowFastFailK:guard_support.obj
 0000:fffae000       .debug$S                   0000000180000000     ntoskrnl:ntoskrnl.exe
 0000:fffae000       .debug$S                   0000000180000000     ntoskrnl:ntoskrnl.exe
 0000:fffae000       .debug$S                   0000000180000000     ntoskrnl:ntoskrnl.exe
 0000:fffae000       .debug$S                   0000000180000000     ntoskrnl:ntoskrnl.exe
 0000:fffae000       .debug$S                   0000000180000000     ntoskrnl:ntoskrnl.exe
 0000:fffae000       .debug$S                   0000000180000000     ntoskrnl:ntoskrnl.exe
 0000:fffae000       .debug$S                   0000000180000000     ntoskrnl:ntoskrnl.exe
 0000:fffae000       .debug$S                   0000000180000000     ntoskrnl:ntoskrnl.exe
 0000:fffae000       .debug$S                   0000000180000000     ntoskrnl:ntoskrnl.exe
 0000:fffae000       .debug$S                   0000000180000000     ntoskrnl:ntoskrnl.exe
 0000:fffae000       .debug$S                   0000000180000000     ntoskrnl:ntoskrnl.exe
 0000:fffae000       .debug$S                   0000000180000000     ntoskrnl:ntoskrnl.exe
 0000:fffae000       .debug$S                   0000000180000000     ntoskrnl:ntoskrnl.exe
 0000:fffae000       .debug$S                   0000000180000000     ntoskrnl:ntoskrnl.exe
 0000:fffae000       .debug$S                   0000000180000000     ntoskrnl:ntoskrnl.exe
 0000:fffae000       .debug$S                   0000000180000000     ntoskrnl:ntoskrnl.exe
 0000:fffae000       .debug$S                   0000000180000000     ntoskrnl:ntoskrnl.exe
 0000:fffae000       .debug$S                   0000000180000000     ntoskrnl:ntoskrnl.exe
 0000:fffae000       .debug$S                   0000000180000000     ntoskrnl:ntoskrnl.exe
 0000:fffae000       .debug$S                   0000000180000000     ntoskrnl:ntoskrnl.exe
 0000:fffae000       .debug$S                   0000000180000000     ntoskrnl:ntoskrnl.exe
 0000:fffae000       .debug$S                   0000000180000000     ntoskrnl:ntoskrnl.exe
 0000:fffae000       .debug$S                   0000000180000000     ntoskrnl:ntoskrnl.exe
 0000:fffae000       .debug$S                   0000000180000000     ntoskrnl:ntoskrnl.exe
 0000:fffae000       .debug$S                   0000000180000000     ntoskrnl:ntoskrnl.exe
 0000:fffae000       .debug$S                   0000000180000000     ntoskrnl:ntoskrnl.exe
 0000:fffae000       .debug$S                   0000000180000000     ntoskrnl:ntoskrnl.exe
 0000:fffae000       .debug$S                   0000000180000000     ntoskrnl:ntoskrnl.exe
 0000:fffae000       .debug$S                   0000000180000000     ntoskrnl:ntoskrnl.exe
 0000:fffae000       .debug$S                   0000000180000000     ntoskrnl:ntoskrnl.exe
 0000:fffae000       .debug$S                   0000000180000000     ntoskrnl:ntoskrnl.exe
 0000:fffae000       .debug$S                   0000000180000000     ntoskrnl:ntoskrnl.exe
 0000:fffae000       .debug$S                   0000000180000000     ntoskrnl:ntoskrnl.exe
 0000:fffae000       .debug$S                   0000000180000000     ntoskrnl:ntoskrnl.exe
 0000:fffae000       .debug$S                   0000000180000000     ntoskrnl:ntoskrnl.exe
 0000:fffae000       .debug$S                   0000000180000000     ntoskrnl:ntoskrnl.exe
 0000:fffae000       .debug$S                   0000000180000000     ntoskrnl:ntoskrnl.exe
 0000:fffae000       .debug$S                   0000000180000000     ntoskrnl:ntoskrnl.exe
 0000:fffae000       .debug$S                   0000000180000000     ntoskrnl:ntoskrnl.exe
 0000:fffae000       .debug$S                   0000000180000000     ntoskrnl:ntoskrnl.exe
 0000:fffae000       .debug$S                   0000000180000000     ntoskrnl:ntoskrnl.exe
 0000:fffae000       .debug$S                   0000000180000000     ntoskrnl:ntoskrnl.exe
 0000:fffae000       .debug$S                   0000000180000000     ntoskrnl:ntoskrnl.exe
 0000:fffae000       .debug$S                   0000000180000000     ntoskrnl:ntoskrnl.exe
 0000:fffae000       .debug$S                   0000000180000000     ntoskrnl:ntoskrnl.exe
 0000:fffae000       .debug$S                   0000000180000000     ntoskrnl:ntoskrnl.exe
 0000:fffae000       .debug$S                   0000000180000000     ntoskrnl:ntoskrnl.exe
 0000:fffae000       .debug$S                   0000000180000000     ntoskrnl:ntoskrnl.exe
 0000:fffae000       .debug$S                   0000000180000000     ntoskrnl:ntoskrnl.exe
 0000:fffae000       .debug$S                   0000000180000000     ntoskrnl:ntoskrnl.exe
 0000:fffae000       .debug$S                   0000000180000000     ntoskrnl:ntoskrnl.exe
 0000:fffae000       .debug$S                   0000000180000000     ntoskrnl:ntoskrnl.exe
 0000:fffae000       .debug$S                   0000000180000000     ntoskrnl:ntoskrnl.exe
 0000:fffae000       .debug$S                   0000000180000000     ntoskrnl:ntoskrnl.exe
 0000:fffae000       .debug$S                   0000000180000000     ntoskrnl:ntoskrnl.exe
 0000:fffae000       .debug$S                   0000000180000000     ntoskrnl:ntoskrnl.exe
 0000:fffae000       .debug$S                   0000000180000000     ntoskrnl:ntoskrnl.exe
 0000:fffae000       .debug$S                   0000000180000000     ntoskrnl:ntoskrnl.exe
 0000:fffae000       .debug$S                   0000000180000000     ntoskrnl:ntoskrnl.exe
 0000:fffae000       .debug$S                   0000000180000000     ntoskrnl:ntoskrnl.exe
 0000:fffae000       .debug$S                   0000000180000000     ntoskrnl:ntoskrnl.exe
 0000:fffae000       .debug$S                   0000000180000000     ntoskrnl:ntoskrnl.exe
 0000:fffae000       .debug$S                   0000000180000000     ntoskrnl:ntoskrnl.exe
 0000:fffae000       .debug$S                   0000000180000000     ntoskrnl:ntoskrnl.exe
 0000:fffae000       .debug$S                   0000000180000000     ntoskrnl:ntoskrnl.exe
 0000:fffae000       .debug$S                   0000000180000000     ntoskrnl:ntoskrnl.exe
 0000:fffae000       .debug$S                   0000000180000000     ntoskrnl:ntoskrnl.exe
 0000:fffae000       .debug$S                   0000000180000000     ntoskrnl:ntoskrnl.exe
 0000:fffae000       .debug$S                   0000000180000000     ntoskrnl:ntoskrnl.exe
 0000:fffae000       .debug$S                   0000000180000000     ntoskrnl:ntoskrnl.exe
 0000:fffae000       .debug$S                   0000000180000000     ntoskrnl:ntoskrnl.exe
 0000:fffae000       .debug$S                   0000000180000000     ntoskrnl:ntoskrnl.exe
 0000:fffae000       .debug$S                   0000000180000000     wpprecorder:WppRecorder.sys
 0000:fffae000       .debug$S                   0000000180000000     wpprecorder:WppRecorder.sys
 0000:fffae000       .debug$S                   0000000180000000     wpprecorder:WppRecorder.sys
 0000:fffae000       .debug$S                   0000000180000000     wpprecorder:WppRecorder.sys
 0000:fffae000       .debug$S                   0000000180000000     wpprecorder:WppRecorder.sys
 0000:fffae000       .debug$S                   0000000180000000     wpprecorder:WppRecorder.sys
 0000:fffae000       .debug$S                   0000000180000000     wpprecorder:WppRecorder.sys
 0000:fffae000       .debug$S                   0000000180000000     wpprecorder:WppRecorder.sys
 0002:fffd9000       __guard_fids_?FxStubBindClasses@@YAJPEAU_WDF_BIND_INFO@@@Z 0000000180000000     WdfDriverEntry:classbind.obj
 0002:fffd9000       __guard_fids_?FxStubUnbindClasses@@YAXPEAU_WDF_BIND_INFO@@@Z 0000000180000000     WdfDriverEntry:classbind.obj
 0002:fffd9000       __guard_fids_FxDriverEntryWorker 0000000180000000     WdfDriverEntry:stub.obj
 0002:fffd9000       __guard_fids_FxStubDriverUnload 0000000180000000     WdfDriverEntry:stub.obj
 0000:fffae000       .debug$S                   0000000180000000     WdfLdr:WDFLDR.SYS
 0000:fffae000       .debug$S                   0000000180000000     WdfLdr:WDFLDR.SYS
 0000:fffae000       .debug$S                   0000000180000000     WdfLdr:WDFLDR.SYS
 0000:fffae000       .debug$S                   0000000180000000     WdfLdr:WDFLDR.SYS
 0000:fffae000       .debug$S                   0000000180000000     WdfLdr:WDFLDR.SYS
 0002:fffd9000       __guard_fids_?DMF_ModuleTreeDestroy@@YAXPEAUDMFMODULE__@@@Z 0000000180000000     DmfK:DmfCall.obj
 0002:fffd9000       __guard_fids_?DMF_Module_ArmWakeFromS0@@YAJPEAUDMFMODULE__@@@Z 0000000180000000     DmfK:DmfCall.obj
 0002:fffd9000       __guard_fids_?DMF_Module_CloseOrUnregisterNotificationOnDestroy@@YAXPEAUDMFMODULE__@@@Z 0000000180000000     DmfK:DmfCall.obj
 0002:fffd9000       __guard_fids_?DMF_Module_DisarmWakeFromS0@@YAXPEAUDMFMODULE__@@@Z 0000000180000000     DmfK:DmfCall.obj
 0002:fffd9000       __guard_fids_?DMF_Module_DisarmWakeFromSx@@YAXPEAUDMFMODULE__@@@Z 0000000180000000     DmfK:DmfCall.obj
 0002:fffd9000       __guard_fids_?DMF_Module_NotificationRegister@@YAJPEAUDMFMODULE__@@@Z 0000000180000000     DmfK:DmfCall.obj
 0002:fffd9000       __guard_fids_?DMF_Module_NotificationUnregister@@YAXPEAUDMFMODULE__@@@Z 0000000180000000     DmfK:DmfCall.obj
 0002:fffd9000       __guard_fids_?DMF_Module_OpenOrRegisterNotificationOnCreate@@YAJPEAUDMFMODULE__@@@Z 0000000180000000     DmfK:DmfCall.obj
 0002:fffd9000       __guard_fids_?DMF_Module_QueryRemove@@YAJPEAUDMFMODULE__@@@Z 0000000180000000     DmfK:DmfCall.obj
 0002:fffd9000       __guard_fids_?DMF_Module_QueryStop@@YAJPEAUDMFMODULE__@@@Z 0000000180000000     DmfK:DmfCall.obj
 0002:fffd9000       __guard_fids_?DMF_Module_SelfManagedIoCleanup@@YAXPEAUDMFMODULE__@@@Z 0000000180000000     DmfK:DmfCall.obj
 0002:fffd9000       __guard_fids_?DMF_Module_SelfManagedIoFlush@@YAXPEAUDMFMODULE__@@@Z 0000000180000000     DmfK:DmfCall.obj
 0002:fffd9000       __guard_fids_?DMF_Module_SelfManagedIoInit@@YAJPEAUDMFMODULE__@@@Z 0000000180000000     DmfK:DmfCall.obj
 0002:fffd9000       __guard_fids_?DMF_Module_SelfManagedIoRestart@@YAJPEAUDMFMODULE__@@@Z 0000000180000000     DmfK:DmfCall.obj
 0002:fffd9000       __guard_fids_?DMF_Module_SelfManagedIoSuspend@@YAJPEAUDMFMODULE__@@@Z 0000000180000000     DmfK:DmfCall.obj
 0002:fffd9000       __guard_fids_?DMF_Module_SurpriseRemoval@@YAXPEAUDMFMODULE__@@@Z 0000000180000000     DmfK:DmfCall.obj
 0002:fffd9000       __guard_fids_?DMF_Module_WakeFromS0Triggered@@YAXPEAUDMFMODULE__@@@Z 0000000180000000     DmfK:DmfCall.obj
 0002:fffd9000       __guard_fids_?DMF_Module_WakeFromSxTriggered@@YAXPEAUDMFMODULE__@@@Z 0000000180000000     DmfK:DmfCall.obj
 0002:fffd9000       __guard_fids_?DmfEvtDynamicModuleCleanupCallback@@YAXPEAX@Z 0000000180000000     DmfK:DmfCall.obj
 0002:fffd9000       __guard_fids__             0000000180000000     DmfK:DmfCall.obj
 0002:fffd9000       __guard_fids_?DMF_ContainerFileObjectConfigInit@@YAXPEAU_WDF_FILEOBJECT_CONFIG@@@Z 0000000180000000     DmfK:DmfContainer.obj
 0002:fffd9000       __guard_fids_?DMF_ContainerPnpPowerCallbacksInit@@YAXPEAU_WDF_PNPPOWER_EVENT_CALLBACKS@@@Z 0000000180000000     DmfK:DmfContainer.obj
 0002:fffd9000       __guard_fids_?DMF_ContainerPowerPolicyCallbacksInit@@YAXPEAU_WDF_POWER_POLICY_EVENT_CALLBACKS@@@Z 0000000180000000     DmfK:DmfContainer.obj
 0002:fffd9000       __guard_fids_?DMF_ContainerQueueConfigCallbacksInit@@YAXPEAU_WDF_IO_QUEUE_CONFIG@@@Z 0000000180000000     DmfK:DmfContainer.obj
 0002:fffd9000       __guard_fids_DmfContainerEvtFileCreate 0000000180000000     DmfK:DmfContainer.obj
 0002:fffd9000       __guard_fids_?DmfCallbacksWdfInitialize@@YAXPEAUDMF_CALLBACKS_WDF@@@Z 0000000180000000     DmfK:DmfCore.obj
 0002:fffd9000       __guard_fids_?DmfModuleCallbacksInitialize@@YAJPEAU_DMF_OBJECT_@@PEAU_DMF_MODULE_ATTRIBUTES@@PEAUDMF_MODULE_DESCRIPTOR@@@Z 0000000180000000     DmfK:DmfCore.obj
 0002:fffd9000       __guard_fids_DMF_ModuleCreate 0000000180000000     DmfK:DmfCore.obj
 0002:fffd9000       __guard_fids__             0000000180000000     DmfK:DmfCore.obj
 0002:fffd9000       __guard_fids_DMF_ModuleInterfaceDescriptorAdd 0000000180000000     DmfK:DmfInterfaceInternal.obj
 0002:fffd9000       __guard_fids_?DMF_ModuleCollectionArmWakeFromS0@@YAJPEAUDMFCOLLECTION__@@@Z 0000000180000000     DmfK:DmfModuleCollection.obj
 0002:fffd9000       __guard_fids_?DMF_ModuleCollectionConfigListInitialize@@YAJPEAUDMF_MODULE_COLLECTION_CONFIG@@@Z 0000000180000000     DmfK:DmfModuleCollection.obj
 0002:fffd9000       __guard_fids_?DMF_ModuleCollectionCreate@@YAJPEAUDMFDEVICE_INIT@@PEAUDMF_MODULE_COLLECTION_CONFIG@@PEAPEAUDMFCOLLECTION__@@@Z 0000000180000000     DmfK:DmfModuleCollection.obj
 0002:fffd9000       __guard_fids_?DMF_ModuleCollectionDisarmWakeFromS0@@YAXPEAUDMFCOLLECTION__@@@Z 0000000180000000     DmfK:DmfModuleCollection.obj
 0002:fffd9000       __guard_fids_?DMF_ModuleCollectionDisarmWakeFromSx@@YAXPEAUDMFCOLLECTION__@@@Z 0000000180000000     DmfK:DmfModuleCollection.obj
 0002:fffd9000       __guard_fids_?DMF_ModuleCollectionQueryRemove@@YAJPEAUDMFCOLLECTION__@@@Z 0000000180000000     DmfK:DmfModuleCollection.obj
 0002:fffd9000       __guard_fids_?DMF_ModuleCollectionQueryStop@@YAJPEAUDMFCOLLECTION__@@@Z 0000000180000000     DmfK:DmfModuleCollection.obj
 0002:fffd9000       __guard_fids_?DMF_ModuleCollectionSelfManagedIoCleanup@@YAXPEAUDMFCOLLECTION__@@@Z 0000000180000000     DmfK:DmfModuleCollection.obj
 0002:fffd9000       __guard_fids_?DMF_ModuleCollectionSelfManagedIoFlush@@YAXPEAUDMFCOLLECTION__@@@Z 0000000180000000     DmfK:DmfModuleCollection.obj
 0002:fffd9000       __guard_fids_?DMF_ModuleCollectionSelfManagedIoInit@@YAJPEAUDMFCOLLECTION__@@@Z 0000000180000000     DmfK:DmfModuleCollection.obj
 0002:fffd9000       __guard_fids_?DMF_ModuleCollectionSelfManagedIoRestart@@YAJPEAUDMFCOLLECTION__@@@Z 0000000180000000     DmfK:DmfModuleCollection.obj
 0002:fffd9000       __guard_fids_?DMF_ModuleCollectionSelfManagedIoSuspend@@YAJPEAUDMFCOLLECTION__@@@Z 0000000180000000     DmfK:DmfModuleCollection.obj
 0002:fffd9000       __guard_fids_?DMF_ModuleCollectionSurpriseRemoval@@YAXPEAUDMFCOLLECTION__@@@Z 0000000180000000     DmfK:DmfModuleCollection.obj
 0002:fffd9000       __guard_fids_?DMF_ModuleCollectionWakeFromS0Triggered@@YAXPEAUDMFCOLLECTION__@@@Z 0000000180000000     DmfK:DmfModuleCollection.obj
 0002:fffd9000       __guard_fids_?DMF_ModuleCollectionWakeFromSxTriggered@@YAXPEAUDMFCOLLECTION__@@@Z 0000000180000000     DmfK:DmfModuleCollection.obj
 0002:fffd9000       __guard_fids_?DMF_ModuleCollection_ModuleValidate@@YAEPEAU_DMF_OBJECT_@@@Z 0000000180000000     DmfK:DmfModuleCollection.obj
 0002:fffd9000       __guard_fids_?BranchTrack_QueryInformation_Details@@YAJPEAUDMFMODULE__@@PEAUWDFREQUEST__@@PEA_K@Z 0000000180000000     DmfK:Dmf_BranchTrack.obj
 0002:fffd9000       __guard_fids_?BranchTrack_QueryInformation_Status@@YAJPEAUDMFMODULE__@@PEAUWDFREQUEST__@@PEA_K@Z 0000000180000000     DmfK:Dmf_BranchTrack.obj
 0002:fffd9000       __guard_fids_?DMF_BranchTrack_ChildModulesAdd@@YAXPEAUDMFMODULE__@@PEAU_DMF_MODULE_ATTRIBUTES@@PEAX@Z 0000000180000000     DmfK:Dmf_BranchTrack.obj
 0002:fffd9000       __guard_fids_DMF_BranchTrack_CheckPointCreate 0000000180000000     DmfK:Dmf_BranchTrack.obj
 0002:fffd9000       __guard_fids_DMF_BranchTrack_CheckPointExecute 0000000180000000     DmfK:Dmf_BranchTrack.obj
 0002:fffd9000       __guard_fids_DMF_BranchTrack_Create 0000000180000000     DmfK:Dmf_BranchTrack.obj
 0002:fffd9000       __guard_fids_?DMF_Bridge_Open@@YAJPEAUDMFMODULE__@@@Z 0000000180000000     DmfK:Dmf_Bridge.obj
 0002:fffd9000       __guard_fids_DMF_Bridge_Create 0000000180000000     DmfK:Dmf_Bridge.obj
 0002:fffd9000       __guard_fids_?BufferPool_BufferPoolEntryCreateAndAddToList@@YAJPEAUDMFMODULE__@@@Z 0000000180000000     DmfK:Dmf_BufferPool.obj
 0002:fffd9000       __guard_fids_DMF_BufferPool_Create 0000000180000000     DmfK:Dmf_BufferPool.obj
 0002:fffd9000       __guard_fids_DMF_BufferPool_Put 0000000180000000     DmfK:Dmf_BufferPool.obj
 0002:fffd9000       __guard_fids_DMF_BufferPool_PutAtHead 0000000180000000     DmfK:Dmf_BufferPool.obj
 0002:fffd9000       __guard_fids_DMF_BufferPool_PutInSinkWithTimer 0000000180000000     DmfK:Dmf_BufferPool.obj
 0002:fffd9000       __guard_fids_?DMF_BufferQueue_ChildModulesAdd@@YAXPEAUDMFMODULE__@@PEAU_DMF_MODULE_ATTRIBUTES@@PEAX@Z 0000000180000000     DmfK:Dmf_BufferQueue.obj
 0002:fffd9000       __guard_fids_DMF_BufferQueue_Create 0000000180000000     DmfK:Dmf_BufferQueue.obj
 0002:fffd9000       __guard_fids_?ContinuousRequestTarget_RequestCreateAndSend@@YAJPEAUDMFMODULE__@@EPEAX_K12W4ContinuousRequestTarget_RequestType@@KKW4ContinuousRequestTarget_CompletionOptions@@PEA_KP6AX011212J@Z1PEAPEAURequestTarget_DmfRequest__@@@Z 0000000180000000     DmfK:Dmf_ContinuousRequestTarget.obj
 0002:fffd9000       __guard_fids_?DMF_ContinuousRequestTarget_ChildModulesAdd@@YAXPEAUDMFMODULE__@@PEAU_DMF_MODULE_ATTRIBUTES@@PEAX@Z 0000000180000000     DmfK:Dmf_ContinuousRequestTarget.obj
 0002:fffd9000       __guard_fids_DMF_ContinuousRequestTarget_Create 0000000180000000     DmfK:Dmf_ContinuousRequestTarget.obj
 0002:fffd9000       __guard_fids_?CrashDump_BugCheckSecondaryDumpDataCallbackRingBuffer@@YAXW4_KBUGCHECK_CALLBACK_REASON@@PEAU_KBUGCHECK_REASON_CALLBACK_RECORD@@PEAXK@Z 0000000180000000     DmfK:Dmf_CrashDump.obj
 0002:fffd9000       __guard_fids_?CrashDump_DataSourceCreateInternal@@YAJPEAUDMFMODULE__@@KKKPEBU_GUID@@@Z 0000000180000000     DmfK:Dmf_CrashDump.obj
 0002:fffd9000       __guard_fids_?CrashDump_DmfCreate_RingBuffer@@YAJPEAUDMFMODULE__@@KKK@Z 0000000180000000     DmfK:Dmf_CrashDump.obj
 0002:fffd9000       __guard_fids_?CrashDump_TriageDataCreateInternal@@YAJPEAUDMFMODULE__@@@Z 0000000180000000     DmfK:Dmf_CrashDump.obj
 0002:fffd9000       __guard_fids_?DMF_CrashDump_ChildModulesAdd@@YAXPEAUDMFMODULE__@@PEAU_DMF_MODULE_ATTRIBUTES@@PEAX@Z 0000000180000000     DmfK:Dmf_CrashDump.obj
 0002:fffd9000       __guard_fids_?DMF_CrashDump_Open@@YAJPEAUDMFMODULE__@@@Z 0000000180000000     DmfK:Dmf_CrashDump.obj
 0002:fffd9000       __guard_fids_DMF_CrashDump_Create 0000000180000000     DmfK:Dmf_CrashDump.obj
 0002:fffd9000       __guard_fids__             0000000180000000     DmfK:Dmf_CrashDump.obj
 0002:fffd9000       __guard_fids_?DMF_DeviceInterfaceTarget_ChildModulesAdd@@YAXPEAUDMFMODULE__@@PEAU_DMF_MODULE_ATTRIBUTES@@PEAX@Z 0000000180000000     DmfK:Dmf_DeviceInterfaceTarget.obj
 0002:fffd9000       __guard_fids_?DMF_DeviceInterfaceTarget_NotificationRegister@@YAJPEAUDMFMODULE__@@@Z 0000000180000000     DmfK:Dmf_DeviceInterfaceTarget.obj
 0002:fffd9000       __guard_fids_?DeviceInterfaceTarget_DeviceCreateNewIoTargetByName@@YAJPEAUDMFMODULE__@@PEAU_UNICODE_STRING@@@Z 0000000180000000     DmfK:Dmf_DeviceInterfaceTarget.obj
 0002:fffd9000       __guard_fids_?DeviceInterfaceTarget_Stream_SendEx@@YAJPEAUDMFMODULE__@@PEAX_K12W4ContinuousRequestTarget_RequestType@@KKP6AX011212J@Z1PEAPEAURequestTarget_DmfRequest__@@@Z 0000000180000000     DmfK:Dmf_DeviceInterfaceTarget.obj
 0002:fffd9000       __guard_fids_?DeviceInterfaceTarget_Target_SendEx@@YAJPEAUDMFMODULE__@@PEAX_K12W4ContinuousRequestTarget_RequestType@@KKP6AX011212J@Z1PEAPEAURequestTarget_DmfRequest__@@@Z 0000000180000000     DmfK:Dmf_DeviceInterfaceTarget.obj
 0002:fffd9000       __guard_fids_DMF_DeviceInterfaceTarget_Create 0000000180000000     DmfK:Dmf_DeviceInterfaceTarget.obj
 0002:fffd9000       __guard_fids_DMF_File_Create 0000000180000000     DmfK:Dmf_File.obj
 0002:fffd9000       __guard_fids_?HashTable_ContextInitialize@@YAJPEAUDMFMODULE__@@@Z 0000000180000000     DmfK:Dmf_HashTable.obj
 0002:fffd9000       __guard_fids_DMF_HashTable_Create 0000000180000000     DmfK:Dmf_HashTable.obj
 0002:fffd9000       __guard_fids_DMF_IoctlHandler_Create 0000000180000000     DmfK:Dmf_IoctlHandler.obj
 0002:fffd9000       __guard_fids_?DMF_LiveKernelDump_ChildModulesAdd@@YAXPEAUDMFMODULE__@@PEAU_DMF_MODULE_ATTRIBUTES@@PEAX@Z 0000000180000000     DmfK:Dmf_LiveKernelDump.obj
 0002:fffd9000       __guard_fids_?LiveKernelDump_DataBufferSourceRemove@@YAXPEAUDMFMODULE__@@PEAXK@Z 0000000180000000     DmfK:Dmf_LiveKernelDump.obj
 0002:fffd9000       __guard_fids_?LiveKernelDump_InsertDmfTriageDataToCrashDump@@YAJPEAUDMFMODULE__@@@Z 0000000180000000     DmfK:Dmf_LiveKernelDump.obj
 0002:fffd9000       __guard_fids_?LiveKernelDump_InsertDmfTriageDataToLiveDump@@YAJPEAUDMFMODULE__@@PEAX@Z 0000000180000000     DmfK:Dmf_LiveKernelDump.obj
 0002:fffd9000       __guard_fids_DMF_LiveKernelDump_Create 0000000180000000     DmfK:Dmf_LiveKernelDump.obj
 0002:fffd9000       __guard_fids__             0000000180000000     DmfK:Dmf_LiveKernelDump.obj
 0002:fffd9000       __guard_fids_?DMF_QueuedWorkItem_ChildModulesAdd@@YAXPEAUDMFMODULE__@@PEAU_DMF_MODULE_ATTRIBUTES@@PEAX@Z 0000000180000000     DmfK:Dmf_QueuedWorkItem.obj
 0002:fffd9000       __guard_fids_DMF_QueuedWorkItem_Create 0000000180000000     DmfK:Dmf_QueuedWorkItem.obj
 0002:fffd9000       __guard_fids_?DMF_RequestTarget_ChildModulesAdd@@YAXPEAUDMFMODULE__@@PEAU_DMF_MODULE_ATTRIBUTES@@PEAX@Z 0000000180000000     DmfK:Dmf_RequestTarget.obj
 0002:fffd9000       __guard_fids_?RequestTarget_RequestCreateAndSend@@YAJPEAUDMFMODULE__@@EPEAX_K12W4ContinuousRequestTarget_RequestType@@KKW4ContinuousRequestTarget_CompletionOptions@@PEA_KP6AX011212J@Z1PEAPEAURequestTarget_DmfRequest__@@@Z 0000000180000000     DmfK:Dmf_RequestTarget.obj
 0002:fffd9000       __guard_fids_DMF_RequestTarget_Create 0000000180000000     DmfK:Dmf_RequestTarget.obj
 0002:fffd9000       __guard_fids_DMF_RingBuffer_Create 0000000180000000     DmfK:Dmf_RingBuffer.obj
 0002:fffd9000       __guard_fids_DMF_RingBuffer_EnumerateToFindItem 0000000180000000     DmfK:Dmf_RingBuffer.obj
 0002:fffd9000       __guard_fids_DMF_RingBuffer_Read 0000000180000000     DmfK:Dmf_RingBuffer.obj
 0002:fffd9000       __guard_fids_DMF_RingBuffer_ReadAll 0000000180000000     DmfK:Dmf_RingBuffer.obj
 0002:fffd9000       __guard_fids_DMF_RingBuffer_SegmentsRead 0000000180000000     DmfK:Dmf_RingBuffer.obj
 0002:fffd9000       __guard_fids_DMF_RingBuffer_SegmentsWrite 0000000180000000     DmfK:Dmf_RingBuffer.obj
 0002:fffd9000       __guard_fids_DMF_RingBuffer_Write 0000000180000000     DmfK:Dmf_RingBuffer.obj
 0002:fffd9000       __guard_fids_DMF_Rundown_Create 0000000180000000     DmfK:Dmf_Rundown.obj
 0002:fffd9000       __guard_fids_?DMF_SamCommunicationViaSsh_BranchTrackInitialize@@YAXPEAUDMFMODULE__@@@Z 0000000180000000     DmfK:Dmf_SamCommunicationViaSsh.obj
 0002:fffd9000       __guard_fids_?DMF_SamCommunicationViaSsh_ChildModulesAdd@@YAXPEAUDMFMODULE__@@PEAU_DMF_MODULE_ATTRIBUTES@@PEAX@Z 0000000180000000     DmfK:Dmf_SamCommunicationViaSsh.obj
 0002:fffd9000       __guard_fids_?SamCommunicationViaSsh_OnDeviceArrivalNotification@@YAXPEAUDMFMODULE__@@@Z 0000000180000000     DmfK:Dmf_SamCommunicationViaSsh.obj
 0002:fffd9000       __guard_fids_?SamCommunicationViaSsh_OnDeviceRemovalNotification@@YAXPEAUDMFMODULE__@@@Z 0000000180000000     DmfK:Dmf_SamCommunicationViaSsh.obj
 0002:fffd9000       __guard_fids_DMF_SamCommunicationViaSsh_Create 0000000180000000     DmfK:Dmf_SamCommunicationViaSsh.obj
 0002:fffd9000       __guard_fids_?DMF_SamNotificationViaSsh_BranchTrackInitialize@@YAXPEAUDMFMODULE__@@@Z 0000000180000000     DmfK:Dmf_SamNotificationViaSsh.obj
 0002:fffd9000       __guard_fids_?DMF_SamNotificationViaSsh_ChildModulesAdd@@YAXPEAUDMFMODULE__@@PEAU_DMF_MODULE_ATTRIBUTES@@PEAX@Z 0000000180000000     DmfK:Dmf_SamNotificationViaSsh.obj
 0002:fffd9000       __guard_fids_?DMF_SamNotificationViaSsh_Close@@YAXPEAUDMFMODULE__@@@Z 0000000180000000     DmfK:Dmf_SamNotificationViaSsh.obj
 0002:fffd9000       __guard_fids_?DMF_SamNotificationViaSsh_ModuleD0Entry@@YAJPEAUDMFMODULE__@@W4_WDF_POWER_DEVICE_STATE@@@Z 0000000180000000     DmfK:Dmf_SamNotificationViaSsh.obj
 0002:fffd9000       __guard_fids_?DMF_SamNotificationViaSsh_ModuleD0Exit@@YAJPEAUDMFMODULE__@@W4_WDF_POWER_DEVICE_STATE@@@Z 0000000180000000     DmfK:Dmf_SamNotificationViaSsh.obj
 0002:fffd9000       __guard_fids_?DMF_SamNotificationViaSsh_Open@@YAJPEAUDMFMODULE__@@@Z 0000000180000000     DmfK:Dmf_SamNotificationViaSsh.obj
 0002:fffd9000       __guard_fids_?SamNotificationViaSsh_LegacyModeQueryAndSet@@YAXPEAUDMFMODULE__@@@Z 0000000180000000     DmfK:Dmf_SamNotificationViaSsh.obj
 0002:fffd9000       __guard_fids_?SamNotificationViaSsh_OnDeviceArrivalNotification@@YAXPEAUDMFMODULE__@@@Z 0000000180000000     DmfK:Dmf_SamNotificationViaSsh.obj
 0002:fffd9000       __guard_fids_?SamNotificationViaSsh_OnDeviceRemovalNotification@@YAXPEAUDMFMODULE__@@@Z 0000000180000000     DmfK:Dmf_SamNotificationViaSsh.obj
 0002:fffd9000       __guard_fids_?SamNotificationViaSsh_RegisterCompletion@@YAXPEAUDMFMODULE__@@PEAX1_K12J@Z 0000000180000000     DmfK:Dmf_SamNotificationViaSsh.obj
 0002:fffd9000       __guard_fids_?SamNotificationViaSsh_RegisterForTargetNotification@@YAJPEAUDMFMODULE__@@E@Z 0000000180000000     DmfK:Dmf_SamNotificationViaSsh.obj
 0002:fffd9000       __guard_fids_?SamNotificationViaSsh_RegisterForTargetNotificationSynchronously@@YAJPEAUDMFMODULE__@@E@Z 0000000180000000     DmfK:Dmf_SamNotificationViaSsh.obj
 0002:fffd9000       __guard_fids_?SamNotificationViaSsh_StreamAsynchronousBufferCallbackInput@@YAXPEAUDMFMODULE__@@PEAXPEA_K1@Z 0000000180000000     DmfK:Dmf_SamNotificationViaSsh.obj
 0002:fffd9000       __guard_fids_?SamNotificationViaSsh_StreamAsynchronousBufferCallbackOutput@@YA?AW4ContinuousRequestTarget_BufferDisposition@@PEAUDMFMODULE__@@PEAX_K1J@Z 0000000180000000     DmfK:Dmf_SamNotificationViaSsh.obj
 0002:fffd9000       __guard_fids_?SamNotificationViaSsh_StreamingStart@@YAJPEAUDMFMODULE__@@@Z 0000000180000000     DmfK:Dmf_SamNotificationViaSsh.obj
 0002:fffd9000       __guard_fids_?SamNotificationViaSsh_StreamingStop@@YAJPEAUDMFMODULE__@@@Z 0000000180000000     DmfK:Dmf_SamNotificationViaSsh.obj
 0002:fffd9000       __guard_fids_?SamNotificationViaSsh_UnregisterCompletion@@YAXPEAUDMFMODULE__@@PEAX1_K12J@Z 0000000180000000     DmfK:Dmf_SamNotificationViaSsh.obj
 0002:fffd9000       __guard_fids_DMF_SamNotificationViaSsh_ControlStream 0000000180000000     DmfK:Dmf_SamNotificationViaSsh.obj
 0002:fffd9000       __guard_fids_DMF_SamNotificationViaSsh_Create 0000000180000000     DmfK:Dmf_SamNotificationViaSsh.obj
 0002:fffd9000       __guard_fids_?DMF_ScheduledTask_ChildModulesAdd@@YAXPEAUDMFMODULE__@@PEAU_DMF_MODULE_ATTRIBUTES@@PEAX@Z 0000000180000000     DmfK:Dmf_ScheduledTask.obj
 0002:fffd9000       __guard_fids_?DMF_ScheduledTask_Open@@YAJPEAUDMFMODULE__@@@Z 0000000180000000     DmfK:Dmf_ScheduledTask.obj
 0002:fffd9000       __guard_fids_DMF_ScheduledTask_Create 0000000180000000     DmfK:Dmf_ScheduledTask.obj
 0002:fffd9000       __guard_fids_DMF_SmbiosWmi_Create 0000000180000000     DmfK:Dmf_SmbiosWmi.obj
 0002:fffd9000       __guard_fids_DMF_String_Create 0000000180000000     DmfK:Dmf_String.obj
 0002:fffd9000       __guard_fids_DMF_String_FindInListExactChar 0000000180000000     DmfK:Dmf_String.obj
 0002:fffd9000       __guard_fids_DMF_String_FindInListLookForLeftMatchChar 0000000180000000     DmfK:Dmf_String.obj
 0002:fffd9000       __guard_fids_DMF_String_MultiSzFindLast 0000000180000000     DmfK:Dmf_String.obj
 0002:fffd9000       __guard_fids_?DMF_SurfaceTelemetryConsentSettingsNotification_ChildModulesAdd@@YAXPEAUDMFMODULE__@@PEAU_DMF_MODULE_ATTRIBUTES@@PEAX@Z 0000000180000000     DmfK:Dmf_SurfaceTelemetryConsentSettingsNotification.obj
 0002:fffd9000       __guard_fids_DMF_SurfaceTelemetryConsentSettingsNotification_Create 0000000180000000     DmfK:Dmf_SurfaceTelemetryConsentSettingsNotification.obj
 0002:fffd9000       __guard_fids__             0000000180000000     DmfK:Dmf_SurfaceTelemetryConsentSettingsNotification.obj
 0002:fffd9008       __guard_fids__             0000000180000008     DmfK:DmfCall.obj
 0002:fffd9018       __guard_fids__             0000000180000018     DmfK:DmfCore.obj
 0002:fffd9028       __guard_fids__             0000000180000028     DmfK:DmfCore.obj
 0002:fffd909c       __guard_fids__             000000018000009c     DmfK:DmfCore.obj
 0002:fffd90b4       __guard_fids__             00000001800000b4     DmfK:DmfCore.obj
 0002:fffd90c4       __guard_fids__             00000001800000c4     DmfK:DmfCore.obj
 0001:00000000       _ZN20surface_hid_mini_lib18generic_hid_module11HidMiniport3new10_tlg_write17h9a5a2466636c6021E 0000000180001000 f   surface_hid_mini.surface_hid_mini.3efcb60154bd7459-cgu.0.rcgu.o
 0001:000000a0       _ZN20surface_hid_mini_lib18generic_hid_module11HidMiniport18get_hid_descriptor17hcc0512e923d8020eE 00000001800010a0 f   surface_hid_mini.surface_hid_mini.3efcb60154bd7459-cgu.0.rcgu.o
 0001:000007b0       _ZN20surface_hid_mini_lib18generic_hid_module11HidMiniport15get_descriptors10_tlg_write17h37e4420442ecbe72E 00000001800017b0 f   surface_hid_mini.surface_hid_mini.3efcb60154bd7459-cgu.0.rcgu.o
 0001:00000860       _ZN20surface_hid_mini_lib18generic_hid_module11HidMiniport15get_descriptors10_tlg_write17h51e4fa681cee9362E 0000000180001860 f   surface_hid_mini.surface_hid_mini.3efcb60154bd7459-cgu.0.rcgu.o
 0001:00000900       _ZN20surface_hid_mini_lib18generic_hid_module11HidMiniport15get_descriptors10_tlg_write17hf564b2c1523f97b1E 0000000180001900 f   surface_hid_mini.surface_hid_mini.3efcb60154bd7459-cgu.0.rcgu.o
 0001:000009d0       _ZN20surface_hid_mini_lib18generic_hid_module27generic_hid_send_completion17hae87df66c0f8daddE 00000001800019d0 f   surface_hid_mini.surface_hid_mini.3efcb60154bd7459-cgu.0.rcgu.o
 0001:00000af0       _ZN20surface_hid_mini_lib18generic_hid_module11HidMiniport10get_report17h937df307f24fef13E 0000000180001af0 f   surface_hid_mini.surface_hid_mini.3efcb60154bd7459-cgu.0.rcgu.o
 0001:00000e50       _ZN20surface_hid_mini_lib18generic_hid_module11HidMiniport10get_report10_tlg_write17h6ed3f4cf02c1e0a1E 0000000180001e50 f   surface_hid_mini.surface_hid_mini.3efcb60154bd7459-cgu.0.rcgu.o
 0001:00000f00       _ZN20surface_hid_mini_lib18generic_hid_module11HidMiniport13input_consume17hbe80a8d155648cb1E 0000000180001f00 f   surface_hid_mini.surface_hid_mini.3efcb60154bd7459-cgu.0.rcgu.o
 0001:00001930       _ZN20surface_hid_mini_lib18generic_hid_module55generic_hid_stream_asynchronous_request_buffer_callback17hfb0c52b1073c052fE 0000000180002930 f   surface_hid_mini.surface_hid_mini.3efcb60154bd7459-cgu.0.rcgu.o
 0001:00001c60       _ZN20surface_hid_mini_lib18generic_hid_module36queuedworkitem_get_string_descriptor17h7f5a487aeffd08a2E 0000000180002c60 f   surface_hid_mini.surface_hid_mini.3efcb60154bd7459-cgu.0.rcgu.o
 0001:00001fe0       _ZN20surface_hid_mini_lib6driver36surface_hid_mini_evt_context_cleanup17h8a7409842904b5fdE 0000000180002fe0 f   surface_hid_mini.surface_hid_mini.3efcb60154bd7459-cgu.0.rcgu.o
 0001:00002220       _ZN20surface_hid_mini_lib5queue47surface_hid_mini_evt_internal_io_device_control17hcac1b47947a6d4eeE 0000000180003220 f   surface_hid_mini.surface_hid_mini.3efcb60154bd7459-cgu.0.rcgu.o
 0001:00003db0       _ZN20surface_hid_mini_lib5queue47surface_hid_mini_evt_internal_io_device_control10_tlg_write17hc69f975f4e7c07abE 0000000180004db0 f   surface_hid_mini.surface_hid_mini.3efcb60154bd7459-cgu.0.rcgu.o
 0001:00003ea0       _ZN20surface_hid_mini_lib5queue47surface_hid_mini_evt_internal_io_device_control10_tlg_write17hd1d680bd08e034b7E 0000000180004ea0 f   surface_hid_mini.surface_hid_mini.3efcb60154bd7459-cgu.0.rcgu.o
 0001:00003f90       _ZN20surface_hid_mini_lib5queue47surface_hid_mini_evt_internal_io_device_control10_tlg_write17h4723c70206d1b14eE 0000000180004f90 f   surface_hid_mini.surface_hid_mini.3efcb60154bd7459-cgu.0.rcgu.o
 0001:00004080       _ZN20surface_hid_mini_lib5queue47surface_hid_mini_evt_internal_io_device_control10_tlg_write17hce61e2ceefbfd63fE 0000000180005080 f   surface_hid_mini.surface_hid_mini.3efcb60154bd7459-cgu.0.rcgu.o
 0001:00004130       _ZN20surface_hid_mini_lib5queue47surface_hid_mini_evt_internal_io_device_control10_tlg_write17h3ef99611eea6525cE 0000000180005130 f   surface_hid_mini.surface_hid_mini.3efcb60154bd7459-cgu.0.rcgu.o
 0001:000041e0       _ZN20surface_hid_mini_lib5queue47surface_hid_mini_evt_internal_io_device_control10_tlg_write17h2df9dcd938be4500E 00000001800051e0 f   surface_hid_mini.surface_hid_mini.3efcb60154bd7459-cgu.0.rcgu.o
 0001:00004290       _ZN20surface_hid_mini_lib5queue47surface_hid_mini_evt_internal_io_device_control10_tlg_write17he44e13736d225bdaE 0000000180005290 f   surface_hid_mini.surface_hid_mini.3efcb60154bd7459-cgu.0.rcgu.o
 0001:00004340       _ZN20surface_hid_mini_lib5queue47surface_hid_mini_evt_internal_io_device_control10_tlg_write17h6bf563a0e1491f33E 0000000180005340 f   surface_hid_mini.surface_hid_mini.3efcb60154bd7459-cgu.0.rcgu.o
 0001:000043f0       _ZN20surface_hid_mini_lib6device32surface_hid_mini_get_instance_id17h87f5f56d3fbee290E 00000001800053f0 f   surface_hid_mini.surface_hid_mini.3efcb60154bd7459-cgu.0.rcgu.o
 0001:00004670       _ZN20surface_hid_mini_lib6device36surface_hid_mini_evt_device_d0_entry17hc04aef7a32727619E 0000000180005670 f   surface_hid_mini.surface_hid_mini.3efcb60154bd7459-cgu.0.rcgu.o
 0001:00004940       _ZN20surface_hid_mini_lib6device35surface_hid_mini_evt_device_d0_exit17h4955d74074ae75dfE 0000000180005940 f   surface_hid_mini.surface_hid_mini.3efcb60154bd7459-cgu.0.rcgu.o
 0001:00004a40       _ZN20surface_hid_mini_lib6device44surface_hid_mini_evt_device_prepare_hardware17h9e1deff4e47c6958E 0000000180005a40 f   surface_hid_mini.surface_hid_mini.3efcb60154bd7459-cgu.0.rcgu.o
 0001:000054c0       _ZN20surface_hid_mini_lib6device44surface_hid_mini_evt_device_release_hardware17h3ad4346eca7f187cE 00000001800064c0 f   surface_hid_mini.surface_hid_mini.3efcb60154bd7459-cgu.0.rcgu.o
 0001:00005710       _ZN20surface_hid_mini_lib6device39surface_hid_mini_device_context_cleanup17hf7769d9bbbba65c8E 0000000180006710 f   surface_hid_mini.surface_hid_mini.3efcb60154bd7459-cgu.0.rcgu.o
 0001:00005800       _ZN20surface_hid_mini_lib6device30surface_hid_mini_create_device10_tlg_write17h734f84a5a1000085E 0000000180006800 f   surface_hid_mini.surface_hid_mini.3efcb60154bd7459-cgu.0.rcgu.o
 0001:000058b0       _ZN20surface_hid_mini_lib6device30surface_hid_mini_create_device10_tlg_write17h046ac4934b2bdb58E 00000001800068b0 f   surface_hid_mini.surface_hid_mini.3efcb60154bd7459-cgu.0.rcgu.o
 0001:00005960       _ZN20surface_hid_mini_lib6device30surface_hid_mini_create_device10_tlg_write17h0169a4ccc1f1af90E 0000000180006960 f   surface_hid_mini.surface_hid_mini.3efcb60154bd7459-cgu.0.rcgu.o
 0001:00005a10       _ZN20surface_hid_mini_lib6device30surface_hid_mini_create_device10_tlg_write17h82d6e9c90a70c381E 0000000180006a10 f   surface_hid_mini.surface_hid_mini.3efcb60154bd7459-cgu.0.rcgu.o
 0001:00005ae0       _ZN20surface_hid_mini_lib6device39surface_hid_mini_power_setting_callback17h1f75742198f87e6aE 0000000180006ae0 f   surface_hid_mini.surface_hid_mini.3efcb60154bd7459-cgu.0.rcgu.o
 0001:00005d30       _ZN12tracelogging6native20ProviderContextInner14outer_callback17h93f4d127a127e0d2E 0000000180006d30 f   surface_hid_mini.surface_hid_mini.3efcb60154bd7459-cgu.0.rcgu.o
 0001:00005da0       _ZN12tracelogging8provider8Provider8register17h18e2a0292224c126E 0000000180006da0 f   surface_hid_mini.surface_hid_mini.3efcb60154bd7459-cgu.0.rcgu.o
 0001:0000a2a0       ?DMF_SamNotificationViaSsh_Close@@YAXPEAUDMFMODULE__@@@Z 000000018000b2a0 f   DmfK:Dmf_SamNotificationViaSsh.obj
 0001:0000a590       ?DMF_SamNotificationViaSsh_ModuleD0Entry@@YAJPEAUDMFMODULE__@@W4_WDF_POWER_DEVICE_STATE@@@Z 000000018000b590 f   DmfK:Dmf_SamNotificationViaSsh.obj
 0001:0000a9a0       ?DMF_SamNotificationViaSsh_ModuleD0Exit@@YAJPEAUDMFMODULE__@@W4_WDF_POWER_DEVICE_STATE@@@Z 000000018000b9a0 f   DmfK:Dmf_SamNotificationViaSsh.obj
 0001:0000ad20       ?DMF_SamNotificationViaSsh_Open@@YAJPEAUDMFMODULE__@@@Z 000000018000bd20 f   DmfK:Dmf_SamNotificationViaSsh.obj
 0001:0000b060       ?SamNotificationViaSsh_OnDeviceArrivalNotification@@YAXPEAUDMFMODULE__@@@Z 000000018000c060 f   DmfK:Dmf_SamNotificationViaSsh.obj
 0001:0000b190       ?SamNotificationViaSsh_OnDeviceRemovalNotification@@YAXPEAUDMFMODULE__@@@Z 000000018000c190 f   DmfK:Dmf_SamNotificationViaSsh.obj
 0001:0000b774       ?SamNotificationViaSsh_RegisterForTargetNotification@@YAJPEAUDMFMODULE__@@E@Z 000000018000c774 f   DmfK:Dmf_SamNotificationViaSsh.obj
 0001:0000bb1c       ?SamNotificationViaSsh_RegisterForTargetNotificationSynchronously@@YAJPEAUDMFMODULE__@@E@Z 000000018000cb1c f   DmfK:Dmf_SamNotificationViaSsh.obj
 0001:0000bee0       ?SamNotificationViaSsh_StreamAsynchronousBufferCallbackInput@@YAXPEAUDMFMODULE__@@PEAXPEA_K1@Z 000000018000cee0 f   DmfK:Dmf_SamNotificationViaSsh.obj
 0001:0000c060       ?SamNotificationViaSsh_StreamAsynchronousBufferCallbackOutput@@YA?AW4ContinuousRequestTarget_BufferDisposition@@PEAUDMFMODULE__@@PEAX_K1J@Z 000000018000d060 f   DmfK:Dmf_SamNotificationViaSsh.obj
 0001:0000c1c8       ?SamNotificationViaSsh_StreamingStart@@YAJPEAUDMFMODULE__@@@Z 000000018000d1c8 f   DmfK:Dmf_SamNotificationViaSsh.obj
 0001:0000c6c4       ?SamNotificationViaSsh_StreamingStop@@YAJPEAUDMFMODULE__@@@Z 000000018000d6c4 f   DmfK:Dmf_SamNotificationViaSsh.obj
 0001:0000dbdc       ?DMF_ModuleCollectionCleanup@@YAXPEAU_DMF_MODULE_COLLECTION_@@W4ModuleOpenedDuringType@@@Z 000000018000ebdc f   DmfK:DmfModuleCollection.obj
 0001:00012260       ?BranchTrack_EVT_DMF_HashTable_Enumerate_DetailsData@@YAEPEAUDMFMODULE__@@PEAEK1KPEAX@Z 0000000180013260 f   DmfK:Dmf_BranchTrack.obj
 0001:00012430       ?BranchTrack_EVT_DMF_HashTable_Enumerate_DetailsSize@@YAEPEAUDMFMODULE__@@PEAEK1KPEAX@Z 0000000180013430 f   DmfK:Dmf_BranchTrack.obj
 0001:00012450       ?BranchTrack_EVT_DMF_HashTable_Enumerate_Status@@YAEPEAUDMFMODULE__@@PEAEK1KPEAX@Z 0000000180013450 f   DmfK:Dmf_BranchTrack.obj
 0001:000124a0       ?BranchTrack_EVT_DMF_HashTable_Find@@YAXPEAUDMFMODULE__@@PEAEK1PEAK@Z 00000001800134a0 f   DmfK:Dmf_BranchTrack.obj
 0001:000124c0       ?BranchTrack_HashTable_CallbackEntryCreate@@YAXPEAUDMFMODULE__@@PEAEK1PEAK@Z 00000001800134c0 f   DmfK:Dmf_BranchTrack.obj
 0001:000124d0       ?BranchTrack_QueryInformation@@YAJPEAUDMFMODULE__@@PEAUWDFREQUEST__@@PEA_K@Z 00000001800134d0 f   DmfK:Dmf_BranchTrack.obj
 0001:000126d8       ?BranchTrack_QueryInformation_Details@@YAJPEAUDMFMODULE__@@PEAUWDFREQUEST__@@PEA_K@Z 00000001800136d8 f   DmfK:Dmf_BranchTrack.obj
 0001:0001294c       ?BranchTrack_QueryInformation_Status@@YAJPEAUDMFMODULE__@@PEAUWDFREQUEST__@@PEA_K@Z 000000018001394c f   DmfK:Dmf_BranchTrack.obj
 0001:00012c50       ?DMF_BranchTrack_ModuleDeviceIoControl@@YAEPEAUDMFMODULE__@@PEAUWDFQUEUE__@@PEAUWDFREQUEST__@@_K3K@Z 0000000180013c50 f   DmfK:Dmf_BranchTrack.obj
 0001:00016d10       ?DMF_ScheduledTask_ModuleD0Entry@@YAJPEAUDMFMODULE__@@W4_WDF_POWER_DEVICE_STATE@@@Z 0000000180017d10 f   DmfK:Dmf_ScheduledTask.obj
 0001:00016f40       ?DMF_ScheduledTask_ModuleD0Exit@@YAJPEAUDMFMODULE__@@W4_WDF_POWER_DEVICE_STATE@@@Z 0000000180017f40 f   DmfK:Dmf_ScheduledTask.obj
 0001:000185f0       ?DMF_Bridge_ModuleD0Entry@@YAJPEAUDMFMODULE__@@W4_WDF_POWER_DEVICE_STATE@@@Z 00000001800195f0 f   DmfK:Dmf_Bridge.obj
 0001:00018720       ?DMF_Bridge_ModuleD0EntryPostInterruptsEnabled@@YAJPEAUDMFMODULE__@@W4_WDF_POWER_DEVICE_STATE@@@Z 0000000180019720 f   DmfK:Dmf_Bridge.obj
 0001:00018850       ?DMF_Bridge_ModuleD0Exit@@YAJPEAUDMFMODULE__@@W4_WDF_POWER_DEVICE_STATE@@@Z 0000000180019850 f   DmfK:Dmf_Bridge.obj
 0001:00018980       ?DMF_Bridge_ModuleD0ExitPreInterruptsDisabled@@YAJPEAUDMFMODULE__@@W4_WDF_POWER_DEVICE_STATE@@@Z 0000000180019980 f   DmfK:Dmf_Bridge.obj
 0001:00018ab0       ?DMF_Bridge_ModuleDeviceIoControl@@YAEPEAUDMFMODULE__@@PEAUWDFQUEUE__@@PEAUWDFREQUEST__@@_K3K@Z 0000000180019ab0 f   DmfK:Dmf_Bridge.obj
 0001:00018bd0       ?DMF_Bridge_ModuleInternalDeviceIoControl@@YAEPEAUDMFMODULE__@@PEAUWDFQUEUE__@@PEAUWDFREQUEST__@@_K3K@Z 0000000180019bd0 f   DmfK:Dmf_Bridge.obj
 0001:00018cf0       ?DMF_Bridge_ModuleQueueIoRead@@YAEPEAUDMFMODULE__@@PEAUWDFQUEUE__@@PEAUWDFREQUEST__@@_K@Z 0000000180019cf0 f   DmfK:Dmf_Bridge.obj
 0001:00018e00       ?DMF_Bridge_ModuleQueueIoWrite@@YAEPEAUDMFMODULE__@@PEAUWDFQUEUE__@@PEAUWDFREQUEST__@@_K@Z 0000000180019e00 f   DmfK:Dmf_Bridge.obj
 0001:00018f10       ?DMF_Bridge_ModuleSelfManagedIoRestart@@YAJPEAUDMFMODULE__@@@Z 0000000180019f10 f   DmfK:Dmf_Bridge.obj
 0001:00019040       ?DMF_Bridge_ModuleSelfManagedIoSuspend@@YAJPEAUDMFMODULE__@@@Z 000000018001a040 f   DmfK:Dmf_Bridge.obj
 0001:00019170       ?DMF_Bridge_ModuleSurpriseRemoval@@YAXPEAUDMFMODULE__@@@Z 000000018001a170 f   DmfK:Dmf_Bridge.obj
 0001:0001a570       ?DMF_IoctlHandler_ModuleDeviceIoControl@@YAEPEAUDMFMODULE__@@PEAUWDFQUEUE__@@PEAUWDFREQUEST__@@_K3K@Z 000000018001b570 f   DmfK:Dmf_IoctlHandler.obj
 0001:0001b170       RtlStringVPrintfWorkerW    000000018001c170 f   DmfK:lkmdtel.obj
 0001:0001b344       ?RingBuffer_Read@@YAJPEAURING_BUFFER@@PEAEKP6AXPEAX1K@Z@Z 000000018001c344 f   DmfK:Dmf_RingBuffer.obj
 0001:0001b3f8       ?RingBuffer_ReadPointerIncrement@@YAXPEAURING_BUFFER@@@Z 000000018001c3f8 f   DmfK:Dmf_RingBuffer.obj
 0001:0001b4bc       ?RingBuffer_Write@@YAJPEAURING_BUFFER@@PEAEKP6AXPEAX1K@Z@Z 000000018001c4bc f   DmfK:Dmf_RingBuffer.obj
 0001:0001dd70       ?HashTable_DataEntryAllocate@@YAJPEAUDMFMODULE__@@PEAU_DMF_CONTEXT_HashTable@@PEAEKPEAK@Z 000000018001ed70 f   DmfK:Dmf_HashTable.obj
 0001:0001de04       ?HashTable_DataEntryFindOrAllocate@@YAJPEAUDMFMODULE__@@PEAEKPEAPEAUDATA_ENTRY@@@Z 000000018001ee04 f   DmfK:Dmf_HashTable.obj
 0001:0001df60       ?HashTable_HashCalculate@@YA_KPEAUDMFMODULE__@@PEAEK@Z 000000018001ef60 f   DmfK:Dmf_HashTable.obj
 0001:0001e768       ?RequestTarget_FormatRequestForRequestType@@YAJPEAUDMFMODULE__@@PEAUWDFREQUEST__@@W4ContinuousRequestTarget_RequestType@@KPEAUWDFMEMORY__@@3@Z 000000018001f768 f   DmfK:Dmf_RequestTarget.obj
 0001:0001ea40       ?RequestTarget_PendingCollectionListAdd@@YAJPEAUDMFMODULE__@@PEAUWDFREQUEST__@@@Z 000000018001fa40 f   DmfK:Dmf_RequestTarget.obj
 0001:0001eba0       ?RequestTarget_PendingCollectionListSearchAndRemove@@YAEPEAUDMFMODULE__@@PEAUWDFREQUEST__@@@Z 000000018001fba0 f   DmfK:Dmf_RequestTarget.obj
 0001:0001f19c       ?RequestTarget_RequestCreateAndSend@@YAJPEAUDMFMODULE__@@EPEAX_K12W4ContinuousRequestTarget_RequestType@@KKW4ContinuousRequestTarget_CompletionOptions@@PEA_KP6AX011212J@Z1PEAPEAURequestTarget_DmfRequest__@@@Z 000000018002019c f   DmfK:Dmf_RequestTarget.obj
 0001:0002006c       ?ContinuousRequestTarget_CompletionParamsInputBufferAndOutputBufferGet@@YAXPEAUDMFMODULE__@@PEAU_WDF_REQUEST_COMPLETION_PARAMS@@W4ContinuousRequestTarget_RequestType@@PEAPEAXPEA_K34@Z 000000018002106c f   DmfK:Dmf_ContinuousRequestTarget.obj
 0001:00020450       ?ContinuousRequestTarget_CreateBuffersAndFormatRequestForRequestType@@YAJPEAUDMFMODULE__@@PEAUWDFREQUEST__@@@Z 0000000180021450 f   DmfK:Dmf_ContinuousRequestTarget.obj
 0001:00020678       ?ContinuousRequestTarget_DecreaseStreamRequestCount@@YAXPEAU_DMF_CONTEXT_ContinuousRequestTarget@@@Z 0000000180021678 f   DmfK:Dmf_ContinuousRequestTarget.obj
 0001:00020738       ?ContinuousRequestTarget_DeleteStreamRequestsFromCollection@@YAXPEAU_DMF_CONTEXT_ContinuousRequestTarget@@@Z 0000000180021738 f   DmfK:Dmf_ContinuousRequestTarget.obj
 0001:000207c0       ?ContinuousRequestTarget_FormatRequestForRequestType@@YAJPEAUDMFMODULE__@@PEAUWDFREQUEST__@@W4ContinuousRequestTarget_RequestType@@KPEAUWDFMEMORY__@@3@Z 00000001800217c0 f   DmfK:Dmf_ContinuousRequestTarget.obj
 0001:00020a98       ?ContinuousRequestTarget_PendingCollectionListAdd@@YAJPEAUDMFMODULE__@@PEAUWDFREQUEST__@@@Z 0000000180021a98 f   DmfK:Dmf_ContinuousRequestTarget.obj
 0001:00020bf8       ?ContinuousRequestTarget_PendingCollectionListSearchAndReference@@YAEPEAUDMFMODULE__@@PEAURequestTarget_DmfRequest__@@PEAPEAUWDFREQUEST__@@@Z 0000000180021bf8 f   DmfK:Dmf_ContinuousRequestTarget.obj
 0001:00020da0       ?ContinuousRequestTarget_PendingCollectionListSearchAndRemove@@YAEPEAUDMFMODULE__@@PEAUWDFREQUEST__@@@Z 0000000180021da0 f   DmfK:Dmf_ContinuousRequestTarget.obj
 0001:0002126c       ?ContinuousRequestTarget_ProcessAsynchronousRequestStream@@YAXPEAUDMFMODULE__@@PEAUWDFREQUEST__@@PEAU_WDF_REQUEST_COMPLETION_PARAMS@@@Z 000000018002226c f   DmfK:Dmf_ContinuousRequestTarget.obj
 0001:0002176c       ?ContinuousRequestTarget_RequestCreateAndSend@@YAJPEAUDMFMODULE__@@EPEAX_K12W4ContinuousRequestTarget_RequestType@@KKW4ContinuousRequestTarget_CompletionOptions@@PEA_KP6AX011212J@Z1PEAPEAURequestTarget_DmfRequest__@@@Z 000000018002276c f   DmfK:Dmf_ContinuousRequestTarget.obj
 0001:00022404       ?ContinuousRequestTarget_StreamRequestSend@@YAJPEAUDMFMODULE__@@PEAUWDFREQUEST__@@@Z 0000000180023404 f   DmfK:Dmf_ContinuousRequestTarget.obj
 0001:000227a0       ?DMF_ContinuousRequestTarget_ModuleD0Entry@@YAJPEAUDMFMODULE__@@W4_WDF_POWER_DEVICE_STATE@@@Z 00000001800237a0 f   DmfK:Dmf_ContinuousRequestTarget.obj
 0001:000228f0       ?DMF_ContinuousRequestTarget_ModuleD0Exit@@YAJPEAUDMFMODULE__@@W4_WDF_POWER_DEVICE_STATE@@@Z 00000001800238f0 f   DmfK:Dmf_ContinuousRequestTarget.obj
 0001:000241d0       $$000000                   00000001800251d0     BufferOverflowFastFailK:amdsecgs.obj
 0001:00024210       $$000000                   0000000180025210     BufferOverflowFastFailK:guard_dispatch.obj
 0001:00024230       $$000000                   0000000180025230     BufferOverflowFastFailK:guard_xfg_dispatch.obj
 0001:00024250       $$000000                   0000000180025250     BufferOverflowFastFailK:dispatchcfg.obj
 0001:00024280       $$000000                   0000000180025280     ntoskrnl:memset.obj
 0001:000242a2       mset10                     00000001800252a2     ntoskrnl:memset.obj
 0001:000242b8       mset20                     00000001800252b8     ntoskrnl:memset.obj
 0001:000242e1       mset30                     00000001800252e1     ntoskrnl:memset.obj
 0001:00024310       mset45                     0000000180025310     ntoskrnl:memset.obj
 0001:00024316       mset46                     0000000180025316     ntoskrnl:memset.obj
 0001:00024340       mset47                     0000000180025340     ntoskrnl:memset.obj
 0001:00024370       mset48                     0000000180025370     ntoskrnl:memset.obj
 0001:00024386       mset50                     0000000180025386     ntoskrnl:memset.obj
 0001:000243c0       $$000000                   00000001800253c0     ntoskrnl:memset.obj
 0001:000243ca       repmovs10                  00000001800253ca     ntoskrnl:memset.obj
 0001:000243fc       repmovs20                  00000001800253fc     ntoskrnl:memset.obj
 0001:00024440       $$000000                   0000000180025440     ntoskrnl:memset.obj
 0001:00024480       $$000000                   0000000180025480     ntoskrnl:memcpy.obj
 0001:000244a0       mcpy00                     00000001800254a0     ntoskrnl:memcpy.obj
 0001:000244c0       mcpy10                     00000001800254c0     ntoskrnl:memcpy.obj
 0001:000244da       mcpy20                     00000001800254da     ntoskrnl:memcpy.obj
 0001:000244e0       mcpy30                     00000001800254e0     ntoskrnl:memcpy.obj
 0001:00024500       xcpy00                     0000000180025500     ntoskrnl:memcpy.obj
 0001:00024531       xcpy10                     0000000180025531     ntoskrnl:memcpy.obj
 0001:00024580       xcpy13                     0000000180025580     ntoskrnl:memcpy.obj
 0001:000245af       xcpy15                     00000001800255af     ntoskrnl:memcpy.obj
 0001:000245d1       xcpy20                     00000001800255d1     ntoskrnl:memcpy.obj
 0001:000245e5       xcpy30                     00000001800255e5     ntoskrnl:memcpy.obj
 0001:00024600       lcpy00                     0000000180025600     ntoskrnl:memcpy.obj
 0001:00024640       lcpy10                     0000000180025640     ntoskrnl:memcpy.obj
 0001:00024680       xmov00                     0000000180025680     ntoskrnl:memcpy.obj
 0001:000246ad       xmov10                     00000001800256ad     ntoskrnl:memcpy.obj
 0001:000246c0       xmov13                     00000001800256c0     ntoskrnl:memcpy.obj
 0001:000246ef       xmov15                     00000001800256ef     ntoskrnl:memcpy.obj
 0001:00024711       xmov20                     0000000180025711     ntoskrnl:memcpy.obj
 0001:00024726       xmov30                     0000000180025726     ntoskrnl:memcpy.obj
 0001:00025a50       _ZN4core9panicking9panic_fmt17hfaa5e12b02d15589E 0000000180026a50 f   surface_hid_mini.surface_hid_mini.3efcb60154bd7459-cgu.0.rcgu.o
 0001:00025a70       _ZN4core6option13expect_failed17hb8b89a9869eeafb0E 0000000180026a70 f   surface_hid_mini.surface_hid_mini.3efcb60154bd7459-cgu.0.rcgu.o
 0001:00025a70       _ZN4core9panicking18panic_bounds_check17he514c840e670f99bE 0000000180026a70 f   surface_hid_mini.surface_hid_mini.3efcb60154bd7459-cgu.0.rcgu.o
 0001:00025a70       _ZN4core9panicking5panic17h3e0319af96206e7cE 0000000180026a70 f   surface_hid_mini.surface_hid_mini.3efcb60154bd7459-cgu.0.rcgu.o
 0001:00025a80       _ZN4spin4once17Once$LT$T$C$R$GT$18try_call_once_slow17h6df211ed18ed61afE 0000000180026a80 f   surface_hid_mini.surface_hid_mini.3efcb60154bd7459-cgu.0.rcgu.o
 0002:00000b30       anon.558d06e7660b46fb1a5372ee215ddf6c.0 0000000180027b30     surface_hid_mini.surface_hid_mini.3efcb60154bd7459-cgu.0.rcgu.o
 0002:00000b53       anon.558d06e7660b46fb1a5372ee215ddf6c.7 0000000180027b53     surface_hid_mini.surface_hid_mini.3efcb60154bd7459-cgu.0.rcgu.o
 0002:00000b88       anon.558d06e7660b46fb1a5372ee215ddf6c.10 0000000180027b88     surface_hid_mini.surface_hid_mini.3efcb60154bd7459-cgu.0.rcgu.o
 0002:00000bb5       anon.558d06e7660b46fb1a5372ee215ddf6c.11 0000000180027bb5     surface_hid_mini.surface_hid_mini.3efcb60154bd7459-cgu.0.rcgu.o
 0002:00000be2       anon.558d06e7660b46fb1a5372ee215ddf6c.15 0000000180027be2     surface_hid_mini.surface_hid_mini.3efcb60154bd7459-cgu.0.rcgu.o
 0002:00000bf8       anon.558d06e7660b46fb1a5372ee215ddf6c.16 0000000180027bf8     surface_hid_mini.surface_hid_mini.3efcb60154bd7459-cgu.0.rcgu.o
 0002:00000c34       anon.558d06e7660b46fb1a5372ee215ddf6c.18 0000000180027c34     surface_hid_mini.surface_hid_mini.3efcb60154bd7459-cgu.0.rcgu.o
 0002:00000c69       anon.558d06e7660b46fb1a5372ee215ddf6c.22 0000000180027c69     surface_hid_mini.surface_hid_mini.3efcb60154bd7459-cgu.0.rcgu.o
 0002:00000c99       anon.558d06e7660b46fb1a5372ee215ddf6c.23 0000000180027c99     surface_hid_mini.surface_hid_mini.3efcb60154bd7459-cgu.0.rcgu.o
 0002:00000cd6       anon.558d06e7660b46fb1a5372ee215ddf6c.25 0000000180027cd6     surface_hid_mini.surface_hid_mini.3efcb60154bd7459-cgu.0.rcgu.o
 0002:00000cfe       anon.558d06e7660b46fb1a5372ee215ddf6c.26 0000000180027cfe     surface_hid_mini.surface_hid_mini.3efcb60154bd7459-cgu.0.rcgu.o
 0002:00000d34       anon.558d06e7660b46fb1a5372ee215ddf6c.29 0000000180027d34     surface_hid_mini.surface_hid_mini.3efcb60154bd7459-cgu.0.rcgu.o
 0002:00000d67       anon.558d06e7660b46fb1a5372ee215ddf6c.30 0000000180027d67     surface_hid_mini.surface_hid_mini.3efcb60154bd7459-cgu.0.rcgu.o
 0002:00000da2       anon.558d06e7660b46fb1a5372ee215ddf6c.31 0000000180027da2     surface_hid_mini.surface_hid_mini.3efcb60154bd7459-cgu.0.rcgu.o
 0002:00000dee       anon.558d06e7660b46fb1a5372ee215ddf6c.32 0000000180027dee     surface_hid_mini.surface_hid_mini.3efcb60154bd7459-cgu.0.rcgu.o
 0002:00000e2a       anon.558d06e7660b46fb1a5372ee215ddf6c.33 0000000180027e2a     surface_hid_mini.surface_hid_mini.3efcb60154bd7459-cgu.0.rcgu.o
 0002:00000e77       anon.558d06e7660b46fb1a5372ee215ddf6c.46 0000000180027e77     surface_hid_mini.surface_hid_mini.3efcb60154bd7459-cgu.0.rcgu.o
 0002:00000eaf       anon.558d06e7660b46fb1a5372ee215ddf6c.48 0000000180027eaf     surface_hid_mini.surface_hid_mini.3efcb60154bd7459-cgu.0.rcgu.o
 0002:00000edf       anon.558d06e7660b46fb1a5372ee215ddf6c.49 0000000180027edf     surface_hid_mini.surface_hid_mini.3efcb60154bd7459-cgu.0.rcgu.o
 0002:00000eff       anon.558d06e7660b46fb1a5372ee215ddf6c.50 0000000180027eff     surface_hid_mini.surface_hid_mini.3efcb60154bd7459-cgu.0.rcgu.o
 0002:00000f50       anon.558d06e7660b46fb1a5372ee215ddf6c.53 0000000180027f50     surface_hid_mini.surface_hid_mini.3efcb60154bd7459-cgu.0.rcgu.o
 0002:00000f73       anon.558d06e7660b46fb1a5372ee215ddf6c.54 0000000180027f73     surface_hid_mini.surface_hid_mini.3efcb60154bd7459-cgu.0.rcgu.o
 0002:00000fd7       anon.558d06e7660b46fb1a5372ee215ddf6c.56 0000000180027fd7     surface_hid_mini.surface_hid_mini.3efcb60154bd7459-cgu.0.rcgu.o
 0002:0000102c       anon.558d06e7660b46fb1a5372ee215ddf6c.57 000000018002802c     surface_hid_mini.surface_hid_mini.3efcb60154bd7459-cgu.0.rcgu.o
 0002:00001089       anon.558d06e7660b46fb1a5372ee215ddf6c.58 0000000180028089     surface_hid_mini.surface_hid_mini.3efcb60154bd7459-cgu.0.rcgu.o
 0002:000010b6       anon.558d06e7660b46fb1a5372ee215ddf6c.59 00000001800280b6     surface_hid_mini.surface_hid_mini.3efcb60154bd7459-cgu.0.rcgu.o
 0002:000010e4       anon.e3a2ac5b3cda3fa87eac5206a81e382b.0 00000001800280e4     surface_hid_mini.surface_hid_mini.3efcb60154bd7459-cgu.0.rcgu.o
 0002:000010f9       anon.e3a2ac5b3cda3fa87eac5206a81e382b.1 00000001800280f9     surface_hid_mini.surface_hid_mini.3efcb60154bd7459-cgu.0.rcgu.o
 0002:00001127       anon.e3a2ac5b3cda3fa87eac5206a81e382b.2 0000000180028127     surface_hid_mini.surface_hid_mini.3efcb60154bd7459-cgu.0.rcgu.o
 0002:00001149       anon.e3a2ac5b3cda3fa87eac5206a81e382b.3 0000000180028149     surface_hid_mini.surface_hid_mini.3efcb60154bd7459-cgu.0.rcgu.o
 0002:00001182       anon.e3a2ac5b3cda3fa87eac5206a81e382b.9 0000000180028182     surface_hid_mini.surface_hid_mini.3efcb60154bd7459-cgu.0.rcgu.o
 0002:000011a1       anon.e3a2ac5b3cda3fa87eac5206a81e382b.10 00000001800281a1     surface_hid_mini.surface_hid_mini.3efcb60154bd7459-cgu.0.rcgu.o
 0002:000011e1       anon.e3a2ac5b3cda3fa87eac5206a81e382b.11 00000001800281e1     surface_hid_mini.surface_hid_mini.3efcb60154bd7459-cgu.0.rcgu.o
 0002:000011f1       anon.e3a2ac5b3cda3fa87eac5206a81e382b.12 00000001800281f1     surface_hid_mini.surface_hid_mini.3efcb60154bd7459-cgu.0.rcgu.o
 0002:00001210       anon.e3a2ac5b3cda3fa87eac5206a81e382b.13 0000000180028210     surface_hid_mini.surface_hid_mini.3efcb60154bd7459-cgu.0.rcgu.o
 0002:00001220       anon.e3a2ac5b3cda3fa87eac5206a81e382b.14 0000000180028220     surface_hid_mini.surface_hid_mini.3efcb60154bd7459-cgu.0.rcgu.o
 0002:0000123f       anon.e3a2ac5b3cda3fa87eac5206a81e382b.15 000000018002823f     surface_hid_mini.surface_hid_mini.3efcb60154bd7459-cgu.0.rcgu.o
 0002:0000124f       anon.e3a2ac5b3cda3fa87eac5206a81e382b.16 000000018002824f     surface_hid_mini.surface_hid_mini.3efcb60154bd7459-cgu.0.rcgu.o
 0002:00001268       anon.e3a2ac5b3cda3fa87eac5206a81e382b.17 0000000180028268     surface_hid_mini.surface_hid_mini.3efcb60154bd7459-cgu.0.rcgu.o
 0002:000012a0       anon.e3a2ac5b3cda3fa87eac5206a81e382b.18 00000001800282a0     surface_hid_mini.surface_hid_mini.3efcb60154bd7459-cgu.0.rcgu.o
 0002:000012c7       anon.e3a2ac5b3cda3fa87eac5206a81e382b.19 00000001800282c7     surface_hid_mini.surface_hid_mini.3efcb60154bd7459-cgu.0.rcgu.o
 0002:000012f1       anon.e3a2ac5b3cda3fa87eac5206a81e382b.20 00000001800282f1     surface_hid_mini.surface_hid_mini.3efcb60154bd7459-cgu.0.rcgu.o
 0002:00001306       anon.e3a2ac5b3cda3fa87eac5206a81e382b.21 0000000180028306     surface_hid_mini.surface_hid_mini.3efcb60154bd7459-cgu.0.rcgu.o
 0002:00001336       anon.e3a2ac5b3cda3fa87eac5206a81e382b.22 0000000180028336     surface_hid_mini.surface_hid_mini.3efcb60154bd7459-cgu.0.rcgu.o
 0002:0000134b       anon.e3a2ac5b3cda3fa87eac5206a81e382b.23 000000018002834b     surface_hid_mini.surface_hid_mini.3efcb60154bd7459-cgu.0.rcgu.o
 0002:0000137b       anon.e3a2ac5b3cda3fa87eac5206a81e382b.24 000000018002837b     surface_hid_mini.surface_hid_mini.3efcb60154bd7459-cgu.0.rcgu.o
 0002:0000138f       anon.e3a2ac5b3cda3fa87eac5206a81e382b.25 000000018002838f     surface_hid_mini.surface_hid_mini.3efcb60154bd7459-cgu.0.rcgu.o
 0002:000013c2       anon.e3a2ac5b3cda3fa87eac5206a81e382b.26 00000001800283c2     surface_hid_mini.surface_hid_mini.3efcb60154bd7459-cgu.0.rcgu.o
 0002:000013dc       anon.e3a2ac5b3cda3fa87eac5206a81e382b.27 00000001800283dc     surface_hid_mini.surface_hid_mini.3efcb60154bd7459-cgu.0.rcgu.o
 0002:0000140a       anon.e3a2ac5b3cda3fa87eac5206a81e382b.28 000000018002840a     surface_hid_mini.surface_hid_mini.3efcb60154bd7459-cgu.0.rcgu.o
 0002:0000144a       anon.e3a2ac5b3cda3fa87eac5206a81e382b.29 000000018002844a     surface_hid_mini.surface_hid_mini.3efcb60154bd7459-cgu.0.rcgu.o
 0002:00001475       anon.e3a2ac5b3cda3fa87eac5206a81e382b.30 0000000180028475     surface_hid_mini.surface_hid_mini.3efcb60154bd7459-cgu.0.rcgu.o
 0002:000014c8       anon.e3a2ac5b3cda3fa87eac5206a81e382b.32 00000001800284c8     surface_hid_mini.surface_hid_mini.3efcb60154bd7459-cgu.0.rcgu.o
 0002:000014d8       anon.e3a2ac5b3cda3fa87eac5206a81e382b.36 00000001800284d8     surface_hid_mini.surface_hid_mini.3efcb60154bd7459-cgu.0.rcgu.o
 0002:000014e8       anon.e3a2ac5b3cda3fa87eac5206a81e382b.40 00000001800284e8     surface_hid_mini.surface_hid_mini.3efcb60154bd7459-cgu.0.rcgu.o
 0002:00001516       anon.e3a2ac5b3cda3fa87eac5206a81e382b.41 0000000180028516     surface_hid_mini.surface_hid_mini.3efcb60154bd7459-cgu.0.rcgu.o
 0002:00001524       anon.e3a2ac5b3cda3fa87eac5206a81e382b.43 0000000180028524     surface_hid_mini.surface_hid_mini.3efcb60154bd7459-cgu.0.rcgu.o
 0002:00001532       anon.e3a2ac5b3cda3fa87eac5206a81e382b.45 0000000180028532     surface_hid_mini.surface_hid_mini.3efcb60154bd7459-cgu.0.rcgu.o
 0002:00001574       anon.e3a2ac5b3cda3fa87eac5206a81e382b.46 0000000180028574     surface_hid_mini.surface_hid_mini.3efcb60154bd7459-cgu.0.rcgu.o
 0002:00001599       anon.75dfd425df8ddff00c3c895f31bc1b57.0 0000000180028599     surface_hid_mini.surface_hid_mini.3efcb60154bd7459-cgu.0.rcgu.o
 0002:000015d6       anon.75dfd425df8ddff00c3c895f31bc1b57.1 00000001800285d6     surface_hid_mini.surface_hid_mini.3efcb60154bd7459-cgu.0.rcgu.o
 0002:00001608       anon.75dfd425df8ddff00c3c895f31bc1b57.2 0000000180028608     surface_hid_mini.surface_hid_mini.3efcb60154bd7459-cgu.0.rcgu.o
 0002:00001618       anon.75dfd425df8ddff00c3c895f31bc1b57.3 0000000180028618     surface_hid_mini.surface_hid_mini.3efcb60154bd7459-cgu.0.rcgu.o
 0002:00001680       anon.75dfd425df8ddff00c3c895f31bc1b57.4 0000000180028680     surface_hid_mini.surface_hid_mini.3efcb60154bd7459-cgu.0.rcgu.o
 0002:00001690       anon.75dfd425df8ddff00c3c895f31bc1b57.5 0000000180028690     surface_hid_mini.surface_hid_mini.3efcb60154bd7459-cgu.0.rcgu.o
 0002:00001710       anon.75dfd425df8ddff00c3c895f31bc1b57.6 0000000180028710     surface_hid_mini.surface_hid_mini.3efcb60154bd7459-cgu.0.rcgu.o
 0002:00001720       anon.75dfd425df8ddff00c3c895f31bc1b57.7 0000000180028720     surface_hid_mini.surface_hid_mini.3efcb60154bd7459-cgu.0.rcgu.o
 0002:000017a0       anon.75dfd425df8ddff00c3c895f31bc1b57.8 00000001800287a0     surface_hid_mini.surface_hid_mini.3efcb60154bd7459-cgu.0.rcgu.o
 0002:000017b0       anon.75dfd425df8ddff00c3c895f31bc1b57.9 00000001800287b0     surface_hid_mini.surface_hid_mini.3efcb60154bd7459-cgu.0.rcgu.o
 0002:00001830       anon.75dfd425df8ddff00c3c895f31bc1b57.10 0000000180028830     surface_hid_mini.surface_hid_mini.3efcb60154bd7459-cgu.0.rcgu.o
 0002:00001840       anon.75dfd425df8ddff00c3c895f31bc1b57.11 0000000180028840     surface_hid_mini.surface_hid_mini.3efcb60154bd7459-cgu.0.rcgu.o
 0002:000018c0       anon.75dfd425df8ddff00c3c895f31bc1b57.12 00000001800288c0     surface_hid_mini.surface_hid_mini.3efcb60154bd7459-cgu.0.rcgu.o
 0002:000018d0       anon.75dfd425df8ddff00c3c895f31bc1b57.15 00000001800288d0     surface_hid_mini.surface_hid_mini.3efcb60154bd7459-cgu.0.rcgu.o
 0002:000018e0       anon.75dfd425df8ddff00c3c895f31bc1b57.21 00000001800288e0     surface_hid_mini.surface_hid_mini.3efcb60154bd7459-cgu.0.rcgu.o
 0002:0000190d       anon.75dfd425df8ddff00c3c895f31bc1b57.22 000000018002890d     surface_hid_mini.surface_hid_mini.3efcb60154bd7459-cgu.0.rcgu.o
 0002:00001958       anon.75dfd425df8ddff00c3c895f31bc1b57.23 0000000180028958     surface_hid_mini.surface_hid_mini.3efcb60154bd7459-cgu.0.rcgu.o
 0002:00001968       anon.75dfd425df8ddff00c3c895f31bc1b57.24 0000000180028968     surface_hid_mini.surface_hid_mini.3efcb60154bd7459-cgu.0.rcgu.o
 0002:00001996       anon.75dfd425df8ddff00c3c895f31bc1b57.25 0000000180028996     surface_hid_mini.surface_hid_mini.3efcb60154bd7459-cgu.0.rcgu.o
 0002:000019b8       anon.75dfd425df8ddff00c3c895f31bc1b57.26 00000001800289b8     surface_hid_mini.surface_hid_mini.3efcb60154bd7459-cgu.0.rcgu.o
 0002:000019b9       anon.75dfd425df8ddff00c3c895f31bc1b57.27 00000001800289b9     surface_hid_mini.surface_hid_mini.3efcb60154bd7459-cgu.0.rcgu.o
 0002:000019e7       anon.75dfd425df8ddff00c3c895f31bc1b57.28 00000001800289e7     surface_hid_mini.surface_hid_mini.3efcb60154bd7459-cgu.0.rcgu.o
 0002:00001a14       anon.75dfd425df8ddff00c3c895f31bc1b57.29 0000000180028a14     surface_hid_mini.surface_hid_mini.3efcb60154bd7459-cgu.0.rcgu.o
 0002:00001a53       anon.75dfd425df8ddff00c3c895f31bc1b57.30 0000000180028a53     surface_hid_mini.surface_hid_mini.3efcb60154bd7459-cgu.0.rcgu.o
 0002:00001a81       anon.75dfd425df8ddff00c3c895f31bc1b57.31 0000000180028a81     surface_hid_mini.surface_hid_mini.3efcb60154bd7459-cgu.0.rcgu.o
 0002:00001ab0       anon.75dfd425df8ddff00c3c895f31bc1b57.32 0000000180028ab0     surface_hid_mini.surface_hid_mini.3efcb60154bd7459-cgu.0.rcgu.o
 0002:00001b00       anon.75dfd425df8ddff00c3c895f31bc1b57.33 0000000180028b00     surface_hid_mini.surface_hid_mini.3efcb60154bd7459-cgu.0.rcgu.o
 0002:00001b08       anon.75dfd425df8ddff00c3c895f31bc1b57.34 0000000180028b08     surface_hid_mini.surface_hid_mini.3efcb60154bd7459-cgu.0.rcgu.o
 0002:00001b10       anon.75dfd425df8ddff00c3c895f31bc1b57.39 0000000180028b10     surface_hid_mini.surface_hid_mini.3efcb60154bd7459-cgu.0.rcgu.o
 0002:00001b20       anon.75dfd425df8ddff00c3c895f31bc1b57.40 0000000180028b20     surface_hid_mini.surface_hid_mini.3efcb60154bd7459-cgu.0.rcgu.o
 0002:00001b55       anon.75dfd425df8ddff00c3c895f31bc1b57.41 0000000180028b55     surface_hid_mini.surface_hid_mini.3efcb60154bd7459-cgu.0.rcgu.o
 0002:00001b94       anon.75dfd425df8ddff00c3c895f31bc1b57.42 0000000180028b94     surface_hid_mini.surface_hid_mini.3efcb60154bd7459-cgu.0.rcgu.o
 0002:00001ba4       anon.75dfd425df8ddff00c3c895f31bc1b57.43 0000000180028ba4     surface_hid_mini.surface_hid_mini.3efcb60154bd7459-cgu.0.rcgu.o
 0002:00001bcf       anon.75dfd425df8ddff00c3c895f31bc1b57.45 0000000180028bcf     surface_hid_mini.surface_hid_mini.3efcb60154bd7459-cgu.0.rcgu.o
 0002:00001c0d       anon.1b8ae7f0ee4e78eae5b03d8aa8b06ca3.0 0000000180028c0d     surface_hid_mini.surface_hid_mini.3efcb60154bd7459-cgu.0.rcgu.o
 0002:00001c1a       anon.1b8ae7f0ee4e78eae5b03d8aa8b06ca3.3 0000000180028c1a     surface_hid_mini.surface_hid_mini.3efcb60154bd7459-cgu.0.rcgu.o
 0002:00002be0       ?CrcTable@@3QBGB           0000000180029be0     DmfK:DmfUtility.obj
 0002:00002f18       PoCompressMethodMap        0000000180029f18     DmfK:stubgen_data.obj
 0002:00003558       $xdatasym                  000000018002a558     BufferOverflowFastFailK:amdsecgs.obj
 0002:00003560       $xdatasym$_guard_dispatch_icall 000000018002a560     BufferOverflowFastFailK:dispatchcfg.obj
 0002:00003560       $xdatasym$_guard_dispatch_icall_nop 000000018002a560     BufferOverflowFastFailK:guard_dispatch.obj
 0002:00003560       $xdatasym$_guard_xfg_dispatch_icall_nop 000000018002a560     BufferOverflowFastFailK:guard_xfg_dispatch.obj
 0002:00003560       $xdatasym$memcpy           000000018002a560     ntoskrnl:memcpy.obj
 0002:00003560       $xdatasym$memset           000000018002a560     ntoskrnl:memset.obj
 0002:00003568       $xdatasym$__memset_repmovs 000000018002a568     ntoskrnl:memset.obj
 0002:00003578       $xdatasym$__memset_query   000000018002a578     ntoskrnl:memset.obj
 0002:00003590       $unwind$__cpu_features_init 000000018002a590     ntoskrnl:cpuinfo.obj
 0002:000035a0       $unwind$?FxStubDriverEntryFailure@@YAXXZ 000000018002a5a0     WdfDriverEntry:stub.obj
 0002:000035ac       $unwind$FxDriverEntryWorker 000000018002a5ac     WdfDriverEntry:stub.obj
 0002:000035c8       $unwind$FxDriverEntry      000000018002a5c8     WdfDriverEntry:stub.obj
 0002:000035c8       $unwind$LkmdTelSubmitReport 000000018002a5c8     DmfK:lkmdtel.obj
 0002:000035d8       $unwind$__GSHandlerCheck   000000018002a5d8     ntoskrnl:gshandler.obj
 0002:000035d8       $unwind$__GSHandlerCheckCommon 000000018002a5d8     ntoskrnl:gshandler.obj
 0002:000035d8       $unwind$?FxStubDriverUnloadCommon@@YAXXZ 000000018002a5d8     WdfDriverEntry:stub.obj
 0002:000035d8       $unwind$FxStubDriverMiniportUnload 000000018002a5d8     WdfDriverEntry:stub.obj
 0002:000035d8       $unwind$FxStubDriverUnload 000000018002a5d8     WdfDriverEntry:stub.obj
 0002:000035d8       $unwind$LkmdTelpAllocateMem 000000018002a5d8     DmfK:lkmdtel.obj
 0002:000035e4       $unwind$?FxStubInitTypes@@YAJXZ 000000018002a5e4     WdfDriverEntry:inittypes.obj
 0002:000035f4       $unwind$?FxStubUnbindClasses@@YAXPEAU_WDF_BIND_INFO@@@Z 000000018002a5f4     WdfDriverEntry:classbind.obj
 0002:00003608       $unwind$?FxStubBindClasses@@YAJPEAU_WDF_BIND_INFO@@@Z 000000018002a608     WdfDriverEntry:classbind.obj
 0002:00003620       $unwind$WppInitialize      000000018002a620     libms_surface_wpp-b83efe80b23bd200:2e40c9e35e9506f4-wpp.o
 0002:00003630       $unwind$WppCleanup         000000018002a630     libms_surface_wpp-b83efe80b23bd200:2e40c9e35e9506f4-wpp.o
 0002:00003638       $unwind$WppLoadTracingSupport 000000018002a638     libms_surface_wpp-b83efe80b23bd200:2e40c9e35e9506f4-wpp.o
 0002:00003640       $unwind$WppTraceCallback   000000018002a640     libms_surface_wpp-b83efe80b23bd200:2e40c9e35e9506f4-wpp.o
 0002:0000365c       $unwind$WppCleanupKm       000000018002a65c     libms_surface_wpp-b83efe80b23bd200:2e40c9e35e9506f4-wpp.o
 0002:0000366c       $chain$0$WppCleanupKm      000000018002a66c     libms_surface_wpp-b83efe80b23bd200:2e40c9e35e9506f4-wpp.o
 0002:00003680       $chain$1$WppCleanupKm      000000018002a680     libms_surface_wpp-b83efe80b23bd200:2e40c9e35e9506f4-wpp.o
 0002:00003690       $unwind$WPP_RECORDER_SF_   000000018002a690     libms_surface_wpp-b83efe80b23bd200:2e40c9e35e9506f4-wpp.o
 0002:000036a8       $unwind$WppInitKm          000000018002a6a8     libms_surface_wpp-b83efe80b23bd200:2e40c9e35e9506f4-wpp.o
 0002:000036b8       $chain$1$WppInitKm         000000018002a6b8     libms_surface_wpp-b83efe80b23bd200:2e40c9e35e9506f4-wpp.o
 0002:000036d0       $chain$2$WppInitKm         000000018002a6d0     libms_surface_wpp-b83efe80b23bd200:2e40c9e35e9506f4-wpp.o
 0002:000036e0       $unwind$WdfObjectAddCustomType_DMF_BranchTrack 000000018002a6e0     DmfK:Dmf_BranchTrack.obj
 0002:000036e0       $unwind$WdfObjectAddCustomType_DMF_Bridge 000000018002a6e0     DmfK:Dmf_Bridge.obj
 0002:000036e0       $unwind$WdfObjectAddCustomType_DMF_BufferPool 000000018002a6e0     DmfK:Dmf_BufferPool.obj
 0002:000036e0       $unwind$WdfObjectAddCustomType_DMF_BufferQueue 000000018002a6e0     DmfK:Dmf_BufferQueue.obj
 0002:000036e0       $unwind$WdfObjectAddCustomType_DMF_ContinuousRequestTarget 000000018002a6e0     DmfK:Dmf_ContinuousRequestTarget.obj
 0002:000036e0       $unwind$WdfObjectAddCustomType_DMF_CrashDump 000000018002a6e0     DmfK:Dmf_CrashDump.obj
 0002:000036e0       $unwind$WdfObjectAddCustomType_DMF_DeviceInterfaceTarget 000000018002a6e0     DmfK:Dmf_DeviceInterfaceTarget.obj
 0002:000036e0       $unwind$WdfObjectAddCustomType_DMF_HashTable 000000018002a6e0     DmfK:Dmf_HashTable.obj
 0002:000036e0       $unwind$WdfObjectAddCustomType_DMF_IoctlHandler 000000018002a6e0     DmfK:Dmf_IoctlHandler.obj
 0002:000036e0       $unwind$WdfObjectAddCustomType_DMF_LiveKernelDump 000000018002a6e0     DmfK:Dmf_LiveKernelDump.obj
 0002:000036e0       $unwind$WdfObjectAddCustomType_DMF_QueuedWorkItem 000000018002a6e0     DmfK:Dmf_QueuedWorkItem.obj
 0002:000036e0       $unwind$WdfObjectAddCustomType_DMF_RequestTarget 000000018002a6e0     DmfK:Dmf_RequestTarget.obj
 0002:000036e0       $unwind$WdfObjectAddCustomType_DMF_RingBuffer 000000018002a6e0     DmfK:Dmf_RingBuffer.obj
 0002:000036e0       $unwind$WdfObjectAddCustomType_DMF_Rundown 000000018002a6e0     DmfK:Dmf_Rundown.obj
 0002:000036e0       $unwind$WdfObjectAddCustomType_DMF_SamCommunicationViaSsh 000000018002a6e0     DmfK:Dmf_SamCommunicationViaSsh.obj
 0002:000036e0       $unwind$WdfObjectAddCustomType_DMF_SamNotificationViaSsh 000000018002a6e0     DmfK:Dmf_SamNotificationViaSsh.obj
 0002:000036e0       $unwind$WdfObjectAddCustomType_DMF_ScheduledTask 000000018002a6e0     DmfK:Dmf_ScheduledTask.obj
 0002:000036e0       $unwind$WdfObjectAddCustomType_DMF_SmbiosWmi 000000018002a6e0     DmfK:Dmf_SmbiosWmi.obj
 0002:000036e0       $unwind$WdfObjectAddCustomType_DMF_String 000000018002a6e0     DmfK:Dmf_String.obj
 0002:000036e0       $unwind$WdfObjectAddCustomType_DMF_SurfaceTelemetryConsentSettingsNotification 000000018002a6e0     DmfK:Dmf_SurfaceTelemetryConsentSettingsNotification.obj
 0002:000036f0       $unwind$DMF_BufferPool_Create 000000018002a6f0     DmfK:Dmf_BufferPool.obj
 0002:000036f0       $unwind$DMF_DeviceInterfaceTarget_Create 000000018002a6f0     DmfK:Dmf_DeviceInterfaceTarget.obj
 0002:00003714       $unwind$DmfContainerEvtDevicePrepareHardware 000000018002a714     DmfK:DmfContainer.obj
 0002:00003714       $unwind$?DMF_ModuleCollectionDestroy@@YAXPEAX@Z 000000018002a714     DmfK:DmfModuleCollection.obj
 0002:00003714       $unwind$?DMF_Bridge_ModuleD0Entry@@YAJPEAUDMFMODULE__@@W4_WDF_POWER_DEVICE_STATE@@@Z 000000018002a714     DmfK:Dmf_Bridge.obj
 0002:00003714       $unwind$?DMF_Bridge_ModuleD0EntryPostInterruptsEnabled@@YAJPEAUDMFMODULE__@@W4_WDF_POWER_DEVICE_STATE@@@Z 000000018002a714     DmfK:Dmf_Bridge.obj
 0002:00003714       $unwind$?DMF_Bridge_ModuleD0Exit@@YAJPEAUDMFMODULE__@@W4_WDF_POWER_DEVICE_STATE@@@Z 000000018002a714     DmfK:Dmf_Bridge.obj
 0002:00003714       $unwind$?DMF_Bridge_ModuleD0ExitPreInterruptsDisabled@@YAJPEAUDMFMODULE__@@W4_WDF_POWER_DEVICE_STATE@@@Z 000000018002a714     DmfK:Dmf_Bridge.obj
 0002:00003714       $unwind$?DMF_Bridge_ModuleFileCleanup@@YAEPEAUDMFMODULE__@@PEAUWDFFILEOBJECT__@@@Z 000000018002a714     DmfK:Dmf_Bridge.obj
 0002:00003714       $unwind$?DMF_Bridge_ModuleFileClose@@YAEPEAUDMFMODULE__@@PEAUWDFFILEOBJECT__@@@Z 000000018002a714     DmfK:Dmf_Bridge.obj
 0002:00003714       $unwind$?DMF_Bridge_ModuleReleaseHardware@@YAJPEAUDMFMODULE__@@PEAUWDFCMRESLIST__@@@Z 000000018002a714     DmfK:Dmf_Bridge.obj
 0002:00003714       $unwind$DMF_BufferPool_ContextGet 000000018002a714     DmfK:Dmf_BufferPool.obj
 0002:00003714       $unwind$DMF_BufferQueue_Dequeue 000000018002a714     DmfK:Dmf_BufferQueue.obj
 0002:00003714       $unwind$DMF_BufferQueue_Fetch 000000018002a714     DmfK:Dmf_BufferQueue.obj
 0002:00003714       $unwind$?DMF_ContinuousRequestTarget_ModuleD0Exit@@YAJPEAUDMFMODULE__@@W4_WDF_POWER_DEVICE_STATE@@@Z 000000018002a714     DmfK:Dmf_ContinuousRequestTarget.obj
 0002:00003730       $unwind$DmfContainerEvtDeviceD0EntryPostInterruptsEnabled 000000018002a730     DmfK:DmfContainer.obj
 0002:00003730       $unwind$DmfContainerEvtDeviceD0Exit 000000018002a730     DmfK:DmfContainer.obj
 0002:00003730       $unwind$DmfContainerEvtDeviceD0ExitPreInterruptsDisabled 000000018002a730     DmfK:DmfContainer.obj
 0002:00003730       $unwind$DmfContainerEvtDeviceReleaseHardware 000000018002a730     DmfK:DmfContainer.obj
 0002:00003730       $unwind$DmfContainerEvtFileCleanup 000000018002a730     DmfK:DmfContainer.obj
 0002:00003730       $unwind$?DmfModuleCallbacksInitialize@@YAJPEAU_DMF_OBJECT_@@PEAU_DMF_MODULE_ATTRIBUTES@@PEAUDMF_MODULE_DESCRIPTOR@@@Z 000000018002a730     DmfK:DmfCore.obj
 0002:00003730       $unwind$?DMF_Bridge_Open@@YAJPEAUDMFMODULE__@@@Z 000000018002a730     DmfK:Dmf_Bridge.obj
 0002:00003730       $unwind$?BufferPool_BufferPoolDestroy@@YAXPEAUDMFMODULE__@@@Z 000000018002a730     DmfK:Dmf_BufferPool.obj
 0002:00003730       $unwind$DMF_BufferPool_Count 000000018002a730     DmfK:Dmf_BufferPool.obj
 0002:00003730       $unwind$DMF_BufferPool_Put 000000018002a730     DmfK:Dmf_BufferPool.obj
 0002:00003730       $unwind$DMF_ContinuousRequestTarget_BufferPut 000000018002a730     DmfK:Dmf_ContinuousRequestTarget.obj
 0002:00003730       $unwind$DMF_ContinuousRequestTarget_StopAndWait 000000018002a730     DmfK:Dmf_ContinuousRequestTarget.obj
 0002:00003730       $unwind$DMF_DeviceInterfaceTarget_StreamStart 000000018002a730     DmfK:Dmf_DeviceInterfaceTarget.obj
 0002:0000374c       $unwind$DMF_Portable_EventCreate 000000018002a74c     DmfK:DmfPortable.obj
 0002:0000374c       $unwind$DMF_BufferPool_Get 000000018002a74c     DmfK:Dmf_BufferPool.obj
 0002:0000374c       $unwind$DMF_ContinuousRequestTarget_IoTargetSet 000000018002a74c     DmfK:Dmf_ContinuousRequestTarget.obj
 0002:0000374c       $unwind$DMF_DeviceInterfaceTarget_BufferPut 000000018002a74c     DmfK:Dmf_DeviceInterfaceTarget.obj
 0002:0000374c       $unwind$DMF_LiveKernelDump_StoreDmfCollectionAsBugcheckParameter 000000018002a74c     DmfK:Dmf_LiveKernelDump.obj
 0002:0000374c       $unwind$?ScheduledTask_DeferredHandlerOnDemand@@YAXPEAUWDFWORKITEM__@@@Z 000000018002a74c     DmfK:Dmf_ScheduledTask.obj
 0002:0000374c       $unwind$DMF_SmbiosWmi_TableType01Get 000000018002a74c     DmfK:Dmf_SmbiosWmi.obj
 0002:00003768       $unwind$?DMF_Bridge_ModuleDeviceIoControl@@YAEPEAUDMFMODULE__@@PEAUWDFQUEUE__@@PEAUWDFREQUEST__@@_K3K@Z 000000018002a768     DmfK:Dmf_Bridge.obj
 0002:00003768       $unwind$?DMF_Bridge_ModuleFileCreate@@YAEPEAUDMFMODULE__@@PEAUWDFDEVICE__@@PEAUWDFREQUEST__@@PEAUWDFFILEOBJECT__@@@Z 000000018002a768     DmfK:Dmf_Bridge.obj
 0002:00003768       $unwind$?DMF_Bridge_ModuleInternalDeviceIoControl@@YAEPEAUDMFMODULE__@@PEAUWDFQUEUE__@@PEAUWDFREQUEST__@@_K3K@Z 000000018002a768     DmfK:Dmf_Bridge.obj
 0002:00003768       $unwind$?DMF_Bridge_ModuleQueueIoRead@@YAEPEAUDMFMODULE__@@PEAUWDFQUEUE__@@PEAUWDFREQUEST__@@_K@Z 000000018002a768     DmfK:Dmf_Bridge.obj
 0002:00003768       $unwind$?DMF_Bridge_ModuleQueueIoWrite@@YAEPEAUDMFMODULE__@@PEAUWDFQUEUE__@@PEAUWDFREQUEST__@@_K@Z 000000018002a768     DmfK:Dmf_Bridge.obj
 0002:00003768       $unwind$?BufferPool_BufferPoolEntryGet@@YAPEAUWDFMEMORY__@@PEAUDMFMODULE__@@PEAPEAUBUFFERPOOL_ENTRY@@@Z 000000018002a768     DmfK:Dmf_BufferPool.obj
 0002:00003768       $unwind$?BufferPool_Put@@YAXPEAUDMFMODULE__@@PEAXP6AXPEAU_DMF_CONTEXT_BufferPool@@PEAUBUFFERPOOL_ENTRY@@@Z@Z 000000018002a768     DmfK:Dmf_BufferPool.obj
 0002:00003768       $unwind$DMF_BufferPool_GetWithMemory 000000018002a768     DmfK:Dmf_BufferPool.obj
 0002:00003768       $unwind$?DeviceInterfaceTarget_EvtIoTargetRemoveComplete@@YAXPEAUWDFIOTARGET__@@@Z 000000018002a768     DmfK:Dmf_DeviceInterfaceTarget.obj
 0002:00003768       $unwind$?DeviceInterfaceTarget_Stream_BufferInput@@YAXPEAUDMFMODULE__@@PEAXPEA_K1@Z 000000018002a768     DmfK:Dmf_DeviceInterfaceTarget.obj
 0002:00003768       $unwind$DMF_LiveKernelDump_DataBufferSourceAdd 000000018002a768     DmfK:Dmf_LiveKernelDump.obj
 0002:00003788       $unwind$WPP_RECORDER_SF_D  000000018002a788     DmfK:DmfPortable.obj
 0002:00003788       $unwind$WPP_RECORDER_SF_d  000000018002a788     DmfK:Dmf_BufferPool.obj
 0002:00003788       $unwind$WPP_RECORDER_SF_q  000000018002a788     DmfK:Dmf_BufferPool.obj
 0002:00003788       $unwind$DMF_HashTable_Find 000000018002a788     DmfK:Dmf_HashTable.obj
 0002:00003788       $unwind$WPP_RECORDER_SF_c  000000018002a788     DmfK:Dmf_SamCommunicationViaSsh.obj
 0002:000037a4       $unwind$WPP_RECORDER_SF_dq 000000018002a7a4     DmfK:DmfInterfaceInternal.obj
 0002:000037a4       $unwind$WPP_RECORDER_SF_qq 000000018002a7a4     DmfK:DmfModuleCollection.obj
 0002:000037a4       $unwind$WPP_RECORDER_SF_dd 000000018002a7a4     DmfK:Dmf_BufferPool.obj
 0002:000037a4       $unwind$WPP_RECORDER_SF_qd 000000018002a7a4     DmfK:Dmf_BufferPool.obj
 0002:000037a4       $unwind$WPP_RECORDER_SF_Dd 000000018002a7a4     DmfK:Dmf_IoctlHandler.obj
 0002:000037a4       $unwind$WPP_RECORDER_SF_dP 000000018002a7a4     DmfK:Dmf_SamNotificationViaSsh.obj
 0002:000037a4       $unwind$WPP_RECORDER_SF_ID 000000018002a7a4     DmfK:SurfaceTelemetry.obj
 0002:000037c0       $unwind$WPP_RECORDER_SF_qdq 000000018002a7c0     DmfK:Dmf_BufferPool.obj
 0002:000037c0       $unwind$WPP_RECORDER_SF_qdd 000000018002a7c0     DmfK:Dmf_DeviceInterfaceTarget.obj
 0002:000037c0       $unwind$WPP_RECORDER_SF_ddd 000000018002a7c0     DmfK:Dmf_IoctlHandler.obj
 0002:000037c0       $unwind$WPP_RECORDER_SF_ddP 000000018002a7c0     DmfK:Dmf_SamNotificationViaSsh.obj
 0002:000037dc       $unwind$?DMF_ModuleTreeDestroy@@YAXPEAUDMFMODULE__@@@Z 000000018002a7dc     DmfK:DmfCall.obj
 0002:000037dc       $unwind$?DMF_Module_CloseOrUnregisterNotificationOnDestroy@@YAXPEAUDMFMODULE__@@@Z 000000018002a7dc     DmfK:DmfCall.obj
 0002:000037dc       $unwind$?DMF_Module_NotificationUnregister@@YAXPEAUDMFMODULE__@@@Z 000000018002a7dc     DmfK:DmfCall.obj
 0002:000037dc       $unwind$?DMF_BranchTrack_LiveKernelDumpInitialize@@YAXPEAUDMFMODULE__@@@Z 000000018002a7dc     DmfK:Dmf_BranchTrack.obj
 0002:000037dc       $unwind$?DMF_Bridge_LiveKernelDumpInitialize@@YAXPEAUDMFMODULE__@@@Z 000000018002a7dc     DmfK:Dmf_Bridge.obj
 0002:000037dc       $unwind$?DMF_BufferPool_LiveKernelDumpInitialize@@YAXPEAUDMFMODULE__@@@Z 000000018002a7dc     DmfK:Dmf_BufferPool.obj
 0002:000037dc       $unwind$?DMF_BufferQueue_LiveKernelDumpInitialize@@YAXPEAUDMFMODULE__@@@Z 000000018002a7dc     DmfK:Dmf_BufferQueue.obj
 0002:000037dc       $unwind$?DMF_ContinuousRequestTarget_LiveKernelDumpInitialize@@YAXPEAUDMFMODULE__@@@Z 000000018002a7dc     DmfK:Dmf_ContinuousRequestTarget.obj
 0002:000037dc       $unwind$?DMF_CrashDump_LiveKernelDumpInitialize@@YAXPEAUDMFMODULE__@@@Z 000000018002a7dc     DmfK:Dmf_CrashDump.obj
 0002:000037dc       $unwind$?DMF_DeviceInterfaceTarget_LiveKernelDumpInitialize@@YAXPEAUDMFMODULE__@@@Z 000000018002a7dc     DmfK:Dmf_DeviceInterfaceTarget.obj
 0002:000037dc       $unwind$?DMF_HashTable_LiveKernelDumpInitialize@@YAXPEAUDMFMODULE__@@@Z 000000018002a7dc     DmfK:Dmf_HashTable.obj
 0002:000037dc       $unwind$?DMF_IoctlHandler_LiveKernelDumpInitialize@@YAXPEAUDMFMODULE__@@@Z 000000018002a7dc     DmfK:Dmf_IoctlHandler.obj
 0002:000037dc       $unwind$?DMF_LiveKernelDump_LiveKernelDumpInitialize@@YAXPEAUDMFMODULE__@@@Z 000000018002a7dc     DmfK:Dmf_LiveKernelDump.obj
 0002:000037dc       $unwind$?DMF_QueuedWorkItem_LiveKernelDumpInitialize@@YAXPEAUDMFMODULE__@@@Z 000000018002a7dc     DmfK:Dmf_QueuedWorkItem.obj
 0002:000037dc       $unwind$?DMF_RequestTarget_LiveKernelDumpInitialize@@YAXPEAUDMFMODULE__@@@Z 000000018002a7dc     DmfK:Dmf_RequestTarget.obj
 0002:000037dc       $unwind$?DMF_RingBuffer_LiveKernelDumpInitialize@@YAXPEAUDMFMODULE__@@@Z 000000018002a7dc     DmfK:Dmf_RingBuffer.obj
 0002:000037dc       $unwind$?DMF_Rundown_LiveKernelDumpInitialize@@YAXPEAUDMFMODULE__@@@Z 000000018002a7dc     DmfK:Dmf_Rundown.obj
 0002:000037dc       $unwind$?DMF_SamCommunicationViaSsh_LiveKernelDumpInitialize@@YAXPEAUDMFMODULE__@@@Z 000000018002a7dc     DmfK:Dmf_SamCommunicationViaSsh.obj
 0002:000037dc       $unwind$?DMF_SamNotificationViaSsh_LiveKernelDumpInitialize@@YAXPEAUDMFMODULE__@@@Z 000000018002a7dc     DmfK:Dmf_SamNotificationViaSsh.obj
 0002:000037dc       $unwind$?DMF_ScheduledTask_LiveKernelDumpInitialize@@YAXPEAUDMFMODULE__@@@Z 000000018002a7dc     DmfK:Dmf_ScheduledTask.obj
 0002:000037dc       $unwind$?DMF_SmbiosWmi_LiveKernelDumpInitialize@@YAXPEAUDMFMODULE__@@@Z 000000018002a7dc     DmfK:Dmf_SmbiosWmi.obj
 0002:000037dc       $unwind$?DMF_SurfaceTelemetryConsentSettingsNotification_LiveKernelDumpInitialize@@YAXPEAUDMFMODULE__@@@Z 000000018002a7dc     DmfK:Dmf_SurfaceTelemetryConsentSettingsNotification.obj
 0002:000037ec       $unwind$?BufferPool_RemoveHeadList@@YAPEAUBUFFERPOOL_ENTRY@@PEAUDMFMODULE__@@PEAU_DMF_CONTEXT_BufferPool@@@Z 000000018002a7ec     DmfK:Dmf_BufferPool.obj
 0002:00003804       $unwind$?DMF_ModuleBranchTrack_ModuleCollectionInitialize@@YAXPEAU_DMF_MODULE_COLLECTION_@@@Z 000000018002a804     DmfK:DmfBranchTrack.obj
 0002:00003804       $unwind$DMF_ModuleRequestCompleteOrForward 000000018002a804     DmfK:DmfCore.obj
 0002:00003804       $unwind$DMF_DmfDeviceInitFree 000000018002a804     DmfK:DmfDeviceInit.obj
 0002:00003804       $unwind$?BufferPool_InsertList@@YAXPEAUDMFMODULE__@@PEAU_DMF_CONTEXT_BufferPool@@PEAUBUFFERPOOL_ENTRY@@P6AX12@Z@Z 000000018002a804     DmfK:Dmf_BufferPool.obj
 0002:00003804       $unwind$?CrashDump_BugCheckSecondaryDumpDataCallbackRingBuffer@@YAXW4_KBUGCHECK_CALLBACK_REASON@@PEAU_KBUGCHECK_REASON_CALLBACK_RECORD@@PEAXK@Z 000000018002a804     DmfK:Dmf_CrashDump.obj
 0002:00003804       $unwind$?CrashDump_FileHandleSlotFree@@YAJPEAUDMFMODULE__@@PEAUWDFFILEOBJECT__@@@Z 000000018002a804     DmfK:Dmf_CrashDump.obj
 0002:00003818       $unwind$?DMF_DmfDeviceInitValidate@@YAEPEAUDMFDEVICE_INIT@@@Z 000000018002a818     DmfK:DmfDeviceInit.obj
 0002:00003818       $unwind$?BranchTrack_EVT_DMF_HashTable_Enumerate_Status@@YAEPEAUDMFMODULE__@@PEAEK1KPEAX@Z 000000018002a818     DmfK:Dmf_BranchTrack.obj
 0002:00003818       $unwind$?BufferPool_BufferPoolEntryGetFromClientBuffer@@YAPEAUBUFFERPOOL_ENTRY@@PEAX@Z 000000018002a818     DmfK:Dmf_BufferPool.obj
 0002:00003824       $unwind$?DMF_Generic_ModulePrepareHardware@@YAJPEAUDMFMODULE__@@PEAUWDFCMRESLIST__@@1@Z 000000018002a824     DmfK:DmfGeneric.obj
 0002:00003824       $unwind$?DMF_ModuleCollectionArmWakeFromSxWithReason@@YAJPEAUDMFCOLLECTION__@@EE@Z 000000018002a824     DmfK:DmfModuleCollection.obj
 0002:00003824       $unwind$?DMF_ModuleCollectionFileCleanup@@YAEPEAUDMFCOLLECTION__@@PEAUWDFFILEOBJECT__@@@Z 000000018002a824     DmfK:DmfModuleCollection.obj
 0002:00003824       $unwind$?DMF_ModuleCollectionFileClose@@YAEPEAUDMFCOLLECTION__@@PEAUWDFFILEOBJECT__@@@Z 000000018002a824     DmfK:DmfModuleCollection.obj
 0002:00003824       $unwind$?DMF_ModuleCollectionFileCreate@@YAEPEAUDMFCOLLECTION__@@PEAUWDFDEVICE__@@PEAUWDFREQUEST__@@PEAUWDFFILEOBJECT__@@@Z 000000018002a824     DmfK:DmfModuleCollection.obj
 0002:00003824       $unwind$?DMF_ModuleCollectionQueueIoRead@@YAEPEAUDMFCOLLECTION__@@PEAUWDFQUEUE__@@PEAUWDFREQUEST__@@_K@Z 000000018002a824     DmfK:DmfModuleCollection.obj
 0002:00003824       $unwind$?DMF_ModuleCollectionQueueIoWrite@@YAEPEAUDMFCOLLECTION__@@PEAUWDFQUEUE__@@PEAUWDFREQUEST__@@_K@Z 000000018002a824     DmfK:DmfModuleCollection.obj
 0002:00003824       $unwind$?DMF_ModuleCollectionUsageNotificationEx@@YAJPEAUDMFCOLLECTION__@@W4_WDF_SPECIAL_FILE_TYPE@@E@Z 000000018002a824     DmfK:DmfModuleCollection.obj
 0002:00003824       $unwind$?BufferPool_BufferPoolEntryPut@@YAXPEAUDMFMODULE__@@PEAUBUFFERPOOL_ENTRY@@P6AXPEAU_DMF_CONTEXT_BufferPool@@1@Z@Z 000000018002a824     DmfK:Dmf_BufferPool.obj
 0002:00003824       $unwind$?ContinuousRequestTarget_RequestsCancel@@YAXPEAUDMFMODULE__@@@Z 000000018002a824     DmfK:Dmf_ContinuousRequestTarget.obj
 0002:00003824       $unwind$?HashTable_DataEntryFindOrAllocate@@YAJPEAUDMFMODULE__@@PEAEKPEAPEAUDATA_ENTRY@@@Z 000000018002a824     DmfK:Dmf_HashTable.obj
 0002:00003824       $unwind$?DMF_SamNotificationViaSsh_BranchTrackInitialize@@YAXPEAUDMFMODULE__@@@Z 000000018002a824     DmfK:Dmf_SamNotificationViaSsh.obj
 0002:00003824       $unwind$?DMF_SamNotificationViaSsh_Close@@YAXPEAUDMFMODULE__@@@Z 000000018002a824     DmfK:Dmf_SamNotificationViaSsh.obj
 0002:00003824       $unwind$?DMF_SamNotificationViaSsh_ModuleD0Entry@@YAJPEAUDMFMODULE__@@W4_WDF_POWER_DEVICE_STATE@@@Z 000000018002a824     DmfK:Dmf_SamNotificationViaSsh.obj
 0002:00003824       $unwind$?DMF_SamNotificationViaSsh_ModuleD0Exit@@YAJPEAUDMFMODULE__@@W4_WDF_POWER_DEVICE_STATE@@@Z 000000018002a824     DmfK:Dmf_SamNotificationViaSsh.obj
 0002:00003824       $unwind$?DMF_SamNotificationViaSsh_Open@@YAJPEAUDMFMODULE__@@@Z 000000018002a824     DmfK:Dmf_SamNotificationViaSsh.obj
 0002:00003824       $unwind$?SamNotificationViaSsh_RegisterCompletion@@YAXPEAUDMFMODULE__@@PEAX1_K12J@Z 000000018002a824     DmfK:Dmf_SamNotificationViaSsh.obj
 0002:00003824       $unwind$?SamNotificationViaSsh_StreamingStart@@YAJPEAUDMFMODULE__@@@Z 000000018002a824     DmfK:Dmf_SamNotificationViaSsh.obj
 0002:00003824       $unwind$?SamNotificationViaSsh_StreamingStop@@YAJPEAUDMFMODULE__@@@Z 000000018002a824     DmfK:Dmf_SamNotificationViaSsh.obj
 0002:00003824       $unwind$?SamNotificationViaSsh_UnregisterCompletion@@YAXPEAUDMFMODULE__@@PEAX1_K12J@Z 000000018002a824     DmfK:Dmf_SamNotificationViaSsh.obj
 0002:00003824       $unwind$DMF_String_FindInListChar 000000018002a824     DmfK:Dmf_String.obj
 0002:00003844       $unwind$?DMF_ModuleCollectionRelationsQuery@@YAXPEAUDMFCOLLECTION__@@W4_DEVICE_RELATION_TYPE@@@Z 000000018002a844     DmfK:DmfModuleCollection.obj
 0002:00003844       $unwind$?BufferPool_BufferPoolEntryTimerHandler@@YAXPEAUWDFTIMER__@@@Z 000000018002a844     DmfK:Dmf_BufferPool.obj
 0002:00003844       $unwind$?DMF_ContinuousRequestTarget_ModuleD0Entry@@YAJPEAUDMFMODULE__@@W4_WDF_POWER_DEVICE_STATE@@@Z 000000018002a844     DmfK:Dmf_ContinuousRequestTarget.obj
 0002:00003844       $unwind$DMF_ContinuousRequestTarget_Start 000000018002a844     DmfK:Dmf_ContinuousRequestTarget.obj
 0002:00003844       $unwind$DMF_RingBuffer_Enumerate 000000018002a844     DmfK:Dmf_RingBuffer.obj
 0002:00003844       $unwind$?Rundown_Close@@YAXPEAUDMFMODULE__@@@Z 000000018002a844     DmfK:Dmf_Rundown.obj
 0002:00003864       $unwind$?BufferPool_BufferPoolEntryCreateAndAddToList@@YAJPEAUDMFMODULE__@@@Z 000000018002a864     DmfK:Dmf_BufferPool.obj
 0002:00003884       $unwind$?BufferPool_BufferGet@@YAPEAXPEAUDMFMODULE__@@@Z 000000018002a884     DmfK:Dmf_BufferPool.obj
 0002:0000389c       $unwind$?BufferPool_BufferPoolCreate@@YAJPEAUDMFMODULE__@@@Z 000000018002a89c     DmfK:Dmf_BufferPool.obj
 0002:0000389c       $unwind$?DMF_QueuedWorkItem_ChildModulesAdd@@YAXPEAUDMFMODULE__@@PEAU_DMF_MODULE_ATTRIBUTES@@PEAX@Z 000000018002a89c     DmfK:Dmf_QueuedWorkItem.obj
 0002:0000389c       $unwind$?DMF_ScheduledTask_Open@@YAJPEAUDMFMODULE__@@@Z 000000018002a89c     DmfK:Dmf_ScheduledTask.obj
 0002:000038c0       $unwind$?BufferPool_ListFlushAndDestroy@@YAXPEAUDMFMODULE__@@@Z 000000018002a8c0     DmfK:Dmf_BufferPool.obj
 0002:000038c0       $unwind$?ContinuousRequestTarget_CompletionParamsInputBufferAndOutputBufferGet@@YAXPEAUDMFMODULE__@@PEAU_WDF_REQUEST_COMPLETION_PARAMS@@W4ContinuousRequestTarget_RequestType@@PEAPEAXPEA_K34@Z 000000018002a8c0     DmfK:Dmf_ContinuousRequestTarget.obj
 0002:000038c0       $unwind$?CrashDump_DataSourceCaptureAuxiliary@@YAJPEAUDMFMODULE__@@PEAUWDFFILEOBJECT__@@PEAEKPEAK@Z 000000018002a8c0     DmfK:Dmf_CrashDump.obj
 0002:000038dc       $unwind$DMF_Portable_EventReset 000000018002a8dc     DmfK:DmfPortable.obj
 0002:000038dc       $unwind$DMF_Portable_EventSet 000000018002a8dc     DmfK:DmfPortable.obj
 0002:000038dc       $unwind$?Bridge_DefaultEvtDeviceArmWakeFromS0@@YAJPEAUWDFDEVICE__@@@Z 000000018002a8dc     DmfK:Dmf_Bridge.obj
 0002:000038dc       $unwind$?Bridge_DefaultEvtDeviceArmWakeFromSxWithReason@@YAJPEAUWDFDEVICE__@@EE@Z 000000018002a8dc     DmfK:Dmf_Bridge.obj
 0002:000038dc       $unwind$?Bridge_DefaultEvtDeviceD0Entry@@YAJPEAUWDFDEVICE__@@W4_WDF_POWER_DEVICE_STATE@@@Z 000000018002a8dc     DmfK:Dmf_Bridge.obj
 0002:000038dc       $unwind$?Bridge_DefaultEvtDeviceD0EntryPostInterruptsEnabled@@YAJPEAUWDFDEVICE__@@W4_WDF_POWER_DEVICE_STATE@@@Z 000000018002a8dc     DmfK:Dmf_Bridge.obj
 0002:000038dc       $unwind$?Bridge_DefaultEvtDeviceD0Exit@@YAJPEAUWDFDEVICE__@@W4_WDF_POWER_DEVICE_STATE@@@Z 000000018002a8dc     DmfK:Dmf_Bridge.obj
 0002:000038dc       $unwind$?Bridge_DefaultEvtDeviceD0ExitPreInterruptsDisabled@@YAJPEAUWDFDEVICE__@@W4_WDF_POWER_DEVICE_STATE@@@Z 000000018002a8dc     DmfK:Dmf_Bridge.obj
 0002:000038dc       $unwind$?Bridge_DefaultEvtDevicePrepareHardware@@YAJPEAUWDFDEVICE__@@PEAUWDFCMRESLIST__@@1@Z 000000018002a8dc     DmfK:Dmf_Bridge.obj
 0002:000038dc       $unwind$?Bridge_DefaultEvtDeviceQueryRemove@@YAJPEAUWDFDEVICE__@@@Z 000000018002a8dc     DmfK:Dmf_Bridge.obj
 0002:000038dc       $unwind$?Bridge_DefaultEvtDeviceQueryStop@@YAJPEAUWDFDEVICE__@@@Z 000000018002a8dc     DmfK:Dmf_Bridge.obj
 0002:000038dc       $unwind$?Bridge_DefaultEvtDeviceReleaseHardware@@YAJPEAUWDFDEVICE__@@PEAUWDFCMRESLIST__@@@Z 000000018002a8dc     DmfK:Dmf_Bridge.obj
 0002:000038dc       $unwind$?Bridge_DefaultEvtDeviceSelfManagedIoInit@@YAJPEAUWDFDEVICE__@@@Z 000000018002a8dc     DmfK:Dmf_Bridge.obj
 0002:000038dc       $unwind$?Bridge_DefaultEvtDeviceSelfManagedIoRestart@@YAJPEAUWDFDEVICE__@@@Z 000000018002a8dc     DmfK:Dmf_Bridge.obj
 0002:000038dc       $unwind$?Bridge_DefaultEvtDeviceSelfManagedIoSuspend@@YAJPEAUWDFDEVICE__@@@Z 000000018002a8dc     DmfK:Dmf_Bridge.obj
 0002:000038dc       $unwind$?Bridge_DefaultEvtDeviceUsageNotificationEx@@YAJPEAUWDFDEVICE__@@W4_WDF_SPECIAL_FILE_TYPE@@E@Z 000000018002a8dc     DmfK:Dmf_Bridge.obj
 0002:000038dc       $unwind$?DMF_BufferPool_Close@@YAXPEAUDMFMODULE__@@@Z 000000018002a8dc     DmfK:Dmf_BufferPool.obj
 0002:000038dc       $unwind$?DMF_BufferPool_Open@@YAJPEAUDMFMODULE__@@@Z 000000018002a8dc     DmfK:Dmf_BufferPool.obj
 0002:000038dc       $unwind$?RingBuffer_ReadPointerIncrement@@YAXPEAURING_BUFFER@@@Z 000000018002a8dc     DmfK:Dmf_RingBuffer.obj
 0002:000038dc       $unwind$?DMF_Rundown_Close@@YAXPEAUDMFMODULE__@@@Z 000000018002a8dc     DmfK:Dmf_Rundown.obj
 0002:000038f0       $unwind$DMF_BufferQueue_Create 000000018002a8f0     DmfK:Dmf_BufferQueue.obj
 0002:000038f0       $unwind$DMF_HashTable_Create 000000018002a8f0     DmfK:Dmf_HashTable.obj
 0002:000038f0       $unwind$DMF_QueuedWorkItem_Create 000000018002a8f0     DmfK:Dmf_QueuedWorkItem.obj
 0002:000038f0       $unwind$DMF_RequestTarget_Create 000000018002a8f0     DmfK:Dmf_RequestTarget.obj
 0002:000038f0       $unwind$DMF_Rundown_Create 000000018002a8f0     DmfK:Dmf_Rundown.obj
 0002:000038f0       $unwind$DMF_SamCommunicationViaSsh_Create 000000018002a8f0     DmfK:Dmf_SamCommunicationViaSsh.obj
 0002:000038f0       $unwind$DMF_SurfaceTelemetryConsentSettingsNotification_Create 000000018002a8f0     DmfK:Dmf_SurfaceTelemetryConsentSettingsNotification.obj
 0002:00003914       $unwind$DMF_SamCommunicationViaSsh_Send 000000018002a914     DmfK:Dmf_SamCommunicationViaSsh.obj
 0002:00003914       $unwind$DMF_SamCommunicationViaSsh_SendSynchronously 000000018002a914     DmfK:Dmf_SamCommunicationViaSsh.obj
 0002:00003934       $unwind$?DMF_Generic_ChildModulesAdd@@YAXPEAUDMFMODULE__@@PEAU_DMF_MODULE_ATTRIBUTES@@PEAX@Z 000000018002a934     DmfK:DmfGeneric.obj
 0002:00003934       $unwind$?DMF_Generic_Destroy@@YAXPEAUDMFMODULE__@@@Z 000000018002a934     DmfK:DmfGeneric.obj
 0002:00003934       $unwind$?DMF_Internal_Close@@YAXPEAUDMFMODULE__@@@Z 000000018002a934     DmfK:DmfInternal.obj
 0002:00003934       $unwind$?DMF_Internal_ModuleArmWakeFromS0@@YAJPEAUDMFMODULE__@@@Z 000000018002a934     DmfK:DmfInternal.obj
 0002:00003934       $unwind$?DMF_Internal_ModuleD0Entry@@YAJPEAUDMFMODULE__@@W4_WDF_POWER_DEVICE_STATE@@@Z 000000018002a934     DmfK:DmfInternal.obj
 0002:00003934       $unwind$?DMF_Internal_ModuleD0EntryPostInterruptsEnabled@@YAJPEAUDMFMODULE__@@W4_WDF_POWER_DEVICE_STATE@@@Z 000000018002a934     DmfK:DmfInternal.obj
 0002:00003934       $unwind$?DMF_Internal_ModuleD0Exit@@YAJPEAUDMFMODULE__@@W4_WDF_POWER_DEVICE_STATE@@@Z 000000018002a934     DmfK:DmfInternal.obj
 0002:00003934       $unwind$?DMF_Internal_ModuleD0ExitPreInterruptsDisabled@@YAJPEAUDMFMODULE__@@W4_WDF_POWER_DEVICE_STATE@@@Z 000000018002a934     DmfK:DmfInternal.obj
 0002:00003934       $unwind$?DMF_Internal_ModuleFileCleanup@@YAEPEAUDMFMODULE__@@PEAUWDFFILEOBJECT__@@@Z 000000018002a934     DmfK:DmfInternal.obj
 0002:00003934       $unwind$?DMF_Internal_ModuleFileClose@@YAEPEAUDMFMODULE__@@PEAUWDFFILEOBJECT__@@@Z 000000018002a934     DmfK:DmfInternal.obj
 0002:00003934       $unwind$?DMF_Internal_ModuleQueryRemove@@YAJPEAUDMFMODULE__@@@Z 000000018002a934     DmfK:DmfInternal.obj
 0002:00003934       $unwind$?DMF_Internal_ModuleQueryStop@@YAJPEAUDMFMODULE__@@@Z 000000018002a934     DmfK:DmfInternal.obj
 0002:00003934       $unwind$?DMF_Internal_ModuleRelationsQuery@@YAXPEAUDMFMODULE__@@W4_DEVICE_RELATION_TYPE@@@Z 000000018002a934     DmfK:DmfInternal.obj
 0002:00003934       $unwind$?DMF_Internal_ModuleReleaseHardware@@YAJPEAUDMFMODULE__@@PEAUWDFCMRESLIST__@@@Z 000000018002a934     DmfK:DmfInternal.obj
 0002:00003934       $unwind$?DMF_Internal_ModuleSelfManagedIoInit@@YAJPEAUDMFMODULE__@@@Z 000000018002a934     DmfK:DmfInternal.obj
 0002:00003934       $unwind$?DMF_Internal_ModuleSelfManagedIoRestart@@YAJPEAUDMFMODULE__@@@Z 000000018002a934     DmfK:DmfInternal.obj
 0002:00003934       $unwind$?DMF_Internal_ModuleSelfManagedIoSuspend@@YAJPEAUDMFMODULE__@@@Z 000000018002a934     DmfK:DmfInternal.obj
 0002:00003934       $unwind$?DMF_Internal_NotificationRegister@@YAJPEAUDMFMODULE__@@@Z 000000018002a934     DmfK:DmfInternal.obj
 0002:00003934       $unwind$?Rundown_ReferenceAdd@@YAJPEAUDMFMODULE__@@@Z 000000018002a934     DmfK:Dmf_Rundown.obj
 0002:00003934       $unwind$?Rundown_ReferenceDelete@@YAJPEAUDMFMODULE__@@@Z 000000018002a934     DmfK:Dmf_Rundown.obj
 0002:00003934       $unwind$?SamCommunicationViaSsh_OnDeviceArrivalNotification@@YAXPEAUDMFMODULE__@@@Z 000000018002a934     DmfK:Dmf_SamCommunicationViaSsh.obj
 0002:00003950       $unwind$?DMF_ModuleReferenceAdd@@YAJPEAUDMFMODULE__@@@Z 000000018002a950     DmfK:DmfCall.obj
 0002:00003950       $unwind$?DMF_ModuleReferenceDelete@@YAJPEAUDMFMODULE__@@@Z 000000018002a950     DmfK:DmfCall.obj
 0002:00003950       $unwind$?DMF_Generic_ModuleArmWakeFromS0@@YAJPEAUDMFMODULE__@@@Z 000000018002a950     DmfK:DmfGeneric.obj
 0002:00003950       $unwind$?DMF_Generic_ModuleArmWakeFromSxWithReason@@YAJPEAUDMFMODULE__@@EE@Z 000000018002a950     DmfK:DmfGeneric.obj
 0002:00003950       $unwind$?DMF_Generic_ModuleDisarmWakeFromS0@@YAXPEAUDMFMODULE__@@@Z 000000018002a950     DmfK:DmfGeneric.obj
 0002:00003950       $unwind$?DMF_Generic_ModuleDisarmWakeFromSx@@YAXPEAUDMFMODULE__@@@Z 000000018002a950     DmfK:DmfGeneric.obj
 0002:00003950       $unwind$?DMF_Generic_ModuleFileCleanup@@YAEPEAUDMFMODULE__@@PEAUWDFFILEOBJECT__@@@Z 000000018002a950     DmfK:DmfGeneric.obj
 0002:00003950       $unwind$?DMF_Generic_ModuleFileClose@@YAEPEAUDMFMODULE__@@PEAUWDFFILEOBJECT__@@@Z 000000018002a950     DmfK:DmfGeneric.obj
 0002:00003950       $unwind$?DMF_Generic_ModuleFileCreate@@YAEPEAUDMFMODULE__@@PEAUWDFDEVICE__@@PEAUWDFREQUEST__@@PEAUWDFFILEOBJECT__@@@Z 000000018002a950     DmfK:DmfGeneric.obj
 0002:00003950       $unwind$?DMF_Generic_ModuleInternalDeviceIoControl@@YAEPEAUDMFMODULE__@@PEAUWDFQUEUE__@@PEAUWDFREQUEST__@@_K3K@Z 000000018002a950     DmfK:DmfGeneric.obj
 0002:00003950       $unwind$?DMF_Generic_ModuleQueryRemove@@YAJPEAUDMFMODULE__@@@Z 000000018002a950     DmfK:DmfGeneric.obj
 0002:00003950       $unwind$?DMF_Generic_ModuleQueryStop@@YAJPEAUDMFMODULE__@@@Z 000000018002a950     DmfK:DmfGeneric.obj
 0002:00003950       $unwind$?DMF_Generic_ModuleQueueIoRead@@YAEPEAUDMFMODULE__@@PEAUWDFQUEUE__@@PEAUWDFREQUEST__@@_K@Z 000000018002a950     DmfK:DmfGeneric.obj
 0002:00003950       $unwind$?DMF_Generic_ModuleQueueIoWrite@@YAEPEAUDMFMODULE__@@PEAUWDFQUEUE__@@PEAUWDFREQUEST__@@_K@Z 000000018002a950     DmfK:DmfGeneric.obj
 0002:00003950       $unwind$?DMF_Generic_ModuleRelationsQuery@@YAXPEAUDMFMODULE__@@W4_DEVICE_RELATION_TYPE@@@Z 000000018002a950     DmfK:DmfGeneric.obj
 0002:00003950       $unwind$?DMF_Generic_ModuleSelfManagedIoCleanup@@YAXPEAUDMFMODULE__@@@Z 000000018002a950     DmfK:DmfGeneric.obj
 0002:00003950       $unwind$?DMF_Generic_ModuleSelfManagedIoFlush@@YAXPEAUDMFMODULE__@@@Z 000000018002a950     DmfK:DmfGeneric.obj
 0002:00003950       $unwind$?DMF_Generic_ModuleSelfManagedIoInit@@YAJPEAUDMFMODULE__@@@Z 000000018002a950     DmfK:DmfGeneric.obj
 0002:00003950       $unwind$?DMF_Generic_ModuleSelfManagedIoRestart@@YAJPEAUDMFMODULE__@@@Z 000000018002a950     DmfK:DmfGeneric.obj
 0002:00003950       $unwind$?DMF_Generic_ModuleSelfManagedIoSuspend@@YAJPEAUDMFMODULE__@@@Z 000000018002a950     DmfK:DmfGeneric.obj
 0002:00003950       $unwind$?DMF_Generic_ModuleSurpriseRemoval@@YAXPEAUDMFMODULE__@@@Z 000000018002a950     DmfK:DmfGeneric.obj
 0002:00003950       $unwind$?DMF_Generic_ModuleUsageNotificationEx@@YAJPEAUDMFMODULE__@@W4_WDF_SPECIAL_FILE_TYPE@@E@Z 000000018002a950     DmfK:DmfGeneric.obj
 0002:00003950       $unwind$?DMF_Generic_ModuleWakeFromS0Triggered@@YAXPEAUDMFMODULE__@@@Z 000000018002a950     DmfK:DmfGeneric.obj
 0002:00003950       $unwind$?DMF_Generic_ModuleWakeFromSxTriggered@@YAXPEAUDMFMODULE__@@@Z 000000018002a950     DmfK:DmfGeneric.obj
 0002:00003950       $unwind$?DMF_Generic_NotificationUnregister@@YAXPEAUDMFMODULE__@@@Z 000000018002a950     DmfK:DmfGeneric.obj
 0002:00003950       $unwind$?DMF_Internal_Destroy@@YAXPEAUDMFMODULE__@@@Z 000000018002a950     DmfK:DmfInternal.obj
 0002:00003950       $unwind$?DMF_Internal_ModuleDisarmWakeFromS0@@YAXPEAUDMFMODULE__@@@Z 000000018002a950     DmfK:DmfInternal.obj
 0002:00003950       $unwind$?DMF_Internal_ModuleDisarmWakeFromSx@@YAXPEAUDMFMODULE__@@@Z 000000018002a950     DmfK:DmfInternal.obj
 0002:00003950       $unwind$?DMF_Internal_ModuleSelfManagedIoCleanup@@YAXPEAUDMFMODULE__@@@Z 000000018002a950     DmfK:DmfInternal.obj
 0002:00003950       $unwind$?DMF_Internal_ModuleSelfManagedIoFlush@@YAXPEAUDMFMODULE__@@@Z 000000018002a950     DmfK:DmfInternal.obj
 0002:00003950       $unwind$?DMF_Internal_ModuleSurpriseRemoval@@YAXPEAUDMFMODULE__@@@Z 000000018002a950     DmfK:DmfInternal.obj
 0002:00003950       $unwind$?DMF_Internal_ModuleWakeFromS0Triggered@@YAXPEAUDMFMODULE__@@@Z 000000018002a950     DmfK:DmfInternal.obj
 0002:00003950       $unwind$?DMF_Internal_ModuleWakeFromSxTriggered@@YAXPEAUDMFMODULE__@@@Z 000000018002a950     DmfK:DmfInternal.obj
 0002:00003950       $unwind$?DMF_Internal_NotificationUnregister@@YAXPEAUDMFMODULE__@@@Z 000000018002a950     DmfK:DmfInternal.obj
 0002:00003950       $unwind$?SamCommunicationViaSsh_OnDeviceRemovalNotification@@YAXPEAUDMFMODULE__@@@Z 000000018002a950     DmfK:Dmf_SamCommunicationViaSsh.obj
 0002:00003950       $unwind$?SamNotificationViaSsh_OnDeviceArrivalNotification@@YAXPEAUDMFMODULE__@@@Z 000000018002a950     DmfK:Dmf_SamNotificationViaSsh.obj
 0002:00003950       $unwind$?SamNotificationViaSsh_OnDeviceRemovalNotification@@YAXPEAUDMFMODULE__@@@Z 000000018002a950     DmfK:Dmf_SamNotificationViaSsh.obj
 0002:00003968       $unwind$?DMF_ChildDispatchSingleParameterNtStatus@@YAJPEAUDMFMODULE__@@P6AJ0@ZPEAU_DMF_ChildObjectGet@@@Z 000000018002a968     DmfK:DmfCall.obj
 0002:00003968       $unwind$?DMF_Module_D0Entry@@YAJPEAUDMFMODULE__@@W4_WDF_POWER_DEVICE_STATE@@@Z 000000018002a968     DmfK:DmfCall.obj
 0002:00003968       $unwind$?DMF_Module_D0EntryPostInterruptsEnabled@@YAJPEAUDMFMODULE__@@W4_WDF_POWER_DEVICE_STATE@@@Z 000000018002a968     DmfK:DmfCall.obj
 0002:00003968       $unwind$?DMF_Module_D0Exit@@YAJPEAUDMFMODULE__@@W4_WDF_POWER_DEVICE_STATE@@@Z 000000018002a968     DmfK:DmfCall.obj
 0002:00003968       $unwind$?DMF_Module_D0ExitPreInterruptsDisabled@@YAJPEAUDMFMODULE__@@W4_WDF_POWER_DEVICE_STATE@@@Z 000000018002a968     DmfK:DmfCall.obj
 0002:00003968       $unwind$?DMF_Module_FileCleanup@@YAEPEAUDMFMODULE__@@PEAUWDFFILEOBJECT__@@@Z 000000018002a968     DmfK:DmfCall.obj
 0002:00003968       $unwind$?DMF_Module_FileClose@@YAEPEAUDMFMODULE__@@PEAUWDFFILEOBJECT__@@@Z 000000018002a968     DmfK:DmfCall.obj
 0002:00003968       $unwind$?DMF_Module_OpenOrRegisterNotificationOnCreate@@YAJPEAUDMFMODULE__@@@Z 000000018002a968     DmfK:DmfCall.obj
 0002:00003968       $unwind$?DMF_Module_ReleaseHardware@@YAJPEAUDMFMODULE__@@PEAUWDFCMRESLIST__@@@Z 000000018002a968     DmfK:DmfCall.obj
 0002:00003968       $unwind$?LiveKernelDump_InsertDataBufferInCrashDump@@YAEPEAUDMFMODULE__@@PEAEKPEAX@Z 000000018002a968     DmfK:Dmf_LiveKernelDump.obj
 0002:00003968       $unwind$?DMF_SamCommunicationViaSsh_BranchTrackInitialize@@YAXPEAUDMFMODULE__@@@Z 000000018002a968     DmfK:Dmf_SamCommunicationViaSsh.obj
 0002:0000397c       $unwind$?DMF_SamCommunicationViaSsh_ChildModulesAdd@@YAXPEAUDMFMODULE__@@PEAU_DMF_MODULE_ATTRIBUTES@@PEAX@Z 000000018002a97c     DmfK:Dmf_SamCommunicationViaSsh.obj
 0002:000039a0       $unwind$?DMF_Module_ArmWakeFromS0@@YAJPEAUDMFMODULE__@@@Z 000000018002a9a0     DmfK:DmfCall.obj
 0002:000039a0       $unwind$?DMF_Module_QueryRemove@@YAJPEAUDMFMODULE__@@@Z 000000018002a9a0     DmfK:DmfCall.obj
 0002:000039a0       $unwind$?DMF_Module_QueryStop@@YAJPEAUDMFMODULE__@@@Z 000000018002a9a0     DmfK:DmfCall.obj
 0002:000039a0       $unwind$?DMF_Module_SelfManagedIoSuspend@@YAJPEAUDMFMODULE__@@@Z 000000018002a9a0     DmfK:DmfCall.obj
 0002:000039a0       $unwind$DMF_ModuleInContextSave 000000018002a9a0     DmfK:DmfCall.obj
 0002:000039a0       $unwind$DMF_DmfDeviceInitHookPnpPowerEventCallbacks 000000018002a9a0     DmfK:DmfDeviceInit.obj
 0002:000039a0       $unwind$DMF_DmfDeviceInitHookPowerPolicyEventCallbacks 000000018002a9a0     DmfK:DmfDeviceInit.obj
 0002:000039a0       $unwind$DMF_DmfDeviceInitHookQueueConfig 000000018002a9a0     DmfK:DmfDeviceInit.obj
 0002:000039a0       $unwind$?DMF_FeatureHandleGetFromModuleCollection@@YAPEAU_DMF_OBJECT_@@PEAUDMFCOLLECTION__@@W4DmfFeatureType@@@Z 000000018002a9a0     DmfK:DmfHelpers.obj
 0002:000039a0       $unwind$?DMF_GenericSpinLockAcquire@@YAXPEA_KPEAE@Z 000000018002a9a0     DmfK:DmfHelpers.obj
 0002:000039a0       $unwind$DMF_IsModuleDynamic 000000018002a9a0     DmfK:DmfHelpers.obj
 0002:000039a0       $unwind$DMF_IsModulePassiveLevel 000000018002a9a0     DmfK:DmfHelpers.obj
 0002:000039a0       $unwind$DMF_ModuleConfigGet 000000018002a9a0     DmfK:DmfHelpers.obj
 0002:000039a0       $unwind$DMF_ModuleIsInFilterDriver 000000018002a9a0     DmfK:DmfHelpers.obj
 0002:000039a0       $unwind$DMF_ParentDeviceGet 000000018002a9a0     DmfK:DmfHelpers.obj
 0002:000039a0       $unwind$DMF_ParentModuleGet 000000018002a9a0     DmfK:DmfHelpers.obj
 0002:000039a0       $unwind$?ContinuousRequestTarget_QueuedWorkitemCallbackSingle@@YA?AW4ScheduledTask_Result_Type@@PEAUDMFMODULE__@@PEAX1@Z 000000018002a9a0     DmfK:Dmf_ContinuousRequestTarget.obj
 0002:000039a0       $unwind$?CrashDump_DmfDestroy_RingBuffer@@YAXPEAUDMFMODULE__@@K@Z 000000018002a9a0     DmfK:Dmf_CrashDump.obj
 0002:000039a0       $unwind$?CrashDump_FileHandleSlotFindForDestroy@@YAJPEAUDMFMODULE__@@PEAUWDFFILEOBJECT__@@@Z 000000018002a9a0     DmfK:Dmf_CrashDump.obj
 0002:000039a0       $unwind$?DMF_LiveKernelDump_Open@@YAJPEAUDMFMODULE__@@@Z 000000018002a9a0     DmfK:Dmf_LiveKernelDump.obj
 0002:000039a0       $unwind$?LiveKernelDump_InsertDmfTriageDataToCrashDump@@YAJPEAUDMFMODULE__@@@Z 000000018002a9a0     DmfK:Dmf_LiveKernelDump.obj
 0002:000039a0       $unwind$?RequestTarget_QueuedWorkitemCallbackSingle@@YA?AW4ScheduledTask_Result_Type@@PEAUDMFMODULE__@@PEAX1@Z 000000018002a9a0     DmfK:Dmf_RequestTarget.obj
 0002:000039a0       $unwind$?DMF_RingBuffer_Close@@YAXPEAUDMFMODULE__@@@Z 000000018002a9a0     DmfK:Dmf_RingBuffer.obj
 0002:000039a0       $unwind$?DMF_SmbiosWmi_Open@@YAJPEAUDMFMODULE__@@@Z 000000018002a9a0     DmfK:Dmf_SmbiosWmi.obj
 0002:000039ac       $unwind$?DMF_Module_SelfManagedIoInit@@YAJPEAUDMFMODULE__@@@Z 000000018002a9ac     DmfK:DmfCall.obj
 0002:000039ac       $unwind$?DMF_Module_SelfManagedIoRestart@@YAJPEAUDMFMODULE__@@@Z 000000018002a9ac     DmfK:DmfCall.obj
 0002:000039ac       $unwind$DMF_ModuleDereference 000000018002a9ac     DmfK:DmfCall.obj
 0002:000039ac       $unwind$?DMF_ModuleTransportSet@@YAXPEAUDMFMODULE__@@0@Z 000000018002a9ac     DmfK:DmfCore.obj
 0002:000039ac       $unwind$?DMF_Generic_AuxiliaryLock_Dispatch@@YAXPEAUDMFMODULE__@@K@Z 000000018002a9ac     DmfK:DmfGeneric.obj
 0002:000039ac       $unwind$?DMF_Generic_AuxiliaryLock_Passive@@YAXPEAUDMFMODULE__@@K@Z 000000018002a9ac     DmfK:DmfGeneric.obj
 0002:000039ac       $unwind$?DMF_Generic_AuxiliaryUnlock_Dispatch@@YAXPEAUDMFMODULE__@@K@Z 000000018002a9ac     DmfK:DmfGeneric.obj
 0002:000039ac       $unwind$?DMF_Generic_AuxiliaryUnlock_Passive@@YAXPEAUDMFMODULE__@@K@Z 000000018002a9ac     DmfK:DmfGeneric.obj
 0002:000039ac       $unwind$DMF_FeatureModuleGetFromModule 000000018002a9ac     DmfK:DmfHelpers.obj
 0002:000039ac       $unwind$DMF_ModuleLockPrivate 000000018002a9ac     DmfK:DmfHelpers.obj
 0002:000039ac       $unwind$?ContinuousRequestTarget_DeleteStreamRequestsFromCollection@@YAXPEAU_DMF_CONTEXT_ContinuousRequestTarget@@@Z 000000018002a9ac     DmfK:Dmf_ContinuousRequestTarget.obj
 0002:000039ac       $unwind$?CrashDump_DataSourceDestroyAuxiliary@@YAJPEAUDMFMODULE__@@PEAUWDFFILEOBJECT__@@@Z 000000018002a9ac     DmfK:Dmf_CrashDump.obj
 0002:000039ac       $unwind$?CrashDump_DataSourceDestroySelf@@YAJPEAUDMFMODULE__@@@Z 000000018002a9ac     DmfK:Dmf_CrashDump.obj
 0002:000039ac       $unwind$?CrashDump_FileHandleSlotFind@@YAJPEAUDMFMODULE__@@PEAUWDFFILEOBJECT__@@W4DataSourceModeType@@@Z 000000018002a9ac     DmfK:Dmf_CrashDump.obj
 0002:000039ac       $unwind$?DMF_CrashDump_FileClose@@YAEPEAUDMFMODULE__@@PEAUWDFFILEOBJECT__@@@Z 000000018002a9ac     DmfK:Dmf_CrashDump.obj
 0002:000039ac       $unwind$?DeviceInterfaceTarget_SymbolicLinkNameClear@@YAXPEAUDMFMODULE__@@@Z 000000018002a9ac     DmfK:Dmf_DeviceInterfaceTarget.obj
 0002:000039ac       $unwind$DMF_RingBuffer_TotalSizeGet 000000018002a9ac     DmfK:Dmf_RingBuffer.obj
 0002:000039ac       $unwind$DMF_Rundown_Reference 000000018002a9ac     DmfK:Dmf_Rundown.obj
 0002:000039bc       $unwind$DMF_ModuleClose    000000018002a9bc     DmfK:DmfCall.obj
 0002:000039bc       $unwind$DMF_ModuleOpen     000000018002a9bc     DmfK:DmfCall.obj
 0002:000039bc       $unwind$DMF_ModuleUnlockPrivate 000000018002a9bc     DmfK:DmfHelpers.obj
 0002:000039c8       $unwind$?DmfEvtDynamicModuleCleanupCallback@@YAXPEAX@Z 000000018002a9c8     DmfK:DmfCall.obj
 0002:000039c8       $unwind$?DMF_GenericMemoryAllocate@@YAPEAX_K0K@Z 000000018002a9c8     DmfK:DmfHelpers.obj
 0002:000039c8       $unwind$?DMF_RequestPassthruWithCompletion@@YAXPEAUWDFDEVICE__@@PEAUWDFREQUEST__@@P6AX1PEAUWDFIOTARGET__@@PEAU_WDF_REQUEST_COMPLETION_PARAMS@@PEAX@Z4@Z 000000018002a9c8     DmfK:DmfHelpers.obj
 0002:000039c8       $unwind$?CrashDump_DataSourceCreateSelf@@YAJPEAUDMFMODULE__@@KKPEBU_GUID@@@Z 000000018002a9c8     DmfK:Dmf_CrashDump.obj
 0002:000039c8       $unwind$?RingBuffer_Read@@YAJPEAURING_BUFFER@@PEAEKP6AXPEAX1K@Z@Z 000000018002a9c8     DmfK:Dmf_RingBuffer.obj
 0002:000039c8       $unwind$?ScheduledTask_TimerRestart@@YAXPEAUDMFMODULE__@@W4ScheduledTask_Result_Type@@@Z 000000018002a9c8     DmfK:Dmf_ScheduledTask.obj
 0002:000039c8       $unwind$DMF_String_FindInListExactChar 000000018002a9c8     DmfK:Dmf_String.obj
 0002:000039c8       $unwind$DMF_String_FindInListLookForLeftMatchChar 000000018002a9c8     DmfK:Dmf_String.obj
 0002:000039e0       $unwind$DMF_ModuleLockIsPassive 000000018002a9e0     DmfK:DmfCall.obj
 0002:000039e0       $unwind$?DMF_GenericSpinLockCreate@@YAJPEAU_WDF_OBJECT_ATTRIBUTES@@PEA_K@Z 000000018002a9e0     DmfK:DmfHelpers.obj
 0002:000039ec       $unwind$?DMF_SynchronizationCreate@@YAJPEAU_DMF_OBJECT_@@E@Z 000000018002a9ec     DmfK:DmfHelpers.obj
 0002:00003a0c       $unwind$?DMF_RequestPassthru@@YAXPEAUWDFDEVICE__@@PEAUWDFREQUEST__@@@Z 000000018002aa0c     DmfK:DmfHelpers.obj
 0002:00003a24       $unwind$WPP_RECORDER_SF_qs 000000018002aa24     DmfK:DmfHelpers.obj
 0002:00003a44       $unwind$WPP_RECORDER_SF_qqs 000000018002aa44     DmfK:DmfGeneric.obj
 0002:00003a44       $unwind$WPP_RECORDER_SF_qsd 000000018002aa44     DmfK:DmfHelpers.obj
 0002:00003a44       $unwind$WPP_RECORDER_SF_qsq 000000018002aa44     DmfK:DmfInternal.obj
 0002:00003a64       $unwind$DMF_ContinuousRequestTarget_Create 000000018002aa64     DmfK:Dmf_ContinuousRequestTarget.obj
 0002:00003a64       $unwind$DMF_SamNotificationViaSsh_Create 000000018002aa64     DmfK:Dmf_SamNotificationViaSsh.obj
 0002:00003a88       $unwind$DmfContainerEvtDeviceArmWakeFromSxWithReason 000000018002aa88     DmfK:DmfContainer.obj
 0002:00003a88       $unwind$DmfContainerEvtDeviceD0Entry 000000018002aa88     DmfK:DmfContainer.obj
 0002:00003a88       $unwind$DmfContainerEvtDeviceUsageNotificationEx 000000018002aa88     DmfK:DmfContainer.obj
 0002:00003a88       $unwind$?DMF_Bridge_ModuleArmWakeFromS0@@YAJPEAUDMFMODULE__@@@Z 000000018002aa88     DmfK:Dmf_Bridge.obj
 0002:00003a88       $unwind$?DMF_Bridge_ModuleQueryRemove@@YAJPEAUDMFMODULE__@@@Z 000000018002aa88     DmfK:Dmf_Bridge.obj
 0002:00003a88       $unwind$?DMF_Bridge_ModuleQueryStop@@YAJPEAUDMFMODULE__@@@Z 000000018002aa88     DmfK:Dmf_Bridge.obj
 0002:00003a88       $unwind$?DMF_Bridge_ModuleRelationsQuery@@YAXPEAUDMFMODULE__@@W4_DEVICE_RELATION_TYPE@@@Z 000000018002aa88     DmfK:Dmf_Bridge.obj
 0002:00003a88       $unwind$?DMF_Bridge_ModuleSelfManagedIoInit@@YAJPEAUDMFMODULE__@@@Z 000000018002aa88     DmfK:Dmf_Bridge.obj
 0002:00003a88       $unwind$?DMF_Bridge_ModuleSelfManagedIoRestart@@YAJPEAUDMFMODULE__@@@Z 000000018002aa88     DmfK:Dmf_Bridge.obj
 0002:00003a88       $unwind$?DMF_Bridge_ModuleSelfManagedIoSuspend@@YAJPEAUDMFMODULE__@@@Z 000000018002aa88     DmfK:Dmf_Bridge.obj
 0002:00003a88       $unwind$DMF_BufferQueue_Enqueue 000000018002aa88     DmfK:Dmf_BufferQueue.obj
 0002:00003a88       $unwind$?ContinuousRequestTarget_StreamCompletionRoutine@@YAXPEAUWDFREQUEST__@@PEAUWDFIOTARGET__@@PEAU_WDF_REQUEST_COMPLETION_PARAMS@@PEAX@Z 000000018002aa88     DmfK:Dmf_ContinuousRequestTarget.obj
 0002:00003a88       $unwind$?DMF_DeviceInterfaceTarget_Open@@YAJPEAUDMFMODULE__@@@Z 000000018002aa88     DmfK:Dmf_DeviceInterfaceTarget.obj
 0002:00003a88       $unwind$?RequestTarget_CompletionRoutine@@YAXPEAUWDFREQUEST__@@PEAUWDFIOTARGET__@@PEAU_WDF_REQUEST_COMPLETION_PARAMS@@PEAX@Z 000000018002aa88     DmfK:Dmf_RequestTarget.obj
 0002:00003a88       $unwind$DMF_RequestTarget_IoTargetSet 000000018002aa88     DmfK:Dmf_RequestTarget.obj
 0002:00003a88       $unwind$DMF_SamNotificationViaSsh_ClientBufferPutOutput 000000018002aa88     DmfK:Dmf_SamNotificationViaSsh.obj
 0002:00003a88       $unwind$?DMF_ScheduledTask_Close@@YAXPEAUDMFMODULE__@@@Z 000000018002aa88     DmfK:Dmf_ScheduledTask.obj
 0002:00003a88       $unwind$DMF_ScheduledTask_Cancel 000000018002aa88     DmfK:Dmf_ScheduledTask.obj
 0002:00003a88       $unwind$SurfaceTelemetry_IsTelemetryEventTypeAllowed 000000018002aa88     DmfK:SurfaceTelemetry.obj
 0002:00003aa4       $unwind$WPP_RECORDER_SF_s  000000018002aaa4     DmfK:Dmf_SamNotificationViaSsh.obj
 0002:00003ac4       $unwind$?SamNotificationViaSsh_LegacyModeQueryAndSet@@YAXPEAUDMFMODULE__@@@Z 000000018002aac4     DmfK:Dmf_SamNotificationViaSsh.obj
 0002:00003af0       $unwind$?ContinuousRequestTarget_CreateBuffersAndFormatRequestForRequestType@@YAJPEAUDMFMODULE__@@PEAUWDFREQUEST__@@@Z 000000018002aaf0     DmfK:Dmf_ContinuousRequestTarget.obj
 0002:00003af0       $unwind$?SamNotificationViaSsh_RegisterForTargetNotification@@YAJPEAUDMFMODULE__@@E@Z 000000018002aaf0     DmfK:Dmf_SamNotificationViaSsh.obj
 0002:00003af0       $unwind$?SamNotificationViaSsh_RegisterForTargetNotificationSynchronously@@YAJPEAUDMFMODULE__@@E@Z 000000018002aaf0     DmfK:Dmf_SamNotificationViaSsh.obj
 0002:00003b0c       $unwind$?DMF_ModuleDestroy@@YAXPEAUDMFMODULE__@@E@Z 000000018002ab0c     DmfK:DmfCore.obj
 0002:00003b0c       $unwind$?DMF_Internal_ModuleArmWakeFromSxWithReason@@YAJPEAUDMFMODULE__@@EE@Z 000000018002ab0c     DmfK:DmfInternal.obj
 0002:00003b0c       $unwind$?DMF_Internal_ModulePrepareHardware@@YAJPEAUDMFMODULE__@@PEAUWDFCMRESLIST__@@1@Z 000000018002ab0c     DmfK:DmfInternal.obj
 0002:00003b0c       $unwind$?DMF_Internal_ModuleUsageNotificationEx@@YAJPEAUDMFMODULE__@@W4_WDF_SPECIAL_FILE_TYPE@@E@Z 000000018002ab0c     DmfK:DmfInternal.obj
 0002:00003b0c       $unwind$?DMF_Internal_ResourcesAssign@@YAJPEAUDMFMODULE__@@PEAUWDFCMRESLIST__@@1@Z 000000018002ab0c     DmfK:DmfInternal.obj
 0002:00003b0c       $unwind$DMF_Portable_LookasideListCreate 000000018002ab0c     DmfK:DmfPortable.obj
 0002:00003b0c       $unwind$?DeviceInterfaceTarget_ModuleCloseReasonSet@@YA?AW4ModuleCloseReason_Type@@PEAUDMFMODULE__@@W41@@Z 000000018002ab0c     DmfK:Dmf_DeviceInterfaceTarget.obj
 0002:00003b0c       $unwind$?SamNotificationViaSsh_StreamAsynchronousBufferCallbackOutput@@YA?AW4ContinuousRequestTarget_BufferDisposition@@PEAUDMFMODULE__@@PEAX_K1J@Z 000000018002ab0c     DmfK:Dmf_SamNotificationViaSsh.obj
 0002:00003b28       $unwind$?DMF_Internal_ModuleDeviceIoControl@@YAEPEAUDMFMODULE__@@PEAUWDFQUEUE__@@PEAUWDFREQUEST__@@_K3K@Z 000000018002ab28     DmfK:DmfInternal.obj
 0002:00003b28       $unwind$?DMF_Internal_ModuleFileCreate@@YAEPEAUDMFMODULE__@@PEAUWDFDEVICE__@@PEAUWDFREQUEST__@@PEAUWDFFILEOBJECT__@@@Z 000000018002ab28     DmfK:DmfInternal.obj
 0002:00003b28       $unwind$?DMF_Internal_ModuleInternalDeviceIoControl@@YAEPEAUDMFMODULE__@@PEAUWDFQUEUE__@@PEAUWDFREQUEST__@@_K3K@Z 000000018002ab28     DmfK:DmfInternal.obj
 0002:00003b28       $unwind$?DMF_Internal_ModuleQueueIoRead@@YAEPEAUDMFMODULE__@@PEAUWDFQUEUE__@@PEAUWDFREQUEST__@@_K@Z 000000018002ab28     DmfK:DmfInternal.obj
 0002:00003b28       $unwind$?DMF_Internal_ModuleQueueIoWrite@@YAEPEAUDMFMODULE__@@PEAUWDFQUEUE__@@PEAUWDFREQUEST__@@_K@Z 000000018002ab28     DmfK:DmfInternal.obj
 0002:00003b28       $unwind$?LiveKernelDump_DataBufferSourceAdd@@YAJPEAUDMFMODULE__@@PEAXK@Z 000000018002ab28     DmfK:Dmf_LiveKernelDump.obj
 0002:00003b28       $unwind$?RingBuffer_Write@@YAJPEAURING_BUFFER@@PEAEKP6AXPEAX1K@Z@Z 000000018002ab28     DmfK:Dmf_RingBuffer.obj
 0002:00003b28       $unwind$?SamNotificationViaSsh_StreamAsynchronousBufferCallbackInput@@YAXPEAUDMFMODULE__@@PEAXPEA_K1@Z 000000018002ab28     DmfK:Dmf_SamNotificationViaSsh.obj
 0002:00003b48       $unwind$?DMF_SamNotificationViaSsh_ChildModulesAdd@@YAXPEAUDMFMODULE__@@PEAU_DMF_MODULE_ATTRIBUTES@@PEAX@Z 000000018002ab48     DmfK:Dmf_SamNotificationViaSsh.obj
 0002:00003b70       $unwind$DmfContainerEvtDeviceRelationsQuery 000000018002ab70     DmfK:DmfContainer.obj
 0002:00003b70       $unwind$?DMF_ModuleCollectionD0EntryCleanup@@YAXPEAUDMFCOLLECTION__@@@Z 000000018002ab70     DmfK:DmfModuleCollection.obj
 0002:00003b70       $unwind$DMF_Portable_LookasideListCreateMemory 000000018002ab70     DmfK:DmfPortable.obj
 0002:00003b70       $unwind$?DMF_BranchTrack_Close@@YAXPEAUDMFMODULE__@@@Z 000000018002ab70     DmfK:Dmf_BranchTrack.obj
 0002:00003b70       $unwind$?DMF_Bridge_ModuleDisarmWakeFromS0@@YAXPEAUDMFMODULE__@@@Z 000000018002ab70     DmfK:Dmf_Bridge.obj
 0002:00003b70       $unwind$?DMF_Bridge_ModuleDisarmWakeFromSx@@YAXPEAUDMFMODULE__@@@Z 000000018002ab70     DmfK:Dmf_Bridge.obj
 0002:00003b70       $unwind$?DMF_Bridge_ModuleSelfManagedIoCleanup@@YAXPEAUDMFMODULE__@@@Z 000000018002ab70     DmfK:Dmf_Bridge.obj
 0002:00003b70       $unwind$?DMF_Bridge_ModuleSelfManagedIoFlush@@YAXPEAUDMFMODULE__@@@Z 000000018002ab70     DmfK:Dmf_Bridge.obj
 0002:00003b70       $unwind$?DMF_Bridge_ModuleSurpriseRemoval@@YAXPEAUDMFMODULE__@@@Z 000000018002ab70     DmfK:Dmf_Bridge.obj
 0002:00003b70       $unwind$?DMF_Bridge_ModuleWakeFromS0Triggered@@YAXPEAUDMFMODULE__@@@Z 000000018002ab70     DmfK:Dmf_Bridge.obj
 0002:00003b70       $unwind$?DMF_Bridge_ModuleWakeFromSxTriggered@@YAXPEAUDMFMODULE__@@@Z 000000018002ab70     DmfK:Dmf_Bridge.obj
 0002:00003b70       $unwind$DMF_BufferQueue_Count 000000018002ab70     DmfK:Dmf_BufferQueue.obj
 0002:00003b70       $unwind$DMF_RequestTarget_IoTargetClear 000000018002ab70     DmfK:Dmf_RequestTarget.obj
 0002:00003b70       $unwind$SurfaceTelemetry_Initialize 000000018002ab70     DmfK:SurfaceTelemetry.obj
 0002:00003b88       $unwind$?DMF_ContinuousRequestTarget_Close@@YAXPEAUDMFMODULE__@@@Z 000000018002ab88     DmfK:Dmf_ContinuousRequestTarget.obj
 0002:00003b88       $unwind$DMF_ContinuousRequestTarget_IoTargetClear 000000018002ab88     DmfK:Dmf_ContinuousRequestTarget.obj
 0002:00003b88       $unwind$DMF_DeviceInterfaceTarget_StreamStop 000000018002ab88     DmfK:Dmf_DeviceInterfaceTarget.obj
 0002:00003b88       $unwind$?HashTable_ContextCleanup@@YAXPEAU_DMF_CONTEXT_HashTable@@@Z 000000018002ab88     DmfK:Dmf_HashTable.obj
 0002:00003b88       $unwind$?DMF_IoctlHandler_Close@@YAXPEAUDMFMODULE__@@@Z 000000018002ab88     DmfK:Dmf_IoctlHandler.obj
 0002:00003b88       $unwind$?DMF_IoctlHandler_FileClose@@YAEPEAUDMFMODULE__@@PEAUWDFFILEOBJECT__@@@Z 000000018002ab88     DmfK:Dmf_IoctlHandler.obj
 0002:00003b88       $unwind$?DMF_RequestTarget_Close@@YAXPEAUDMFMODULE__@@@Z 000000018002ab88     DmfK:Dmf_RequestTarget.obj
 0002:00003b88       $unwind$?DMF_Rundown_Open@@YAJPEAUDMFMODULE__@@@Z 000000018002ab88     DmfK:Dmf_Rundown.obj
 0002:00003b88       $unwind$SurfaceTelemetry_Update 000000018002ab88     DmfK:SurfaceTelemetry.obj
 0002:00003ba0       $unwind$?SurfaceTelemetry_ReadConsentFile@@YAJXZ 000000018002aba0     DmfK:SurfaceTelemetry.obj
 0002:00003bb8       $unwind$?DMF_ModuleCollectionReleaseHardware@@YAJPEAUDMFCOLLECTION__@@PEAUWDFCMRESLIST__@@@Z 000000018002abb8     DmfK:DmfModuleCollection.obj
 0002:00003bb8       $unwind$DMF_QueuedWorkItem_Enqueue 000000018002abb8     DmfK:Dmf_QueuedWorkItem.obj
 0002:00003bd8       $unwind$?QueuedWorkItem_CallbackScheduledTask@@YA?AW4ScheduledTask_Result_Type@@PEAUDMFMODULE__@@PEAXW4_WDF_POWER_DEVICE_STATE@@@Z 000000018002abd8     DmfK:Dmf_QueuedWorkItem.obj
 0002:00003bf4       $unwind$DMF_ModulesCreate  000000018002abf4     DmfK:DmfModuleCollection.obj
 0002:00003c14       $unwind$?DMF_ModuleBranchTrack_ModuleInitialize@@YAXPEAU_DMF_OBJECT_@@@Z 000000018002ac14     DmfK:DmfBranchTrack.obj
 0002:00003c14       $unwind$?DMF_ModuleCollectionHandleSet@@YAXPEAU_DMF_OBJECT_@@@Z 000000018002ac14     DmfK:DmfModuleCollection.obj
 0002:00003c20       $unwind$?DMF_ModuleCollectionHandlePropagate@@YAXPEAU_DMF_MODULE_COLLECTION_@@J@Z 000000018002ac20     DmfK:DmfModuleCollection.obj
 0002:00003c34       $unwind$?DMF_ModuleCollectionCreate@@YAJPEAUDMFDEVICE_INIT@@PEAUDMF_MODULE_COLLECTION_CONFIG@@PEAPEAUDMFCOLLECTION__@@@Z 000000018002ac34     DmfK:DmfModuleCollection.obj
 0002:00003c54       $unwind$?DMF_ModuleCollectionPostCreate@@YAJPEAUDMF_MODULE_COLLECTION_CONFIG@@PEAUDMFCOLLECTION__@@@Z 000000018002ac54     DmfK:DmfModuleCollection.obj
 0002:00003c74       $unwind$?DMF_ModuleCollectionFeatureHandleGet@@YAPEAU_DMF_OBJECT_@@PEAU_DMF_MODULE_COLLECTION_@@W4DmfFeatureType@@@Z 000000018002ac74     DmfK:DmfModuleCollection.obj
 0002:00003c74       $unwind$?ContinuousRequestTarget_PendingCollectionListSearchAndRemove@@YAEPEAUDMFMODULE__@@PEAUWDFREQUEST__@@@Z 000000018002ac74     DmfK:Dmf_ContinuousRequestTarget.obj
 0002:00003c74       $unwind$?RequestTarget_PendingCollectionListSearchAndRemove@@YAEPEAUDMFMODULE__@@PEAUWDFREQUEST__@@@Z 000000018002ac74     DmfK:Dmf_RequestTarget.obj
 0002:00003c90       $unwind$?DMF_ModuleCollectionPrepareHardware@@YAJPEAUDMFCOLLECTION__@@PEAUWDFCMRESLIST__@@1@Z 000000018002ac90     DmfK:DmfModuleCollection.obj
 0002:00003cb0       $unwind$?DMF_ModuleCollectionD0Entry@@YAJPEAUDMFCOLLECTION__@@W4_WDF_POWER_DEVICE_STATE@@@Z 000000018002acb0     DmfK:DmfModuleCollection.obj
 0002:00003cb0       $unwind$?DMF_ModuleCollectionD0EntryPostInterruptsEnabled@@YAJPEAUDMFCOLLECTION__@@W4_WDF_POWER_DEVICE_STATE@@@Z 000000018002acb0     DmfK:DmfModuleCollection.obj
 0002:00003cd0       $unwind$?DMF_ModuleCollectionD0Exit@@YAJPEAUDMFCOLLECTION__@@W4_WDF_POWER_DEVICE_STATE@@@Z 000000018002acd0     DmfK:DmfModuleCollection.obj
 0002:00003cd0       $unwind$?DMF_ModuleCollectionD0ExitPreInterruptsDisabled@@YAJPEAUDMFCOLLECTION__@@W4_WDF_POWER_DEVICE_STATE@@@Z 000000018002acd0     DmfK:DmfModuleCollection.obj
 0002:00003cf0       $unwind$?DMF_ModuleCollectionDeviceIoControl@@YAEPEAUDMFCOLLECTION__@@PEAUWDFQUEUE__@@PEAUWDFREQUEST__@@_K3K@Z 000000018002acf0     DmfK:DmfModuleCollection.obj
 0002:00003cf0       $unwind$?DMF_ModuleCollectionInternalDeviceIoControl@@YAEPEAUDMFCOLLECTION__@@PEAUWDFQUEUE__@@PEAUWDFREQUEST__@@_K3K@Z 000000018002acf0     DmfK:DmfModuleCollection.obj
 0002:00003d0c       $unwind$?DMF_ModuleCollectionDisarmWakeFromS0@@YAXPEAUDMFCOLLECTION__@@@Z 000000018002ad0c     DmfK:DmfModuleCollection.obj
 0002:00003d0c       $unwind$?DMF_ModuleCollectionDisarmWakeFromSx@@YAXPEAUDMFCOLLECTION__@@@Z 000000018002ad0c     DmfK:DmfModuleCollection.obj
 0002:00003d0c       $unwind$?DMF_ModuleCollectionSelfManagedIoCleanup@@YAXPEAUDMFCOLLECTION__@@@Z 000000018002ad0c     DmfK:DmfModuleCollection.obj
 0002:00003d0c       $unwind$?DMF_ModuleCollectionSelfManagedIoFlush@@YAXPEAUDMFCOLLECTION__@@@Z 000000018002ad0c     DmfK:DmfModuleCollection.obj
 0002:00003d0c       $unwind$?DMF_ModuleCollectionSurpriseRemoval@@YAXPEAUDMFCOLLECTION__@@@Z 000000018002ad0c     DmfK:DmfModuleCollection.obj
 0002:00003d0c       $unwind$?DMF_ModuleCollectionWakeFromS0Triggered@@YAXPEAUDMFCOLLECTION__@@@Z 000000018002ad0c     DmfK:DmfModuleCollection.obj
 0002:00003d0c       $unwind$?DMF_ModuleCollectionWakeFromSxTriggered@@YAXPEAUDMFCOLLECTION__@@@Z 000000018002ad0c     DmfK:DmfModuleCollection.obj
 0002:00003d20       $unwind$?DMF_Generic_Close@@YAXPEAUDMFMODULE__@@@Z 000000018002ad20     DmfK:DmfGeneric.obj
 0002:00003d20       $unwind$?DMF_Generic_Open@@YAJPEAUDMFMODULE__@@@Z 000000018002ad20     DmfK:DmfGeneric.obj
 0002:00003d20       $unwind$?DMF_ModuleCollectionArmWakeFromS0@@YAJPEAUDMFCOLLECTION__@@@Z 000000018002ad20     DmfK:DmfModuleCollection.obj
 0002:00003d20       $unwind$?DMF_ModuleCollectionQueryRemove@@YAJPEAUDMFCOLLECTION__@@@Z 000000018002ad20     DmfK:DmfModuleCollection.obj
 0002:00003d20       $unwind$?DMF_ModuleCollectionQueryStop@@YAJPEAUDMFCOLLECTION__@@@Z 000000018002ad20     DmfK:DmfModuleCollection.obj
 0002:00003d20       $unwind$?DMF_ModuleCollectionSelfManagedIoInit@@YAJPEAUDMFCOLLECTION__@@@Z 000000018002ad20     DmfK:DmfModuleCollection.obj
 0002:00003d20       $unwind$?DMF_ModuleCollectionSelfManagedIoRestart@@YAJPEAUDMFCOLLECTION__@@@Z 000000018002ad20     DmfK:DmfModuleCollection.obj
 0002:00003d20       $unwind$?DMF_ModuleCollectionSelfManagedIoSuspend@@YAJPEAUDMFCOLLECTION__@@@Z 000000018002ad20     DmfK:DmfModuleCollection.obj
 0002:00003d20       $unwind$?ContinuousRequestTarget_DecreaseStreamRequestCount@@YAXPEAU_DMF_CONTEXT_ContinuousRequestTarget@@@Z 000000018002ad20     DmfK:Dmf_ContinuousRequestTarget.obj
 0002:00003d3c       $unwind$?DMF_ModuleCollectionCleanup@@YAXPEAU_DMF_MODULE_COLLECTION_@@W4ModuleOpenedDuringType@@@Z 000000018002ad3c     DmfK:DmfModuleCollection.obj
 0002:00003d5c       $unwind$?DMF_ModuleCollectionDispatchNtStatus@@YAJPEAU_DMF_MODULE_COLLECTION_@@P6AJPEAUDMFMODULE__@@@Z@Z 000000018002ad5c     DmfK:DmfModuleCollection.obj
 0002:00003d5c       $unwind$DMF_HashTable_Enumerate 000000018002ad5c     DmfK:Dmf_HashTable.obj
 0002:00003d7c       $unwind$?DMF_ModuleCollectionDispatchVoid@@YAXPEAU_DMF_MODULE_COLLECTION_@@P6AXPEAUDMFMODULE__@@@Z@Z 000000018002ad7c     DmfK:DmfModuleCollection.obj
 0002:00003d7c       $unwind$?DMF_Bridge_ModuleArmWakeFromSxWithReason@@YAJPEAUDMFMODULE__@@EE@Z 000000018002ad7c     DmfK:Dmf_Bridge.obj
 0002:00003d7c       $unwind$?DMF_Bridge_ModulePrepareHardware@@YAJPEAUDMFMODULE__@@PEAUWDFCMRESLIST__@@1@Z 000000018002ad7c     DmfK:Dmf_Bridge.obj
 0002:00003d7c       $unwind$?DMF_Bridge_ModuleUsageNotificationEx@@YAJPEAUDMFMODULE__@@W4_WDF_SPECIAL_FILE_TYPE@@E@Z 000000018002ad7c     DmfK:Dmf_Bridge.obj
 0002:00003d7c       $unwind$?DMF_IoctlHandler_FileCleanup@@YAEPEAUDMFMODULE__@@PEAUWDFFILEOBJECT__@@@Z 000000018002ad7c     DmfK:Dmf_IoctlHandler.obj
 0002:00003d9c       $unwind$?DMF_ModuleCollectionConfigListInitialize@@YAJPEAUDMF_MODULE_COLLECTION_CONFIG@@@Z 000000018002ad9c     DmfK:DmfModuleCollection.obj
 0002:00003dbc       $unwind$?DMF_ModuleCollectionConfigAddAttributes@@YAXPEAUDMF_MODULE_COLLECTION_CONFIG@@PEAU_DMF_MODULE_ATTRIBUTES@@PEAU_WDF_OBJECT_ATTRIBUTES@@PEAPEAUDMFMODULE__@@@Z 000000018002adbc     DmfK:DmfModuleCollection.obj
 0002:00003dbc       $unwind$DMF_File_ReadEx    000000018002adbc     DmfK:Dmf_File.obj
 0002:00003ddc       $unwind$?SurfaceTelemetryConsentSettingsNotification_IoctlClientCallback_TelemetryConsentChanged@@YAJPEAUDMFMODULE__@@PEAUWDFQUEUE__@@PEAUWDFREQUEST__@@KPEAX_K34PEA_K@Z 000000018002addc     DmfK:Dmf_SurfaceTelemetryConsentSettingsNotification.obj
 0002:00003df0       $unwind$?DMF_SurfaceTelemetryConsentSettingsNotification_ChildModulesAdd@@YAXPEAUDMFMODULE__@@PEAU_DMF_MODULE_ATTRIBUTES@@PEAX@Z 000000018002adf0     DmfK:Dmf_SurfaceTelemetryConsentSettingsNotification.obj
 0002:00003e14       $unwind$DMF_DmfDeviceInitAllocate 000000018002ae14     DmfK:DmfDeviceInit.obj
 0002:00003e2c       $unwind$DMF_DmfDeviceInitHookFileObjectConfig 000000018002ae2c     DmfK:DmfDeviceInit.obj
 0002:00003e2c       $unwind$DMF_ScheduledTask_TimesRunGet 000000018002ae2c     DmfK:Dmf_ScheduledTask.obj
 0002:00003e3c       $unwind$DMF_LiveKernelDump_Create 000000018002ae3c     DmfK:Dmf_LiveKernelDump.obj
 0002:00003e3c       $unwind$DMF_RingBuffer_Create 000000018002ae3c     DmfK:Dmf_RingBuffer.obj
 0002:00003e60       $unwind$WPP_RECORDER_SF_qddd 000000018002ae60     DmfK:Dmf_CrashDump.obj
 0002:00003e60       $unwind$WPP_RECORDER_SF_DDDD 000000018002ae60     DmfK:Dmf_HashTable.obj
 0002:00003e60       $unwind$WPP_RECORDER_SF_qddD 000000018002ae60     DmfK:Dmf_LiveKernelDump.obj
 0002:00003e7c       $unwind$?LiveKernelDump_InsertDataBufferInLiveDump@@YAEPEAUDMFMODULE__@@PEAEKPEAX@Z 000000018002ae7c     DmfK:Dmf_LiveKernelDump.obj
 0002:00003e98       $unwind$?LiveKernelDump_InsertDmfTriageDataToLiveDump@@YAJPEAUDMFMODULE__@@PEAX@Z 000000018002ae98     DmfK:Dmf_LiveKernelDump.obj
 0002:00003eb4       $unwind$?LiveKernelDump_InsertClientTriageDataToLiveDump@@YAJPEAXKPEAULIVEKERNELDUMP_CLIENT_STRUCTURE@@@Z 000000018002aeb4     DmfK:Dmf_LiveKernelDump.obj
 0002:00003ed4       $unwind$?LiveKernelDump_LiveKernelMemoryDumpCreate@@YAJPEAUDMFMODULE__@@K_KEKPEAULIVEKERNELDUMP_CLIENT_STRUCTURE@@KPEAX@Z 000000018002aed4     DmfK:Dmf_LiveKernelDump.obj
 0002:00003ef8       $unwind$?DMF_Generic_ModuleD0ExitPreInterruptsDisabled@@YAJPEAUDMFMODULE__@@W4_WDF_POWER_DEVICE_STATE@@@Z 000000018002aef8     DmfK:DmfGeneric.obj
 0002:00003ef8       $unwind$?CrashDump_IoctlHandler@@YAJPEAUDMFMODULE__@@PEAUWDFQUEUE__@@PEAUWDFREQUEST__@@KPEAX_K34PEA_K@Z 000000018002aef8     DmfK:Dmf_CrashDump.obj
 0002:00003ef8       $unwind$?LiveKernelDump_IoctlHandler@@YAJPEAUDMFMODULE__@@PEAUWDFQUEUE__@@PEAUWDFREQUEST__@@KPEAX_K34PEA_K@Z 000000018002aef8     DmfK:Dmf_LiveKernelDump.obj
 0002:00003f14       $unwind$?DMF_LiveKernelDump_ChildModulesAdd@@YAXPEAUDMFMODULE__@@PEAU_DMF_MODULE_ATTRIBUTES@@PEAX@Z 000000018002af14     DmfK:Dmf_LiveKernelDump.obj
 0002:00003f38       $unwind$DMF_Portable_EventWaitForSingleObject 000000018002af38     DmfK:DmfPortable.obj
 0002:00003f54       $unwind$DMF_Portable_EventClose 000000018002af54     DmfK:DmfPortable.obj
 0002:00003f54       $unwind$?Bridge_DefaultEvtDeviceContextCleanup@@YAXPEAX@Z 000000018002af54     DmfK:Dmf_Bridge.obj
 0002:00003f54       $unwind$?Bridge_DefaultEvtDeviceDisarmWakeFromS0@@YAXPEAUWDFDEVICE__@@@Z 000000018002af54     DmfK:Dmf_Bridge.obj
 0002:00003f54       $unwind$?Bridge_DefaultEvtDeviceDisarmWakeFromSx@@YAXPEAUWDFDEVICE__@@@Z 000000018002af54     DmfK:Dmf_Bridge.obj
 0002:00003f54       $unwind$?Bridge_DefaultEvtDeviceRelationsQuery@@YAXPEAUWDFDEVICE__@@W4_DEVICE_RELATION_TYPE@@@Z 000000018002af54     DmfK:Dmf_Bridge.obj
 0002:00003f54       $unwind$?Bridge_DefaultEvtDeviceSelfManagedIoCleanup@@YAXPEAUWDFDEVICE__@@@Z 000000018002af54     DmfK:Dmf_Bridge.obj
 0002:00003f54       $unwind$?Bridge_DefaultEvtDeviceSelfManagedIoFlush@@YAXPEAUWDFDEVICE__@@@Z 000000018002af54     DmfK:Dmf_Bridge.obj
 0002:00003f54       $unwind$?Bridge_DefaultEvtDeviceSurpriseRemoval@@YAXPEAUWDFDEVICE__@@@Z 000000018002af54     DmfK:Dmf_Bridge.obj
 0002:00003f54       $unwind$?Bridge_DefaultEvtDeviceWakeFromS0Triggered@@YAXPEAUWDFDEVICE__@@@Z 000000018002af54     DmfK:Dmf_Bridge.obj
 0002:00003f54       $unwind$?Bridge_DefaultEvtDeviceWakeFromSxTriggered@@YAXPEAUWDFDEVICE__@@@Z 000000018002af54     DmfK:Dmf_Bridge.obj
 0002:00003f64       $unwind$?RtlStringCbPrintfA@@YAJPEAD_KPEBDZZ 000000018002af64     DmfK:DmfCore.obj
 0002:00003f74       $unwind$DMF_ModuleCreate   000000018002af74     DmfK:DmfCore.obj
 0002:00003f94       $unwind$?DmfModuleInstanceNameInitialize@@YAJPEAU_DMF_OBJECT_@@PEAUWDFMEMORY__@@PEAU_DMF_MODULE_ATTRIBUTES@@@Z 000000018002af94     DmfK:DmfCore.obj
 0002:00003f94       $unwind$?DMF_Bridge_Destroy@@YAXPEAUDMFMODULE__@@@Z 000000018002af94     DmfK:Dmf_Bridge.obj
 0002:00003f94       $unwind$?ContinuousRequestTarget_PendingCollectionListAdd@@YAJPEAUDMFMODULE__@@PEAUWDFREQUEST__@@@Z 000000018002af94     DmfK:Dmf_ContinuousRequestTarget.obj
 0002:00003f94       $unwind$DMF_ContinuousRequestTarget_Cancel 000000018002af94     DmfK:Dmf_ContinuousRequestTarget.obj
 0002:00003f94       $unwind$?RequestTarget_PendingCollectionListAdd@@YAJPEAUDMFMODULE__@@PEAUWDFREQUEST__@@@Z 000000018002af94     DmfK:Dmf_RequestTarget.obj
 0002:00003f94       $unwind$DMF_Rundown_Start  000000018002af94     DmfK:Dmf_Rundown.obj
 0002:00003f94       $unwind$DMF_ScheduledTask_ExecuteNowDeferred 000000018002af94     DmfK:Dmf_ScheduledTask.obj
 0002:00003fa8       $unwind$?DmfModuleChildObjectsInitialize@@YAJPEAU_DMF_OBJECT_@@PEAUWDFMEMORY__@@PEAU_DMF_MODULE_ATTRIBUTES@@PEAUDMF_MODULE_DESCRIPTOR@@@Z 000000018002afa8     DmfK:DmfCore.obj
 0002:00003fc0       $unwind$?DmfModuleParentUpdate@@YAJPEAUWDFDEVICE__@@PEAXPEAU_DMF_OBJECT_@@PEAU_DMF_MODULE_ATTRIBUTES@@@Z 000000018002afc0     DmfK:DmfCore.obj
 0002:00003fc0       $unwind$DMF_RingBuffer_Read 000000018002afc0     DmfK:Dmf_RingBuffer.obj
 0002:00003fc0       $unwind$DMF_RingBuffer_Write 000000018002afc0     DmfK:Dmf_RingBuffer.obj
 0002:00003fd8       $unwind$?DmfModuleInFlightRecorderInitialize@@YAXPEAU_DMF_OBJECT_@@@Z 000000018002afd8     DmfK:DmfCore.obj
 0002:00003ff0       $unwind$DMF_ModuleReference 000000018002aff0     DmfK:DmfCall.obj
 0002:00004008       $unwind$?DMF_ModuleWaitForReferenceCountToClear@@YAXPEAUDMFMODULE__@@@Z 000000018002b008     DmfK:DmfCall.obj
 0002:00004024       $unwind$?DMF_ChildDispatchSingleParameterVoid@@YAXPEAUDMFMODULE__@@P6AX0@ZPEAU_DMF_ChildObjectGet@@@Z 000000018002b024     DmfK:DmfCall.obj
 0002:00004024       $unwind$?CrashDump_BugCheckTriageDumpDataCallback@@YAXW4_KBUGCHECK_CALLBACK_REASON@@PEAU_KBUGCHECK_REASON_CALLBACK_RECORD@@PEAXK@Z 000000018002b024     DmfK:Dmf_CrashDump.obj
 0002:00004034       $unwind$?DMF_Module_ArmWakeFromSxWithReason@@YAJPEAUDMFMODULE__@@EE@Z 000000018002b034     DmfK:DmfCall.obj
 0002:00004034       $unwind$?DMF_Module_PrepareHardware@@YAJPEAUDMFMODULE__@@PEAUWDFCMRESLIST__@@1@Z 000000018002b034     DmfK:DmfCall.obj
 0002:00004034       $unwind$?DMF_Module_UsageNotificationEx@@YAJPEAUDMFMODULE__@@W4_WDF_SPECIAL_FILE_TYPE@@E@Z 000000018002b034     DmfK:DmfCall.obj
 0002:0000404c       $unwind$?DMF_Module_FileCreate@@YAEPEAUDMFMODULE__@@PEAUWDFDEVICE__@@PEAUWDFREQUEST__@@PEAUWDFFILEOBJECT__@@@Z 000000018002b04c     DmfK:DmfCall.obj
 0002:0000404c       $unwind$?DMF_Module_QueueIoRead@@YAEPEAUDMFMODULE__@@PEAUWDFQUEUE__@@PEAUWDFREQUEST__@@_K@Z 000000018002b04c     DmfK:DmfCall.obj
 0002:0000404c       $unwind$?DMF_Module_QueueIoWrite@@YAEPEAUDMFMODULE__@@PEAUWDFQUEUE__@@PEAUWDFREQUEST__@@_K@Z 000000018002b04c     DmfK:DmfCall.obj
 0002:00004068       $unwind$?DMF_Module_DeviceIoControl@@YAEPEAUDMFMODULE__@@PEAUWDFQUEUE__@@PEAUWDFREQUEST__@@_K3K@Z 000000018002b068     DmfK:DmfCall.obj
 0002:00004068       $unwind$?DMF_Module_InternalDeviceIoControl@@YAEPEAUDMFMODULE__@@PEAUWDFQUEUE__@@PEAUWDFREQUEST__@@_K3K@Z 000000018002b068     DmfK:DmfCall.obj
 0002:00004068       $unwind$DMF_DeviceInterfaceTarget_Send 000000018002b068     DmfK:Dmf_DeviceInterfaceTarget.obj
 0002:00004068       $unwind$DMF_DeviceInterfaceTarget_SendEx 000000018002b068     DmfK:Dmf_DeviceInterfaceTarget.obj
 0002:00004088       $unwind$?DMF_Module_SelfManagedIoCleanup@@YAXPEAUDMFMODULE__@@@Z 000000018002b088     DmfK:DmfCall.obj
 0002:00004088       $unwind$?DMF_Module_SelfManagedIoFlush@@YAXPEAUDMFMODULE__@@@Z 000000018002b088     DmfK:DmfCall.obj
 0002:00004088       $unwind$?DMF_Module_SurpriseRemoval@@YAXPEAUDMFMODULE__@@@Z 000000018002b088     DmfK:DmfCall.obj
 0002:00004088       $unwind$?DeviceInterfaceTarget_StreamStopAndModuleClose@@YAXPEAUDMFMODULE__@@@Z 000000018002b088     DmfK:Dmf_DeviceInterfaceTarget.obj
 0002:00004088       $unwind$?DeviceInterfaceTarget_Stream_Cancel@@YAEPEAUDMFMODULE__@@PEAURequestTarget_DmfRequest__@@@Z 000000018002b088     DmfK:Dmf_DeviceInterfaceTarget.obj
 0002:00004088       $unwind$?DeviceInterfaceTarget_Stream_IoTargetSet@@YAXPEAUDMFMODULE__@@PEAUWDFIOTARGET__@@@Z 000000018002b088     DmfK:Dmf_DeviceInterfaceTarget.obj
 0002:00004088       $unwind$?DeviceInterfaceTarget_Target_Cancel@@YAEPEAUDMFMODULE__@@PEAURequestTarget_DmfRequest__@@@Z 000000018002b088     DmfK:Dmf_DeviceInterfaceTarget.obj
 0002:00004088       $unwind$?DeviceInterfaceTarget_Target_IoTargetSet@@YAXPEAUDMFMODULE__@@PEAUWDFIOTARGET__@@@Z 000000018002b088     DmfK:Dmf_DeviceInterfaceTarget.obj
 0002:00004088       $unwind$DMF_Rundown_Dereference 000000018002b088     DmfK:Dmf_Rundown.obj
 0002:00004094       $unwind$?DMF_Module_RelationsQuery@@YAXPEAUDMFMODULE__@@W4_DEVICE_RELATION_TYPE@@@Z 000000018002b094     DmfK:DmfCall.obj
 0002:000040a8       $unwind$?DMF_Module_DisarmWakeFromS0@@YAXPEAUDMFMODULE__@@@Z 000000018002b0a8     DmfK:DmfCall.obj
 0002:000040a8       $unwind$?DMF_Module_DisarmWakeFromSx@@YAXPEAUDMFMODULE__@@@Z 000000018002b0a8     DmfK:DmfCall.obj
 0002:000040a8       $unwind$?DMF_Module_WakeFromS0Triggered@@YAXPEAUDMFMODULE__@@@Z 000000018002b0a8     DmfK:DmfCall.obj
 0002:000040a8       $unwind$?DMF_Module_WakeFromSxTriggered@@YAXPEAUDMFMODULE__@@@Z 000000018002b0a8     DmfK:DmfCall.obj
 0002:000040b8       $unwind$DMF_BranchTrack_Create 000000018002b0b8     DmfK:Dmf_BranchTrack.obj
 0002:000040b8       $unwind$DMF_CrashDump_Create 000000018002b0b8     DmfK:Dmf_CrashDump.obj
 0002:000040b8       $unwind$DMF_IoctlHandler_Create 000000018002b0b8     DmfK:Dmf_IoctlHandler.obj
 0002:000040b8       $unwind$DMF_ScheduledTask_Create 000000018002b0b8     DmfK:Dmf_ScheduledTask.obj
 0002:000040dc       $unwind$DMF_BranchTrack_CheckPointCreate 000000018002b0dc     DmfK:Dmf_BranchTrack.obj
 0002:000040dc       $unwind$DMF_BranchTrack_CheckPointExecute 000000018002b0dc     DmfK:Dmf_BranchTrack.obj
 0002:000040fc       $unwind$?BranchTrack_EVT_DMF_HashTable_Enumerate_DetailsData@@YAEPEAUDMFMODULE__@@PEAEK1KPEAX@Z 000000018002b0fc     DmfK:Dmf_BranchTrack.obj
 0002:0000411c       $unwind$?DMF_ModuleInterfaceFindAndRemove@@YAEPEAUDMFMODULE__@@0PEAPEAU_DMF_INTERFACE_OBJECT@@@Z 000000018002b11c     DmfK:DmfInterfaceInternal.obj
 0002:0000411c       $unwind$?BranchTrack_QueryInformation@@YAJPEAUDMFMODULE__@@PEAUWDFREQUEST__@@PEA_K@Z 000000018002b11c     DmfK:Dmf_BranchTrack.obj
 0002:0000411c       $unwind$?BranchTrack_QueryInformation_Status@@YAJPEAUDMFMODULE__@@PEAUWDFREQUEST__@@PEA_K@Z 000000018002b11c     DmfK:Dmf_BranchTrack.obj
 0002:0000413c       $unwind$?BranchTrack_QueryInformation_Details@@YAJPEAUDMFMODULE__@@PEAUWDFREQUEST__@@PEA_K@Z 000000018002b13c     DmfK:Dmf_BranchTrack.obj
 0002:00004158       $unwind$?BranchTrack_CheckPointProcess@@YAXPEAUDMFMODULE__@@PEAD11KP6AE01_K2@Z2P6AX0PEAEK4PEAK@Z@Z 000000018002b158     DmfK:Dmf_BranchTrack.obj
 0002:00004174       $unwind$?DMF_BranchTrack_ChildModulesAdd@@YAXPEAUDMFMODULE__@@PEAU_DMF_MODULE_ATTRIBUTES@@PEAX@Z 000000018002b174     DmfK:Dmf_BranchTrack.obj
 0002:0000419c       $unwind$?DMF_Generic_ModuleReleaseHardware@@YAJPEAUDMFMODULE__@@PEAUWDFCMRESLIST__@@@Z 000000018002b19c     DmfK:DmfGeneric.obj
 0002:0000419c       $unwind$?DMF_BranchTrack_ModuleDeviceIoControl@@YAEPEAUDMFMODULE__@@PEAUWDFQUEUE__@@PEAUWDFREQUEST__@@_K3K@Z 000000018002b19c     DmfK:Dmf_BranchTrack.obj
 0002:000041b8       $unwind$?DMF_BranchTrack_Open@@YAJPEAUDMFMODULE__@@@Z 000000018002b1b8     DmfK:Dmf_BranchTrack.obj
 0002:000041b8       $unwind$?ContinuousRequestTarget_FormatRequestForRequestType@@YAJPEAUDMFMODULE__@@PEAUWDFREQUEST__@@W4ContinuousRequestTarget_RequestType@@KPEAUWDFMEMORY__@@3@Z 000000018002b1b8     DmfK:Dmf_ContinuousRequestTarget.obj
 0002:000041b8       $unwind$?RequestTarget_FormatRequestForRequestType@@YAJPEAUDMFMODULE__@@PEAUWDFREQUEST__@@W4ContinuousRequestTarget_RequestType@@KPEAUWDFMEMORY__@@3@Z 000000018002b1b8     DmfK:Dmf_RequestTarget.obj
 0002:000041d8       $unwind$?RtlUnicodeStringCopy@@YAJPEAU_UNICODE_STRING@@PEBU1@@Z 000000018002b1d8     DmfK:Dmf_DeviceInterfaceTarget.obj
 0002:000041ec       $unwind$?DMF_Generic_ModuleD0Entry@@YAJPEAUDMFMODULE__@@W4_WDF_POWER_DEVICE_STATE@@@Z 000000018002b1ec     DmfK:DmfGeneric.obj
 0002:000041ec       $unwind$DMF_DeviceInterfaceTarget_SendSynchronously 000000018002b1ec     DmfK:Dmf_DeviceInterfaceTarget.obj
 0002:0000420c       $unwind$WPP_RECORDER_SF_S  000000018002b20c     DmfK:Dmf_DeviceInterfaceTarget.obj
 0002:00004228       $unwind$WPP_RECORDER_SF__guid_ 000000018002b228     DmfK:Dmf_DeviceInterfaceTarget.obj
 0002:00004244       $unwind$?DeviceInterfaceTarget_SendCompletion@@YAXPEAUDMFMODULE__@@PEAX1_K12J@Z 000000018002b244     DmfK:Dmf_DeviceInterfaceTarget.obj
 0002:00004260       $unwind$?DeviceInterfaceTarget_SymbolicLinkNameStore@@YAJPEAUDMFMODULE__@@PEAU_UNICODE_STRING@@@Z 000000018002b260     DmfK:Dmf_DeviceInterfaceTarget.obj
 0002:00004280       $unwind$?DeviceInterfaceTarget_Stream_SendSynchronously@@YAJPEAUDMFMODULE__@@PEAX_K12W4ContinuousRequestTarget_RequestType@@KKPEA_K@Z 000000018002b280     DmfK:Dmf_DeviceInterfaceTarget.obj
 0002:00004280       $unwind$?DeviceInterfaceTarget_Target_SendSynchronously@@YAJPEAUDMFMODULE__@@PEAX_K12W4ContinuousRequestTarget_RequestType@@KKPEA_K@Z 000000018002b280     DmfK:Dmf_DeviceInterfaceTarget.obj
 0002:00004294       $unwind$?DeviceInterfaceTarget_Stream_SendEx@@YAJPEAUDMFMODULE__@@PEAX_K12W4ContinuousRequestTarget_RequestType@@KKP6AX011212J@Z1PEAPEAURequestTarget_DmfRequest__@@@Z 000000018002b294     DmfK:Dmf_DeviceInterfaceTarget.obj
 0002:00004294       $unwind$?DeviceInterfaceTarget_Target_SendEx@@YAJPEAUDMFMODULE__@@PEAX_K12W4ContinuousRequestTarget_RequestType@@KKP6AX011212J@Z1PEAPEAURequestTarget_DmfRequest__@@@Z 000000018002b294     DmfK:Dmf_DeviceInterfaceTarget.obj
 0002:000042b0       $unwind$?DeviceInterfaceTarget_Stream_Send@@YAJPEAUDMFMODULE__@@PEAX_K12W4ContinuousRequestTarget_RequestType@@KKP6AX011212J@Z1@Z 000000018002b2b0     DmfK:Dmf_DeviceInterfaceTarget.obj
 0002:000042bc       $unwind$?DeviceInterfaceTarget_Stream_IoTargetClear@@YAXPEAUDMFMODULE__@@@Z 000000018002b2bc     DmfK:Dmf_DeviceInterfaceTarget.obj
 0002:000042bc       $unwind$?DeviceInterfaceTarget_Target_IoTargetClear@@YAXPEAUDMFMODULE__@@@Z 000000018002b2bc     DmfK:Dmf_DeviceInterfaceTarget.obj
 0002:000042c8       $unwind$?DeviceInterfaceTarget_Target_Send@@YAJPEAUDMFMODULE__@@PEAX_K12W4ContinuousRequestTarget_RequestType@@KKP6AX011212J@Z1@Z 000000018002b2c8     DmfK:Dmf_DeviceInterfaceTarget.obj
 0002:000042e0       $unwind$?DeviceInterfaceTarget_Stream_BufferOutput@@YA?AW4ContinuousRequestTarget_BufferDisposition@@PEAUDMFMODULE__@@PEAX_K1J@Z 000000018002b2e0     DmfK:Dmf_DeviceInterfaceTarget.obj
 0002:000042e0       $unwind$?IoctlHandler_DeviceInterfaceCreate@@YAJPEAUDMFMODULE__@@@Z 000000018002b2e0     DmfK:Dmf_IoctlHandler.obj
 0002:00004300       $unwind$?DeviceInterfaceTarget_EvtIoTargetQueryRemove@@YAJPEAUWDFIOTARGET__@@@Z 000000018002b300     DmfK:Dmf_DeviceInterfaceTarget.obj
 0002:0000431c       $unwind$?DeviceInterfaceTarget_EvtIoTargetRemoveCancel@@YAXPEAUWDFIOTARGET__@@@Z 000000018002b31c     DmfK:Dmf_DeviceInterfaceTarget.obj
 0002:00004340       $unwind$?DeviceInterfaceTarget_DeviceCreateNewIoTargetByName@@YAJPEAUDMFMODULE__@@PEAU_UNICODE_STRING@@@Z 000000018002b340     DmfK:Dmf_DeviceInterfaceTarget.obj
 0002:00004364       $unwind$?DeviceInterfaceTarget_InterfaceArrivalRemovalCallback@@YAJPEAX0@Z 000000018002b364     DmfK:Dmf_DeviceInterfaceTarget.obj
 0002:00004384       $unwind$?DMF_DeviceInterfaceTarget_NotificationRegister@@YAJPEAUDMFMODULE__@@@Z 000000018002b384     DmfK:Dmf_DeviceInterfaceTarget.obj
 0002:000043a0       $unwind$?DMF_DeviceInterfaceTarget_NotificationUnregister@@YAXPEAUDMFMODULE__@@@Z 000000018002b3a0     DmfK:Dmf_DeviceInterfaceTarget.obj
 0002:000043bc       $unwind$?DMF_DeviceInterfaceTarget_Close@@YAXPEAUDMFMODULE__@@@Z 000000018002b3bc     DmfK:Dmf_DeviceInterfaceTarget.obj
 0002:000043d8       $unwind$?DMF_DeviceInterfaceTarget_ChildModulesAdd@@YAXPEAUDMFMODULE__@@PEAU_DMF_MODULE_ATTRIBUTES@@PEAX@Z 000000018002b3d8     DmfK:Dmf_DeviceInterfaceTarget.obj
 0002:00004400       $unwind$DMF_String_Create  000000018002b400     DmfK:Dmf_String.obj
 0002:00004420       $unwind$WPP_RECORDER_SF_Dss 000000018002b420     DmfK:Dmf_String.obj
 0002:0000443c       $unwind$?String_FindInListLeftLookForMatchCharCallback@@YAJPEAUDMFMODULE__@@PEAD1@Z 000000018002b43c     DmfK:Dmf_String.obj
 0002:00004448       $unwind$DMF_SmbiosWmi_Create 000000018002b448     DmfK:Dmf_SmbiosWmi.obj
 0002:00004468       $unwind$WPP_RECORDER_SF_DDDDDDDDDDDDDDDD 000000018002b468     DmfK:Dmf_SmbiosWmi.obj
 0002:0000448c       $unwind$?SmbioWmi_TablesSet@@YAJPEAUDMFMODULE__@@@Z 000000018002b48c     DmfK:Dmf_SmbiosWmi.obj
 0002:000044a8       $unwind$?SmbiosWmi_Read@@YAJPEAUDMFMODULE__@@@Z 000000018002b4a8     DmfK:Dmf_SmbiosWmi.obj
 0002:000044d4       $unwind$DMF_File_FileExists 000000018002b4d4     DmfK:Dmf_File.obj
 0002:000044f0       $unwind$DMF_File_Read      000000018002b4f0     DmfK:Dmf_File.obj
 0002:00004518       $unwind$WPP_RECORDER_SF_Sd 000000018002b518     DmfK:Dmf_File.obj
 0002:00004534       $unwind$DMF_BufferQueue_Flush 000000018002b534     DmfK:Dmf_BufferQueue.obj
 0002:0000454c       $unwind$DMF_BufferQueue_Reuse 000000018002b54c     DmfK:Dmf_BufferQueue.obj
 0002:00004568       $unwind$?DMF_BufferQueue_ChildModulesAdd@@YAXPEAUDMFMODULE__@@PEAU_DMF_MODULE_ATTRIBUTES@@PEAX@Z 000000018002b568     DmfK:Dmf_BufferQueue.obj
 0002:0000458c       $unwind$DmfContainerEvtDeviceArmWakeFromS0 000000018002b58c     DmfK:DmfContainer.obj
 0002:0000458c       $unwind$DmfContainerEvtDeviceDisarmWakeFromS0 000000018002b58c     DmfK:DmfContainer.obj
 0002:0000458c       $unwind$DmfContainerEvtDeviceDisarmWakeFromSx 000000018002b58c     DmfK:DmfContainer.obj
 0002:0000458c       $unwind$DmfContainerEvtDeviceQueryRemove 000000018002b58c     DmfK:DmfContainer.obj
 0002:0000458c       $unwind$DmfContainerEvtDeviceQueryStop 000000018002b58c     DmfK:DmfContainer.obj
 0002:0000458c       $unwind$DmfContainerEvtDeviceSelfManagedIoCleanup 000000018002b58c     DmfK:DmfContainer.obj
 0002:0000458c       $unwind$DmfContainerEvtDeviceSelfManagedIoFlush 000000018002b58c     DmfK:DmfContainer.obj
 0002:0000458c       $unwind$DmfContainerEvtDeviceSelfManagedIoInit 000000018002b58c     DmfK:DmfContainer.obj
 0002:0000458c       $unwind$DmfContainerEvtDeviceSelfManagedIoRestart 000000018002b58c     DmfK:DmfContainer.obj
 0002:0000458c       $unwind$DmfContainerEvtDeviceSelfManagedIoSuspend 000000018002b58c     DmfK:DmfContainer.obj
 0002:0000458c       $unwind$DmfContainerEvtDeviceSurpriseRemoval 000000018002b58c     DmfK:DmfContainer.obj
 0002:0000458c       $unwind$DmfContainerEvtDeviceWakeFromS0Triggered 000000018002b58c     DmfK:DmfContainer.obj
 0002:0000458c       $unwind$DmfContainerEvtDeviceWakeFromSxTriggered 000000018002b58c     DmfK:DmfContainer.obj
 0002:0000458c       $unwind$?DMF_BufferQueue_Close@@YAXPEAUDMFMODULE__@@@Z 000000018002b58c     DmfK:Dmf_BufferQueue.obj
 0002:0000458c       $unwind$?DMF_CrashDump_SurpriseRemoval@@YAXPEAUDMFMODULE__@@@Z 000000018002b58c     DmfK:Dmf_CrashDump.obj
 0002:0000458c       $unwind$?DMF_HashTable_Close@@YAXPEAUDMFMODULE__@@@Z 000000018002b58c     DmfK:Dmf_HashTable.obj
 0002:0000458c       $unwind$?DMF_HashTable_Open@@YAJPEAUDMFMODULE__@@@Z 000000018002b58c     DmfK:Dmf_HashTable.obj
 0002:000045a0       $unwind$DMF_ScheduledTask_TimesRunSet 000000018002b5a0     DmfK:Dmf_ScheduledTask.obj
 0002:000045b8       $unwind$DMF_Invoke_DeviceCallbacksDestroy 000000018002b5b8     DmfK:DmfContainer.obj
 0002:000045b8       $unwind$?ContinuousRequestTarget_PendingCollectionListSearchAndReference@@YAEPEAUDMFMODULE__@@PEAURequestTarget_DmfRequest__@@PEAPEAUWDFREQUEST__@@@Z 000000018002b5b8     DmfK:Dmf_ContinuousRequestTarget.obj
 0002:000045b8       $unwind$?DMF_CrashDump_Close@@YAXPEAUDMFMODULE__@@@Z 000000018002b5b8     DmfK:Dmf_CrashDump.obj
 0002:000045b8       $unwind$DMF_RequestTarget_Cancel 000000018002b5b8     DmfK:Dmf_RequestTarget.obj
 0002:000045b8       $unwind$?DMF_ScheduledTask_ModuleD0Entry@@YAJPEAUDMFMODULE__@@W4_WDF_POWER_DEVICE_STATE@@@Z 000000018002b5b8     DmfK:Dmf_ScheduledTask.obj
 0002:000045b8       $unwind$?DMF_ScheduledTask_ModulePrepareHardware@@YAJPEAUDMFMODULE__@@PEAUWDFCMRESLIST__@@1@Z 000000018002b5b8     DmfK:Dmf_ScheduledTask.obj
 0002:000045b8       $unwind$?ScheduledTask_ClientWorkDo@@YA?AW4ScheduledTask_Result_Type@@PEAUDMFMODULE__@@PEAXW4_WDF_POWER_DEVICE_STATE@@@Z 000000018002b5b8     DmfK:Dmf_ScheduledTask.obj
 0002:000045d8       $unwind$DmfContainerEvtFileClose 000000018002b5d8     DmfK:DmfContainer.obj
 0002:000045d8       $unwind$?ScheduledTask_TimerHandler@@YAXPEAUWDFTIMER__@@@Z 000000018002b5d8     DmfK:Dmf_ScheduledTask.obj
 0002:000045f0       $unwind$?DMF_ScheduledTask_ModuleD0Exit@@YAJPEAUDMFMODULE__@@W4_WDF_POWER_DEVICE_STATE@@@Z 000000018002b5f0     DmfK:Dmf_ScheduledTask.obj
 0002:000045f0       $unwind$?DMF_ScheduledTask_ModuleReleaseHardware@@YAJPEAUDMFMODULE__@@PEAUWDFCMRESLIST__@@@Z 000000018002b5f0     DmfK:Dmf_ScheduledTask.obj
 0002:00004608       $unwind$?DMF_ScheduledTask_ChildModulesAdd@@YAXPEAUDMFMODULE__@@PEAU_DMF_MODULE_ATTRIBUTES@@PEAX@Z 000000018002b608     DmfK:Dmf_ScheduledTask.obj
 0002:00004624       $unwind$DmfContainerEvtQueueIoRead 000000018002b624     DmfK:DmfContainer.obj
 0002:00004624       $unwind$DmfContainerEvtQueueIoWrite 000000018002b624     DmfK:DmfContainer.obj
 0002:00004640       $unwind$DmfContainerEvtDeviceIoControl 000000018002b640     DmfK:DmfContainer.obj
 0002:00004640       $unwind$DmfContainerEvtInternalDeviceIoControl 000000018002b640     DmfK:DmfContainer.obj
 0002:00004660       $unwind$DmfContainerEvtFileCreate 000000018002b660     DmfK:DmfContainer.obj
 0002:00004660       $unwind$?ContinuousRequestTarget_CompletionRoutine@@YAXPEAUWDFREQUEST__@@PEAUWDFIOTARGET__@@PEAU_WDF_REQUEST_COMPLETION_PARAMS@@PEAX@Z 000000018002b660     DmfK:Dmf_ContinuousRequestTarget.obj
 0002:0000467c       $unwind$DMF_Bridge_Create  000000018002b67c     DmfK:Dmf_Bridge.obj
 0002:0000469c       $unwind$?DMF_ModuleBranchTrack_HasClientEnabledBranchTrack@@YAKPEAUWDFDEVICE__@@@Z 000000018002b69c     DmfK:DmfBranchTrack.obj
 0002:000046bc       $unwind$?DMF_ModuleLiveKernelDump_ModuleCollectionInitialize@@YAXPEAU_DMF_MODULE_COLLECTION_@@@Z 000000018002b6bc     DmfK:DmfLiveKernelDump.obj
 0002:000046d8       $unwind$?DMF_LiveKernelDump_ModuleInitialize@@YAXPEAU_DMF_OBJECT_@@@Z 000000018002b6d8     DmfK:DmfLiveKernelDump.obj
 0002:000046f4       $unwind$?EVT_DMF_MODULE_Generic_OnDeviceNotificationPostOpen@@YAXPEAUDMFMODULE__@@@Z 000000018002b6f4     DmfK:DmfGeneric.obj
 0002:000046f4       $unwind$?EVT_DMF_MODULE_Generic_OnDeviceNotificationPreClose@@YAXPEAUDMFMODULE__@@@Z 000000018002b6f4     DmfK:DmfGeneric.obj
 0002:0000470c       $unwind$?DMF_Generic_ModuleD0EntryPostInterruptsEnabled@@YAJPEAUDMFMODULE__@@W4_WDF_POWER_DEVICE_STATE@@@Z 000000018002b70c     DmfK:DmfGeneric.obj
 0002:00004728       $unwind$?DMF_Generic_ModuleD0Exit@@YAJPEAUDMFMODULE__@@W4_WDF_POWER_DEVICE_STATE@@@Z 000000018002b728     DmfK:DmfGeneric.obj
 0002:00004748       $unwind$?DMF_Generic_ModuleDeviceIoControl@@YAEPEAUDMFMODULE__@@PEAUWDFQUEUE__@@PEAUWDFREQUEST__@@_K3K@Z 000000018002b748     DmfK:DmfGeneric.obj
 0002:00004760       $unwind$?DMF_Generic_ResourcesAssign@@YAJPEAUDMFMODULE__@@PEAUWDFCMRESLIST__@@1@Z 000000018002b760     DmfK:DmfGeneric.obj
 0002:0000477c       $unwind$?DMF_Generic_NotificationRegister@@YAJPEAUDMFMODULE__@@@Z 000000018002b77c     DmfK:DmfGeneric.obj
 0002:00004798       $unwind$WPP_RECORDER_SF_qqsd 000000018002b798     DmfK:DmfGeneric.obj
 0002:000047b8       $unwind$?IoctlHandler_RequestForward@@YAJPEAUDMFMODULE__@@PEAUWDFREQUEST__@@@Z 000000018002b7b8     DmfK:Dmf_IoctlHandler.obj
 0002:000047d4       $unwind$?IoctlHandler_AssociatedFileObjectsLookUp@@YAEPEAUDMFMODULE__@@PEAUWDFFILEOBJECT__@@E@Z 000000018002b7d4     DmfK:Dmf_IoctlHandler.obj
 0002:000047f4       $unwind$?DMF_IoctlHandler_ModuleDeviceIoControl@@YAEPEAUDMFMODULE__@@PEAUWDFQUEUE__@@PEAUWDFREQUEST__@@_K3K@Z 000000018002b7f4     DmfK:Dmf_IoctlHandler.obj
 0002:00004818       $unwind$?DMF_IoctlHandler_FileCreate@@YAEPEAUDMFMODULE__@@PEAUWDFDEVICE__@@PEAUWDFREQUEST__@@PEAUWDFFILEOBJECT__@@@Z 000000018002b818     DmfK:Dmf_IoctlHandler.obj
 0002:0000483c       $unwind$?DMF_IoctlHandler_Open@@YAJPEAUDMFMODULE__@@@Z 000000018002b83c     DmfK:Dmf_IoctlHandler.obj
 0002:00004864       $unwind$LkmdTelpWriteDumpFile 000000018002b864     DmfK:lkmdtel.obj
 0002:0000487c       $unwind$LkmdTelInsertTriageDataBlock 000000018002b87c     DmfK:lkmdtel.obj
 0002:0000487c       $unwind$LkmdTelSetSecondaryData 000000018002b87c     DmfK:lkmdtel.obj
 0002:0000487c       $unwind$RtlStringVPrintfWorkerW 000000018002b87c     DmfK:lkmdtel.obj
 0002:00004898       $unwind$LkmdTelpSetMaxSize 000000018002b898     DmfK:lkmdtel.obj
 0002:000048a4       $unwind$LkmdTelpGetRegistryUlongValue 000000018002b8a4     DmfK:lkmdtel.obj
 0002:000048bc       $unwind$LkmdTelpGetRegistryKey 000000018002b8bc     DmfK:lkmdtel.obj
 0002:000048d8       $unwind$LkmdTelCreateReport 000000018002b8d8     DmfK:lkmdtel.obj
 0002:000048fc       $unwind$LkmdTelCloseHandle 000000018002b8fc     DmfK:lkmdtel.obj
 0002:00004908       $unwind$RtlStringCbPrintfW 000000018002b908     DmfK:lkmdtel.obj
 0002:00004914       $unwind$DMF_Utility_DelayMilliseconds 000000018002b914     DmfK:DmfUtility.obj
 0002:00004928       $unwind$DMF_RingBuffer_ReadAll 000000018002b928     DmfK:Dmf_RingBuffer.obj
 0002:00004928       $unwind$DMF_RingBuffer_Reorder 000000018002b928     DmfK:Dmf_RingBuffer.obj
 0002:00004944       $unwind$?DMF_RingBuffer_Open@@YAJPEAUDMFMODULE__@@@Z 000000018002b944     DmfK:Dmf_RingBuffer.obj
 0002:00004964       $unwind$DMF_CrashDump_TriageDumpDataAdd 000000018002b964     DmfK:Dmf_CrashDump.obj
 0002:00004988       $unwind$?CrashDump_BugCheckSecondaryDumpDataCallbackAdditional@@YAXW4_KBUGCHECK_CALLBACK_REASON@@PEAU_KBUGCHECK_REASON_CALLBACK_RECORD@@PEAXK@Z 000000018002b988     DmfK:Dmf_CrashDump.obj
 0002:00004994       $unwind$?CrashDump_DataSourceCaptureInternal@@YAJPEAUDMFMODULE__@@KPEAEKPEAK@Z 000000018002b994     DmfK:Dmf_CrashDump.obj
 0002:00004994       $unwind$?CrashDump_DataSourceOrphanCreate@@YAXPEAUDMFMODULE__@@PEAUWDFFILEOBJECT__@@@Z 000000018002b994     DmfK:Dmf_CrashDump.obj
 0002:00004994       $unwind$?CrashDump_DataSourceReadInternal@@YAJPEAUDMFMODULE__@@KPEAEK@Z 000000018002b994     DmfK:Dmf_CrashDump.obj
 0002:00004994       $unwind$?CrashDump_DataSourceWriteInternal@@YAJPEAUDMFMODULE__@@KPEAEK@Z 000000018002b994     DmfK:Dmf_CrashDump.obj
 0002:000049a8       $unwind$?CrashDump_DmfCreate_RingBuffer@@YAJPEAUDMFMODULE__@@KKK@Z 000000018002b9a8     DmfK:Dmf_CrashDump.obj
 0002:000049d0       $unwind$?CrashDump_DataSourceCreateInternal@@YAJPEAUDMFMODULE__@@KKKPEBU_GUID@@@Z 000000018002b9d0     DmfK:Dmf_CrashDump.obj
 0002:000049f0       $unwind$?ContinuousRequestTarget_QueuedWorkitemCallbackStream@@YA?AW4ScheduledTask_Result_Type@@PEAUDMFMODULE__@@PEAX1@Z 000000018002b9f0     DmfK:Dmf_ContinuousRequestTarget.obj
 0002:000049f0       $unwind$?CrashDump_DataSourceDestroyAuxiliaryInternal@@YAJPEAUDMFMODULE__@@PEAUWDFFILEOBJECT__@@@Z 000000018002b9f0     DmfK:Dmf_CrashDump.obj
 0002:000049f0       $unwind$?CrashDump_DataSourceDestroyInternal@@YAJPEAUDMFMODULE__@@K@Z 000000018002b9f0     DmfK:Dmf_CrashDump.obj
 0002:000049f0       $unwind$?HashTable_DataEntryAllocate@@YAJPEAUDMFMODULE__@@PEAU_DMF_CONTEXT_HashTable@@PEAEKPEAK@Z 000000018002b9f0     DmfK:Dmf_HashTable.obj
 0002:00004a00       $unwind$?CrashDump_DataSourceCreateAuxiliary@@YAJPEAUDMFMODULE__@@PEAUWDFFILEOBJECT__@@KKPEBU_GUID@@@Z 000000018002ba00     DmfK:Dmf_CrashDump.obj
 0002:00004a24       $unwind$?CrashDump_DataSourceOpenAuxiliary@@YAJPEAUDMFMODULE__@@PEAUWDFFILEOBJECT__@@PEAKPEBU_GUID@@@Z 000000018002ba24     DmfK:Dmf_CrashDump.obj
 0002:00004a48       $unwind$?CrashDump_TriageDataCreateInternal@@YAJPEAUDMFMODULE__@@@Z 000000018002ba48     DmfK:Dmf_CrashDump.obj
 0002:00004a74       $unwind$?CrashDump_DataSourceReadAuxiliary@@YAJPEAUDMFMODULE__@@PEAUWDFFILEOBJECT__@@PEAEK@Z 000000018002ba74     DmfK:Dmf_CrashDump.obj
 0002:00004a74       $unwind$?CrashDump_DataSourceWriteAuxiliary@@YAJPEAUDMFMODULE__@@PEAUWDFFILEOBJECT__@@PEAEK@Z 000000018002ba74     DmfK:Dmf_CrashDump.obj
 0002:00004a90       $unwind$?CrashDump_DataSourceCreateFromRequest@@YAJPEAUDMFMODULE__@@PEAUWDFREQUEST__@@PEA_K@Z 000000018002ba90     DmfK:Dmf_CrashDump.obj
 0002:00004aa4       $unwind$?CrashDump_DataSourceOpenFromRequest@@YAJPEAUDMFMODULE__@@PEAUWDFREQUEST__@@PEA_K@Z 000000018002baa4     DmfK:Dmf_CrashDump.obj
 0002:00004ac0       $unwind$?CrashDump_DataSourceReadFromRequest@@YAJPEAUDMFMODULE__@@PEAUWDFREQUEST__@@PEA_K@Z 000000018002bac0     DmfK:Dmf_CrashDump.obj
 0002:00004ac0       $unwind$?CrashDump_DataSourceWriteFromRequest@@YAJPEAUDMFMODULE__@@PEAUWDFREQUEST__@@PEA_K@Z 000000018002bac0     DmfK:Dmf_CrashDump.obj
 0002:00004ad4       $unwind$?CrashDump_DataSourceCaptureFromRequest@@YAJPEAUDMFMODULE__@@PEAUWDFREQUEST__@@PEA_K@Z 000000018002bad4     DmfK:Dmf_CrashDump.obj
 0002:00004ae8       $unwind$?DMF_CrashDump_Open@@YAJPEAUDMFMODULE__@@@Z 000000018002bae8     DmfK:Dmf_CrashDump.obj
 0002:00004b08       $unwind$?DMF_CrashDump_ChildModulesAdd@@YAXPEAUDMFMODULE__@@PEAU_DMF_MODULE_ATTRIBUTES@@PEAX@Z 000000018002bb08     DmfK:Dmf_CrashDump.obj
 0002:00004b2c       $unwind$?DMF_Internal_Open@@YAJPEAUDMFMODULE__@@@Z 000000018002bb2c     DmfK:DmfInternal.obj
 0002:00004b4c       $unwind$?DMF_ModuleInterfacesUnbind@@YAXPEAUDMFMODULE__@@@Z 000000018002bb4c     DmfK:DmfInterfaceInternal.obj
 0002:00004b4c       $unwind$?DMF_ModuleIsClosed@@YAEPEAUDMFMODULE__@@@Z 000000018002bb4c     DmfK:DmfInternal.obj
 0002:00004b60       $unwind$DMF_ModuleInterfaceUnbind 000000018002bb60     DmfK:DmfInterfaceInternal.obj
 0002:00004b78       $unwind$?DMF_ModuleInterfaceDestroy@@YAXPEAU_DMF_INTERFACE_OBJECT@@@Z 000000018002bb78     DmfK:DmfInterfaceInternal.obj
 0002:00004b88       $unwind$?DMF_ModuleInterfaceWaitToClose@@YAXPEAU_DMF_INTERFACE_OBJECT@@@Z 000000018002bb88     DmfK:DmfInterfaceInternal.obj
 0002:00004ba0       $unwind$?HashTable_ContextInitialize@@YAJPEAUDMFMODULE__@@@Z 000000018002bba0     DmfK:Dmf_HashTable.obj
 0002:00004bc4       $unwind$DMF_ContinuousRequestTarget_SendSynchronously 000000018002bbc4     DmfK:Dmf_ContinuousRequestTarget.obj
 0002:00004bc4       $unwind$DMF_RequestTarget_SendEx 000000018002bbc4     DmfK:Dmf_RequestTarget.obj
 0002:00004be4       $unwind$DMF_RequestTarget_SendSynchronously 000000018002bbe4     DmfK:Dmf_RequestTarget.obj
 0002:00004c04       $unwind$?ContinuousRequestTarget_ProcessAsynchronousRequestSingle@@YAXPEAUDMFMODULE__@@PEAUWDFREQUEST__@@PEAU_WDF_REQUEST_COMPLETION_PARAMS@@PEAUContinuousRequestTarget_SingleAsynchronousRequestContext@@@Z 000000018002bc04     DmfK:Dmf_ContinuousRequestTarget.obj
 0002:00004c04       $unwind$?RequestTarget_ProcessAsynchronousRequestSingle@@YAXPEAUDMFMODULE__@@PEAUWDFREQUEST__@@PEAU_WDF_REQUEST_COMPLETION_PARAMS@@PEAURequestTarget_SingleAsynchronousRequestContext@@@Z 000000018002bc04     DmfK:Dmf_RequestTarget.obj
 0002:00004c20       $unwind$?RequestTarget_CompletionRoutinePassive@@YAXPEAUWDFREQUEST__@@PEAUWDFIOTARGET__@@PEAU_WDF_REQUEST_COMPLETION_PARAMS@@PEAX@Z 000000018002bc20     DmfK:Dmf_RequestTarget.obj
 0002:00004c40       $unwind$?ContinuousRequestTarget_RequestCreateAndSend@@YAJPEAUDMFMODULE__@@EPEAX_K12W4ContinuousRequestTarget_RequestType@@KKW4ContinuousRequestTarget_CompletionOptions@@PEA_KP6AX011212J@Z1PEAPEAURequestTarget_DmfRequest__@@@Z 000000018002bc40     DmfK:Dmf_ContinuousRequestTarget.obj
 0002:00004c40       $unwind$?RequestTarget_RequestCreateAndSend@@YAJPEAUDMFMODULE__@@EPEAX_K12W4ContinuousRequestTarget_RequestType@@KKW4ContinuousRequestTarget_CompletionOptions@@PEA_KP6AX011212J@Z1PEAPEAURequestTarget_DmfRequest__@@@Z 000000018002bc40     DmfK:Dmf_RequestTarget.obj
 0002:00004c68       $unwind$?DMF_RequestTarget_ChildModulesAdd@@YAXPEAUDMFMODULE__@@PEAU_DMF_MODULE_ATTRIBUTES@@PEAX@Z 000000018002bc68     DmfK:Dmf_RequestTarget.obj
 0002:00004c8c       $unwind$?DMF_RequestTarget_Open@@YAJPEAUDMFMODULE__@@@Z 000000018002bc8c     DmfK:Dmf_RequestTarget.obj
 0002:00004ca0       $unwind$DMF_ContinuousRequestTarget_SendEx 000000018002bca0     DmfK:Dmf_ContinuousRequestTarget.obj
 0002:00004cc0       $unwind$?ContinuousRequestTarget_CompletionRoutinePassive@@YAXPEAUWDFREQUEST__@@PEAUWDFIOTARGET__@@PEAU_WDF_REQUEST_COMPLETION_PARAMS@@PEAX@Z 000000018002bcc0     DmfK:Dmf_ContinuousRequestTarget.obj
 0002:00004ce0       $unwind$?ContinuousRequestTarget_StreamRequestSend@@YAJPEAUDMFMODULE__@@PEAUWDFREQUEST__@@@Z 000000018002bce0     DmfK:Dmf_ContinuousRequestTarget.obj
 0002:00004d00       $unwind$?ContinuousRequestTarget_ProcessAsynchronousRequestStream@@YAXPEAUDMFMODULE__@@PEAUWDFREQUEST__@@PEAU_WDF_REQUEST_COMPLETION_PARAMS@@@Z 000000018002bd00     DmfK:Dmf_ContinuousRequestTarget.obj
 0002:00004d20       $unwind$?ContinuousRequestTarget_StreamCompletionRoutinePassive@@YAXPEAUWDFREQUEST__@@PEAUWDFIOTARGET__@@PEAU_WDF_REQUEST_COMPLETION_PARAMS@@PEAX@Z 000000018002bd20     DmfK:Dmf_ContinuousRequestTarget.obj
 0002:00004d38       $unwind$?ContinuousRequestTarget_StopAndWait@@YAXPEAUDMFMODULE__@@@Z 000000018002bd38     DmfK:Dmf_ContinuousRequestTarget.obj
 0002:00004d54       $unwind$?DMF_ContinuousRequestTarget_ChildModulesAdd@@YAXPEAUDMFMODULE__@@PEAU_DMF_MODULE_ATTRIBUTES@@PEAX@Z 000000018002bd54     DmfK:Dmf_ContinuousRequestTarget.obj
 0002:00004d7c       $unwind$?DMF_ContinuousRequestTarget_Open@@YAJPEAUDMFMODULE__@@@Z 000000018002bd7c     DmfK:Dmf_ContinuousRequestTarget.obj
 0002:00004da0       $unwind$DMF_Rundown_EndAndWait 000000018002bda0     DmfK:Dmf_Rundown.obj
 0003:00000000       _ZN20surface_hid_mini_lib39WDF_DRIVER_CONTEXT_TYPE_INFO_FIXED_SIZE17h2721a098ded43cd5E 000000018002c000     surface_hid_mini.surface_hid_mini.3efcb60154bd7459-cgu.0.rcgu.o
 0003:00000028       _ZN20surface_hid_mini_lib39WDF_DEVICE_CONTEXT_TYPE_INFO_FIXED_SIZE17h444be84c7413bebeE 000000018002c028     surface_hid_mini.surface_hid_mini.3efcb60154bd7459-cgu.0.rcgu.o
 0003:00000050       _ZN20surface_hid_mini_lib24SURFACE_HIDMINI_PROVIDER17hc9ffeec2aad7c9a4E 000000018002c050     surface_hid_mini.surface_hid_mini.3efcb60154bd7459-cgu.0.rcgu.o
 0003:000000a0       _ZN20surface_hid_mini_lib34SURFACE_HIDMINI_TELEMETRY_PROVIDER17h5b5d2603e4fc5bf6E 000000018002c0a0     surface_hid_mini.surface_hid_mini.3efcb60154bd7459-cgu.0.rcgu.o
 0003:000009b0       ?DmfModuleDescriptor_Generic@@3UDMF_MODULE_DESCRIPTOR@@A 000000018002c9b0     DmfK:DmfCore.obj
 0003:00000d78       ?__KMDF_CLASS_BIND_LAST_BOUND@@3PEAU_WDF_CLASS_BIND_INFO@@EA 000000018002cd78     WdfDriverEntry:classbind.obj
 0003:00000da0       _ZN76_$LT$wdk_sys..wdf..WDF_FUNCTION_TABLE$u20$as$u20$core..ops..deref..Deref$GT$5deref11__stability4LAZY17h228b5f2ccbb3549dE 000000018002cda0     surface_hid_mini.surface_hid_mini.3efcb60154bd7459-cgu.0.rcgu.o
 0003:00000dc0       WdfDriverStubRegistryPathBuffer 000000018002cdc0     WdfDriverEntry:stub.obj
 0003:00000fd8       WdfDriverStubRegistryPath  000000018002cfd8     WdfDriverEntry:stub.obj
 0003:00000ff8       WdfDriverStubDriverObject  000000018002cff8     WdfDriverEntry:stub.obj
 0003:00001000       WdfDriverStubDisplacedDriverUnload 000000018002d000     WdfDriverEntry:stub.obj
 0003:00001038       ?internalExAllocatePool2@?1??DMF_GenericMemoryAllocate@@YAPEAX_K0K@Z@4P6APEAX00K@ZEA 000000018002d038     DmfK:DmfHelpers.obj
 0003:00001040       ?internalExAllocatePoolWithTag@?1??DMF_GenericMemoryAllocate@@YAPEAX_K0K@Z@4P6APEAXW4_POOL_TYPE@@0K@ZEA 000000018002d040     DmfK:DmfHelpers.obj
 0003:00001144       ?numberOfDataBuffers@?1??LiveKernelDump_InsertDataBufferInLiveDump@@YAEPEAUDMFMODULE__@@PEAEKPEAX@Z@4KA 000000018002d144     DmfK:Dmf_LiveKernelDump.obj
 0003:00001148       ?telemetryDataSize@?1??LiveKernelDump_InsertDataBufferInLiveDump@@YAEPEAUDMFMODULE__@@PEAEKPEAX@Z@4KA 000000018002d148     DmfK:Dmf_LiveKernelDump.obj
 0005:00000000       _ZN20surface_hid_mini_lib18generic_hid_module11HidMiniport14get_descriptor17h4f5ccb44f9ba9516E 0000000180031000 f   surface_hid_mini.surface_hid_mini.3efcb60154bd7459-cgu.0.rcgu.o
 0005:000003e0       _ZN20surface_hid_mini_lib13dmf_interface22dmf_device_modules_add17h4556ec1b3649fb66E 00000001800313e0 f   surface_hid_mini.surface_hid_mini.3efcb60154bd7459-cgu.0.rcgu.o
 0005:000008c0       _ZN20surface_hid_mini_lib6device30surface_hid_mini_create_device17heaa3a2b63226fc26E 00000001800318c0 f   surface_hid_mini.surface_hid_mini.3efcb60154bd7459-cgu.0.rcgu.o
 0005:00002178       $LN60                      0000000180033178     libms_surface_wpp-b83efe80b23bd200:2e40c9e35e9506f4-wpp.o
 0005:000022a0       ?DMF_BufferPool_Close@@YAXPEAUDMFMODULE__@@@Z 00000001800332a0 f   DmfK:Dmf_BufferPool.obj
 0005:00002340       ?DMF_BufferPool_Open@@YAJPEAUDMFMODULE__@@@Z 0000000180033340 f   DmfK:Dmf_BufferPool.obj
 0005:00006480       ?SurfaceTelemetryConsentSettingsNotification_IoctlClientCallback_TelemetryConsentChanged@@YAJPEAUDMFMODULE__@@PEAUWDFQUEUE__@@PEAUWDFREQUEST__@@KPEAX_K34PEA_K@Z 0000000180037480 f   DmfK:Dmf_SurfaceTelemetryConsentSettingsNotification.obj
 0005:00007540       ?DMF_LiveKernelDump_Open@@YAJPEAUDMFMODULE__@@@Z 0000000180038540 f   DmfK:Dmf_LiveKernelDump.obj
 0005:00007ff0       ?DmfCallbacksWdfInitialize@@YAXPEAUDMF_CALLBACKS_WDF@@@Z 0000000180038ff0 f   DmfK:DmfCore.obj
 0005:00008164       ?DmfModuleCallbacksInitialize@@YAJPEAU_DMF_OBJECT_@@PEAU_DMF_MODULE_ATTRIBUTES@@PEAUDMF_MODULE_DESCRIPTOR@@@Z 0000000180039164 f   DmfK:DmfCore.obj
 0005:00008944       ?DmfModuleChildObjectsInitialize@@YAJPEAU_DMF_OBJECT_@@PEAUWDFMEMORY__@@PEAU_DMF_MODULE_ATTRIBUTES@@PEAUDMF_MODULE_DESCRIPTOR@@@Z 0000000180039944 f   DmfK:DmfCore.obj
 0005:00008a60       ?DmfModuleInFlightRecorderInitialize@@YAXPEAU_DMF_OBJECT_@@@Z 0000000180039a60 f   DmfK:DmfCore.obj
 0005:00008b88       ?DmfModuleInstanceNameInitialize@@YAJPEAU_DMF_OBJECT_@@PEAUWDFMEMORY__@@PEAU_DMF_MODULE_ATTRIBUTES@@@Z 0000000180039b88 f   DmfK:DmfCore.obj
 0005:00008c48       ?DmfModuleParentUpdate@@YAJPEAUWDFDEVICE__@@PEAXPEAU_DMF_OBJECT_@@PEAU_DMF_MODULE_ATTRIBUTES@@@Z 0000000180039c48 f   DmfK:DmfCore.obj
 0005:000098c0       ?DMF_BranchTrack_Close@@YAXPEAUDMFMODULE__@@@Z 000000018003a8c0 f   DmfK:Dmf_BranchTrack.obj
 0005:00009990       ?DMF_BranchTrack_Open@@YAJPEAUDMFMODULE__@@@Z 000000018003a990 f   DmfK:Dmf_BranchTrack.obj
 0005:0000a330       ?DMF_DeviceInterfaceTarget_Close@@YAXPEAUDMFMODULE__@@@Z 000000018003b330 f   DmfK:Dmf_DeviceInterfaceTarget.obj
 0005:0000a4e0       ?DMF_DeviceInterfaceTarget_NotificationRegister@@YAJPEAUDMFMODULE__@@@Z 000000018003b4e0 f   DmfK:Dmf_DeviceInterfaceTarget.obj
 0005:0000a620       ?DMF_DeviceInterfaceTarget_NotificationUnregister@@YAXPEAUDMFMODULE__@@@Z 000000018003b620 f   DmfK:Dmf_DeviceInterfaceTarget.obj
 0005:0000a7a0       ?DMF_DeviceInterfaceTarget_Open@@YAJPEAUDMFMODULE__@@@Z 000000018003b7a0 f   DmfK:Dmf_DeviceInterfaceTarget.obj
 0005:0000a898       ?DeviceInterfaceTarget_DeviceCreateNewIoTargetByName@@YAJPEAUDMFMODULE__@@PEAU_UNICODE_STRING@@@Z 000000018003b898 f   DmfK:Dmf_DeviceInterfaceTarget.obj
 0005:0000ab80       ?DeviceInterfaceTarget_InterfaceArrivalRemovalCallback@@YAJPEAX0@Z 000000018003bb80 f   DmfK:Dmf_DeviceInterfaceTarget.obj
 0005:0000af0c       ?DeviceInterfaceTarget_StreamStopAndModuleClose@@YAXPEAUDMFMODULE__@@@Z 000000018003bf0c f   DmfK:Dmf_DeviceInterfaceTarget.obj
 0005:0000b190       ?DMF_SmbiosWmi_Open@@YAJPEAUDMFMODULE__@@@Z 000000018003c190 f   DmfK:Dmf_SmbiosWmi.obj
 0005:0000bf40       ?DMF_BufferQueue_Close@@YAXPEAUDMFMODULE__@@@Z 000000018003cf40 f   DmfK:Dmf_BufferQueue.obj
 0005:0000c330       ?DMF_ScheduledTask_Close@@YAXPEAUDMFMODULE__@@@Z 000000018003d330 f   DmfK:Dmf_ScheduledTask.obj
 0005:0000c480       ?DMF_ScheduledTask_ModulePrepareHardware@@YAJPEAUDMFMODULE__@@PEAUWDFCMRESLIST__@@1@Z 000000018003d480 f   DmfK:Dmf_ScheduledTask.obj
 0005:0000c6b0       ?DMF_ScheduledTask_ModuleReleaseHardware@@YAJPEAUDMFMODULE__@@PEAUWDFCMRESLIST__@@@Z 000000018003d6b0 f   DmfK:Dmf_ScheduledTask.obj
 0005:0000c7e0       ?DMF_ScheduledTask_Open@@YAJPEAUDMFMODULE__@@@Z 000000018003d7e0 f   DmfK:Dmf_ScheduledTask.obj
 0005:0000f4e0       ?DMF_Bridge_Destroy@@YAXPEAUDMFMODULE__@@@Z 00000001800404e0 f   DmfK:Dmf_Bridge.obj
 0005:0000f590       ?DMF_Bridge_ModuleArmWakeFromS0@@YAJPEAUDMFMODULE__@@@Z 0000000180040590 f   DmfK:Dmf_Bridge.obj
 0005:0000f6c0       ?DMF_Bridge_ModuleArmWakeFromSxWithReason@@YAJPEAUDMFMODULE__@@EE@Z 00000001800406c0 f   DmfK:Dmf_Bridge.obj
 0005:0000f800       ?DMF_Bridge_ModuleDisarmWakeFromS0@@YAXPEAUDMFMODULE__@@@Z 0000000180040800 f   DmfK:Dmf_Bridge.obj
 0005:0000f8e0       ?DMF_Bridge_ModuleDisarmWakeFromSx@@YAXPEAUDMFMODULE__@@@Z 00000001800408e0 f   DmfK:Dmf_Bridge.obj
 0005:0000f9c0       ?DMF_Bridge_ModuleFileCleanup@@YAEPEAUDMFMODULE__@@PEAUWDFFILEOBJECT__@@@Z 00000001800409c0 f   DmfK:Dmf_Bridge.obj
 0005:0000fab0       ?DMF_Bridge_ModuleFileClose@@YAEPEAUDMFMODULE__@@PEAUWDFFILEOBJECT__@@@Z 0000000180040ab0 f   DmfK:Dmf_Bridge.obj
 0005:0000fba0       ?DMF_Bridge_ModuleFileCreate@@YAEPEAUDMFMODULE__@@PEAUWDFDEVICE__@@PEAUWDFREQUEST__@@PEAUWDFFILEOBJECT__@@@Z 0000000180040ba0 f   DmfK:Dmf_Bridge.obj
 0005:0000fcb0       ?DMF_Bridge_ModulePrepareHardware@@YAJPEAUDMFMODULE__@@PEAUWDFCMRESLIST__@@1@Z 0000000180040cb0 f   DmfK:Dmf_Bridge.obj
 0005:0000fdf0       ?DMF_Bridge_ModuleQueryRemove@@YAJPEAUDMFMODULE__@@@Z 0000000180040df0 f   DmfK:Dmf_Bridge.obj
 0005:0000ff20       ?DMF_Bridge_ModuleQueryStop@@YAJPEAUDMFMODULE__@@@Z 0000000180040f20 f   DmfK:Dmf_Bridge.obj
 0005:00010050       ?DMF_Bridge_ModuleRelationsQuery@@YAXPEAUDMFMODULE__@@W4_DEVICE_RELATION_TYPE@@@Z 0000000180041050 f   DmfK:Dmf_Bridge.obj
 0005:00010140       ?DMF_Bridge_ModuleReleaseHardware@@YAJPEAUDMFMODULE__@@PEAUWDFCMRESLIST__@@@Z 0000000180041140 f   DmfK:Dmf_Bridge.obj
 0005:00010270       ?DMF_Bridge_ModuleSelfManagedIoCleanup@@YAXPEAUDMFMODULE__@@@Z 0000000180041270 f   DmfK:Dmf_Bridge.obj
 0005:00010350       ?DMF_Bridge_ModuleSelfManagedIoFlush@@YAXPEAUDMFMODULE__@@@Z 0000000180041350 f   DmfK:Dmf_Bridge.obj
 0005:00010430       ?DMF_Bridge_ModuleSelfManagedIoInit@@YAJPEAUDMFMODULE__@@@Z 0000000180041430 f   DmfK:Dmf_Bridge.obj
 0005:00010560       ?DMF_Bridge_ModuleUsageNotificationEx@@YAJPEAUDMFMODULE__@@W4_WDF_SPECIAL_FILE_TYPE@@E@Z 0000000180041560 f   DmfK:Dmf_Bridge.obj
 0005:000106a0       ?DMF_Bridge_ModuleWakeFromS0Triggered@@YAXPEAUDMFMODULE__@@@Z 00000001800416a0 f   DmfK:Dmf_Bridge.obj
 0005:00010780       ?DMF_Bridge_ModuleWakeFromSxTriggered@@YAXPEAUDMFMODULE__@@@Z 0000000180041780 f   DmfK:Dmf_Bridge.obj
 0005:00010860       ?DMF_Bridge_Open@@YAJPEAUDMFMODULE__@@@Z 0000000180041860 f   DmfK:Dmf_Bridge.obj
 0005:00012f00       ?DMF_IoctlHandler_Close@@YAXPEAUDMFMODULE__@@@Z 0000000180043f00 f   DmfK:Dmf_IoctlHandler.obj
 0005:00012ff0       ?DMF_IoctlHandler_FileCleanup@@YAEPEAUDMFMODULE__@@PEAUWDFFILEOBJECT__@@@Z 0000000180043ff0 f   DmfK:Dmf_IoctlHandler.obj
 0005:00013210       ?DMF_IoctlHandler_FileClose@@YAEPEAUDMFMODULE__@@PEAUWDFFILEOBJECT__@@@Z 0000000180044210 f   DmfK:Dmf_IoctlHandler.obj
 0005:000132d0       ?DMF_IoctlHandler_FileCreate@@YAEPEAUDMFMODULE__@@PEAUWDFDEVICE__@@PEAUWDFREQUEST__@@PEAUWDFFILEOBJECT__@@@Z 00000001800442d0 f   DmfK:Dmf_IoctlHandler.obj
 0005:00013970       ?DMF_IoctlHandler_Open@@YAJPEAUDMFMODULE__@@@Z 0000000180044970 f   DmfK:Dmf_IoctlHandler.obj
 0005:00014880       ?DMF_RingBuffer_Close@@YAXPEAUDMFMODULE__@@@Z 0000000180045880 f   DmfK:Dmf_RingBuffer.obj
 0005:000148e0       ?DMF_RingBuffer_Open@@YAJPEAUDMFMODULE__@@@Z 00000001800458e0 f   DmfK:Dmf_RingBuffer.obj
 0005:00014fac       ?CrashDump_DataSourceCaptureFromRequest@@YAJPEAUDMFMODULE__@@PEAUWDFREQUEST__@@PEA_K@Z 0000000180045fac f   DmfK:Dmf_CrashDump.obj
 0005:00015390       ?CrashDump_DataSourceCreateFromRequest@@YAJPEAUDMFMODULE__@@PEAUWDFREQUEST__@@PEA_K@Z 0000000180046390 f   DmfK:Dmf_CrashDump.obj
 0005:0001548c       ?CrashDump_DataSourceCreateInternal@@YAJPEAUDMFMODULE__@@KKKPEBU_GUID@@@Z 000000018004648c f   DmfK:Dmf_CrashDump.obj
 0005:00015988       ?CrashDump_DataSourceDestroyInternal@@YAJPEAUDMFMODULE__@@K@Z 0000000180046988 f   DmfK:Dmf_CrashDump.obj
 0005:00015cfc       ?CrashDump_DataSourceOpenFromRequest@@YAJPEAUDMFMODULE__@@PEAUWDFREQUEST__@@PEA_K@Z 0000000180046cfc f   DmfK:Dmf_CrashDump.obj
 0005:000161d4       ?CrashDump_DataSourceReadFromRequest@@YAJPEAUDMFMODULE__@@PEAUWDFREQUEST__@@PEA_K@Z 00000001800471d4 f   DmfK:Dmf_CrashDump.obj
 0005:00016454       ?CrashDump_DataSourceWriteFromRequest@@YAJPEAUDMFMODULE__@@PEAUWDFREQUEST__@@PEA_K@Z 0000000180047454 f   DmfK:Dmf_CrashDump.obj
 0005:00016518       ?CrashDump_DmfCreate_RingBuffer@@YAJPEAUDMFMODULE__@@KKK@Z 0000000180047518 f   DmfK:Dmf_CrashDump.obj
 0005:00016778       ?CrashDump_DmfDestroy_RingBuffer@@YAXPEAUDMFMODULE__@@K@Z 0000000180047778 f   DmfK:Dmf_CrashDump.obj
 0005:000167e4       ?CrashDump_FileHandleSlotFind@@YAJPEAUDMFMODULE__@@PEAUWDFFILEOBJECT__@@W4DataSourceModeType@@@Z 00000001800477e4 f   DmfK:Dmf_CrashDump.obj
 0005:00016858       ?CrashDump_FileHandleSlotFindForDestroy@@YAJPEAUDMFMODULE__@@PEAUWDFFILEOBJECT__@@@Z 0000000180047858 f   DmfK:Dmf_CrashDump.obj
 0005:000168c4       ?CrashDump_FileHandleSlotFree@@YAJPEAUDMFMODULE__@@PEAUWDFFILEOBJECT__@@@Z 00000001800478c4 f   DmfK:Dmf_CrashDump.obj
 0005:00016e50       ?DMF_CrashDump_Close@@YAXPEAUDMFMODULE__@@@Z 0000000180047e50 f   DmfK:Dmf_CrashDump.obj
 0005:00017170       ?DMF_CrashDump_Destroy@@YAXPEAUDMFMODULE__@@@Z 0000000180048170 f   DmfK:Dmf_CrashDump.obj
 0005:000171e0       ?DMF_CrashDump_Open@@YAJPEAUDMFMODULE__@@@Z 00000001800481e0 f   DmfK:Dmf_CrashDump.obj
 0005:00018f70       ?DMF_HashTable_Close@@YAXPEAUDMFMODULE__@@@Z 0000000180049f70 f   DmfK:Dmf_HashTable.obj
 0005:00019030       ?DMF_HashTable_Open@@YAJPEAUDMFMODULE__@@@Z 000000018004a030 f   DmfK:Dmf_HashTable.obj
 0005:00019100       ?HashTable_ContextCleanup@@YAXPEAU_DMF_CONTEXT_HashTable@@@Z 000000018004a100 f   DmfK:Dmf_HashTable.obj
 0005:000191f0       ?HashTable_ContextInitialize@@YAJPEAUDMFMODULE__@@@Z 000000018004a1f0 f   DmfK:Dmf_HashTable.obj
 0005:000199f0       ?DMF_RequestTarget_Close@@YAXPEAUDMFMODULE__@@@Z 000000018004a9f0 f   DmfK:Dmf_RequestTarget.obj
 0005:00019ae0       ?DMF_RequestTarget_Open@@YAJPEAUDMFMODULE__@@@Z 000000018004aae0 f   DmfK:Dmf_RequestTarget.obj
 0005:0001a410       ?DMF_ContinuousRequestTarget_Close@@YAXPEAUDMFMODULE__@@@Z 000000018004b410 f   DmfK:Dmf_ContinuousRequestTarget.obj
 0005:0001a540       ?DMF_ContinuousRequestTarget_Open@@YAJPEAUDMFMODULE__@@@Z 000000018004b540 f   DmfK:Dmf_ContinuousRequestTarget.obj
 0005:0001ab50       ?DMF_Rundown_Close@@YAXPEAUDMFMODULE__@@@Z 000000018004bb50 f   DmfK:Dmf_Rundown.obj
 0005:0001abf0       ?DMF_Rundown_Open@@YAJPEAUDMFMODULE__@@@Z 000000018004bbf0 f   DmfK:Dmf_Rundown.obj
 0007:00000000       .edata                     000000018004e000     surface_hid_mini.dll.exp
 0007:00000028       rgpv                       000000018004e028     surface_hid_mini.dll.exp
 0007:00000034       rgszName                   000000018004e034     surface_hid_mini.dll.exp
 0007:00000040       rgwOrd                     000000018004e040     surface_hid_mini.dll.exp
 0007:00000046       szName                     000000018004e046     surface_hid_mini.dll.exp
 0007:0000005b       $N00001                    000000018004e05b     surface_hid_mini.dll.exp
 0007:00000067       $N00002                    000000018004e067     surface_hid_mini.dll.exp
 0007:0000007a       $N00003                    000000018004e07a     surface_hid_mini.dll.exp
 0008:00000a0c       .idata$6                   000000018004fa0c     ntoskrnl:ntoskrnl.exe
 0008:00000aa6       .idata$6                   000000018004faa6     DmfK:ext-ms-win-ntos-werkernel-l1-1-1.dll
 0008:00000b9a       .idata$6                   000000018004fb9a     wpprecorder:WppRecorder.sys
 0008:00001038       .idata$6                   0000000180050038     WdfLdr:WDFLDR.SYS

 Exports

  ordinal    name

        1    DriverEntry
        2    __CxxFrameHandler3
        3    _fltused
